 3DFileAccess

 Timestamp is 56cd4ba8 (Wed Feb 24 15:20:24 2016)

 Preferred load address is 10000000

 Start         Length     Name                   Class
 0001:00000000 0003eb66H .text                   CODE
 0001:0003eb70 000012d2H .text$x                 CODE
 0001:0003fe50 0000000cH .text$yc                CODE
 0001:0003fe60 0000004aH .text$yd                CODE
 0002:00000000 00000180H .idata$5                DATA
 0002:00000180 00000004H .CRT$XCA                DATA
 0002:00000184 00000004H .CRT$XCU                DATA
 0002:00000188 00000004H .CRT$XCZ                DATA
 0002:0000018c 00000004H .CRT$XIA                DATA
 0002:00000190 00000014H .CRT$XIC                DATA
 0002:000001a4 00000004H .CRT$XIZ                DATA
 0002:000001a8 00000004H .CRT$XPA                DATA
 0002:000001ac 00000004H .CRT$XPX                DATA
 0002:000001b0 00000004H .CRT$XPXA               DATA
 0002:000001b4 00000004H .CRT$XPZ                DATA
 0002:000001b8 00000004H .CRT$XTA                DATA
 0002:000001bc 00000004H .CRT$XTZ                DATA
 0002:000001c0 000063b8H .rdata                  DATA
 0002:00006578 00000073H .rdata$debug            DATA
 0002:000065ec 000006bcH .rdata$r                DATA
 0002:00006cb0 000001b8H .rdata$sxdata           DATA
 0002:00006e68 00000004H .rtc$IAA                DATA
 0002:00006e6c 00000004H .rtc$IZZ                DATA
 0002:00006e70 00000004H .rtc$TAA                DATA
 0002:00006e74 00000004H .rtc$TZZ                DATA
 0002:00006e78 00001ea4H .xdata$x                DATA
 0002:00008d1c 00000028H .idata$2                DATA
 0002:00008d44 00000014H .idata$3                DATA
 0002:00008d58 00000180H .idata$4                DATA
 0002:00008ed8 000006aeH .idata$6                DATA
 0002:00009590 00001c29H .edata                  DATA
 0003:00000000 000019c0H .data                   DATA
 0003:000019c0 00005260H .bss                    DATA
 0004:00000000 00000058H .rsrc$01                DATA
 0004:00000060 00000320H .rsrc$02                DATA

  Address         Publics by Value              Rva+Base       Lib:Object

 0000:00000000       __except_list              00000000     <absolute>
 0000:0000006e       ___safe_se_handler_count   0000006e     <absolute>
 0000:00000000       ___ImageBase               10000000     <linker-defined>
 0001:00000000       ?SetHasBVInfo@CWzUnitEditable@@QAEXH@Z 10001000 f i dllaccess.obj
 0001:00000017       ?EnableLodByForce@CWzUnitEditable@@QAEX_N@Z 10001017 f i dllaccess.obj
 0001:0000002e       ?GetNumSoundSet@WzAnimationInfo@@QBEHXZ 1000102e f i dllaccess.obj
 0001:00000050       ?GetNumEffectInfo@WzAnimationInfo@@QBEHXZ 10001050 f i dllaccess.obj
 0001:00000075       ?GetNumCustomInfo@WzAnimationInfo@@QBEHXZ 10001075 f i dllaccess.obj
 0001:0000009c       ?SetScale@CWzUnitDraw@@QAEXABUWzVector@@H@Z 1000109c f i dllaccess.obj
 0001:000000e9       ?SetScale@CWzUnitSkeleton@@QAEXABUWzVector@@H@Z 100010e9 f i dllaccess.obj
 0001:0000014b       ??8WzVector@@QBEHABU0@@Z   1000114b f i dllaccess.obj
 0001:000001cf       ?SetScale@CWzUnitDraw@@QAEXMMMH@Z 100011cf f i dllaccess.obj
 0001:0000023b       ?SetScale@CWzUnitDraw@@QAEXMH@Z 1000123b f i dllaccess.obj
 0001:000002a7       ?SetRotation@CWzUnitDraw@@QAEXABUWzVector@@H@Z 100012a7 f i dllaccess.obj
 0001:000002f4       ?SetRotation@CWzUnitSkeleton@@QAEXABUWzVector@@H@Z 100012f4 f i dllaccess.obj
 0001:00000356       ?SetRotation@CWzUnitDraw@@QAEXMMMH@Z 10001356 f i dllaccess.obj
 0001:000003c2       ?SetPosition@CWzUnitDraw@@QAEXABUWzVector@@H@Z 100013c2 f i dllaccess.obj
 0001:0000040f       ?SetPosition@CWzUnitSkeleton@@QAEXABUWzVector@@H@Z 1000140f f i dllaccess.obj
 0001:00000471       ?SetPosition@CWzUnitDraw@@QAEXMMMH@Z 10001471 f i dllaccess.obj
 0001:000004dd       ?SetBoundingVolume@CWzUnitDraw@@QAEXABUWzBoundingVolume@@@Z 100014dd f i dllaccess.obj
 0001:00000555       ?UpdateBoundingVolumeWithMatrix@CWzUnitDraw@@QAEXPAUWzMatrix@@@Z 10001555 f i dllaccess.obj
 0001:000005a3       ?ResetBVExtra@CWzUnitDraw@@QAEXXZ 100015a3 f i dllaccess.obj
 0001:00000617       ?SetCurrentAnimation@CWzUnitDraw@@QAEXKHHH@Z 10001617 f i dllaccess.obj
 0001:0000066a       ?SetCurrentBlendAnimation@CWzUnitDraw@@QAEXKHHMHM@Z 1000166a f i dllaccess.obj
 0001:000006c4       ?UnSetBlendAnimation@CWzUnitDraw@@QAEXXZ 100016c4 f i dllaccess.obj
 0001:00000709       ?UnsetBlendAnimation@CWzUnitSkeleton@@QAEXXZ 10001709 f i dllaccess.obj
 0001:00000740       ?SetInterpolationFrame@CWzUnitDraw@@QAEXH@Z 10001740 f i dllaccess.obj
 0001:0000079c       ?SetBlendInterpolationFrame@CWzUnitDraw@@QAEXHH@Z 1000179c f i dllaccess.obj
 0001:000007f3       ?GetTransformBuffer@CWzUnitDraw@@QAEPAUWzMatrix@@H@Z 100017f3 f i dllaccess.obj
 0001:0000084f       ?GetInverseAndTransformBuffer@CWzUnitDraw@@QAEPAUWzMatrix@@H@Z 1000184f f i dllaccess.obj
 0001:000008ab       _Func_ContactWzd           100018ab f   dllaccess.obj
 0001:00001008       ?Instance@CWzdShareInfo@@SAPAV1@XZ 10002008 f i dllaccess.obj
 0001:00001070       _DllMain@12                10002070 f   dllentry.obj
 0001:0000108e       ??0CWzdAnimation@@QAE@XZ   1000208e f   wzdanimation.obj
 0001:00001119       ??1CWzdAnimation@@UAE@XZ   10002119 f   wzdanimation.obj
 0001:0000116d       ?InitVariables@CWzdAnimation@@AAEXXZ 1000216d f   wzdanimation.obj
 0001:00001189       ?Release@CWzdAnimation@@AAEXXZ 10002189 f   wzdanimation.obj
 0001:00001262       ?Destroy@CWzdAnimation@@UAEXXZ 10002262 f   wzdanimation.obj
 0001:00001283       ?AllocBones@CWzdAnimation@@UAEXG@Z 10002283 f   wzdanimation.obj
 0001:000013b3       ?SetBoneInfo@CWzdAnimation@@UAEXGHPBD@Z 100023b3 f   wzdanimation.obj
 0001:00001431       ?CompareBoneStructure@CWzdAnimation@@UAEHPBVCWzdBase@@@Z 10002431 f   wzdanimation.obj
 0001:00001551       ?CompareBoneList@CWzdAnimation@@UAEHPBVCWzdBase@@@Z 10002551 f   wzdanimation.obj
 0001:000015fa       ?AllocKeyFrames@CWzdAnimation@@UAEXXZ 100025fa f   wzdanimation.obj
 0001:000016f6       ?AllocKeyTransforms@CWzdAnimation@@UAEXGG@Z 100026f6 f   wzdanimation.obj
 0001:00001857       ?SetRealFrame@CWzdAnimation@@UAEXGGG@Z 10002857 f   wzdanimation.obj
 0001:00001885       ?SetKeyTransformInfo@CWzdAnimation@@UAEXGGABUWzVector@@ABUWzQuaternion@@@Z 10002885 f   wzdanimation.obj
 0001:000018db       ?CreateTransformArrayByFrame@CWzdAnimation@@UAEXPAUWzTransform@@M@Z 100028db f   wzdanimation.obj
 0001:0000192f       ?CreateTransformByFrame@CWzdAnimation@@UAEXPAUWzTransform@@GM@Z 1000292f f   wzdanimation.obj
 0001:00001b55       ?CalcTransformMatrixT@CWzdAnimation@@UAEXPAUWzMatrix@@PBUWzTransform@@PBUWzTransformParam@@@Z 10002b55 f   wzdanimation.obj
 0001:00001bbb       ?CalcBoneTransformMatrixT@CWzdAnimation@@AAEXGPAUWzMatrix@@PBUWzTransform@@PBUWzTransformParam@@@Z 10002bbb f   wzdanimation.obj
 0001:00001f45       ?AnimationSlerp@CWzdAnimation@@UAEXPAUWzTransform@@PBU2@1M@Z 10002f45 f   wzdanimation.obj
 0001:00001f97       ?Serialize@CWzdAnimation@@MAEHPAVCWzArchive@@@Z 10002f97 f   wzdanimation.obj
 0001:00002d42       ?Save_Text@CWzdAnimation@@IAEHPAVCWzArchive@@@Z 10003d42 f   wzdanimation.obj
 0001:000030ed       ?AddTriangle@CWzdBase@@UAEXPBDQBUWzSkinningInfo@@QBUWzVector@@2QBUWzUVVert@@0QBK4@Z 100040ed f i wzdanimation.obj
 0001:000030f8       ?GetNumberOfVertex@CWzdBase@@UBEHXZ 100040f8 f i wzdanimation.obj
 0001:000030f8       ?GetNumberOfMeshGroup@CWzdBase@@UBEHXZ 100040f8 f i wzdanimation.obj
 0001:000030f8       ?GetNumFrame@CWzdBase@@UBEGXZ 100040f8 f i wzdbase.obj
 0001:000030f8       ?GetInverseOfDefaultTransform@CWzdBase@@UBEPBUWzMatrix@@XZ 100040f8 f i wzdanimation.obj
 0001:000030f8       ?GetTotalVertPack@CWzdBase@@UBEKXZ 100040f8 f i wzdanimation.obj
 0001:000030f8       ?GetSkinningInfo@CWzdBase@@UBEPAUWzSkinningInfo@@XZ 100040f8 f i wzdanimation.obj
 0001:000030f8       ?GetKeyFramesList@CWzdBase@@UBEPAUWzKeyFrame@@XZ 100040f8 f i wzdbase.obj
 0001:000030f8       ?AllocForMesh@CWzdBase@@UAEHXZ 100040f8 f i wzdanimation.obj
 0001:000030f8       ?GetBonesList@CWzdBase@@UBEPAUWzNode@@XZ 100040f8 f i wzdbase.obj
 0001:000030f8       ?GetMaxMeshGroup@CWzdBase@@UBEHXZ 100040f8 f i wzdanimation.obj
 0001:000030f8       ?GetBlendedCount@CWzdBase@@UBEHXZ 100040f8 f i wzdanimation.obj
 0001:000030f8       ?GetNumNode@CWzdBase@@UBEGXZ 100040f8 f i wzdbase.obj
 0001:000030f8       ?GetVertexList@CWzdBase@@UBEPAUWzMeshVertex@@XZ 100040f8 f i wzdanimation.obj
 0001:000030f8       ?GetBoneExtraInfoList@CWzdBase@@UBEPAUWzNodeExtra@@XZ 100040f8 f i wzdbase.obj
 0001:00003103       ?SetAnimationSpeedRate@CWzdBase@@UAEXM@Z 10004103 f i wzdbase.obj
 0001:00003103       ?GetIdentity@CWzdBase@@UAEXQAE@Z 10004103 f i wzdbase.obj
 0001:00003103       ?DestroyShadowVolume@CWzdBase@@UAEXPAVCWzShadowVolume@@@Z 10004103 f i wzdanimation.obj
 0001:00003103       ?AllocBones@CWzdBase@@UAEXG@Z 10004103 f i wzdbase.obj
 0001:00003103       ?DestroySilhouette@CWzdBase@@UAEXPAVCWzSilhouette@@@Z 10004103 f i wzdanimation.obj
 0001:0000310e       ?CreateVertexShaderConstantInfo@CWzdBase@@UAEHHH@Z 1000410e f i wzdanimation.obj
 0001:0000311b       ?CreateTransformArrayByFrame@CWzdBase@@UAEXPAUWzTransform@@M@Z 1000411b f i wzdbase.obj
 0001:0000311b       ?CalcSkinMatrix@CWzdBase@@UAEXPAUWzMatrix@@PBU2@@Z 1000411b f i wzdanimation.obj
 0001:0000311b       ?CalcTransformMatrixD@CWzdBase@@UAEXPAUWzMatrix@@PBUWzTransformParam@@@Z 1000411b f i wzdanimation.obj
 0001:0000311b       ?SetOwnVertexBuffer@CWzdBase@@UAEXHPAX@Z 1000411b f i wzdanimation.obj
 0001:0000311b       ?OnAniStateNotice@CWzAniStateCB@@UAEXHK@Z 1000411b f i wzunitskeleton.obj
 0001:0000311b       ?SetOwnIndexBuffer@CWzdBase@@UAEXHPAX@Z 1000411b f i wzdanimation.obj
 0001:0000311b       ?AllocKeyTransforms@CWzdBase@@UAEXGG@Z 1000411b f i wzdbase.obj
 0001:00003126       ?GetOwnVertexBuffer@CWzdBase@@UBEPAXH@Z 10004126 f i wzdanimation.obj
 0001:00003126       ?GetOwnIndexBuffer@CWzdBase@@UBEPAXH@Z 10004126 f i wzdanimation.obj
 0001:00003134       ?GetBvAABB@CWzdBase@@UBEABUBvAABB@@XZ 10004134 f i wzdanimation.obj
 0001:00003142       ?GetBvSphere@CWzdBase@@UBEABUBvSphere@@XZ 10004142 f i wzdanimation.obj
 0001:00003150       ?GetIdentity@CWzdAnimation@@UAEXQAE@Z 10004150 f i wzdanimation.obj
 0001:00003166       ?CheckIdentity@CWzdAnimation@@UBEHPBE@Z 10004166 f i wzdanimation.obj
 0001:00003184       ?GetNumNode@CWzdAnimation@@UBEGXZ 10004184 f i wzdanimation.obj
 0001:00003197       ?GetBonesList@CWzdAnimation@@UBEPAUWzNode@@XZ 10004197 f i wzdanimation.obj
 0001:000031a9       ?GetBoneExtraInfoList@CWzdAnimation@@UBEPAUWzNodeExtra@@XZ 100041a9 f i wzdanimation.obj
 0001:000031bb       ?GetKeyFramesList@CWzdAnimation@@UBEPAUWzKeyFrame@@XZ 100041bb f i wzdanimation.obj
 0001:000031cd       ?GetNumFrame@CWzdAnimation@@UBEGXZ 100041cd f i wzdanimation.obj
 0001:000031f7       ?GetNumBoneFrame@CWzdAnimation@@UBEGG@Z 100041f7 f i wzdanimation.obj
 0001:00003217       ?SetAnimationSpeedRate@CWzdAnimation@@UAEXM@Z 10004217 f i wzdanimation.obj
 0001:00003232       ?GetAnimationSpeedRate@CWzdAnimation@@UBEMXZ 10004232 f i wzdanimation.obj
 0001:00003244       ??_ECWzdAnimation@@UAEPAXI@Z 10004244 f i wzdanimation.obj
 0001:00003244       ??_GCWzdAnimation@@UAEPAXI@Z 10004244 f i wzdanimation.obj
 0001:0000326b       ??_EWzKeyFrame@@QAEPAXI@Z  1000426b f i wzdanimation.obj
 0001:000032ce       ??1WzKeyFrame@@QAE@XZ      100042ce f i wzdanimation.obj
 0001:0000331a       ??0WzKeyFrame@@QAE@XZ      1000431a f i wzdanimation.obj
 0001:0000333a       ?QuaternionToMatrix@@YAPAUWzMatrix@@PAU1@PBUWzQuaternion@@@Z 1000433a f i wzdanimation.obj
 0001:0000350e       ?InterpolateVector@@YAPAUWzVector@@PAU1@PBU1@1M@Z 1000450e f i wzdanimation.obj
 0001:0000356c       ?find@?$_Tree@V?$_Tmap_traits@HUWzVector@@U?$less@H@std@@V?$allocator@U?$pair@$$CBHUWzVector@@@std@@@3@$0A@@std@@@std@@QBE?AVconst_iterator@12@ABH@Z 1000456c f i wzdanimation.obj
 0001:0000363b       ??0const_iterator@?$_Tree@V?$_Tmap_traits@HUWzVector@@U?$less@H@std@@V?$allocator@U?$pair@$$CBHUWzVector@@@std@@@3@$0A@@std@@@std@@QAE@PAU_Node@?$_Tree_nod@V?$_Tmap_traits@HUWzVector@@U?$less@H@std@@V?$allocator@U?$pair@$$CBHUWzVector@@@std@@@3@$0A@@std@@@2@PBV12@@Z 1000463b f i wzdanimation.obj
 0001:00003671       ??Dconst_iterator@?$_Tree@V?$_Tmap_traits@HUWzVector@@U?$less@H@std@@V?$allocator@U?$pair@$$CBHUWzVector@@@std@@@3@$0A@@std@@@std@@QBEABU?$pair@$$CBHUWzVector@@@2@XZ 10004671 f i wzdanimation.obj
 0001:000036db       ?_Lbound@?$_Tree@V?$_Tmap_traits@HUWzVector@@U?$less@H@std@@V?$allocator@U?$pair@$$CBHUWzVector@@@std@@@3@$0A@@std@@@std@@IBEPAU_Node@?$_Tree_nod@V?$_Tmap_traits@HUWzVector@@U?$less@H@std@@V?$allocator@U?$pair@$$CBHUWzVector@@@std@@@3@$0A@@std@@@2@ABH@Z 100046db f i wzdanimation.obj
 0001:0000373d       ??0CWzdBase@@QAE@XZ        1000473d f   wzdbase.obj
 0001:00003764       ??1CWzdBase@@UAE@XZ        10004764 f   wzdbase.obj
 0001:0000377e       ?InitVariables@CWzdBase@@AAEXXZ 1000477e f   wzdbase.obj
 0001:000037b3       ?Release@CWzdBase@@AAEXXZ  100047b3 f   wzdbase.obj
 0001:000037bc       ?Destroy@CWzdBase@@UAEXXZ  100047bc f   wzdbase.obj
 0001:000037d5       ?Create@CWzdBase@@UAEHPBDPAEH@Z 100047d5 f   wzdbase.obj
 0001:000038f2       ?Create@CWzdBase@@UAEHPBDPAX@Z 100048f2 f   wzdbase.obj
 0001:0000396e       ?Create@CWzdBase@@UAEHPBD@Z 1000496e f   wzdbase.obj
 0001:000039c8       ?Save@CWzdBase@@UAEHPBDH@Z 100049c8 f   wzdbase.obj
 0001:00003ac3       ?Save@CWzdBase@@UAEHPBDPAXH@Z 10004ac3 f   wzdbase.obj
 0001:00003bc1       ?Serialize@CWzdBase@@MAEHPAVCWzArchive@@@Z 10004bc1 f   wzdbase.obj
 0001:00003db2       ?CreateShadowVolume@CWzdBase@@UAEXPAVCWzShadowVolume@@ABUWzVector@@PBU3@K@Z 10004db2 f i wzdanimation.obj
 0001:00003db2       ?SetKeyTransformInfo@CWzdBase@@UAEXGGABUWzVector@@ABUWzQuaternion@@@Z 10004db2 f i wzdbase.obj
 0001:00003db2       ?AnimationSlerp@CWzdBase@@UAEXPAUWzTransform@@PBU2@1M@Z 10004db2 f i wzdbase.obj
 0001:00003db2       ?FillVertexShaderConstantInfo@CWzdBase@@UAEXHHHPAH@Z 10004db2 f i wzdanimation.obj
 0001:00003dbd       ?SetBoneInfo@CWzdBase@@UAEXGHPBD@Z 10004dbd f i wzdbase.obj
 0001:00003dbd       ?SetRealFrame@CWzdBase@@UAEXGGG@Z 10004dbd f i wzdbase.obj
 0001:00003dbd       ?CreateSilhouette@CWzdBase@@UAEXPAVCWzSilhouette@@ABUWzVector@@PBU3@@Z 10004dbd f i wzdanimation.obj
 0001:00003dbd       ?CreateTransformByFrame@CWzdBase@@UAEXPAUWzTransform@@GM@Z 10004dbd f i wzdbase.obj
 0001:00003dbd       ?CalcTransformMatrixT@CWzdBase@@UAEXPAUWzMatrix@@PBUWzTransform@@PBUWzTransformParam@@@Z 10004dbd f i wzdbase.obj
 0001:00003dc8       ?GetAnimationSpeedRate@CWzdBase@@UBEMXZ 10004dc8 f i wzdbase.obj
 0001:00003dd3       ?GetMeshGroupInfo@CWzdBase@@UBEPAUWzMeshGroup@@H@Z 10004dd3 f i wzdanimation.obj
 0001:00003dd3       ?CompareBoneList@CWzdBase@@UAEHPBV1@@Z 10004dd3 f i wzdbase.obj
 0001:00003dd3       ?GetNumBoneFrame@CWzdBase@@UBEGG@Z 10004dd3 f i wzdbase.obj
 0001:00003dd3       ?CompareBoneStructure@CWzdBase@@UAEHPBV1@@Z 10004dd3 f i wzdbase.obj
 0001:00003dd3       ?CheckIdentity@CWzdBase@@UBEHPBE@Z 10004dd3 f i wzdbase.obj
 0001:00003de0       ?CheckDiscAccessExistence@CWzdBase@@SAPAVCDiscAccess@@XZ 10004de0 f i wzdbase.obj
 0001:00003e5b       ??0CWzdMesh@@QAE@XZ        10004e5b f   wzdmesh.obj
 0001:00003ec6       ??1CWzdMesh@@UAE@XZ        10004ec6 f   wzdmesh.obj
 0001:00003f1a       ?InitVariables@CWzdMesh@@AAEXXZ 10004f1a f   wzdmesh.obj
 0001:00003fe6       ?Release@CWzdMesh@@AAEXXZ  10004fe6 f   wzdmesh.obj
 0001:00003ff7       ?Destroy@CWzdMesh@@UAEXXZ  10004ff7 f   wzdmesh.obj
 0001:00004018       ?ReleaseDefTransformMat@CWzdMesh@@AAEXXZ 10005018 f   wzdmesh.obj
 0001:00004079       ?InitDefTransformMat@CWzdMesh@@AAEXXZ 10005079 f   wzdmesh.obj
 0001:000041bc       ?CalcDefBoneTransformMatrix@CWzdMesh@@AAEXGPAUWzMatrix@@@Z 100051bc f   wzdmesh.obj
 0001:000042ba       ?CalcTransformMatrixD@CWzdMesh@@UAEXPAUWzMatrix@@PBUWzTransformParam@@@Z 100052ba f   wzdmesh.obj
 0001:0000431d       ?CalcBoneTransformMatrixD@CWzdMesh@@AAEXGPAUWzMatrix@@PBUWzTransformParam@@@Z 1000531d f   wzdmesh.obj
 0001:0000467c       ?CalcSkinMatrix@CWzdMesh@@UAEXPAUWzMatrix@@PBU2@@Z 1000567c f   wzdmesh.obj
 0001:000046e6       ?CreateSilhouette@CWzdMesh@@UAEXPAVCWzSilhouette@@ABUWzVector@@PBU3@@Z 100056e6 f   wzdmesh.obj
 0001:00004737       ?DestroySilhouette@CWzdMesh@@UAEXPAVCWzSilhouette@@@Z 10005737 f   wzdmesh.obj
 0001:00004750       ?CreateShadowVolume@CWzdMesh@@UAEXPAVCWzShadowVolume@@ABUWzVector@@PBU3@K@Z 10005750 f   wzdmesh.obj
 0001:000047a4       ?DestroyShadowVolume@CWzdMesh@@UAEXPAVCWzShadowVolume@@@Z 100057a4 f   wzdmesh.obj
 0001:000047bd       ?CreateVertexShaderConstantInfo@CWzdMesh@@UAEHHH@Z 100057bd f   wzdmesh.obj
 0001:00004903       ?FillVertexShaderConstantInfo@CWzdMesh@@UAEXHHHPAH@Z 10005903 f   wzdmesh.obj
 0001:000049ed       ?UpdateBoundingVolume@CWzdMesh@@IAEXXZ 100059ed f   wzdmesh.obj
 0001:00004a54       ?Serialize@CWzdMesh@@MAEHPAVCWzArchive@@@Z 10005a54 f   wzdmesh.obj
 0001:00004bc8       ?SerializeVertexList@CWzdMesh@@IAEHPAVCWzArchive@@@Z 10005bc8 f   wzdmesh.obj
 0001:00005047       ?SerializeMeshGroup@CWzdMesh@@IAEHPAVCWzArchive@@@Z 10006047 f   wzdmesh.obj
 0001:00005fdc       ?SerializeSkinningInfo@CWzdMesh@@IAEHPAVCWzArchive@@@Z 10006fdc f   wzdmesh.obj
 0001:00006370       ?ReadOldVersionAndConvert@CWzdMesh@@IAEHPAVCWzArchive@@@Z 10007370 f   wzdmesh.obj
 0001:00006dff       ?GetNumberOfVertex@CWzdMeshConstructor@@UBEHXZ 10007dff f i wzdmesh.obj
 0001:00006e11       ?GetVertexList@CWzdMeshConstructor@@UBEPAUWzMeshVertex@@XZ 10007e11 f i wzdmesh.obj
 0001:00006e23       ?GetNumberOfMeshGroup@CWzdMeshConstructor@@UBEHXZ 10007e23 f i wzdmesh.obj
 0001:00006e35       ?GetMaxMeshGroup@CWzdMeshConstructor@@UBEHXZ 10007e35 f i wzdmesh.obj
 0001:00006e47       ?GetTotalVertPack@CWzdMeshConstructor@@UBEKXZ 10007e47 f i wzdmesh.obj
 0001:00006e59       ?GetBlendedCount@CWzdMeshConstructor@@UBEHXZ 10007e59 f i wzdmesh.obj
 0001:00006e6b       ?GetSkinningInfo@CWzdMeshConstructor@@UBEPAUWzSkinningInfo@@XZ 10007e6b f i wzdmesh.obj
 0001:00006e7d       ?GetIdentity@CWzdMesh@@UAEXQAE@Z 10007e7d f i wzdmesh.obj
 0001:00006e93       ?CheckIdentity@CWzdMesh@@UBEHPBE@Z 10007e93 f i wzdmesh.obj
 0001:00006eb1       ?GetInverseOfDefaultTransform@CWzdMesh@@UBEPBUWzMatrix@@XZ 10007eb1 f i wzdmesh.obj
 0001:00006ec3       ?SetOwnVertexBuffer@CWzdMesh@@UAEXHPAX@Z 10007ec3 f i wzdmesh.obj
 0001:00006eea       ?GetOwnVertexBuffer@CWzdMesh@@UBEPAXH@Z 10007eea f i wzdmesh.obj
 0001:00006f27       ?SetOwnIndexBuffer@CWzdMesh@@UAEXHPAX@Z 10007f27 f i wzdmesh.obj
 0001:00006f4e       ?GetOwnIndexBuffer@CWzdMesh@@UBEPAXH@Z 10007f4e f i wzdmesh.obj
 0001:00006f8b       ?GetBvAABB@CWzdMesh@@UBEABUBvAABB@@XZ 10007f8b f i wzdmesh.obj
 0001:00006f9c       ?GetBvSphere@CWzdMesh@@UBEABUBvSphere@@XZ 10007f9c f i wzdmesh.obj
 0001:00006fad       ??_GCWzdMesh@@UAEPAXI@Z    10007fad f i wzdmesh.obj
 0001:00006fad       ??_ECWzdMesh@@UAEPAXI@Z    10007fad f i wzdmesh.obj
 0001:00006fd4       ??1WzVertexShaderConstantInfo@@QAE@XZ 10007fd4 f i wzdmesh.obj
 0001:00007076       ?VectorNormalize@@YAPAUWzVector@@PAU1@PBU1@@Z 10008076 f i wzdmesh.obj
 0001:000070d1       ?VectorLength@@YAMPBUWzVector@@@Z 100080d1 f i wzdmesh.obj
 0001:000070f2       ?VectorLength2@@YAMPBUWzVector@@@Z 100080f2 f i wzdmesh.obj
 0001:00007124       ??0WzMeshGroup@@QAE@XZ     10008124 f i wzdmesh.obj
 0001:000071eb       ??0CWzdMeshConstructor@@QAE@XZ 100081eb f   wzdmeshconstructor.obj
 0001:00007260       ??1CWzdMeshConstructor@@UAE@XZ 10008260 f   wzdmeshconstructor.obj
 0001:000072b4       ?InitVariables@CWzdMeshConstructor@@AAEXXZ 100082b4 f   wzdmeshconstructor.obj
 0001:0000730d       ?Release@CWzdMeshConstructor@@AAEXXZ 1000830d f   wzdmeshconstructor.obj
 0001:00007376       ?ReleaseMeshGroup@CWzdMeshConstructor@@IAEXXZ 10008376 f   wzdmeshconstructor.obj
 0001:0000750d       ?Destroy@CWzdMeshConstructor@@UAEXXZ 1000850d f   wzdmeshconstructor.obj
 0001:0000752e       ?AllocForMesh@CWzdMeshConstructor@@UAEHXZ 1000852e f   wzdmeshconstructor.obj
 0001:000076cc       ?AddTriangle@CWzdMeshConstructor@@UAEXPBDQBUWzSkinningInfo@@QBUWzVector@@2QBUWzUVVert@@0QBK4@Z 100086cc f   wzdmeshconstructor.obj
 0001:00007857       ?GetIndexOfVertex@CWzdMeshConstructor@@IAEKHABUWzVector@@@Z 10008857 f   wzdmeshconstructor.obj
 0001:00007926       ?MakeSureSizeOfVertices@CWzdMeshConstructor@@IAEXH@Z 10008926 f   wzdmeshconstructor.obj
 0001:000079d8       ?GetMeshGroupOfTexture@CWzdMeshConstructor@@IAEHPBD0@Z 100089d8 f   wzdmeshconstructor.obj
 0001:00007b42       ?AddMeshGroup@CWzdMeshConstructor@@IAEXHPBD0@Z 10008b42 f   wzdmeshconstructor.obj
 0001:00007d24       ?MakeSureMeshGroupSize@CWzdMeshConstructor@@IAEXH@Z 10008d24 f   wzdmeshconstructor.obj
 0001:00007e55       ?GetMeshGroupInfo@CWzdMeshConstructor@@UBEPAUWzMeshGroup@@H@Z 10008e55 f   wzdmeshconstructor.obj
 0001:00007e96       ?GetIndexOfVertPack@CWzdMeshConstructor@@IAEKPAUWzMeshGroup@@PBUWzMeshVertPack@@@Z 10008e96 f   wzdmeshconstructor.obj
 0001:00007f81       ?IsSameVertPack@CWzdMeshConstructor@@IBEHPBUWzMeshVertPack@@0@Z 10008f81 f   wzdmeshconstructor.obj
 0001:00008059       ?MakeSureSizeOfVertPack@CWzdMeshConstructor@@IAEXPAUWzMeshGroup@@H@Z 10009059 f   wzdmeshconstructor.obj
 0001:0000810b       ?GenerateNearFaceInfo@CWzdMeshConstructor@@IAEXXZ 1000910b f   wzdmeshconstructor.obj
 0001:000081ab       ?SetNearFaceOfTheDirection@CWzdMeshConstructor@@IAEXHHH@Z 100091ab f   wzdmeshconstructor.obj
 0001:00008304       ?MakeSureSizeOfFace@CWzdMeshConstructor@@IAEXPAUWzMeshGroup@@H@Z 10009304 f   wzdmeshconstructor.obj
 0001:000083b6       ?GetSkinningIndex@CWzdMeshConstructor@@IAEHPBUWzSkinningInfo@@@Z 100093b6 f   wzdmeshconstructor.obj
 0001:00008459       ?MakeSureSIListSize@CWzdMeshConstructor@@IAEXH@Z 10009459 f   wzdmeshconstructor.obj
 0001:0000850b       ?CalculateTangent@@YAXPAUWzVector@@PAEPBU1@22PBUWzUVVert@@332@Z 1000950b f   wzdmeshconstructor.obj
 0001:000088ad       ??_ECWzdMeshConstructor@@UAEPAXI@Z 100098ad f i wzdmeshconstructor.obj
 0001:000088ad       ??_GCWzdMeshConstructor@@UAEPAXI@Z 100098ad f i wzdmeshconstructor.obj
 0001:000088d4       ??HWzVector@@QBE?AU0@ABU0@@Z 100098d4 f i wzdmeshconstructor.obj
 0001:0000891c       ?VectorDotProduct@@YAMPBUWzVector@@0@Z 1000991c f i wzdmeshconstructor.obj
 0001:0000894e       ??8@YAHABUWzSkinningInfo@@0@Z 1000994e f i wzdmeshconstructor.obj
 0001:000089c1       ??GWzVector@@QBE?AU0@ABU0@@Z 100099c1 f i wzdmeshconstructor.obj
 0001:00008a09       ?VectorCrossProduct@@YAPAUWzVector@@PAU1@PBU1@1@Z 10009a09 f i wzdmeshconstructor.obj
 0001:00008a6c       ??0CWzdMeshSorter@@QAE@XZ  10009a6c f   wzdmeshsorter.obj
 0001:00008a7e       ??1CWzdMeshSorter@@QAE@XZ  10009a7e f   wzdmeshsorter.obj
 0001:00008a87       ?Sort@CWzdMeshSorter@@QAEXPAVCWzdMesh@@@Z 10009a87 f   wzdmeshsorter.obj
 0001:00008c16       ?InitBoneConnection@CWzdMeshSorter@@AAEHPAUSt_BoneConnection@@@Z 10009c16 f   wzdmeshsorter.obj
 0001:00008f14       ?InitBoneRelation@CWzdMeshSorter@@AAEHPAUSt_BoneConnection@@H@Z 10009f14 f   wzdmeshsorter.obj
 0001:00009266       ?SortBones@CWzdMeshSorter@@AAEHPAHPAUSt_BoneConnection@@@Z 1000a266 f   wzdmeshsorter.obj
 0001:00009b53       ?SortFaces@CWzdMeshSorter@@AAEXHPBH@Z 1000ab53 f   wzdmeshsorter.obj
 0001:00009edb       ?DecreaseCost@CWzdMeshSorter@@AAEXPAUSt_BoneConnection@@H@Z 1000aedb f   wzdmeshsorter.obj
 0001:0000a02b       ?GetMaxRelatedBone@CWzdMeshSorter@@AAEHPBUSt_BoneConnection@@PBH@Z 1000b02b f   wzdmeshsorter.obj
 0001:0000a0a4       ?CanAddBone@CWzdMeshSorter@@AAEHHPBUSt_BoneConnection@@PBH1H@Z 1000b0a4 f   wzdmeshsorter.obj
 0001:0000a148       ?GetMinCostBone@CWzdMeshSorter@@AAEHPBUSt_BoneConnection@@H@Z 1000b148 f   wzdmeshsorter.obj
 0001:0000a22d       ?CanAddFace@CWzdMeshSorter@@AAEHHPBUWzFace@@PBH@Z 1000b22d f   wzdmeshsorter.obj
 0001:0000a2ee       ??0?$vector@HV?$allocator@H@std@@@std@@QAE@XZ 1000b2ee f i wzdmeshsorter.obj
 0001:0000a370       ??1?$vector@HV?$allocator@H@std@@@std@@QAE@XZ 1000b370 f i wzdmeshsorter.obj
 0001:0000a3c6       ?push_back@?$vector@HV?$allocator@H@std@@@std@@QAEXABH@Z 1000b3c6 f i wzdmeshsorter.obj
 0001:0000a490       ??0?$list@HV?$allocator@H@std@@@std@@QAE@XZ 1000b490 f i wzdmeshsorter.obj
 0001:0000a505       ??1?$list@HV?$allocator@H@std@@@std@@QAE@XZ 1000b505 f i wzdmeshsorter.obj
 0001:0000a55b       ?begin@?$list@HV?$allocator@H@std@@@std@@QAE?AV?$_Iterator@$00@12@XZ 1000b55b f i wzdmeshsorter.obj
 0001:0000a5a9       ?end@?$list@HV?$allocator@H@std@@@std@@QAE?AV?$_Iterator@$00@12@XZ 1000b5a9 f i wzdmeshsorter.obj
 0001:0000a5ee       ?push_back@?$list@HV?$allocator@H@std@@@std@@QAEXABH@Z 1000b5ee f i wzdmeshsorter.obj
 0001:0000a647       ?erase@?$list@HV?$allocator@H@std@@@std@@QAE?AV?$_Iterator@$00@12@V?$_Const_iterator@$00@12@@Z 1000b647 f i wzdmeshsorter.obj
 0001:0000a6f8       ??1?$_Vector_val@HV?$allocator@H@std@@@std@@QAE@XZ 1000b6f8 f i wzdmeshsorter.obj
 0001:0000a6f8       ??1?$_List_val@HV?$allocator@H@std@@@std@@QAE@XZ 1000b6f8 f i wzdmeshsorter.obj
 0001:0000a6f8       ??1?$_Vector_val@UWzSoundInfo@@V?$allocator@UWzSoundInfo@@@std@@@std@@QAE@XZ 1000b6f8 f i wzanimationInfo.obj
 0001:0000a6f8       ??1?$_Vector_val@UWzEffectInfo@@V?$allocator@UWzEffectInfo@@@std@@@std@@QAE@XZ 1000b6f8 f i wzanimationInfo.obj
 0001:0000a6f8       ??1?$_Tree_val@V?$_Tmap_traits@HUWzVector@@U?$less@H@std@@V?$allocator@U?$pair@$$CBHUWzVector@@@std@@@3@$0A@@std@@@std@@QAE@XZ 1000b6f8 f i wzunitskeleton.obj
 0001:0000a6f8       ??1?$_Vector_val@UWzCustomInfo@@V?$allocator@UWzCustomInfo@@@std@@@std@@QAE@XZ 1000b6f8 f i wzanimationInfo.obj
 0001:0000a713       ?end@?$vector@UWzSoundInfo@@V?$allocator@UWzSoundInfo@@@std@@@std@@QAE?AV?$_Vector_iterator@UWzSoundInfo@@V?$allocator@UWzSoundInfo@@@std@@@2@XZ 1000b713 f i wzanimationInfo.obj
 0001:0000a713       ?end@?$vector@HV?$allocator@H@std@@@std@@QAE?AV?$_Vector_iterator@HV?$allocator@H@std@@@2@XZ 1000b713 f i wzdmeshsorter.obj
 0001:0000a713       ?end@?$vector@HV?$allocator@H@std@@@std@@QBE?AV?$_Vector_const_iterator@HV?$allocator@H@std@@@2@XZ 1000b713 f i wzanimationInfo.obj
 0001:0000a713       ?end@?$vector@UWzCustomInfo@@V?$allocator@UWzCustomInfo@@@std@@@std@@QAE?AV?$_Vector_iterator@UWzCustomInfo@@V?$allocator@UWzCustomInfo@@@std@@@2@XZ 1000b713 f i wzanimationInfo.obj
 0001:0000a713       ?end@?$vector@UWzEffectInfo@@V?$allocator@UWzEffectInfo@@@std@@@std@@QAE?AV?$_Vector_iterator@UWzEffectInfo@@V?$allocator@UWzEffectInfo@@@std@@@2@XZ 1000b713 f i wzanimationInfo.obj
 0001:0000a769       ?insert@?$vector@HV?$allocator@H@std@@@std@@QAE?AV?$_Vector_iterator@HV?$allocator@H@std@@@2@V?$_Vector_const_iterator@HV?$allocator@H@std@@@2@ABH@Z 1000b769 f i wzdmeshsorter.obj
 0001:0000a7f9       ?_Buy@?$vector@HV?$allocator@H@std@@@std@@IAE_NI@Z 1000b7f9 f i wzdmeshsorter.obj
 0001:0000a8ab       ?_Tidy@?$vector@HV?$allocator@H@std@@@std@@IAEXXZ 1000b8ab f i wzdmeshsorter.obj
 0001:0000a91c       ?_Insert@?$list@HV?$allocator@H@std@@@std@@QAEXV?$_Const_iterator@$00@12@ABH@Z 1000b91c f i wzdmeshsorter.obj
 0001:0000a96a       ?_Buynode@?$list@HV?$allocator@H@std@@@std@@IAEPAU_Node@?$_List_nod@HV?$allocator@H@std@@@2@XZ 1000b96a f i wzdmeshsorter.obj
 0001:0000aa4c       ?_Tidy@?$list@HV?$allocator@H@std@@@std@@IAEXXZ 1000ba4c f i wzdmeshsorter.obj
 0001:0000aa81       ??D?$_Const_iterator@$00@?$list@HV?$allocator@H@std@@@std@@QBEABHXZ 1000ba81 f i wzdmeshsorter.obj
 0001:0000aaf5       ??E?$_Const_iterator@$00@?$list@HV?$allocator@H@std@@@std@@QAEAAV012@XZ 1000baf5 f i wzdmeshsorter.obj
 0001:0000ab77       ??8?$_Const_iterator@$00@?$list@HV?$allocator@H@std@@@std@@QBE_NABV012@@Z 1000bb77 f i wzdmeshsorter.obj
 0001:0000abc9       ?_Insert_n@?$vector@HV?$allocator@H@std@@@std@@IAEXV?$_Vector_const_iterator@HV?$allocator@H@std@@@2@IABH@Z 1000bbc9 f i wzdmeshsorter.obj
 0001:0000b1d7       ??0logic_error@std@@QAE@ABV?$basic_string@DU?$char_traits@D@std@@V?$allocator@D@2@@1@@Z 1000c1d7 f i wzdmeshsorter.obj
 0001:0000b252       ?what@logic_error@std@@UBEPBDXZ 1000c252 f i wzdmeshsorter.obj
 0001:0000b286       ??_Glogic_error@std@@UAEPAXI@Z 1000c286 f i wzdmeshsorter.obj
 0001:0000b286       ??_Elogic_error@std@@UAEPAXI@Z 1000c286 f i wzdmeshsorter.obj
 0001:0000b2af       ??1logic_error@std@@UAE@XZ 1000c2af f i wzdmeshsorter.obj
 0001:0000b2da       ??1length_error@std@@UAE@XZ 1000c2da f i wzdmeshsorter.obj
 0001:0000b2f6       ??_Elength_error@std@@UAEPAXI@Z 1000c2f6 f i wzdmeshsorter.obj
 0001:0000b2f6       ??_Glength_error@std@@UAEPAXI@Z 1000c2f6 f i wzdmeshsorter.obj
 0001:0000b328       ??1?$basic_string@DU?$char_traits@D@std@@V?$allocator@D@2@@std@@QAE@XZ 1000c328 f i wzdmeshsorter.obj
 0001:0000b33f       ?assign@?$basic_string@DU?$char_traits@D@std@@V?$allocator@D@2@@std@@QAEAAV12@ABV12@II@Z 1000c33f f i wzdmeshsorter.obj
 0001:0000b462       ?_Tidy@?$basic_string@DU?$char_traits@D@std@@V?$allocator@D@2@@std@@IAEX_NI@Z 1000c462 f i wzdmeshsorter.obj
 0001:0000b505       ?erase@?$basic_string@DU?$char_traits@D@std@@V?$allocator@D@2@@std@@QAEAAV12@II@Z 1000c505 f i wzdmeshsorter.obj
 0001:0000b609       ?_Grow@?$basic_string@DU?$char_traits@D@std@@V?$allocator@D@2@@std@@IAE_NI_N@Z 1000c609 f i wzdmeshsorter.obj
 0001:0000b6ea       ??0?$_Container_base_aux_alloc_real@V?$allocator@UWzEffectInfo@@@std@@@std@@IAE@V?$allocator@UWzEffectInfo@@@1@@Z 1000c6ea f i wzanimationInfo.obj
 0001:0000b6ea       ??0?$_Container_base_aux_alloc_real@V?$allocator@H@std@@@std@@IAE@V?$allocator@H@1@@Z 1000c6ea f i wzdmeshsorter.obj
 0001:0000b6ea       ??0?$_Container_base_aux_alloc_real@V?$allocator@UWzCustomInfo@@@std@@@std@@IAE@V?$allocator@UWzCustomInfo@@@1@@Z 1000c6ea f i wzanimationInfo.obj
 0001:0000b6ea       ??0?$_Container_base_aux_alloc_real@V?$allocator@UWzSoundInfo@@@std@@@std@@IAE@V?$allocator@UWzSoundInfo@@@1@@Z 1000c6ea f i wzanimationInfo.obj
 0001:0000b6ea       ??0?$_Container_base_aux_alloc_real@V?$allocator@U?$pair@$$CBHUWzVector@@@std@@@std@@@std@@IAE@V?$allocator@U?$pair@$$CBHUWzVector@@@std@@@1@@Z 1000c6ea f i wzunitskeleton.obj
 0001:0000b768       ?clear@?$list@HV?$allocator@H@std@@@std@@QAEXXZ 1000c768 f i wzdmeshsorter.obj
 0001:0000b7d4       ?_Buynode@?$list@HV?$allocator@H@std@@@std@@IAEPAU_Node@?$_List_nod@HV?$allocator@H@std@@@2@PAU342@0ABH@Z 1000c7d4 f i wzdmeshsorter.obj
 0001:0000b8d8       ?_Incsize@?$list@HV?$allocator@H@std@@@std@@IAEXI@Z 1000c8d8 f i wzdmeshsorter.obj
 0001:0000b9a2       ??0?$_List_ptr@HV?$allocator@H@std@@@std@@IAE@V?$allocator@H@1@@Z 1000c9a2 f i wzdmeshsorter.obj
 0001:0000b9d2       ??G?$_Vector_const_iterator@HV?$allocator@H@std@@@std@@QBEHABV01@@Z 1000c9d2 f i wzdmeshsorter.obj
 0001:0000ba1d       ??0length_error@std@@QAE@ABV01@@Z 1000ca1d f i wzdmeshsorter.obj
 0001:0000ba41       ??0logic_error@std@@QAE@ABV01@@Z 1000ca41 f i wzdmeshsorter.obj
 0001:0000bac3       ??0?$basic_string@DU?$char_traits@D@std@@V?$allocator@D@2@@std@@QAE@PBD@Z 1000cac3 f i wzdmeshsorter.obj
 0001:0000bb1a       ?_Copy@?$basic_string@DU?$char_traits@D@std@@V?$allocator@D@2@@std@@IAEXII@Z 1000cb1a f i wzdmeshsorter.obj
 0001:0000bd46       ??Y?$_Vector_const_iterator@HV?$allocator@H@std@@@std@@QAEAAV01@H@Z 1000cd46 f i wzdmeshsorter.obj
 0001:0000bdfc       ?assign@?$basic_string@DU?$char_traits@D@std@@V?$allocator@D@2@@std@@QAEAAV12@PBDI@Z 1000cdfc f i wzdmeshsorter.obj
 0001:0000bede       ?_Inside@?$basic_string@DU?$char_traits@D@std@@V?$allocator@D@2@@std@@IAE_NPBD@Z 1000cede f i wzdmeshsorter.obj
 0001:0000bf49       ??1bad_alloc@std@@UAE@XZ   1000cf49 f i wzdmeshsorter.obj
 0001:0000bf63       ??_Gbad_alloc@std@@UAEPAXI@Z 1000cf63 f i wzdmeshsorter.obj
 0001:0000bf63       ??_Ebad_alloc@std@@UAEPAXI@Z 1000cf63 f i wzdmeshsorter.obj
 0001:0000bf93       ??$_Umove@PAH@?$vector@HV?$allocator@H@std@@@std@@IAEPAHPAH00@Z 1000cf93 f i wzdmeshsorter.obj
 0001:0000bff0       ??$_Unchecked_move_backward@PAHPAH@stdext@@YAPAHPAH00@Z 1000cff0 f i wzdmeshsorter.obj
 0001:0000c087       ??$_Allocate@U_Node@?$_List_nod@HV?$allocator@H@std@@@std@@@std@@YAPAU_Node@?$_List_nod@HV?$allocator@H@std@@@0@IPAU120@@Z 1000d087 f i wzdmeshsorter.obj
 0001:0000c0da       ??$_Allocate@H@std@@YAPAHIPAH@Z 1000d0da f i wzdmeshsorter.obj
 0001:0000c0da       ??$_Allocate@V_Aux_cont@std@@@std@@YAPAV_Aux_cont@0@IPAV10@@Z 1000d0da f i wzdmeshsorter.obj
 0001:0000c12d       ??$_Allocate@D@std@@YAPADIPAD@Z 1000d12d f i wzdmeshsorter.obj
 0001:0000c17c       ??0bad_alloc@std@@QAE@ABV01@@Z 1000d17c f i wzdmeshsorter.obj
 0001:0000c19e       ??$_Sort@PAHH@std@@YAXPAH0H@Z 1000d19e f i wzdmeshsorter.obj
 0001:0000c26c       ??$_Unchecked_uninitialized_move@PAHPAHV?$allocator@H@std@@@stdext@@YAPAHPAH00AAV?$allocator@H@std@@@Z 1000d26c f i wzdmeshsorter.obj
 0001:0000c2ae       ??$_Unguarded_partition@PAH@std@@YA?AU?$pair@PAHPAH@0@PAH0@Z 1000d2ae f i wzdmeshsorter.obj
 0001:0000c5a3       ??$make_heap@PAH@std@@YAXPAH0@Z 1000d5a3 f i wzdmeshsorter.obj
 0001:0000c605       ??$sort_heap@PAH@std@@YAXPAH0@Z 1000d605 f i wzdmeshsorter.obj
 0001:0000c647       ??$unchecked_fill_n@PAHIH@stdext@@YAXPAHIABH@Z 1000d647 f i wzdmeshsorter.obj
 0001:0000c6b1       ??$_Median@PAH@std@@YAXPAH00@Z 1000d6b1 f i wzdmeshsorter.obj
 0001:0000ca04       ??$_Insertion_sort1@PAHH@std@@YAXPAH00@Z 1000da04 f i wzdmeshsorter.obj
 0001:0000caa5       ??$unchecked_uninitialized_copy@PAHPAHV?$allocator@H@std@@@stdext@@YAPAHPAH00AAV?$allocator@H@std@@@Z 1000daa5 f i wzdmeshsorter.obj
 0001:0000cb10       ??$_Adjust_heap@PAHHH@std@@YAXPAHHHH@Z 1000db10 f i wzdmeshsorter.obj
 0001:0000cbaa       ??$pop_heap@PAH@std@@YAXPAH0@Z 1000dbaa f i wzdmeshsorter.obj
 0001:0000cbfd       ??$unchecked_copy_backward@PAHPAH@stdext@@YAPAHPAH00@Z 1000dbfd f i wzdmeshsorter.obj
 0001:0000cc70       ??$_Push_heap@PAHHH@std@@YAXPAHHHH@Z 1000dc70 f i wzdmeshsorter.obj
 0001:0000ccce       ??0CWzdShareInfo@@AAE@XZ   1000dcce f   wzdshareinfo.obj
 0001:0000cce8       ??1CWzdShareInfo@@AAE@XZ   1000dce8 f   wzdshareinfo.obj
 0001:0000ccf1       ?Initialize@CWzdShareInfo@@AAEXXZ 1000dcf1 f   wzdshareinfo.obj
 0001:0000ce44       ?OnCameraDirChange@CWzdShareInfo@@QAEXXZ 1000de44 f   wzdshareinfo.obj
 0001:0000cea2       ?SetLightDir@CWzdShareInfo@@QAEXABUWzVector@@@Z 1000dea2 f   wzdshareinfo.obj
 0001:0000cedd       ?CalculateBlinnVector@CWzdShareInfo@@AAEXXZ 1000dedd f   wzdshareinfo.obj
 0001:0000cfc0       ??0WzAnimationInfo@@QAE@XZ 1000dfc0 f   wzanimationInfo.obj
 0001:0000d0be       ??1WzAnimationInfo@@QAE@XZ 1000e0be f   wzanimationInfo.obj
 0001:0000d1c1       ?AddSoundInfo@WzAnimationInfo@@QAEXPBUWzSoundInfo@@@Z 1000e1c1 f   wzanimationInfo.obj
 0001:0000d1dc       ?GetSoundInfo@WzAnimationInfo@@QAEPAUWzSoundInfo@@H@Z 1000e1dc f   wzanimationInfo.obj
 0001:0000d242       ?GetNumSoundInfo@WzAnimationInfo@@QBEHXZ 1000e242 f   wzanimationInfo.obj
 0001:0000d264       ?AddSound@WzAnimationInfo@@QAEXHMH@Z 1000e264 f   wzanimationInfo.obj
 0001:0000d3c7       ?DelSoundIndex@WzAnimationInfo@@QAEXHH@Z 1000e3c7 f   wzanimationInfo.obj
 0001:0000d52e       ?ClearSoundIndex@WzAnimationInfo@@QAEXH@Z 1000e52e f   wzanimationInfo.obj
 0001:0000d599       ?GetNumSound@WzAnimationInfo@@QBEHH@Z 1000e599 f   wzanimationInfo.obj
 0001:0000d61a       ?GetSound@WzAnimationInfo@@QBEHHH@Z 1000e61a f   wzanimationInfo.obj
 0001:0000d71a       ?SetSoundFrame@WzAnimationInfo@@QAEXMH@Z 1000e71a f   wzanimationInfo.obj
 0001:0000d786       ?GetSoundFrame@WzAnimationInfo@@QBEMH@Z 1000e786 f   wzanimationInfo.obj
 0001:0000d7ef       ?SetVoiceChannel@WzAnimationInfo@@QAEXHH@Z 1000e7ef f   wzanimationInfo.obj
 0001:0000d858       ?IsVoiceChannel@WzAnimationInfo@@QBEHH@Z 1000e858 f   wzanimationInfo.obj
 0001:0000d8c2       ?DelSoundSetIndex@WzAnimationInfo@@QAEXH@Z 1000e8c2 f   wzanimationInfo.obj
 0001:0000d959       ?ClearAllSound@WzAnimationInfo@@QAEXXZ 1000e959 f   wzanimationInfo.obj
 0001:0000d96f       ?AddEffectInfo@WzAnimationInfo@@QAEXPBUWzEffectInfo@@@Z 1000e96f f   wzanimationInfo.obj
 0001:0000d990       ?SetEffectInfo@WzAnimationInfo@@QAEXPBUWzEffectInfo@@H@Z 1000e990 f   wzanimationInfo.obj
 0001:0000da0c       ?DelEffectIndex@WzAnimationInfo@@QAEXH@Z 1000ea0c f   wzanimationInfo.obj
 0001:0000da97       ?GetEffectInfo@WzAnimationInfo@@QAEPAUWzEffectInfo@@H@Z 1000ea97 f   wzanimationInfo.obj
 0001:0000db03       ?AddCustomInfo@WzAnimationInfo@@QAEXPBUWzCustomInfo@@@Z 1000eb03 f   wzanimationInfo.obj
 0001:0000db27       ?SetCustomInfo@WzAnimationInfo@@QAEXPBUWzCustomInfo@@H@Z 1000eb27 f   wzanimationInfo.obj
 0001:0000dba7       ?DelCustomIndex@WzAnimationInfo@@QAEXH@Z 1000eba7 f   wzanimationInfo.obj
 0001:0000dc3e       ?GetCustomInfo@WzAnimationInfo@@QAEPAUWzCustomInfo@@H@Z 1000ec3e f   wzanimationInfo.obj
 0001:0000dcae       ?AddBV@WzAnimationInfo@@QAEXPBUBvAABB@@@Z 1000ecae f   wzanimationInfo.obj
 0001:0000dcf0       ?DeleteAllBV@WzAnimationInfo@@QAEXXZ 1000ecf0 f   wzanimationInfo.obj
 0001:0000dd57       ??4WzAnimationInfo@@QAEAAV0@ABV0@@Z 1000ed57 f   wzanimationInfo.obj
 0001:0000de8f       ??1WzSoundInfo@@QAE@XZ     1000ee8f f i wzanimationInfo.obj
 0001:0000deee       ?erase@?$vector@HV?$allocator@H@std@@@std@@QAE?AV?$_Vector_iterator@HV?$allocator@H@std@@@2@V?$_Vector_const_iterator@HV?$allocator@H@std@@@2@@Z 1000eeee f i wzanimationInfo.obj
 0001:0000df8a       ?clear@?$vector@HV?$allocator@H@std@@@std@@QAEXXZ 1000ef8a f i wzanimationInfo.obj
 0001:0000dfdb       ??0?$vector@UWzSoundInfo@@V?$allocator@UWzSoundInfo@@@std@@@std@@QAE@XZ 1000efdb f i wzanimationInfo.obj
 0001:0000e05d       ??1?$vector@UWzSoundInfo@@V?$allocator@UWzSoundInfo@@@std@@@std@@QAE@XZ 1000f05d f i wzanimationInfo.obj
 0001:0000e0b3       ??4?$vector@UWzSoundInfo@@V?$allocator@UWzSoundInfo@@@std@@@std@@QAEAAV01@ABV01@@Z 1000f0b3 f i wzanimationInfo.obj
 0001:0000e3cc       ?begin@?$vector@UWzCustomInfo@@V?$allocator@UWzCustomInfo@@@std@@@std@@QAE?AV?$_Vector_iterator@UWzCustomInfo@@V?$allocator@UWzCustomInfo@@@std@@@2@XZ 1000f3cc f i wzanimationInfo.obj
 0001:0000e3cc       ?begin@?$vector@UWzSoundInfo@@V?$allocator@UWzSoundInfo@@@std@@@std@@QAE?AV?$_Vector_iterator@UWzSoundInfo@@V?$allocator@UWzSoundInfo@@@std@@@2@XZ 1000f3cc f i wzanimationInfo.obj
 0001:0000e3cc       ?begin@?$vector@HV?$allocator@H@std@@@std@@QAE?AV?$_Vector_iterator@HV?$allocator@H@std@@@2@XZ 1000f3cc f i wzdmeshsorter.obj
 0001:0000e3cc       ?begin@?$vector@UWzEffectInfo@@V?$allocator@UWzEffectInfo@@@std@@@std@@QAE?AV?$_Vector_iterator@UWzEffectInfo@@V?$allocator@UWzEffectInfo@@@std@@@2@XZ 1000f3cc f i wzanimationInfo.obj
 0001:0000e3cc       ?begin@?$vector@HV?$allocator@H@std@@@std@@QBE?AV?$_Vector_const_iterator@HV?$allocator@H@std@@@2@XZ 1000f3cc f i wzanimationInfo.obj
 0001:0000e422       ?push_back@?$vector@UWzSoundInfo@@V?$allocator@UWzSoundInfo@@@std@@@std@@QAEXABUWzSoundInfo@@@Z 1000f422 f i wzanimationInfo.obj
 0001:0000e4e1       ?erase@?$vector@UWzSoundInfo@@V?$allocator@UWzSoundInfo@@@std@@@std@@QAE?AV?$_Vector_iterator@UWzSoundInfo@@V?$allocator@UWzSoundInfo@@@std@@@2@V?$_Vector_const_iterator@UWzSoundInfo@@V?$allocator@UWzSoundInfo@@@std@@@2@@Z 1000f4e1 f i wzanimationInfo.obj
 0001:0000e5dc       ?clear@?$vector@UWzSoundInfo@@V?$allocator@UWzSoundInfo@@@std@@@std@@QAEXXZ 1000f5dc f i wzanimationInfo.obj
 0001:0000e62d       ??0?$vector@UWzEffectInfo@@V?$allocator@UWzEffectInfo@@@std@@@std@@QAE@XZ 1000f62d f i wzanimationInfo.obj
 0001:0000e6af       ??1?$vector@UWzEffectInfo@@V?$allocator@UWzEffectInfo@@@std@@@std@@QAE@XZ 1000f6af f i wzanimationInfo.obj
 0001:0000e705       ??4?$vector@UWzEffectInfo@@V?$allocator@UWzEffectInfo@@@std@@@std@@QAEAAV01@ABV01@@Z 1000f705 f i wzanimationInfo.obj
 0001:0000ea10       ?push_back@?$vector@UWzEffectInfo@@V?$allocator@UWzEffectInfo@@@std@@@std@@QAEXABUWzEffectInfo@@@Z 1000fa10 f i wzanimationInfo.obj
 0001:0000ead5       ?erase@?$vector@UWzEffectInfo@@V?$allocator@UWzEffectInfo@@@std@@@std@@QAE?AV?$_Vector_iterator@UWzEffectInfo@@V?$allocator@UWzEffectInfo@@@std@@@2@V?$_Vector_const_iterator@UWzEffectInfo@@V?$allocator@UWzEffectInfo@@@std@@@2@@Z 1000fad5 f i wzanimationInfo.obj
 0001:0000eb8c       ??0?$vector@UWzCustomInfo@@V?$allocator@UWzCustomInfo@@@std@@@std@@QAE@XZ 1000fb8c f i wzanimationInfo.obj
 0001:0000ec0e       ??1?$vector@UWzCustomInfo@@V?$allocator@UWzCustomInfo@@@std@@@std@@QAE@XZ 1000fc0e f i wzanimationInfo.obj
 0001:0000ec64       ??4?$vector@UWzCustomInfo@@V?$allocator@UWzCustomInfo@@@std@@@std@@QAEAAV01@ABV01@@Z 1000fc64 f i wzanimationInfo.obj
 0001:0000ef6f       ?push_back@?$vector@UWzCustomInfo@@V?$allocator@UWzCustomInfo@@@std@@@std@@QAEXABUWzCustomInfo@@@Z 1000ff6f f i wzanimationInfo.obj
 0001:0000f034       ?erase@?$vector@UWzCustomInfo@@V?$allocator@UWzCustomInfo@@@std@@@std@@QAE?AV?$_Vector_iterator@UWzCustomInfo@@V?$allocator@UWzCustomInfo@@@std@@@2@V?$_Vector_const_iterator@UWzCustomInfo@@V?$allocator@UWzCustomInfo@@@std@@@2@@Z 10010034 f i wzanimationInfo.obj
 0001:0000f0eb       ?erase@?$vector@HV?$allocator@H@std@@@std@@QAE?AV?$_Vector_iterator@HV?$allocator@H@std@@@2@V?$_Vector_const_iterator@HV?$allocator@H@std@@@2@0@Z 100100eb f i wzanimationInfo.obj
 0001:0000f17b       ?insert@?$vector@UWzSoundInfo@@V?$allocator@UWzSoundInfo@@@std@@@std@@QAE?AV?$_Vector_iterator@UWzSoundInfo@@V?$allocator@UWzSoundInfo@@@std@@@2@V?$_Vector_const_iterator@UWzSoundInfo@@V?$allocator@UWzSoundInfo@@@std@@@2@ABUWzSoundInfo@@@Z 1001017b f i wzanimationInfo.obj
 0001:0000f20b       ?erase@?$vector@UWzSoundInfo@@V?$allocator@UWzSoundInfo@@@std@@@std@@QAE?AV?$_Vector_iterator@UWzSoundInfo@@V?$allocator@UWzSoundInfo@@@std@@@2@V?$_Vector_const_iterator@UWzSoundInfo@@V?$allocator@UWzSoundInfo@@@std@@@2@0@Z 1001020b f i wzanimationInfo.obj
 0001:0000f314       ?_Buy@?$vector@UWzSoundInfo@@V?$allocator@UWzSoundInfo@@@std@@@std@@IAE_NI@Z 10010314 f i wzanimationInfo.obj
 0001:0000f3c6       ?_Tidy@?$vector@UWzSoundInfo@@V?$allocator@UWzSoundInfo@@@std@@@std@@IAEXXZ 100103c6 f i wzanimationInfo.obj
 0001:0000f462       ?insert@?$vector@UWzEffectInfo@@V?$allocator@UWzEffectInfo@@@std@@@std@@QAE?AV?$_Vector_iterator@UWzEffectInfo@@V?$allocator@UWzEffectInfo@@@std@@@2@V?$_Vector_const_iterator@UWzEffectInfo@@V?$allocator@UWzEffectInfo@@@std@@@2@ABUWzEffectInfo@@@Z 10010462 f i wzanimationInfo.obj
 0001:0000f4f5       ?clear@?$vector@UWzEffectInfo@@V?$allocator@UWzEffectInfo@@@std@@@std@@QAEXXZ 100104f5 f i wzanimationInfo.obj
 0001:0000f546       ?_Buy@?$vector@UWzEffectInfo@@V?$allocator@UWzEffectInfo@@@std@@@std@@IAE_NI@Z 10010546 f i wzanimationInfo.obj
 0001:0000f5f8       ?_Tidy@?$vector@UWzEffectInfo@@V?$allocator@UWzEffectInfo@@@std@@@std@@IAEXXZ 100105f8 f i wzanimationInfo.obj
 0001:0000f687       ?insert@?$vector@UWzCustomInfo@@V?$allocator@UWzCustomInfo@@@std@@@std@@QAE?AV?$_Vector_iterator@UWzCustomInfo@@V?$allocator@UWzCustomInfo@@@std@@@2@V?$_Vector_const_iterator@UWzCustomInfo@@V?$allocator@UWzCustomInfo@@@std@@@2@ABUWzCustomInfo@@@Z 10010687 f i wzanimationInfo.obj
 0001:0000f71a       ?clear@?$vector@UWzCustomInfo@@V?$allocator@UWzCustomInfo@@@std@@@std@@QAEXXZ 1001071a f i wzanimationInfo.obj
 0001:0000f76b       ?_Buy@?$vector@UWzCustomInfo@@V?$allocator@UWzCustomInfo@@@std@@@std@@IAE_NI@Z 1001076b f i wzanimationInfo.obj
 0001:0000f81d       ?_Tidy@?$vector@UWzCustomInfo@@V?$allocator@UWzCustomInfo@@@std@@@std@@IAEXXZ 1001081d f i wzanimationInfo.obj
 0001:0000f8ac       ?_Insert_n@?$vector@UWzSoundInfo@@V?$allocator@UWzSoundInfo@@@std@@@std@@IAEXV?$_Vector_const_iterator@UWzSoundInfo@@V?$allocator@UWzSoundInfo@@@std@@@2@IABUWzSoundInfo@@@Z 100108ac f i wzanimationInfo.obj
 0001:00010020       ?_Xlen@?$vector@HV?$allocator@H@std@@@std@@KAXXZ 10011020 f i wzdmeshsorter.obj
 0001:00010020       ?_Xlen@?$vector@UWzSoundInfo@@V?$allocator@UWzSoundInfo@@@std@@@std@@KAXXZ 10011020 f i wzanimationInfo.obj
 0001:00010020       ?_Xlen@?$vector@UWzEffectInfo@@V?$allocator@UWzEffectInfo@@@std@@@std@@KAXXZ 10011020 f i wzanimationInfo.obj
 0001:00010020       ?_Xlen@?$vector@UWzCustomInfo@@V?$allocator@UWzCustomInfo@@@std@@@std@@KAXXZ 10011020 f i wzanimationInfo.obj
 0001:00010097       ?erase@?$vector@UWzEffectInfo@@V?$allocator@UWzEffectInfo@@@std@@@std@@QAE?AV?$_Vector_iterator@UWzEffectInfo@@V?$allocator@UWzEffectInfo@@@std@@@2@V?$_Vector_const_iterator@UWzEffectInfo@@V?$allocator@UWzEffectInfo@@@std@@@2@0@Z 10011097 f i wzanimationInfo.obj
 0001:00010142       ?_Insert_n@?$vector@UWzEffectInfo@@V?$allocator@UWzEffectInfo@@@std@@@std@@IAEXV?$_Vector_const_iterator@UWzEffectInfo@@V?$allocator@UWzEffectInfo@@@std@@@2@IABUWzEffectInfo@@@Z 10011142 f i wzanimationInfo.obj
 0001:00010860       ?erase@?$vector@UWzCustomInfo@@V?$allocator@UWzCustomInfo@@@std@@@std@@QAE?AV?$_Vector_iterator@UWzCustomInfo@@V?$allocator@UWzCustomInfo@@@std@@@2@V?$_Vector_const_iterator@UWzCustomInfo@@V?$allocator@UWzCustomInfo@@@std@@@2@0@Z 10011860 f i wzanimationInfo.obj
 0001:0001090b       ?_Insert_n@?$vector@UWzCustomInfo@@V?$allocator@UWzCustomInfo@@@std@@@std@@IAEXV?$_Vector_const_iterator@UWzCustomInfo@@V?$allocator@UWzCustomInfo@@@std@@@2@IABUWzCustomInfo@@@Z 1001190b f i wzanimationInfo.obj
 0001:0001101a       ??0?$_Vector_const_iterator@UWzSoundInfo@@V?$allocator@UWzSoundInfo@@@std@@@std@@QAE@PAUWzSoundInfo@@PBV_Container_base_aux@1@@Z 1001201a f i wzanimationInfo.obj
 0001:0001101a       ??0?$_Vector_const_iterator@UWzCustomInfo@@V?$allocator@UWzCustomInfo@@@std@@@std@@QAE@PAUWzCustomInfo@@PBV_Container_base_aux@1@@Z 1001201a f i wzanimationInfo.obj
 0001:0001101a       ??0?$_Vector_const_iterator@UWzEffectInfo@@V?$allocator@UWzEffectInfo@@@std@@@std@@QAE@PAUWzEffectInfo@@PBV_Container_base_aux@1@@Z 1001201a f i wzanimationInfo.obj
 0001:0001101a       ??0?$_Vector_const_iterator@HV?$allocator@H@std@@@std@@QAE@PAHPBV_Container_base_aux@1@@Z 1001201a f i wzanimationInfo.obj
 0001:00011066       ??Y?$_Vector_const_iterator@UWzSoundInfo@@V?$allocator@UWzSoundInfo@@@std@@@std@@QAEAAV01@H@Z 10012066 f i wzanimationInfo.obj
 0001:0001111c       ??G?$_Vector_const_iterator@UWzSoundInfo@@V?$allocator@UWzSoundInfo@@@std@@@std@@QBEHABV01@@Z 1001211c f i wzanimationInfo.obj
 0001:00011167       ??Y?$_Vector_const_iterator@UWzEffectInfo@@V?$allocator@UWzEffectInfo@@@std@@@std@@QAEAAV01@H@Z 10012167 f i wzanimationInfo.obj
 0001:0001121d       ??G?$_Vector_const_iterator@UWzEffectInfo@@V?$allocator@UWzEffectInfo@@@std@@@std@@QBEHABV01@@Z 1001221d f i wzanimationInfo.obj
 0001:0001126b       ??Y?$_Vector_const_iterator@UWzCustomInfo@@V?$allocator@UWzCustomInfo@@@std@@@std@@QAEAAV01@H@Z 1001226b f i wzanimationInfo.obj
 0001:00011321       ??G?$_Vector_const_iterator@UWzCustomInfo@@V?$allocator@UWzCustomInfo@@@std@@@std@@QBEHABV01@@Z 10012321 f i wzanimationInfo.obj
 0001:0001136f       ??0?$vector@HV?$allocator@H@std@@@std@@QAE@ABV01@@Z 1001236f f i wzanimationInfo.obj
 0001:000114e9       ??8const_iterator@?$_Tree@V?$_Tmap_traits@HUWzVector@@U?$less@H@std@@V?$allocator@U?$pair@$$CBHUWzVector@@@std@@@3@$0A@@std@@@std@@QBE_NABV012@@Z 100124e9 f i wzdanimation.obj
 0001:000114e9       ??8?$_Vector_const_iterator@HV?$allocator@H@std@@@std@@QBE_NABV01@@Z 100124e9 f i wzanimationInfo.obj
 0001:000114e9       ??8?$_Vector_const_iterator@UWzEffectInfo@@V?$allocator@UWzEffectInfo@@@std@@@std@@QBE_NABV01@@Z 100124e9 f i wzanimationInfo.obj
 0001:000114e9       ??8?$_Vector_const_iterator@UWzCustomInfo@@V?$allocator@UWzCustomInfo@@@std@@@std@@QBE_NABV01@@Z 100124e9 f i wzanimationInfo.obj
 0001:000114e9       ??8?$_Vector_const_iterator@UWzSoundInfo@@V?$allocator@UWzSoundInfo@@@std@@@std@@QBE_NABV01@@Z 100124e9 f i wzanimationInfo.obj
 0001:00011536       ??0?$CWzArray@PAUBvAABB@@@@QAE@XZ 10012536 f i wzanimationInfo.obj
 0001:0001159e       ?Clear@?$CWzArray@PAUWzBVExtraInfo@@@@QAEXXZ 1001259e f i wzunit.obj
 0001:0001159e       ?Clear@?$CWzArray@PAUWzBoneScaling@@@@QAEXXZ 1001259e f i wzunitsubtype.obj
 0001:0001159e       ?Clear@?$CWzArray@PAUWzTexAniMappingInfo@@@@QAEXXZ 1001259e f i wzunit.obj
 0001:0001159e       ?Clear@?$CWzArray@PAUWzMappingInfo@@@@QAEXXZ 1001259e f i wzunit.obj
 0001:0001159e       ?Clear@?$CWzArray@PAUWzDecoration@@@@QAEXXZ 1001259e f i wzunitsubtype.obj
 0001:0001159e       ?Clear@?$CWzArray@PAVCWzUnitSubType@@@@QAEXXZ 1001259e f i wzunit.obj
 0001:0001159e       ?Clear@?$CWzArray@PAUBvAABB@@@@QAEXXZ 1001259e f i wzanimationInfo.obj
 0001:0001159e       ?Clear@?$CWzArray@PAUWzTexAniSetInfo@@@@QAEXXZ 1001259e f i wzunit.obj
 0001:0001159e       ?Clear@?$CWzArray@K@@QAEXXZ 1001259e f i wzunit.obj
 0001:0001159e       ?Clear@?$CWzArray@PAUMeshGroupNameInfo@@@@QAEXXZ 1001259e f i wzunit.obj
 0001:0001159e       ?Clear@?$CWzArray@PAVWzAnimationInfo@@@@QAEXXZ 1001259e f i wzunit.obj
 0001:0001159e       ?Clear@?$CWzArray@PAUWzRenderInfo@@@@QAEXXZ 1001259e f i wzunitsubtype.obj
 0001:0001159e       ?Clear@?$CWzArray@PAUWzUnitEffectInfo@@@@QAEXXZ 1001259e f i wzunitdraw.obj
 0001:0001159e       ?Clear@?$CWzArray@PAUWzBoneInfo@@@@QAEXXZ 1001259e f i wzunit.obj
 0001:000115c7       ?Get@?$CWzArray@PAUBvAABB@@@@QBEAAPAUBvAABB@@H@Z 100125c7 f i wzanimationInfo.obj
 0001:000115f6       ??$unchecked_copy@PAHPAH@stdext@@YAPAHPAH00@Z 100125f6 f i wzanimationInfo.obj
 0001:00011667       ??$unchecked_copy@PAUWzSoundInfo@@PAU1@@stdext@@YAPAUWzSoundInfo@@PAU1@00@Z 10012667 f i wzanimationInfo.obj
 0001:000116a3       ??$_Ucopy@PAUWzSoundInfo@@@?$vector@UWzSoundInfo@@V?$allocator@UWzSoundInfo@@@std@@@std@@IAEPAUWzSoundInfo@@PAU2@00@Z 100126a3 f i wzanimationInfo.obj
 0001:000116fa       ??$unchecked_copy@PAUWzEffectInfo@@PAU1@@stdext@@YAPAUWzEffectInfo@@PAU1@00@Z 100126fa f i wzanimationInfo.obj
 0001:00011795       ??$_Ucopy@PAUWzEffectInfo@@@?$vector@UWzEffectInfo@@V?$allocator@UWzEffectInfo@@@std@@@std@@IAEPAUWzEffectInfo@@PAU2@00@Z 10012795 f i wzanimationInfo.obj
 0001:000117ec       ??$unchecked_copy@PAUWzCustomInfo@@PAU1@@stdext@@YAPAUWzCustomInfo@@PAU1@00@Z 100127ec f i wzanimationInfo.obj
 0001:00011887       ??$_Ucopy@PAUWzCustomInfo@@@?$vector@UWzCustomInfo@@V?$allocator@UWzCustomInfo@@@std@@@std@@IAEPAUWzCustomInfo@@PAU2@00@Z 10012887 f i wzanimationInfo.obj
 0001:000118de       ??$_Umove@PAUWzSoundInfo@@@?$vector@UWzSoundInfo@@V?$allocator@UWzSoundInfo@@@std@@@std@@IAEPAUWzSoundInfo@@PAU2@00@Z 100128de f i wzanimationInfo.obj
 0001:00011903       ??$fill@PAUWzSoundInfo@@U1@@std@@YAXPAUWzSoundInfo@@0ABU1@@Z 10012903 f i wzanimationInfo.obj
 0001:00011954       ??$_Unchecked_move_backward@PAUWzSoundInfo@@PAU1@@stdext@@YAPAUWzSoundInfo@@PAU1@00@Z 10012954 f i wzanimationInfo.obj
 0001:000119b4       ??$_Umove@PAUWzEffectInfo@@@?$vector@UWzEffectInfo@@V?$allocator@UWzEffectInfo@@@std@@@std@@IAEPAUWzEffectInfo@@PAU2@00@Z 100129b4 f i wzanimationInfo.obj
 0001:000119d9       ??$_Unchecked_move_backward@PAUWzEffectInfo@@PAU1@@stdext@@YAPAUWzEffectInfo@@PAU1@00@Z 100129d9 f i wzanimationInfo.obj
 0001:00011a15       ??$_Allocate@UWzEffectInfo@@@std@@YAPAUWzEffectInfo@@IPAU1@@Z 10012a15 f i wzanimationInfo.obj
 0001:00011a68       ??$_Umove@PAUWzCustomInfo@@@?$vector@UWzCustomInfo@@V?$allocator@UWzCustomInfo@@@std@@@std@@IAEPAUWzCustomInfo@@PAU2@00@Z 10012a68 f i wzanimationInfo.obj
 0001:00011a8d       ??$_Unchecked_move_backward@PAUWzCustomInfo@@PAU1@@stdext@@YAPAUWzCustomInfo@@PAU1@00@Z 10012a8d f i wzanimationInfo.obj
 0001:00011ac9       ??$_Allocate@UWzCustomInfo@@@std@@YAPAUWzCustomInfo@@IPAU1@@Z 10012ac9 f i wzanimationInfo.obj
 0001:00011b1c       ??$_Copy_opt@PAUWzSoundInfo@@PAU1@@std@@YAPAUWzSoundInfo@@PAU1@00Urandom_access_iterator_tag@0@U_Nonscalar_ptr_iterator_tag@0@U_Range_checked_iterator_tag@0@@Z 10012b1c f i wzanimationInfo.obj
 0001:00011ba5       ??$_Copy_opt@PAUWzEffectInfo@@PAU1@@std@@YAPAUWzEffectInfo@@PAU1@00Urandom_access_iterator_tag@0@U_Nonscalar_ptr_iterator_tag@0@U_Range_checked_iterator_tag@0@@Z 10012ba5 f i wzanimationInfo.obj
 0001:00011c16       ??$_Copy_opt@PAUWzCustomInfo@@PAU1@@std@@YAPAUWzCustomInfo@@PAU1@00Urandom_access_iterator_tag@0@U_Nonscalar_ptr_iterator_tag@0@U_Range_checked_iterator_tag@0@@Z 10012c16 f i wzanimationInfo.obj
 0001:00011c87       ??$_Uninit_fill_n@PAUWzSoundInfo@@IU1@V?$allocator@UWzSoundInfo@@@std@@@std@@YAXPAUWzSoundInfo@@IABU1@AAV?$allocator@UWzSoundInfo@@@0@U_Nonscalar_ptr_iterator_tag@0@U_Range_checked_iterator_tag@0@@Z 10012c87 f i wzanimationInfo.obj
 0001:00011d2c       ??$_Uninit_fill_n@PAUWzEffectInfo@@IU1@V?$allocator@UWzEffectInfo@@@std@@@std@@YAXPAUWzEffectInfo@@IABU1@AAV?$allocator@UWzEffectInfo@@@0@U_Nonscalar_ptr_iterator_tag@0@U_Range_checked_iterator_tag@0@@Z 10012d2c f i wzanimationInfo.obj
 0001:00011de3       ??$_Uninit_fill_n@PAUWzCustomInfo@@IU1@V?$allocator@UWzCustomInfo@@@std@@@std@@YAXPAUWzCustomInfo@@IABU1@AAV?$allocator@UWzCustomInfo@@@0@U_Nonscalar_ptr_iterator_tag@0@U_Range_checked_iterator_tag@0@@Z 10012de3 f i wzanimationInfo.obj
 0001:00011e9a       ??$_Unchecked_uninitialized_move@PAUWzSoundInfo@@PAU1@V?$allocator@UWzSoundInfo@@@std@@@stdext@@YAPAUWzSoundInfo@@PAU1@00AAV?$allocator@UWzSoundInfo@@@std@@@Z 10012e9a f i wzanimationInfo.obj
 0001:00011f0c       ??$_Unchecked_uninitialized_move@PAUWzEffectInfo@@PAU1@V?$allocator@UWzEffectInfo@@@std@@@stdext@@YAPAUWzEffectInfo@@PAU1@00AAV?$allocator@UWzEffectInfo@@@std@@@Z 10012f0c f i wzanimationInfo.obj
 0001:00011f7e       ??$_Move_backward_opt@PAUWzEffectInfo@@PAU1@Urandom_access_iterator_tag@std@@U_Undefined_move_tag@3@@std@@YAPAUWzEffectInfo@@PAU1@00Urandom_access_iterator_tag@0@U_Undefined_move_tag@0@U_Range_checked_iterator_tag@0@@Z 10012f7e f i wzanimationInfo.obj
 0001:0001200d       ??$_Unchecked_uninitialized_move@PAUWzCustomInfo@@PAU1@V?$allocator@UWzCustomInfo@@@std@@@stdext@@YAPAUWzCustomInfo@@PAU1@00AAV?$allocator@UWzCustomInfo@@@std@@@Z 1001300d f i wzanimationInfo.obj
 0001:0001207f       ??$_Move_backward_opt@PAUWzCustomInfo@@PAU1@Urandom_access_iterator_tag@std@@U_Undefined_move_tag@3@@std@@YAPAUWzCustomInfo@@PAU1@00Urandom_access_iterator_tag@0@U_Undefined_move_tag@0@U_Range_checked_iterator_tag@0@@Z 1001307f f i wzanimationInfo.obj
 0001:0001210e       ??$unchecked_uninitialized_copy@V?$_Vector_const_iterator@HV?$allocator@H@std@@@std@@PAHV?$allocator@H@2@@stdext@@YAPAHV?$_Vector_const_iterator@HV?$allocator@H@std@@@std@@0PAHAAV?$allocator@H@2@@Z 1001310e f i wzanimationInfo.obj
 0001:00012179       ??4?$vector@HV?$allocator@H@std@@@std@@QAEAAV01@ABV01@@Z 10013179 f i wzanimationInfo.obj
 0001:00012432       ??$_Uninit_copy@PAUWzSoundInfo@@PAU1@V?$allocator@UWzSoundInfo@@@std@@@std@@YAPAUWzSoundInfo@@PAU1@00AAV?$allocator@UWzSoundInfo@@@0@U_Nonscalar_ptr_iterator_tag@0@U_Range_checked_iterator_tag@0@@Z 10013432 f i wzanimationInfo.obj
 0001:000124de       ??$_Uninit_copy@PAUWzEffectInfo@@PAU1@V?$allocator@UWzEffectInfo@@@std@@@std@@YAPAUWzEffectInfo@@PAU1@00AAV?$allocator@UWzEffectInfo@@@0@U_Nonscalar_ptr_iterator_tag@0@U_Range_checked_iterator_tag@0@@Z 100134de f i wzanimationInfo.obj
 0001:0001259c       ??$_Uninit_copy@PAUWzCustomInfo@@PAU1@V?$allocator@UWzCustomInfo@@@std@@@std@@YAPAUWzCustomInfo@@PAU1@00AAV?$allocator@UWzCustomInfo@@@0@U_Nonscalar_ptr_iterator_tag@0@U_Range_checked_iterator_tag@0@@Z 1001359c f i wzanimationInfo.obj
 0001:0001265a       ??$_Copy_backward_opt@PAUWzSoundInfo@@PAU1@@std@@YAPAUWzSoundInfo@@PAU1@00Urandom_access_iterator_tag@0@U_Nonscalar_ptr_iterator_tag@0@U_Range_checked_iterator_tag@0@@Z 1001365a f i wzanimationInfo.obj
 0001:000126e3       ??$_Construct@UWzSoundInfo@@U1@@std@@YAXPAUWzSoundInfo@@ABU1@@Z 100136e3 f i wzanimationInfo.obj
 0001:00012769       ??3@YAXPAX0@Z              10013769 f i wzanimationInfo.obj
 0001:0001276e       ??_GWzSoundInfo@@QAEPAXI@Z 1001376e f i wzanimationInfo.obj
 0001:000127e3       ??0CWzAniState@@QAE@XZ     100137e3 f   wzanistate.obj
 0001:0001287b       ??1CWzAniState@@UAE@XZ     1001387b f   wzanistate.obj
 0001:000128fa       ?InitVariables@CWzAniState@@AAEXXZ 100138fa f   wzanistate.obj
 0001:000129c3       ?Release@CWzAniState@@AAEXXZ 100139c3 f   wzanistate.obj
 0001:000129ef       ?Initialize@CWzAniState@@QAEXXZ 100139ef f   wzanistate.obj
 0001:00012a08       ?SetAnimationInfo@CWzAniState@@QAEXPAVWzAnimationInfo@@_N1H1@Z 10013a08 f   wzanistate.obj
 0001:00012aa7       ?CheckAnimationData@CWzAniState@@AAE_NXZ 10013aa7 f   wzanistate.obj
 0001:00012e89       ?ProgressFrame@CWzAniState@@QAE?AW4ENUM_ANI_FRAME_STATUS@@MPAUWzEvent@@MPAVWzAnimationInfo@@@Z 10013e89 f   wzanistate.obj
 0001:00013131       ?AnimateSimple@CWzAniState@@QAE_NPAUWzTransform@@@Z 10014131 f   wzanistate.obj
 0001:00013169       ?Animate@CWzAniState@@QAE_NPAUWzTransform@@PBU2@@Z 10014169 f   wzanistate.obj
 0001:000132cf       ?AnimateBlend@CWzAniState@@QAE_NPAUWzTransform@@@Z 100142cf f   wzanistate.obj
 0001:00013636       ?BlendTransform_typeS@CWzAniState@@AAEXPAUWzTransform@@HM@Z 10014636 f   wzanistate.obj
 0001:000136a9       ?BlendTransform_typeSD@CWzAniState@@AAEXPAUWzTransform@@HM@Z 100146a9 f   wzanistate.obj
 0001:0001381b       ?BlendTransform_typeE@CWzAniState@@AAEXPAUWzTransform@@HM@Z 1001481b f   wzanistate.obj
 0001:00013895       ?BlendTransform_typeED@CWzAniState@@AAEXPAUWzTransform@@HM@Z 10014895 f   wzanistate.obj
 0001:00013a18       ?BlendTransform_typeN@CWzAniState@@AAEXPAUWzTransform@@H@Z 10014a18 f   wzanistate.obj
 0001:00013a4b       ?BlendTransform_typeND@CWzAniState@@AAEXPAUWzTransform@@H@Z 10014a4b f   wzanistate.obj
 0001:00013b4d       ?CalcTransformMatrix@CWzAniState@@QAEXPAUWzMatrix@@PBUWzTransform@@PBUWzTransformParam@@@Z 10014b4d f   wzanistate.obj
 0001:00013b7b       ?SetBlendBoneIndex@CWzAniState@@QAEXH@Z 10014b7b f   wzanistate.obj
 0001:00013b97       ?ResetBlendBoneList@CWzAniState@@AAEXXZ 10014b97 f   wzanistate.obj
 0001:00013be4       ?AddBlendBone@CWzAniState@@AAEXPBUWzNode@@H@Z 10014be4 f   wzanistate.obj
 0001:00013c5c       ?SetEvents@CWzAniState@@AAEXPAUWzEvent@@@Z 10014c5c f   wzanistate.obj
 0001:000140d3       ??_ECWzAniState@@UAEPAXI@Z 100150d3 f i wzanistate.obj
 0001:000140d3       ??_GCWzAniState@@UAEPAXI@Z 100150d3 f i wzanistate.obj
 0001:000140fa       ?InitEventPlayFlags@CWzAniState@@AAEXXZ 100150fa f i wzanistate.obj
 0001:0001411b       ?FindWzd@CManagerWzdLoader@@QAEPAXPBD@Z 1001511b f i wzanistate.obj
 0001:000141b7       ??1CWzSync@@QAE@XZ         100151b7 f i wzanistate.obj
 0001:000141da       ?GetWzdInfo@CManagerWzdLoader@@QAEPAUSt_WzdContainer@@PAX@Z 100151da f i wzanistate.obj
 0001:00014295       ??YWzVector@@QAEAAU0@ABU0@@Z 10015295 f i wzanistate.obj
 0001:000142d6       ??DWzVector@@QBE?AU0@M@Z   100152d6 f i wzanistate.obj
 0001:00014316       ??1?$CWzFlag@K@@QAE@XZ     10015316 f i wzanistate.obj
 0001:00014316       ??1_Container_base_aux@std@@QAE@XZ 10015316 f i wzdmeshsorter.obj
 0001:00014316       ?AllocKeyFrames@CWzdBase@@UAEXXZ 10015316 f i wzdbase.obj
 0001:0001431f       ?GetData@?$CWzHandleManager@PAUSt_WzdContainer@@@@QBEABQAUSt_WzdContainer@@PAX@Z 1001531f f i wzanistate.obj
 0001:00014357       ?GetC@?$CWzHashTableStr@PAX@@QBEABQAXPBD@Z 10015357 f i wzanistate.obj
 0001:00014421       ??1CKey_HashTableStr@@QAE@XZ 10015421 f i wzanistate.obj
 0001:0001444a       ?SetStr@CKey_HashTableStr@@QAEXPBD@Z 1001544a f i wzanistate.obj
 0001:000144f7       ?Get@?$CWzArray@G@@QBEAAGH@Z 100154f7 f i wzanistate.obj
 0001:00014526       ?Get@?$CWzArray@PAUSt_WzdContainer@@@@QBEAAPAUSt_WzdContainer@@H@Z 10015526 f i wzanistate.obj
 0001:00014555       ?IsSameKey@?$CWzHashTable@PAXVCKey_HashTableStr@@@@IBEHABVCKey_HashTableStr@@0@Z 10015555 f i wzanistate.obj
 0001:000145e0       ??0CWzShadowVolume@@QAE@XZ 100155e0 f   wzshadowvolume.obj
 0001:00014619       ??1CWzShadowVolume@@QAE@XZ 10015619 f   wzshadowvolume.obj
 0001:0001464d       ?Create@CWzShadowVolume@@QAEHABUWzVector@@HPAUWzMeshGroup@@PBU2@K@Z 1001564d f   wzshadowvolume.obj
 0001:0001470b       ?Destroy@CWzShadowVolume@@QAEXXZ 1001570b f   wzshadowvolume.obj
 0001:00014723       ?GenerateResult@CWzShadowVolume@@AAEXPBUWzVector@@@Z 10015723 f   wzshadowvolume.obj
 0001:00014987       ??0CWzSilhouette@@QAE@XZ   10015987 f   wzsilhouette.obj
 0001:000149bd       ??1CWzSilhouette@@QAE@XZ   100159bd f   wzsilhouette.obj
 0001:00014a0c       ?Create@CWzSilhouette@@QAEHABUWzVector@@HPAUWzMeshGroup@@PBU2@@Z 10015a0c f   wzsilhouette.obj
 0001:00014a92       ?Destroy@CWzSilhouette@@QAEXXZ 10015a92 f   wzsilhouette.obj
 0001:00014aa9       ?DetermineSilhouette@CWzSilhouette@@AAEXPAUWzMeshGroup@@HPBUWzVector@@HPAUWzFace@@PAM@Z 10015aa9 f   wzsilhouette.obj
 0001:00014e23       ?GenerateResult@CWzSilhouette@@AAEXPBUWzVector@@@Z 10015e23 f   wzsilhouette.obj
 0001:000150c8       ?MakeSureSilhouetteLineBuffer@CWzSilhouette@@AAEXH@Z 100160c8 f   wzsilhouette.obj
 0001:00015189       ?CalculateNormal@@YAPAUWzVector@@PAU1@PBU1@11@Z 10016189 f i wzsilhouette.obj
 0001:000151d4       ??0CWzUnit@@QAE@XZ         100161d4 f   wzunit.obj
 0001:00015301       ??1CWzUnit@@UAE@XZ         10016301 f   wzunit.obj
 0001:00015421       ?InitVariables@CWzUnit@@AAEXXZ 10016421 f   wzunit.obj
 0001:00015584       ?Release@CWzUnit@@AAEXXZ   10016584 f   wzunit.obj
 0001:00015bc3       ?Create@CWzUnit@@UAEHXZ    10016bc3 f   wzunit.obj
 0001:00015bcf       ?Destroy@CWzUnit@@UAEXXZ   10016bcf f   wzunit.obj
 0001:00015be8       ?AddWzdFileName@CWzUnit@@QAEXPBD@Z 10016be8 f   wzunit.obj
 0001:00015ce5       ?GetWzdFileName@CWzUnit@@QAEXPADH@Z 10016ce5 f   wzunit.obj
 0001:00015d4c       ?FindWzdPtr@CWzUnit@@AAEXH@Z 10016d4c f   wzunit.obj
 0001:00015dd3       ?CheckLoadState@CWzUnit@@AAEXXZ 10016dd3 f   wzunit.obj
 0001:00015ed2       ?AddAnimationInfo@CWzUnit@@QAEXABVWzAnimationInfo@@@Z 10016ed2 f   wzunit.obj
 0001:00015f5c       ?GetAnimationInfo@CWzUnit@@QAEPAVWzAnimationInfo@@K@Z 10016f5c f   wzunit.obj
 0001:00015fdf       ?AddBoneInfo@CWzUnit@@QAEXABUWzBoneInfo@@@Z 10016fdf f   wzunit.obj
 0001:00016047       ?GetBoneInfo@CWzUnit@@QAEPAUWzBoneInfo@@K@Z 10017047 f   wzunit.obj
 0001:000160c9       ?CreateSubType@CWzUnit@@QAEPAVCWzUnitSubType@@XZ 100170c9 f   wzunit.obj
 0001:00016151       ?GetMeshGroupIndexByName@CWzUnit@@QAEHPBD@Z 10017151 f   wzunit.obj
 0001:00016263       ?AddDiffuseMapInfo@CWzUnit@@QAEXHABUWzMappingInfo@@@Z 10017263 f   wzunit.obj
 0001:00016309       ?AddSpecularMapInfo@CWzUnit@@QAEXHABUWzMappingInfo@@@Z 10017309 f   wzunit.obj
 0001:000163af       ?AddNormalMapInfo@CWzUnit@@QAEXHABUWzMappingInfo@@@Z 100173af f   wzunit.obj
 0001:00016455       ?AddGlowMapInfo@CWzUnit@@QAEXHABUWzMappingInfo@@@Z 10017455 f   wzunit.obj
 0001:000164fe       ?AddInternalMapInfo@CWzUnit@@QAEXHABUWzMappingInfo@@@Z 100174fe f   wzunit.obj
 0001:000165a7       ?AddFilterInfo@CWzUnit@@QAEXHABUWzMappingInfo@@@Z 100175a7 f   wzunit.obj
 0001:00016650       ?AddTexAniMapInfo@CWzUnit@@QAEXHABUWzTexAniMappingInfo@@@Z 10017650 f   wzunit.obj
 0001:00016724       ?AddTexAniSetInfo@CWzUnit@@QAEXABUWzTexAniSetInfo@@@Z 10017724 f   wzunit.obj
 0001:000167d1       ?GetTexAniSetInfo@CWzUnit@@QAEPAUWzTexAniSetInfo@@K@Z 100177d1 f   wzunit.obj
 0001:0001682d       ?AddBVExtraInfo@CWzUnit@@QAEXABUWzBVExtraInfo@@@Z 1001782d f   wzunit.obj
 0001:000168cf       ?OnNotify@CWzUnit@@UAEXHKK@Z 100178cf f   wzunit.obj
 0001:00016950       ??_ECWzUnit@@UAEPAXI@Z     10017950 f i wzunit.obj
 0001:00016950       ??_GCWzUnit@@UAEPAXI@Z     10017950 f i wzunit.obj
 0001:00016977       ?AddMeshGroupNameInfo@CWzUnit@@QAEXABUMeshGroupNameInfo@@@Z 10017977 f i wzunit.obj
 0001:000169b6       ??0WzTexAniSetInfo@@QAE@XZ 100179b6 f i wzunit.obj
 0001:00016a20       ??0?$CWzArray@K@@QAE@XZ    10017a20 f i wzunit.obj
 0001:00016a88       ??4?$CWzArray@K@@QAEAAV0@ABV0@@Z 10017a88 f i wzunit.obj
 0001:00016b3c       ??0?$CWzArray@PAVWzAnimationInfo@@@@QAE@XZ 10017b3c f i wzunit.obj
 0001:00016ba4       ?Get@?$CWzArray@PAVWzAnimationInfo@@@@QBEAAPAVWzAnimationInfo@@H@Z 10017ba4 f i wzunit.obj
 0001:00016bd3       ??0?$CWzArray@PAUWzBoneInfo@@@@QAE@XZ 10017bd3 f i wzunit.obj
 0001:00016c3b       ?Get@?$CWzArray@PAUWzBoneInfo@@@@QBEAAPAUWzBoneInfo@@H@Z 10017c3b f i wzunit.obj
 0001:00016c6a       ??0?$CWzArray@PAVCWzUnitSubType@@@@QAE@XZ 10017c6a f i wzunit.obj
 0001:00016cd2       ?Get@?$CWzArray@PAVCWzUnitSubType@@@@QBEAAPAVCWzUnitSubType@@H@Z 10017cd2 f i wzunit.obj
 0001:00016d01       ??0?$CWzArray@PAUMeshGroupNameInfo@@@@QAE@XZ 10017d01 f i wzunit.obj
 0001:00016d69       ?Get@?$CWzArray@PAUMeshGroupNameInfo@@@@QBEAAPAUMeshGroupNameInfo@@H@Z 10017d69 f i wzunit.obj
 0001:00016d98       ??0?$CWzArray@PAUWzMappingInfo@@@@QAE@XZ 10017d98 f i wzunit.obj
 0001:00016e00       ?SetE@?$CWzArray@PAUWzTexAniMappingInfo@@@@QAEXHABQAUWzTexAniMappingInfo@@@Z 10017e00 f i wzunit.obj
 0001:00016e00       ?SetE@?$CWzArray@PAUWzMappingInfo@@@@QAEXHABQAUWzMappingInfo@@@Z 10017e00 f i wzunit.obj
 0001:00016e51       ?Get@?$CWzArray@PAUWzMappingInfo@@@@QBEAAPAUWzMappingInfo@@H@Z 10017e51 f i wzunit.obj
 0001:00016e80       ??0?$CWzArray@PAUWzTexAniMappingInfo@@@@QAE@XZ 10017e80 f i wzunit.obj
 0001:00016ee8       ?Get@?$CWzArray@PAUWzTexAniMappingInfo@@@@QBEAAPAUWzTexAniMappingInfo@@H@Z 10017ee8 f i wzunit.obj
 0001:00016f17       ??0?$CWzArray@PAUWzTexAniSetInfo@@@@QAE@XZ 10017f17 f i wzunit.obj
 0001:00016f7f       ?Get@?$CWzArray@PAUWzTexAniSetInfo@@@@QBEAAPAUWzTexAniSetInfo@@H@Z 10017f7f f i wzunit.obj
 0001:00016fae       ??0?$CWzArray@PAUWzBVExtraInfo@@@@QAE@XZ 10017fae f i wzunit.obj
 0001:00017016       ?Get@?$CWzArray@PAUWzBVExtraInfo@@@@QBEAAPAUWzBVExtraInfo@@H@Z 10018016 f i wzunit.obj
 0001:00017045       ?Add@?$CWzArray@PAVCWzUnitSubType@@@@QAEHABQAVCWzUnitSubType@@@Z 10018045 f i wzunit.obj
 0001:00017045       ?Add@?$CWzArray@PAUWzBoneInfo@@@@QAEHABQAUWzBoneInfo@@@Z 10018045 f i wzunit.obj
 0001:00017045       ?Add@?$CWzArray@PAUWzTexAniSetInfo@@@@QAEHABQAUWzTexAniSetInfo@@@Z 10018045 f i wzunit.obj
 0001:00017045       ?Add@?$CWzArray@PAUWzBVExtraInfo@@@@QAEHABQAUWzBVExtraInfo@@@Z 10018045 f i wzunit.obj
 0001:00017045       ?Add@?$CWzArray@PAUWzUnitEffectInfo@@@@QAEHABQAUWzUnitEffectInfo@@@Z 10018045 f i wzunitdraw.obj
 0001:00017045       ?Add@?$CWzArray@PAVWzAnimationInfo@@@@QAEHABQAVWzAnimationInfo@@@Z 10018045 f i wzunit.obj
 0001:00017045       ?Add@?$CWzArray@K@@QAEHABK@Z 10018045 f i wzunit_loadsave.obj
 0001:00017045       ?Add@?$CWzArray@PAUBvAABB@@@@QAEHABQAUBvAABB@@@Z 10018045 f i wzanimationInfo.obj
 0001:00017045       ?Add@?$CWzArray@PAUMeshGroupNameInfo@@@@QAEHABQAUMeshGroupNameInfo@@@Z 10018045 f i wzunit.obj
 0001:00017066       ?Set@?$CWzArray@PAUWzTexAniMappingInfo@@@@QAEXHABQAUWzTexAniMappingInfo@@@Z 10018066 f i wzunit.obj
 0001:00017066       ?Set@?$CWzArray@PAUWzTexAniSetInfo@@@@QAEXHABQAUWzTexAniSetInfo@@@Z 10018066 f i wzunit.obj
 0001:00017066       ?Set@?$CWzArray@PAVCWzUnitSubType@@@@QAEXHABQAVCWzUnitSubType@@@Z 10018066 f i wzunit.obj
 0001:00017066       ?Set@?$CWzArray@PAUWzUnitEffectInfo@@@@QAEXHABQAUWzUnitEffectInfo@@@Z 10018066 f i wzunitdraw.obj
 0001:00017066       ?Set@?$CWzArray@PAUMeshGroupNameInfo@@@@QAEXHABQAUMeshGroupNameInfo@@@Z 10018066 f i wzunit.obj
 0001:00017066       ?Set@?$CWzArray@PAUWzMappingInfo@@@@QAEXHABQAUWzMappingInfo@@@Z 10018066 f i wzunit.obj
 0001:00017066       ?Set@?$CWzArray@PAUWzBoneInfo@@@@QAEXHABQAUWzBoneInfo@@@Z 10018066 f i wzunit.obj
 0001:00017066       ?Set@?$CWzArray@PAUBvAABB@@@@QAEXHABQAUBvAABB@@@Z 10018066 f i wzanimationInfo.obj
 0001:00017066       ?Set@?$CWzArray@PAUWzBVExtraInfo@@@@QAEXHABQAUWzBVExtraInfo@@@Z 10018066 f i wzunit.obj
 0001:00017066       ?Set@?$CWzArray@PAVWzAnimationInfo@@@@QAEXHABQAVWzAnimationInfo@@@Z 10018066 f i wzunit.obj
 0001:00017066       ?Set@?$CWzArray@K@@QAEXHABK@Z 10018066 f i wzunit_loadsave.obj
 0001:000170b2       ?MakeSureDimensionSize@?$CWzArray@PAUMeshGroupNameInfo@@@@AAEXH@Z 100180b2 f i wzunit.obj
 0001:000170b2       ?MakeSureDimensionSize@?$CWzArray@PAUWzTexAniMappingInfo@@@@AAEXH@Z 100180b2 f i wzunit.obj
 0001:000170b2       ?MakeSureDimensionSize@?$CWzArray@PAUWzTexAniSetInfo@@@@AAEXH@Z 100180b2 f i wzunit.obj
 0001:000170b2       ?MakeSureDimensionSize@?$CWzArray@PAUWzMappingInfo@@@@AAEXH@Z 100180b2 f i wzunit.obj
 0001:000170b2       ?MakeSureDimensionSize@?$CWzArray@PAUWzBVExtraInfo@@@@AAEXH@Z 100180b2 f i wzunit.obj
 0001:000170b2       ?MakeSureDimensionSize@?$CWzArray@PAUBvAABB@@@@AAEXH@Z 100180b2 f i wzanimationInfo.obj
 0001:000170b2       ?MakeSureDimensionSize@?$CWzArray@PAVWzAnimationInfo@@@@AAEXH@Z 100180b2 f i wzunit.obj
 0001:000170b2       ?MakeSureDimensionSize@?$CWzArray@PAUWzUnitEffectInfo@@@@AAEXH@Z 100180b2 f i wzunitdraw.obj
 0001:000170b2       ?MakeSureDimensionSize@?$CWzArray@PAUWzBoneInfo@@@@AAEXH@Z 100180b2 f i wzunit.obj
 0001:000170b2       ?MakeSureDimensionSize@?$CWzArray@K@@AAEXH@Z 100180b2 f i wzunit_loadsave.obj
 0001:000170b2       ?MakeSureDimensionSize@?$CWzArray@PAVCWzUnitSubType@@@@AAEXH@Z 100180b2 f i wzunit.obj
 0001:00017180       ?Save@CWzUnit@@UAEHPBD@Z   10018180 f   wzunit_loadsave.obj
 0001:0001726f       ?Load@CWzUnit@@UAEHPBD@Z   1001826f f   wzunit_loadsave.obj
 0001:0001736f       ?SerializeHeader@CWzUnit@@AAEHPAVCWzArchive@@@Z 1001836f f   wzunit_loadsave.obj
 0001:0001743a       ?SerializeLODInfo@CWzUnit@@AAEHPAVCWzArchive@@@Z 1001843a f   wzunit_loadsave.obj
 0001:000174e2       ?SerializeAnimInfo@CWzUnit@@AAEHPAVCWzArchive@@@Z 100184e2 f   wzunit_loadsave.obj
 0001:00017ed8       ?SerializeBoneInfo@CWzUnit@@AAEHPAVCWzArchive@@@Z 10018ed8 f   wzunit_loadsave.obj
 0001:00017fc3       ?SerializeMappingInfo@CWzUnit@@AAEHPAVCWzArchive@@@Z 10018fc3 f   wzunit_loadsave.obj
 0001:00018954       ?SerializeComboInfo@CWzUnit@@AAEHPAVCWzArchive@@@Z 10019954 f   wzunit_loadsave.obj
 0001:00018a09       ?SerializeForceLODInfo@CWzUnit@@AAEHPAVCWzArchive@@@Z 10019a09 f   wzunit_loadsave.obj
 0001:00018a65       ?SerializeBVInfo@CWzUnit@@AAEHPAVCWzArchive@@@Z 10019a65 f   wzunit_loadsave.obj
 0001:00018e73       ?SerializeMorphMeshInfo@CWzUnit@@AAEHPAVCWzArchive@@@Z 10019e73 f   wzunit_loadsave.obj
 0001:00018f39       ?SerializeIKInfo@CWzUnit@@AAEHPAVCWzArchive@@@Z 10019f39 f   wzunit_loadsave.obj
 0001:00019023       ?SerializeDefaultInfo@CWzUnit@@AAEHPAVCWzArchive@@@Z 1001a023 f   wzunit_loadsave.obj
 0001:00019174       ?SerializeSubType@CWzUnit@@AAEHPAVCWzArchive@@@Z 1001a174 f   wzunit_loadsave.obj
 0001:00019273       ?SerializeMeshGroup@CWzUnit@@AAEHPAVCWzArchive@@@Z 1001a273 f   wzunit_loadsave.obj
 0001:000193b3       ?SerializeUnitOffset@CWzUnit@@AAEHPAVCWzArchive@@@Z 1001a3b3 f   wzunit_loadsave.obj
 0001:000194b4       ?Serialize@CWzUnit@@UAEHPAVCWzArchive@@@Z 1001a4b4 f   wzunit_loadsave.obj
 0001:00019521       ??1WzTexAniSetInfo@@QAE@XZ 1001a521 f i wzunit_loadsave.obj
 0001:00019535       ??0WzBVExtraInfo@@QAE@XZ   1001a535 f i wzunit_loadsave.obj
 0001:00019587       ?Get@?$CWzArray@K@@QBEAAKH@Z 1001a587 f i wzunit_loadsave.obj
 0001:000195b6       ??0CWzUnitDraw@@QAE@K@Z    1001a5b6 f   wzunitdraw.obj
 0001:000196ca       ??1CWzUnitDraw@@UAE@XZ     1001a6ca f   wzunitdraw.obj
 0001:00019730       ?InitVariables@CWzUnitDraw@@AAEXXZ 1001a730 f   wzunitdraw.obj
 0001:000197f6       ?Release@CWzUnitDraw@@AAEXXZ 1001a7f6 f   wzunitdraw.obj
 0001:00019943       ?Destroy@CWzUnitDraw@@UAEXXZ 1001a943 f   wzunitdraw.obj
 0001:0001995c       ?SetWzUnit@CWzUnitDraw@@QAEXPAVCWzUnit@@H@Z 1001a95c f   wzunitdraw.obj
 0001:000199d2       ?SetSubType@CWzUnitDraw@@QAEXH@Z 1001a9d2 f   wzunitdraw.obj
 0001:00019a5f       ?SetAniRefUnitDraw@CWzUnitDraw@@QAEXPAV1@@Z 1001aa5f f   wzunitdraw.obj
 0001:00019b68       ?ProgressFrame@CWzUnitDraw@@QAE?AW4ENUM_ANI_FRAME_STATUS@@MPAUWzEvent@@PAM@Z 1001ab68 f   wzunitdraw.obj
 0001:00019bf6       ?Process@CWzUnitDraw@@QAEXPBUWzMatrix@@@Z 1001abf6 f   wzunitdraw.obj
 0001:00019c4e       ?UpdateWzdLOD@CWzUnitDraw@@AAEXXZ 1001ac4e f   wzunitdraw.obj
 0001:00019da0       ?ProcessEffect@CWzUnitDraw@@AAEXXZ 1001ada0 f   wzunitdraw.obj
 0001:00019e05       ?UpdateSilhouette@CWzUnitDraw@@QAEXPAVCWzdBase@@ABUWzVector@@PBU3@@Z 1001ae05 f   wzunitdraw.obj
 0001:00019eae       ?UpdateShadowVolume@CWzUnitDraw@@QAEXPAVCWzdBase@@ABUWzVector@@PBU3@K@Z 1001aeae f   wzunitdraw.obj
 0001:00019f5a       ?InitShadowCastRecvInfo@CWzUnitDraw@@QAEXXZ 1001af5a f   wzunitdraw.obj
 0001:0001a0b4       ?EnableShadowCast@CWzUnitDraw@@QAEXHH@Z 1001b0b4 f   wzunitdraw.obj
 0001:0001a16e       ?IsEnableShadowCast@CWzUnitDraw@@QAEHH@Z 1001b16e f   wzunitdraw.obj
 0001:0001a1f7       ?EnableShadowReceive@CWzUnitDraw@@QAEXHH@Z 1001b1f7 f   wzunitdraw.obj
 0001:0001a2b1       ?IsEnableShadowReceive@CWzUnitDraw@@QAEHH@Z 1001b2b1 f   wzunitdraw.obj
 0001:0001a33a       ?AddUnitEffectInfo@CWzUnitDraw@@QAEXPBUWzUnitEffectInfo@@@Z 1001b33a f   wzunitdraw.obj
 0001:0001a376       ?ClearAllUnitEffectInfo@CWzUnitDraw@@QAEXXZ 1001b376 f   wzunitdraw.obj
 0001:0001a3dd       ?RemoveUnitEffectInfo@CWzUnitDraw@@QAEXH@Z 1001b3dd f   wzunitdraw.obj
 0001:0001a43a       ?SetEffectScale@CWzUnitDraw@@QAEXPAXABUWzVector@@@Z 1001b43a f   wzunitdraw.obj
 0001:0001a4a1       ?SetEffectRotation@CWzUnitDraw@@QAEXPAXABUWzQuaternion@@@Z 1001b4a1 f   wzunitdraw.obj
 0001:0001a509       ?SetEffectPosition@CWzUnitDraw@@QAEXPAXABUWzVector@@@Z 1001b509 f   wzunitdraw.obj
 0001:0001a570       ?SetEffectApplyRotation@CWzUnitDraw@@QAEXPAXH@Z 1001b570 f   wzunitdraw.obj
 0001:0001a5d0       ??_GCWzUnitDraw@@UAEPAXI@Z 1001b5d0 f i wzunitdraw.obj
 0001:0001a5d0       ??_ECWzUnitDraw@@UAEPAXI@Z 1001b5d0 f i wzunitdraw.obj
 0001:0001a5f7       ?IsUnitFullLoaded@CWzUnitDraw@@QBEHXZ 1001b5f7 f i wzunitdraw.obj
 0001:0001a641       ?Get@?$CWzArray@PAUWzRenderInfo@@@@QBEAAPAUWzRenderInfo@@H@Z 1001b641 f i wzunitdraw.obj
 0001:0001a670       ??0?$CWzArray@PAUWzUnitEffectInfo@@@@QAE@XZ 1001b670 f i wzunitdraw.obj
 0001:0001a6d8       ?Get@?$CWzArray@PAUWzUnitEffectInfo@@@@QBEAAPAUWzUnitEffectInfo@@H@Z 1001b6d8 f i wzunitdraw.obj
 0001:0001a707       ?GetCount@?$CWzArray@PAUWzBoneInfo@@@@QBEHXZ 1001b707 f i wzunit.obj
 0001:0001a707       ?GetCount@?$CWzArray@PAUWzBoneScaling@@@@QBEHXZ 1001b707 f i wzunitskeleton.obj
 0001:0001a707       ?GetCount@?$CWzArray@PAUWzUnitEffectInfo@@@@QBEHXZ 1001b707 f i wzunitdraw.obj
 0001:0001a707       ?GetCount@?$CWzArray@PAVCWzUnitSubType@@@@QBEHXZ 1001b707 f i wzunit.obj
 0001:0001a707       ?GetCount@?$CWzArray@PAVWzAnimationInfo@@@@QBEHXZ 1001b707 f i wzunit.obj
 0001:0001a707       ?GetCount@?$CWzArray@PAUWzTexAniMappingInfo@@@@QBEHXZ 1001b707 f i wzunit.obj
 0001:0001a707       ?GetCount@?$CWzArray@PAUWzTexAniSetInfo@@@@QBEHXZ 1001b707 f i wzunit.obj
 0001:0001a707       ?GetCount@?$CWzArray@PAUWzRenderInfo@@@@QBEHXZ 1001b707 f i wzunitdraw.obj
 0001:0001a707       ?GetCount@?$CWzArray@PAUWzBVExtraInfo@@@@QBEHXZ 1001b707 f i wzunit.obj
 0001:0001a707       ?GetCount@?$CWzArray@PAUWzDecoration@@@@QBEHXZ 1001b707 f i wzunitsubtype.obj
 0001:0001a707       ?GetCount@?$CWzArray@PAUMeshGroupNameInfo@@@@QBEHXZ 1001b707 f i wzunit.obj
 0001:0001a707       ?GetCount@?$CWzArray@K@@QBEHXZ 1001b707 f i wzunit_loadsave.obj
 0001:0001a707       ?GetCount@?$CWzArray@PAUWzMappingInfo@@@@QBEHXZ 1001b707 f i wzunit.obj
 0001:0001a707       ?GetCount@?$CWzArray@PAUBvAABB@@@@QBEHXZ 1001b707 f i wzanimationInfo.obj
 0001:0001a715       ??0CWzUnitEditable@@QAE@XZ 1001b715 f   wzuniteditable.obj
 0001:0001a732       ??1CWzUnitEditable@@UAE@XZ 1001b732 f   wzuniteditable.obj
 0001:0001a74c       ?SetWzdFileName@CWzUnitEditable@@QAEXPBDH@Z 1001b74c f   wzuniteditable.obj
 0001:0001a7a7       ?DelWzdFileName@CWzUnitEditable@@QAEXH@Z 1001b7a7 f   wzuniteditable.obj
 0001:0001a87e       ?SetAnimationInfoByIndex@CWzUnitEditable@@QAEXPBVWzAnimationInfo@@H@Z 1001b87e f   wzuniteditable.obj
 0001:0001a8be       ?DelAnimationInfoByIndex@CWzUnitEditable@@QAEXH@Z 1001b8be f   wzuniteditable.obj
 0001:0001a943       ?SetBoneInfoByIndex@CWzUnitEditable@@QAEXPBUWzBoneInfo@@H@Z 1001b943 f   wzuniteditable.obj
 0001:0001a988       ?DelBoneInfoByIndex@CWzUnitEditable@@QAEXH@Z 1001b988 f   wzuniteditable.obj
 0001:0001a9e5       ?SetDiffuseMapInfoByIndex@CWzUnitEditable@@QAEXPBUWzMappingInfo@@H@Z 1001b9e5 f   wzuniteditable.obj
 0001:0001aa5d       ?SetSpecularMapInfoByIndex@CWzUnitEditable@@QAEXPBUWzMappingInfo@@H@Z 1001ba5d f   wzuniteditable.obj
 0001:0001aad5       ?SetNormalMapInfoByIndex@CWzUnitEditable@@QAEXPBUWzMappingInfo@@H@Z 1001bad5 f   wzuniteditable.obj
 0001:0001ab4d       ?SetGlowMapInfoByIndex@CWzUnitEditable@@QAEXPBUWzMappingInfo@@H@Z 1001bb4d f   wzuniteditable.obj
 0001:0001abcb       ?SetInternalMapInfoByIndex@CWzUnitEditable@@QAEXPBUWzMappingInfo@@H@Z 1001bbcb f   wzuniteditable.obj
 0001:0001ac49       ?DelInternalMapInfoByIndex@CWzUnitEditable@@QAEXH@Z 1001bc49 f   wzuniteditable.obj
 0001:0001acaf       ?SetTexAniMapInfoByIndex@CWzUnitEditable@@QAEXPBUWzTexAniMappingInfo@@H@Z 1001bcaf f   wzuniteditable.obj
 0001:0001ad3e       ?DelTexAniMapInfoByIndex@CWzUnitEditable@@QAEXH@Z 1001bd3e f   wzuniteditable.obj
 0001:0001ada4       ?SetTexAniSetInfoByIndex@CWzUnitEditable@@QAEXPBUWzTexAniSetInfo@@H@Z 1001bda4 f   wzuniteditable.obj
 0001:0001ae07       ?DelTexAniSetInfoByIndex@CWzUnitEditable@@QAEXH@Z 1001be07 f   wzuniteditable.obj
 0001:0001ae98       ?AddTexAniID@CWzUnitEditable@@QAEXK@Z 1001be98 f   wzuniteditable.obj
 0001:0001af06       ?AddTexIDInTexAniSetInfo@CWzUnitEditable@@QAEXKH@Z 1001bf06 f   wzuniteditable.obj
 0001:0001af6f       ?DelTexIDInTexAniSetInfo@CWzUnitEditable@@QAEXHH@Z 1001bf6f f   wzuniteditable.obj
 0001:0001afed       ?CreateSubType@CWzUnitEditable@@QAEPAVCWzUnitSubType@@XZ 1001bfed f   wzuniteditable.obj
 0001:0001b075       ?DelSubType@CWzUnitEditable@@QAEXH@Z 1001c075 f   wzuniteditable.obj
 0001:0001b106       ?CopySubType@CWzUnitEditable@@QAEXHH@Z 1001c106 f   wzuniteditable.obj
 0001:0001b190       ?SetBVExtraInfoByIndex@CWzUnitEditable@@QAEXPBUWzBVExtraInfo@@H@Z 1001c190 f   wzuniteditable.obj
 0001:0001b1da       ?DelBVExtraInfoByIndex@CWzUnitEditable@@QAEXH@Z 1001c1da f   wzuniteditable.obj
 0001:0001b240       ??_ECWzUnitEditable@@UAEPAXI@Z 1001c240 f i wzuniteditable.obj
 0001:0001b240       ??_GCWzUnitEditable@@UAEPAXI@Z 1001c240 f i wzuniteditable.obj
 0001:0001b267       ??4WzMappingInfo@@QAEAAU0@ABU0@@Z 1001c267 f i wzuniteditable.obj
 0001:0001b2b9       ?Remove@?$CWzArray@PAUWzMappingInfo@@@@QAEXH@Z 1001c2b9 f i wzuniteditable.obj
 0001:0001b2b9       ?Remove@?$CWzArray@PAUWzRenderInfo@@@@QAEXH@Z 1001c2b9 f i wzunitsubtypeeditable.obj
 0001:0001b2b9       ?Remove@?$CWzArray@PAUWzBVExtraInfo@@@@QAEXH@Z 1001c2b9 f i wzuniteditable.obj
 0001:0001b2b9       ?Remove@?$CWzArray@PAUWzDecoration@@@@QAEXH@Z 1001c2b9 f i wzunitsubtypeeditable.obj
 0001:0001b2b9       ?Remove@?$CWzArray@K@@QAEXH@Z 1001c2b9 f i wzuniteditable.obj
 0001:0001b2b9       ?Remove@?$CWzArray@PAVCWzUnitSubType@@@@QAEXH@Z 1001c2b9 f i wzuniteditable.obj
 0001:0001b2b9       ?Remove@?$CWzArray@PAUWzUnitEffectInfo@@@@QAEXH@Z 1001c2b9 f i wzunitdraw.obj
 0001:0001b2b9       ?Remove@?$CWzArray@PAUWzTexAniSetInfo@@@@QAEXH@Z 1001c2b9 f i wzuniteditable.obj
 0001:0001b2b9       ?Remove@?$CWzArray@PAVWzAnimationInfo@@@@QAEXH@Z 1001c2b9 f i wzuniteditable.obj
 0001:0001b2b9       ?Remove@?$CWzArray@PAUWzBoneScaling@@@@QAEXH@Z 1001c2b9 f i wzunitsubtypeeditable.obj
 0001:0001b2b9       ?Remove@?$CWzArray@PAUWzBoneInfo@@@@QAEXH@Z 1001c2b9 f i wzuniteditable.obj
 0001:0001b2b9       ?Remove@?$CWzArray@PAUWzTexAniMappingInfo@@@@QAEXH@Z 1001c2b9 f i wzuniteditable.obj
 0001:0001b312       ??0CWzUnitSkeleton@@AAE@XZ 1001c312 f   wzunitskeleton.obj
 0001:0001b3c6       ??0CWzUnitSkeleton@@QAE@PAVCWzUnitDraw@@@Z 1001c3c6 f   wzunitskeleton.obj
 0001:0001b6a3       ??1CWzUnitSkeleton@@UAE@XZ 1001c6a3 f   wzunitskeleton.obj
 0001:0001b765       ?Release@CWzUnitSkeleton@@AAEXXZ 1001c765 f   wzunitskeleton.obj
 0001:0001b77e       ?OnWzUnitSet@CWzUnitSkeleton@@QAEXH@Z 1001c77e f   wzunitskeleton.obj
 0001:0001b83c       ?OnSubTypeChange@CWzUnitSkeleton@@QAEXXZ 1001c83c f   wzunitskeleton.obj
 0001:0001b8ad       ?SetCurAnimation@CWzUnitSkeleton@@QAEXKHHH@Z 1001c8ad f   wzunitskeleton.obj
 0001:0001b95e       ?SetCurBlendAnimation@CWzUnitSkeleton@@QAEXKHHMH@Z 1001c95e f   wzunitskeleton.obj
 0001:0001ba33       ?ProgressFrame@CWzUnitSkeleton@@QAE?AW4ENUM_ANI_FRAME_STATUS@@MPAUWzEvent@@PAM@Z 1001ca33 f   wzunitskeleton.obj
 0001:0001bb51       ?PreProcess@CWzUnitSkeleton@@AAEXPBUWzMatrix@@@Z 1001cb51 f   wzunitskeleton.obj
 0001:0001bb6f       ?Process@CWzUnitSkeleton@@QAEXPBUWzMatrix@@@Z 1001cb6f f   wzunitskeleton.obj
 0001:0001bdad       ?PostProcess@CWzUnitSkeleton@@AAEXXZ 1001cdad f   wzunitskeleton.obj
 0001:0001bdbe       ?InitTransformParam@CWzUnitSkeleton@@AAEXXZ 1001cdbe f   wzunitskeleton.obj
 0001:0001bef5       ?UpdateTransformParam@CWzUnitSkeleton@@AAEHPBUWzMatrix@@@Z 1001cef5 f   wzunitskeleton.obj
 0001:0001c047       ?FreeTransformBuf@CWzUnitSkeleton@@AAEXXZ 1001d047 f   wzunitskeleton.obj
 0001:0001c108       ?ResizeTransformBuf@CWzUnitSkeleton@@AAEXH@Z 1001d108 f   wzunitskeleton.obj
 0001:0001c4e8       ?OnAniStateNotice@CWzUnitSkeleton@@UAEXHK@Z 1001d4e8 f   wzunitskeleton.obj
 0001:0001c533       ?InitBaseBV@CWzUnitSkeleton@@AAEXW4ENUM_BVTYPE@@@Z 1001d533 f   wzunitskeleton.obj
 0001:0001c5ad       ?UpdateBV@CWzUnitSkeleton@@QAEXHPBUWzMatrix@@H@Z 1001d5ad f   wzunitskeleton.obj
 0001:0001caf9       ?ReleaseBVExtra@CWzUnitSkeleton@@AAEXXZ 1001daf9 f   wzunitskeleton.obj
 0001:0001cb69       ?InitBVExtra@CWzUnitSkeleton@@QAEXXZ 1001db69 f   wzunitskeleton.obj
 0001:0001cc81       ?UpdateBVExtra@CWzUnitSkeleton@@QAEXXZ 1001dc81 f   wzunitskeleton.obj
 0001:0001d04d       ?UpdateLOD@CWzUnitSkeleton@@AAEXPBUWzMatrix@@@Z 1001e04d f   wzunitskeleton.obj
 0001:0001d307       ?AdjustOwnerOption@CWzUnitSkeleton@@AAEXXZ 1001e307 f   wzunitskeleton.obj
 0001:0001d6bb       ?UpdateAreaLight@CWzUnitSkeleton@@AAEXXZ 1001e6bb f   wzunitskeleton.obj
 0001:0001d741       ??1CWzAniStateCB@@UAE@XZ   1001e741 f i wzunitskeleton.obj
 0001:0001d753       ??_GCWzUnitSkeleton@@UAEPAXI@Z 1001e753 f i wzunitskeleton.obj
 0001:0001d753       ??_ECWzUnitSkeleton@@UAEPAXI@Z 1001e753 f i wzunitskeleton.obj
 0001:0001d77a       ??1WzTransformParam@@QAE@XZ 1001e77a f i wzunitskeleton.obj
 0001:0001d7cf       ?MatrixIdentity@@YAPAUWzMatrix@@PAU1@@Z 1001e7cf f i wzunitskeleton.obj
 0001:0001d8d6       ?SaveLastTransform@CWzUnitSkeleton@@AAEXXZ 1001e8d6 f i wzunitskeleton.obj
 0001:0001d912       ?GetValidWzdPtr@CWzUnit@@QAEPAVCWzdBase@@XZ 1001e912 f i wzunitskeleton.obj
 0001:0001d94e       ?GetWzdPtr@CWzUnit@@QAEPAVCWzdBase@@H@Z 1001e94e f i wzunitskeleton.obj
 0001:0001d990       ?GetRotationMatrix@CWzUnitSkeleton@@QAEXPAUWzMatrix@@@Z 1001e990 f i wzunitskeleton.obj
 0001:0001da45       ?VectorTransformCoord@@YAPAUWzVector@@PAU1@PBU1@PBUWzMatrix@@@Z 1001ea45 f i wzunitskeleton.obj
 0001:0001dae4       ?MatrixSRT@@YAPAUWzMatrix@@PAU1@ABUWzVector@@PBU1@1@Z 1001eae4 f i wzunitskeleton.obj
 0001:0001dbac       ?insert@?$_Tree@V?$_Tmap_traits@HUWzVector@@U?$less@H@std@@V?$allocator@U?$pair@$$CBHUWzVector@@@std@@@3@$0A@@std@@@std@@QAE?AU?$pair@Viterator@?$_Tree@V?$_Tmap_traits@HUWzVector@@U?$less@H@std@@V?$allocator@U?$pair@$$CBHUWzVector@@@std@@@3@$0A@@std@@@std@@_N@2@ABU?$pair@$$CBHUWzVector@@@2@@Z 1001ebac f i wzunitskeleton.obj
 0001:0001dd7c       ?clear@?$_Tree@V?$_Tmap_traits@HUWzVector@@U?$less@H@std@@V?$allocator@U?$pair@$$CBHUWzVector@@@std@@@3@$0A@@std@@@std@@QAEXXZ 1001ed7c f i wzunitskeleton.obj
 0001:0001ddd1       ??0?$_Tree@V?$_Tmap_traits@HUWzVector@@U?$less@H@std@@V?$allocator@U?$pair@$$CBHUWzVector@@@std@@@3@$0A@@std@@@std@@QAE@ABU?$less@H@1@ABV?$allocator@U?$pair@$$CBHUWzVector@@@std@@@1@@Z 1001edd1 f i wzunitskeleton.obj
 0001:0001de32       ?_Erase@?$_Tree@V?$_Tmap_traits@HUWzVector@@U?$less@H@std@@V?$allocator@U?$pair@$$CBHUWzVector@@@std@@@3@$0A@@std@@@std@@IAEXPAU_Node@?$_Tree_nod@V?$_Tmap_traits@HUWzVector@@U?$less@H@std@@V?$allocator@U?$pair@$$CBHUWzVector@@@std@@@3@$0A@@std@@@2@@Z 1001ee32 f i wzunitskeleton.obj
 0001:0001de78       ?_Insert@?$_Tree@V?$_Tmap_traits@HUWzVector@@U?$less@H@std@@V?$allocator@U?$pair@$$CBHUWzVector@@@std@@@3@$0A@@std@@@std@@IAE?AViterator@12@_NPAU_Node@?$_Tree_nod@V?$_Tmap_traits@HUWzVector@@U?$less@H@std@@V?$allocator@U?$pair@$$CBHUWzVector@@@std@@@3@$0A@@std@@@2@ABU?$pair@$$CBHUWzVector@@@2@@Z 1001ee78 f i wzunitskeleton.obj
 0001:0001e233       ?_Tidy@?$_Tree@V?$_Tmap_traits@HUWzVector@@U?$less@H@std@@V?$allocator@U?$pair@$$CBHUWzVector@@@std@@@3@$0A@@std@@@std@@IAEXXZ 1001f233 f i wzunitskeleton.obj
 0001:0001e2f3       ?erase@?$_Tree@V?$_Tmap_traits@HUWzVector@@U?$less@H@std@@V?$allocator@U?$pair@$$CBHUWzVector@@@std@@@3@$0A@@std@@@std@@QAE?AViterator@12@Vconst_iterator@12@0@Z 1001f2f3 f i wzunitskeleton.obj
 0001:0001e4ad       ?_Init@?$_Tree@V?$_Tmap_traits@HUWzVector@@U?$less@H@std@@V?$allocator@U?$pair@$$CBHUWzVector@@@std@@@3@$0A@@std@@@std@@IAEXXZ 1001f4ad f i wzunitskeleton.obj
 0001:0001e508       ?_Lrotate@?$_Tree@V?$_Tmap_traits@HUWzVector@@U?$less@H@std@@V?$allocator@U?$pair@$$CBHUWzVector@@@std@@@3@$0A@@std@@@std@@IAEXPAU_Node@?$_Tree_nod@V?$_Tmap_traits@HUWzVector@@U?$less@H@std@@V?$allocator@U?$pair@$$CBHUWzVector@@@std@@@3@$0A@@std@@@2@@Z 1001f508 f i wzunitskeleton.obj
 0001:0001e5ac       ?_Rrotate@?$_Tree@V?$_Tmap_traits@HUWzVector@@U?$less@H@std@@V?$allocator@U?$pair@$$CBHUWzVector@@@std@@@3@$0A@@std@@@std@@IAEXPAU_Node@?$_Tree_nod@V?$_Tmap_traits@HUWzVector@@U?$less@H@std@@V?$allocator@U?$pair@$$CBHUWzVector@@@std@@@3@$0A@@std@@@2@@Z 1001f5ac f i wzunitskeleton.obj
 0001:0001e64d       ?_Buynode@?$_Tree@V?$_Tmap_traits@HUWzVector@@U?$less@H@std@@V?$allocator@U?$pair@$$CBHUWzVector@@@std@@@3@$0A@@std@@@std@@IAEPAU_Node@?$_Tree_nod@V?$_Tmap_traits@HUWzVector@@U?$less@H@std@@V?$allocator@U?$pair@$$CBHUWzVector@@@std@@@3@$0A@@std@@@2@PAU342@00ABU?$pair@$$CBHUWzVector@@@2@D@Z 1001f64d f i wzunitskeleton.obj
 0001:0001e71a       ??0?$_Tree_val@V?$_Tmap_traits@HUWzVector@@U?$less@H@std@@V?$allocator@U?$pair@$$CBHUWzVector@@@std@@@3@$0A@@std@@@std@@IAE@ABU?$less@H@1@V?$allocator@U?$pair@$$CBHUWzVector@@@std@@@1@@Z 1001f71a f i wzunitskeleton.obj
 0001:0001e741       ?erase@?$_Tree@V?$_Tmap_traits@HUWzVector@@U?$less@H@std@@V?$allocator@U?$pair@$$CBHUWzVector@@@std@@@3@$0A@@std@@@std@@QAE?AViterator@12@Vconst_iterator@12@@Z 1001f741 f i wzunitskeleton.obj
 0001:0001ed1c       ??1out_of_range@std@@UAE@XZ 1001fd1c f i wzunitskeleton.obj
 0001:0001ed38       ??_Gout_of_range@std@@UAEPAXI@Z 1001fd38 f i wzunitskeleton.obj
 0001:0001ed38       ??_Eout_of_range@std@@UAEPAXI@Z 1001fd38 f i wzunitskeleton.obj
 0001:0001ed6a       ??0out_of_range@std@@QAE@ABV01@@Z 1001fd6a f i wzunitskeleton.obj
 0001:0001ed8e       ?_Buynode@?$_Tree@V?$_Tmap_traits@HUWzVector@@U?$less@H@std@@V?$allocator@U?$pair@$$CBHUWzVector@@@std@@@3@$0A@@std@@@std@@IAEPAU_Node@?$_Tree_nod@V?$_Tmap_traits@HUWzVector@@U?$less@H@std@@V?$allocator@U?$pair@$$CBHUWzVector@@@std@@@3@$0A@@std@@@2@XZ 1001fd8e f i wzunitskeleton.obj
 0001:0001eea8       ??0?$_Tree_ptr@V?$_Tmap_traits@HUWzVector@@U?$less@H@std@@V?$allocator@U?$pair@$$CBHUWzVector@@@std@@@3@$0A@@std@@@std@@IAE@ABU?$less@H@1@V?$allocator@U?$pair@$$CBHUWzVector@@@std@@@1@@Z 1001fea8 f i wzunitskeleton.obj
 0001:0001eeec       ??9const_iterator@?$_Tree@V?$_Tmap_traits@HUWzVector@@U?$less@H@std@@V?$allocator@U?$pair@$$CBHUWzVector@@@std@@@3@$0A@@std@@@std@@QBE_NABV012@@Z 1001feec f i wzunitskeleton.obj
 0001:0001ef41       ?_Dec@const_iterator@?$_Tree@V?$_Tmap_traits@HUWzVector@@U?$less@H@std@@V?$allocator@U?$pair@$$CBHUWzVector@@@std@@@3@$0A@@std@@@std@@QAEXXZ 1001ff41 f i wzunitskeleton.obj
 0001:0001f034       ?_Inc@const_iterator@?$_Tree@V?$_Tmap_traits@HUWzVector@@U?$less@H@std@@V?$allocator@U?$pair@$$CBHUWzVector@@@std@@@3@$0A@@std@@@std@@QAEXXZ 10020034 f i wzunitskeleton.obj
 0001:0001f0fa       ?Get@?$CWzArray@PAUWzBoneScaling@@@@QBEAAPAUWzBoneScaling@@H@Z 100200fa f i wzunitskeleton.obj
 0001:0001f129       ??$_Allocate@UWzSoundInfo@@@std@@YAPAUWzSoundInfo@@IPAU1@@Z 10020129 f i wzanimationInfo.obj
 0001:0001f129       ??$_Allocate@U_Node@?$_Tree_nod@V?$_Tmap_traits@HUWzVector@@U?$less@H@std@@V?$allocator@U?$pair@$$CBHUWzVector@@@std@@@3@$0A@@std@@@std@@@std@@YAPAU_Node@?$_Tree_nod@V?$_Tmap_traits@HUWzVector@@U?$less@H@std@@V?$allocator@U?$pair@$$CBHUWzVector@@@std@@@3@$0A@@std@@@0@IPAU120@@Z 10020129 f i wzunitskeleton.obj
 0001:0001f17c       ??0CWzUnitSubType@@QAE@XZ  1002017c f   wzunitsubtype.obj
 0001:0001f1f4       ??1CWzUnitSubType@@UAE@XZ  100201f4 f   wzunitsubtype.obj
 0001:0001f26c       ?InitVariables@CWzUnitSubType@@AAEXXZ 1002026c f   wzunitsubtype.obj
 0001:0001f2dc       ?Release@CWzUnitSubType@@AAEXXZ 100202dc f   wzunitsubtype.obj
 0001:0001f3fb       ?Create@CWzUnitSubType@@UAEHXZ 100203fb f   wzunitsubtype.obj
 0001:0001f407       ?Destroy@CWzUnitSubType@@UAEXXZ 10020407 f   wzunitsubtype.obj
 0001:0001f420       ?AddBoneScaling@CWzUnitSubType@@QAEXPBUWzBoneScaling@@@Z 10020420 f   wzunitsubtype.obj
 0001:0001f4b7       ?AddDecoration@CWzUnitSubType@@QAEXPBUWzDecoration@@@Z 100204b7 f   wzunitsubtype.obj
 0001:0001f520       ?AddRenderInfo@CWzUnitSubType@@QAEXPBUWzRenderInfo@@@Z 10020520 f   wzunitsubtype.obj
 0001:0001f5b1       ?Copy@CWzUnitSubType@@QAEXABV1@@Z 100205b1 f   wzunitsubtype.obj
 0001:0001f6d7       ?Serialize@CWzUnitSubType@@UAEHPAVCWzArchive@@@Z 100206d7 f   wzunitsubtype.obj
 0001:0002043e       ??_ECWzUnitSubType@@UAEPAXI@Z 1002143e f i wzunitsubtype.obj
 0001:0002043e       ??_GCWzUnitSubType@@UAEPAXI@Z 1002143e f i wzunitsubtype.obj
 0001:00020465       ??0WzRenderInfo@@QAE@XZ    10021465 f i wzunitsubtype.obj
 0001:000205ee       ??0?$CWzArray@PAUWzBoneScaling@@@@QAE@XZ 100215ee f i wzunitsubtype.obj
 0001:00020656       ?Add@?$CWzArray@PAUWzDecoration@@@@QAEHABQAUWzDecoration@@@Z 10021656 f i wzunitsubtype.obj
 0001:00020656       ?Add@?$CWzArray@PAUWzRenderInfo@@@@QAEHABQAUWzRenderInfo@@@Z 10021656 f i wzunitsubtype.obj
 0001:00020656       ?Add@?$CWzArray@PAUWzBoneScaling@@@@QAEHABQAUWzBoneScaling@@@Z 10021656 f i wzunitsubtype.obj
 0001:00020677       ??0?$CWzArray@PAUWzDecoration@@@@QAE@XZ 10021677 f i wzunitsubtype.obj
 0001:000206df       ?Get@?$CWzArray@PAUWzDecoration@@@@QBEAAPAUWzDecoration@@H@Z 100216df f i wzunitsubtype.obj
 0001:0002070e       ??0?$CWzArray@PAUWzRenderInfo@@@@QAE@XZ 1002170e f i wzunitsubtype.obj
 0001:00020776       ??1?$CWzArray@PAUWzRenderInfo@@@@QAE@XZ 10021776 f i wzunitsubtype.obj
 0001:00020776       ??1?$CWzArray@PAUWzBoneScaling@@@@QAE@XZ 10021776 f i wzunitsubtype.obj
 0001:00020776       ??1?$CWzArray@PAUWzDecoration@@@@QAE@XZ 10021776 f i wzunitsubtype.obj
 0001:00020787       ?Set@?$CWzArray@PAUWzDecoration@@@@QAEXHABQAUWzDecoration@@@Z 10021787 f i wzunitsubtype.obj
 0001:00020787       ?Set@?$CWzArray@PAUWzBoneScaling@@@@QAEXHABQAUWzBoneScaling@@@Z 10021787 f i wzunitsubtype.obj
 0001:00020787       ?Set@?$CWzArray@PAUWzRenderInfo@@@@QAEXHABQAUWzRenderInfo@@@Z 10021787 f i wzunitsubtype.obj
 0001:000207d3       ?Release@?$CWzArray@PAUWzBoneScaling@@@@AAEXXZ 100217d3 f i wzunitsubtype.obj
 0001:000207d3       ?Release@?$CWzArray@PAUWzDecoration@@@@AAEXXZ 100217d3 f i wzunitsubtype.obj
 0001:000207d3       ?Release@?$CWzArray@PAUWzRenderInfo@@@@AAEXXZ 100217d3 f i wzunitsubtype.obj
 0001:0002080c       ?MakeSureDimensionSize@?$CWzArray@PAUWzBoneScaling@@@@AAEXH@Z 1002180c f i wzunitsubtype.obj
 0001:0002080c       ?MakeSureDimensionSize@?$CWzArray@PAUWzRenderInfo@@@@AAEXH@Z 1002180c f i wzunitsubtype.obj
 0001:0002080c       ?MakeSureDimensionSize@?$CWzArray@PAUWzDecoration@@@@AAEXH@Z 1002180c f i wzunitsubtype.obj
 0001:000208da       ??0CWzUnitSubTypeEditable@@QAE@XZ 100218da f   wzunitsubtypeeditable.obj
 0001:000208f7       ??1CWzUnitSubTypeEditable@@UAE@XZ 100218f7 f   wzunitsubtypeeditable.obj
 0001:00020911       ?SetBoneScaling@CWzUnitSubTypeEditable@@QAEXPBUWzBoneScaling@@H@Z 10021911 f   wzunitsubtypeeditable.obj
 0001:00020954       ?DelBoneScaling@CWzUnitSubTypeEditable@@QAEXH@Z 10021954 f   wzunitsubtypeeditable.obj
 0001:000209b1       ?SetDecoration@CWzUnitSubTypeEditable@@QAEXPBUWzDecoration@@H@Z 100219b1 f   wzunitsubtypeeditable.obj
 0001:000209f5       ?DelDecoration@CWzUnitSubTypeEditable@@QAEXH@Z 100219f5 f   wzunitsubtypeeditable.obj
 0001:00020a52       ?SetRenderInfo@CWzUnitSubTypeEditable@@QAEXPBUWzRenderInfo@@H@Z 10021a52 f   wzunitsubtypeeditable.obj
 0001:00020a96       ?DelRenderInfo@CWzUnitSubTypeEditable@@QAEXH@Z 10021a96 f   wzunitsubtypeeditable.obj
 0001:00020af3       ??_ECWzUnitSubTypeEditable@@UAEPAXI@Z 10021af3 f i wzunitsubtypeeditable.obj
 0001:00020af3       ??_GCWzUnitSubTypeEditable@@UAEPAXI@Z 10021af3 f i wzunitsubtypeeditable.obj
 0001:00020b1a       ?IsCPUID@FastMath@@YA_NXZ  10021b1a f   common:wzfastmath.obj
 0001:00020b8e       ?IsCPUSupport@FastMath@@YA_NW4SlIntrinsic@1@@Z 10021b8e f   common:wzfastmath.obj
 0001:00020c68       ?IsOSSupport@FastMath@@YA_NW4SlIntrinsic@1@@Z 10021c68 f   common:wzfastmath.obj
 0001:00020d23       ?GetCPUCaps@FastMath@@YAXPAUCPUCaps@1@@Z 10021d23 f   common:wzfastmath.obj
 0001:00020e47       ?Startup@FastMath@@YAXXZ   10021e47 f   common:wzfastmath.obj
 0001:00020ee0       ?MatrixRotationX_Scalar@@YAPAUWzMatrix@@PAU1@M@Z 10021ee0 f i common:wzmath.obj
 0001:00020ff4       ?MatrixRotationY_Scalar@@YAPAUWzMatrix@@PAU1@M@Z 10021ff4 f i common:wzmath.obj
 0001:00021107       ?MatrixRotationZ_Scalar@@YAPAUWzMatrix@@PAU1@M@Z 10022107 f i common:wzmath.obj
 0001:0002121b       ?QuaternionMultiply_Scalar@@YAPAUWzQuaternion@@PAU1@PBU1@1@Z 1002221b f i common:wzmath.obj
 0001:0002130a       ?MatrixInverse@@YAPAUWzMatrix@@PAU1@PBU1@@Z 1002230a f   common:wzmath.obj
 0001:00021bb8       ?MatrixRotationZYX@@YAPAUWzMatrix@@PAU1@PBUWzVector@@@Z 10022bb8 f   common:wzmath.obj
 0001:00021d84       ?MatrixRotationZXY@@YAPAUWzMatrix@@PAU1@PBUWzVector@@@Z 10022d84 f   common:wzmath.obj
 0001:00021f4d       ?MatrixMultiply_Scalar@@YAPAUWzMatrix@@PAU1@PBU1@1@Z 10022f4d f   common:wzmath.obj
 0001:0002230c       ?MatrixMultiply4x3_Scalar@@YAPAUWzMatrix@@PAU1@PBU1@1@Z 1002330c f   common:wzmath.obj
 0001:00022586       ?MatrixRotationX_SSE@@YAPAUWzMatrix@@PAU1@M@Z 10023586 f   common:wzmath.obj
 0001:000225bd       ?MatrixRotationY_SSE@@YAPAUWzMatrix@@PAU1@M@Z 100235bd f   common:wzmath.obj
 0001:000225f1       ?MatrixRotationZ_SSE@@YAPAUWzMatrix@@PAU1@M@Z 100235f1 f   common:wzmath.obj
 0001:00022625       ?MatrixMultiply_SSE@@YAPAUWzMatrix@@PAU1@PBU1@1@Z 10023625 f   common:wzmath.obj
 0001:00022740       ?MatrixRotationX_3DNOW@@YAPAUWzMatrix@@PAU1@M@Z 10023740 f   common:wzmath.obj
 0001:0002278b       ?MatrixRotationY_3DNOW@@YAPAUWzMatrix@@PAU1@M@Z 1002378b f   common:wzmath.obj
 0001:000227d3       ?MatrixRotationZ_3DNOW@@YAPAUWzMatrix@@PAU1@M@Z 100237d3 f   common:wzmath.obj
 0001:0002281b       ?MatrixMultiply_3DNOW@@YAPAUWzMatrix@@PAU1@PBU1@1@Z 1002381b f   common:wzmath.obj
 0001:000229df       ?RotationToQuaternion@@YAPAUWzQuaternion@@PAU1@PBUWzVector@@@Z 100239df f   common:wzmath.obj
 0001:00022ae3       ?GetQuaternionToConvertVector@@YAPAUWzQuaternion@@PAU1@PBUWzVector@@1@Z 10023ae3 f   common:wzmath.obj
 0001:00022c2c       ?MatrixToQuaternion@@YAPAUWzQuaternion@@PAU1@PBUWzMatrix@@@Z 10023c2c f   common:wzmath.obj
 0001:00022e0d       ?QuaternionToAxisAngle@@YAXPAUWzVector@@PAMPBUWzQuaternion@@@Z 10023e0d f   common:wzmath.obj
 0001:00022f03       ?QuaternionSlerp@@YAPAUWzQuaternion@@PAU1@PBU1@1M@Z 10023f03 f   common:wzmath.obj
 0001:00023079       ?QuaternionMultiply_SSE@@YAPAUWzQuaternion@@PAU1@PBU1@1@Z 10024079 f   common:wzmath.obj
 0001:000230eb       ?QuaternionMultiply_3DNOWEXT@@YAPAUWzQuaternion@@PAU1@PBU1@1@Z 100240eb f   common:wzmath.obj
 0001:00023194       ?MatrixSetZero@@YAPAUWzMatrix@@PAU1@@Z 10024194 f i common:wzmath.obj
 0001:0002329b       ?QuaternionRotation@@YAPAUWzQuaternion@@PAU1@PBUWzVector@@M@Z 1002429b f i common:wzmath.obj
 0001:0002331e       ?TransformRay@@YAPAUWzRay@@PAU1@PBU1@PBUWzMatrix@@@Z 1002431e f   common:boundingvolume.obj
 0001:00023363       ?Generate_Frustum@@YAPAUWzFrustum@@PAU1@ABUWzVector@@111MMMM@Z 10024363 f   common:boundingvolume.obj
 0001:00023697       ?Generate_Frustum_Orthogonal@@YAPAUWzFrustum@@PAU1@ABUWzVector@@111MMMMMM@Z 10024697 f   common:boundingvolume.obj
 0001:00023871       ?CutTriangleWithFrustum@@YAHPAUWzVector@@PAHPBU1@PBUWzFrustum@@@Z 10024871 f   common:boundingvolume.obj
 0001:0002397d       ?Intersect_Ray_Triangle@@YAGPBUWzRay@@PBUWzVector@@11PAMH@Z 1002497d f   common:boundingvolume.obj
 0001:00023b61       ?Intersect_Ray_TriangleList@@YAHPBUWzRay@@PBUWzVector@@HPAMHH@Z 10024b61 f   common:boundingvolume.obj
 0001:00023c2a       ?Intersect_Ray_TriangleListIndexed@@YAHPBUWzRay@@PBUWzVector@@PBHHPAMHHPAU2@@Z 10024c2a f   common:boundingvolume.obj
 0001:00023d9d       ?Intersect_Ray_Plane@@YAGPBUWzRay@@PBUWzPlane@@PAM@Z 10024d9d f   common:boundingvolume.obj
 0001:00023e00       ?Intersect_Ray_AABB@@YAGPBUWzRay@@PBUBvAABB@@PAM@Z 10024e00 f   common:boundingvolume.obj
 0001:00023f82       ?Intersect_Ray_Sphere@@YAGPBUWzRay@@PBUBvSphere@@PAM@Z 10024f82 f   common:boundingvolume.obj
 0001:0002404c       ?Intersect_Ray_Bv@@YAGPBUWzRay@@PBUWzBoundingVolume@@PAM@Z 1002504c f   common:boundingvolume.obj
 0001:00024098       ?Intersect_Frustum_AABB@@YAGPBUWzFrustum@@PBUBvAABB@@@Z 10025098 f   common:boundingvolume.obj
 0001:00024213       ?Intersect_Frustum_Sphere@@YAGPBUWzFrustum@@PBUBvSphere@@@Z 10025213 f   common:boundingvolume.obj
 0001:0002428d       ?Intersect_AABB_AABB@@YAGPBUBvAABB@@0@Z 1002528d f   common:boundingvolume.obj
 0001:00024399       ?Intersect_AABB_Sphere@@YAGPBUBvAABB@@PBUBvSphere@@@Z 10025399 f   common:boundingvolume.obj
 0001:00024497       ?Intersect_Sphere_AABB@@YAGPBUBvSphere@@PBUBvAABB@@@Z 10025497 f   common:boundingvolume.obj
 0001:00024747       ?Intersect_Sphere_Sphere@@YAGPBUBvSphere@@0@Z 10025747 f   common:boundingvolume.obj
 0001:000247be       ?Intersect_Bv_Bv@@YAGPBUWzBoundingVolume@@0@Z 100257be f   common:boundingvolume.obj
 0001:0002486b       ?Contain_AABB_AABB@@YAHPBUBvAABB@@0@Z 1002586b f   common:boundingvolume.obj
 0001:000248f5       ?Contain_AABB_Sphere@@YAHPBUBvAABB@@PBUBvSphere@@@Z 100258f5 f   common:boundingvolume.obj
 0001:00024954       ?Contain_Sphere_AABB@@YAHPBUBvSphere@@PBUBvAABB@@@Z 10025954 f   common:boundingvolume.obj
 0001:00024989       ?Contain_Sphere_Sphere@@YAHPBUBvSphere@@0@Z 10025989 f   common:boundingvolume.obj
 0001:000249d2       ?Contain_Bv_Bv@@YAHPBUWzBoundingVolume@@0@Z 100259d2 f   common:boundingvolume.obj
 0001:00024a7f       ?Generate_BvAABB@@YAXPAUBvAABB@@PBUWzVector@@HH@Z 10025a7f f   common:boundingvolume.obj
 0001:00024b8a       ?Generate_BvAABB@@YAXPAUBvAABB@@PBUWzVector@@PBHHH@Z 10025b8a f   common:boundingvolume.obj
 0001:00024c9b       ?Generate_BvSphere@@YAXPAUBvSphere@@PBUWzVector@@HH@Z 10025c9b f   common:boundingvolume.obj
 0001:00025021       ?Generate_BvSphere@@YAXPAUBvSphere@@PBUWzVector@@PBHHH@Z 10026021 f   common:boundingvolume.obj
 0001:000253b3       ?VectorTransformNormal@@YAPAUWzVector@@PAU1@PBU1@PBUWzMatrix@@@Z 100263b3 f i common:boundingvolume.obj
 0001:00025440       ?Distance_Plane_Vertex@@YAMPBUWzPlane@@ABUWzVector@@@Z 10026440 f i common:boundingvolume.obj
 0001:00025478       ?Contain_Sphere_Vertex@@YAHPBUBvSphere@@ABUWzVector@@@Z 10026478 f i common:boundingvolume.obj
 0001:000254be       ?Math_GetOrthogonalVectors@@YAXPAUWzVector@@0PBU1@@Z 100264be f   common:mathassistant.obj
 0001:00025530       ?Math_GetRandomDirection@@YAPAUWzVector@@PAU1@PBU1@M@Z 10026530 f   common:mathassistant.obj
 0001:00025644       ?Math_GetRandomPosInBoundingVolume@@YAXPAUWzVector@@PBUWzBoundingVolume@@@Z 10026644 f   common:mathassistant.obj
 0001:0002576e       ?Math_GetRandomFloatBetween@@YAMMM@Z 1002676e f i common:mathassistant.obj
 0001:000257a4       ?CutPolygonWithPlane@@YAHPAUWzVector@@PAHPBU1@HPBUWzPlane@@@Z 100267a4 f   common:wzutil.obj
 0001:0002593e       ?As2D_TestCrossTwoSegment@@YAHPBUWzVector@@000PAH@Z 1002693e f   common:wzutil.obj
 0001:00025a79       ?As2D_GetLine@@YAPAUWzVector@@PAU1@PBU1@1@Z 10026a79 f i common:wzutil.obj
 0001:00025b19       ?As2D_Distance_Line_Vertex@@YAMPBUWzVector@@ABU1@@Z 10026b19 f i common:wzutil.obj
 0001:00025b43       ?As2D_GetCrossPointOfTwoLine@@YAPAUWzVector@@PAU1@PBU1@1@Z 10026b43 f i common:wzutil.obj
 0001:00025c8b       ?GetModuleTitle@?A0x5958724f@WzLog@@YAPBDXZ 10026c8b f   programcommonlibforengine:wzlogsystem.obj
 0001:00025d4a       ??0WzLogSystem@WzLog@@QAE@XZ 10026d4a f   programcommonlibforengine:wzlogsystem.obj
 0001:00025d98       ??1WzLogSystem@WzLog@@UAE@XZ 10026d98 f   programcommonlibforengine:wzlogsystem.obj
 0001:00025dba       ?AddLogHandler@WzLogSystem@WzLog@@QAEXPAVWzLogHandler@2@@Z 10026dba f   programcommonlibforengine:wzlogsystem.obj
 0001:00025dff       ?Initialize@WzLogSystem@WzLog@@QAEXXZ 10026dff f   programcommonlibforengine:wzlogsystem.obj
 0001:00025e5f       ?Release@WzLogSystem@WzLog@@QAEXXZ 10026e5f f   programcommonlibforengine:wzlogsystem.obj
 0001:00025e8b       ?WriteLog@WzLogSystem@WzLog@@QAEXW4WZLOG_TYPE@WzLogType@@PBD@Z 10026e8b f   programcommonlibforengine:wzlogsystem.obj
 0001:00025ed4       ?InitializeWzLogSystem@@YAXXZ 10026ed4 f   programcommonlibforengine:wzlogsystem.obj
 0001:00025f4f       ?ReleaseWzLogSystem@@YAXXZ 10026f4f f   programcommonlibforengine:wzlogsystem.obj
 0001:00025f94       ?AddWzLogHandler@@YAXPAVWzLogHandler@WzLog@@@Z 10026f94 f   programcommonlibforengine:wzlogsystem.obj
 0001:00025fb3       ?OutputWzLog@@YAXW4WZLOG_TYPE@WzLogType@@PBDZZ 10026fb3 f   programcommonlibforengine:wzlogsystem.obj
 0001:00026002       ??_GWzLogSystem@WzLog@@UAEPAXI@Z 10027002 f i programcommonlibforengine:wzlogsystem.obj
 0001:00026002       ??_EWzLogSystem@WzLog@@UAEPAXI@Z 10027002 f i programcommonlibforengine:wzlogsystem.obj
 0001:00026029       ??_G?$CWzSingleton@VWzLogSystem@WzLog@@@@UAEPAXI@Z 10027029 f i programcommonlibforengine:wzlogsystem.obj
 0001:00026029       ??_E?$CWzSingleton@VWzLogSystem@WzLog@@@@UAEPAXI@Z 10027029 f i programcommonlibforengine:wzlogsystem.obj
 0001:00026058       ??0CWzArchive@@QAE@XZ      10027058 f   programcommonlibforengine:wzarchive.obj
 0001:000260ca       ??1CWzArchive@@QAE@XZ      100270ca f   programcommonlibforengine:wzarchive.obj
 0001:00026120       ?CreateDiscAccess@CWzArchive@@AAEXXZ 10027120 f   programcommonlibforengine:wzarchive.obj
 0001:000261a2       ?ReleaseDiscAccess@CWzArchive@@AAEXXZ 100271a2 f   programcommonlibforengine:wzarchive.obj
 0001:00026204       ?Clear@CWzArchive@@AAEXXZ  10027204 f   programcommonlibforengine:wzarchive.obj
 0001:00026260       ?SetDiscAccess@CWzArchive@@QAEXPAVCDiscAccess@@@Z 10027260 f   programcommonlibforengine:wzarchive.obj
 0001:00026282       ?GetDiscAccess@CWzArchive@@QAEXPAPAVCDiscAccess@@@Z 10027282 f   programcommonlibforengine:wzarchive.obj
 0001:00026297       ?LoadFile@CWzArchive@@QAEHPBD@Z 10027297 f   programcommonlibforengine:wzarchive.obj
 0001:000263c6       ?LoadFile@CWzArchive@@QAEHPBDPAEH@Z 100273c6 f   programcommonlibforengine:wzarchive.obj
 0001:00026457       ?SaveFile@CWzArchive@@QAEHPBD@Z 10027457 f   programcommonlibforengine:wzarchive.obj
 0001:00026500       ?SaveFile@CWzArchive@@QAEHPBDPAX@Z 10027500 f   programcommonlibforengine:wzarchive.obj
 0001:00026574       ?Close@CWzArchive@@QAEXXZ  10027574 f   programcommonlibforengine:wzarchive.obj
 0001:000265fe       ?Read@CWzArchive@@QAEIPAXI@Z 100275fe f   programcommonlibforengine:wzarchive.obj
 0001:0002666d       ?Write@CWzArchive@@QAEIPBXI@Z 1002766d f   programcommonlibforengine:wzarchive.obj
 0001:0002669b       ?ReadName@CWzArchive@@QAEIPADPAPAD@Z 1002769b f   programcommonlibforengine:wzarchive.obj
 0001:000267ce       ?WriteName@CWzArchive@@QAEIPBD@Z 100277ce f   programcommonlibforengine:wzarchive.obj
 0001:00026848       ?WriteText@CWzArchive@@QAAXPBDZZ 10027848 f   programcommonlibforengine:wzarchive.obj
 0001:000268ea       ?WriteHexText@CWzArchive@@QAEXPBXH@Z 100278ea f   programcommonlibforengine:wzarchive.obj
 0001:00026b12       ?Seek@CWzArchive@@QAEKJW4ENUM_SEEK_ORIGIN@@@Z 10027b12 f   programcommonlibforengine:wzarchive.obj
 0001:00026ba4       ?SetBeginningOfChunk@CWzArchive@@QAEXG@Z 10027ba4 f   programcommonlibforengine:wzarchive.obj
 0001:00026bef       ?SetEndOfChunk@CWzArchive@@QAEXXZ 10027bef f   programcommonlibforengine:wzarchive.obj
 0001:00026c51       ?ReadChunk@CWzArchive@@QAE?AUSt_ChunkInfo@@XZ 10027c51 f   programcommonlibforengine:wzarchive.obj
 0001:00026c86       ?SkipCurrentChunk@CWzArchive@@QAEXUSt_ChunkInfo@@@Z 10027c86 f   programcommonlibforengine:wzarchive.obj
 0001:00026ca8       ??0?$CWzList@USt_ChunkStack@@@@QAE@XZ 10027ca8 f i programcommonlibforengine:wzarchive.obj
 0001:00026d6d       ??1?$CWzList@USt_ChunkStack@@@@UAE@XZ 10027d6d f i programcommonlibforengine:wzarchive.obj
 0001:00026e0d       ?AddTail@?$CWzList@USt_ChunkStack@@@@QAEPAV?$CWzNode@USt_ChunkStack@@@@ABUSt_ChunkStack@@@Z 10027e0d f i programcommonlibforengine:wzarchive.obj
 0001:00026ed1       ?RemoveTail@?$CWzList@USt_ChunkStack@@@@QAE?AUSt_ChunkStack@@XZ 10027ed1 f i programcommonlibforengine:wzarchive.obj
 0001:00026fa5       ?RemoveAll@?$CWzList@USt_ChunkStack@@@@QAEXXZ 10027fa5 f i programcommonlibforengine:wzarchive.obj
 0001:00027043       ??_E?$CWzList@USt_ChunkStack@@@@UAEPAXI@Z 10028043 f i programcommonlibforengine:wzarchive.obj
 0001:00027043       ??_G?$CWzList@USt_ChunkStack@@@@UAEPAXI@Z 10028043 f i programcommonlibforengine:wzarchive.obj
 0001:0002706a       ?Write@@YAXPAXPBDZZ        1002806a f   programcommonlibforengine:filenbuffer.obj
 0001:00027115       ?HexWrite@@YAXPAXPBXH@Z    10028115 f   programcommonlibforengine:filenbuffer.obj
 0001:00027344       ?GetFloatString@@YAXPADMH@Z 10028344 f   programcommonlibforengine:filenbuffer.obj
 0001:0002738b       ?GetFromBuffer@@YAHPAXPBEHHPAH@Z 1002838b f   programcommonlibforengine:filenbuffer.obj
 0001:000273c8       ?GetFolderOfFilePath@@YAHPADPBD@Z 100283c8 f   programcommonlibforengine:filenbuffer.obj
 0001:000273f8       ?GetFileNameOfFilePath@@YAHPADPBD@Z 100283f8 f   programcommonlibforengine:filenbuffer.obj
 0001:00027469       ??0CDiscAccess@@QAE@XZ     10028469 f   programcommonlibforengine:discaccess.obj
 0001:000274f2       ??1CDiscAccess@@QAE@XZ     100284f2 f   programcommonlibforengine:discaccess.obj
 0001:00027568       ?Create@CDiscAccess@@QAEHXZ 10028568 f   programcommonlibforengine:discaccess.obj
 0001:0002759a       ?Destroy@CDiscAccess@@QAEXXZ 1002859a f   programcommonlibforengine:discaccess.obj
 0001:000275d1       ?OpenDisc_Hard@CDiscAccess@@QAEHKPBD@Z 100285d1 f   programcommonlibforengine:discaccess.obj
 0001:000276e6       ?OpenDisc_Packer@CDiscAccess@@QAEHKPBD0W4ENUM_OPEN_PACKER_TYPE@@@Z 100286e6 f   programcommonlibforengine:discaccess.obj
 0001:0002795e       ?CloseDisc@CDiscAccess@@QAEXK@Z 1002895e f   programcommonlibforengine:discaccess.obj
 0001:00027a7f       ?SetActiveDisc@CDiscAccess@@QAEHK@Z 10028a7f f   programcommonlibforengine:discaccess.obj
 0001:00027b2d       ?GetActiveDisc@CDiscAccess@@QAEKXZ 10028b2d f   programcommonlibforengine:discaccess.obj
 0001:00027b78       ?FixFileName@CDiscAccess@@AAEXPADPBD@Z 10028b78 f   programcommonlibforengine:discaccess.obj
 0001:00027c29       ?OpenFile@CDiscAccess@@QAEPAXKPBDKKW4ENUM_OPEN_DISPOSITION@@@Z 10028c29 f   programcommonlibforengine:discaccess.obj
 0001:0002802c       ?CloseFile@CDiscAccess@@QAEHPAX@Z 1002902c f   programcommonlibforengine:discaccess.obj
 0001:00028192       ?SeekFile@CDiscAccess@@QAEKPAXJW4ENUM_SEEK_ORIGIN@@@Z 10029192 f   programcommonlibforengine:discaccess.obj
 0001:00028347       ?ReadFile@CDiscAccess@@QAEKPAX0K@Z 10029347 f   programcommonlibforengine:discaccess.obj
 0001:000284d8       ?WriteFile@CDiscAccess@@QAEKPAXPBXK@Z 100294d8 f   programcommonlibforengine:discaccess.obj
 0001:00028669       ?FileExists@CDiscAccess@@QAEHKPBD@Z 10029669 f   programcommonlibforengine:discaccess.obj
 0001:000289e8       ?GetFileSize@CDiscAccess@@QAEKPAX@Z 100299e8 f   programcommonlibforengine:discaccess.obj
 0001:00028b3d       ?GetFileInformationByHandle@CDiscAccess@@QAEHPAXPAUSt_FileInformation@@@Z 10029b3d f   programcommonlibforengine:discaccess.obj
 0001:00028dee       ?CopyFileA@CDiscAccess@@QAEHKPBD0@Z 10029dee f   programcommonlibforengine:discaccess.obj
 0001:00029096       ?DeleteFileA@CDiscAccess@@QAEHKPBD@Z 1002a096 f   programcommonlibforengine:discaccess.obj
 0001:00029336       ?CreateDirectoryA@CDiscAccess@@QAEHKPBD@Z 1002a336 f   programcommonlibforengine:discaccess.obj
 0001:000295d8       ?RemoveDirectoryA@CDiscAccess@@QAEHKPBD@Z 1002a5d8 f   programcommonlibforengine:discaccess.obj
 0001:00029878       ??1CWzCriticalSection@@QAE@XZ 1002a878 f i programcommonlibforengine:discaccess.obj
 0001:00029893       ??0?$CWzHandleManager@USt_DAFileInfo@@@@QAE@XZ 1002a893 f i programcommonlibforengine:discaccess.obj
 0001:0002991f       ??1?$CWzHandleManager@USt_DAFileInfo@@@@UAE@XZ 1002a91f f i programcommonlibforengine:discaccess.obj
 0001:0002998b       ?Add@?$CWzHandleManager@USt_DAFileInfo@@@@QAEPAXABUSt_DAFileInfo@@@Z 1002a98b f i programcommonlibforengine:discaccess.obj
 0001:00029a5f       ?Release@?$CWzHandleManager@USt_DAFileInfo@@@@QAEHPAX@Z 1002aa5f f i programcommonlibforengine:discaccess.obj
 0001:00029b0b       ?GetData@?$CWzHandleManager@USt_DAFileInfo@@@@QBEABUSt_DAFileInfo@@PAX@Z 1002ab0b f i programcommonlibforengine:discaccess.obj
 0001:00029b43       ?IsValidHandle@?$CWzHandleManager@PAUSt_WzdContainer@@@@QBEHPAX@Z 1002ab43 f i wzanistate.obj
 0001:00029b43       ?IsValidHandle@?$CWzHandleManager@USt_DAFileInfo@@@@QBEHPAX@Z 1002ab43 f i programcommonlibforengine:discaccess.obj
 0001:00029b92       ??_G?$CWzHandleManager@USt_DAFileInfo@@@@UAEPAXI@Z 1002ab92 f i programcommonlibforengine:discaccess.obj
 0001:00029b92       ??_E?$CWzHandleManager@USt_DAFileInfo@@@@UAEPAXI@Z 1002ab92 f i programcommonlibforengine:discaccess.obj
 0001:00029bb9       ?Clear@?$CWzHandleManager@USt_DAFileInfo@@@@QAEXXZ 1002abb9 f i programcommonlibforengine:discaccess.obj
 0001:00029bff       ??0?$CWzArray@USt_DAFileInfo@@@@QAE@XZ 1002abff f i programcommonlibforengine:discaccess.obj
 0001:00029c68       ??1?$CWzArray@PAUWzMappingInfo@@@@QAE@XZ 1002ac68 f i wzunit.obj
 0001:00029c68       ??1?$CWzArray@K@@QAE@XZ    1002ac68 f i wzunit.obj
 0001:00029c68       ??1?$CWzArray@PAUBvAABB@@@@QAE@XZ 1002ac68 f i wzanimationInfo.obj
 0001:00029c68       ??1?$CWzArray@USt_DAFileInfo@@@@QAE@XZ 1002ac68 f i programcommonlibforengine:discaccess.obj
 0001:00029c68       ??1?$CWzArray@PAUWzUnitEffectInfo@@@@QAE@XZ 1002ac68 f i wzunitdraw.obj
 0001:00029c68       ??1?$CWzArray@PAVCWzUnitSubType@@@@QAE@XZ 1002ac68 f i wzunit.obj
 0001:00029c68       ??1?$CWzArray@G@@QAE@XZ    1002ac68 f i programcommonlibforengine:discaccess.obj
 0001:00029c68       ??1?$CWzArray@PAUWzTexAniMappingInfo@@@@QAE@XZ 1002ac68 f i wzunit.obj
 0001:00029c68       ??1?$CWzArray@PAUWzBVExtraInfo@@@@QAE@XZ 1002ac68 f i wzunit.obj
 0001:00029c68       ??1?$CWzArray@PAUWzTexAniSetInfo@@@@QAE@XZ 1002ac68 f i wzunit.obj
 0001:00029c68       ??1?$CWzArray@PAUWzBoneInfo@@@@QAE@XZ 1002ac68 f i wzunit.obj
 0001:00029c68       ??1?$CWzArray@PAVWzAnimationInfo@@@@QAE@XZ 1002ac68 f i wzunit.obj
 0001:00029c68       ??1?$CWzArray@PAUMeshGroupNameInfo@@@@QAE@XZ 1002ac68 f i wzunit.obj
 0001:00029c79       ?Set@?$CWzArray@USt_DAFileInfo@@@@QAEXHABUSt_DAFileInfo@@@Z 1002ac79 f i programcommonlibforengine:discaccess.obj
 0001:00029cce       ?Get@?$CWzArray@USt_DAFileInfo@@@@QBEAAUSt_DAFileInfo@@H@Z 1002acce f i programcommonlibforengine:discaccess.obj
 0001:00029cfd       ??0?$CWzArray@G@@QAE@XZ    1002acfd f i programcommonlibforengine:discaccess.obj
 0001:00029d65       ?Set@?$CWzArray@G@@QAEXHABG@Z 1002ad65 f i programcommonlibforengine:discaccess.obj
 0001:00029db3       ?Clear@?$CWzArray@USt_DAFileInfo@@@@QAEXXZ 1002adb3 f i programcommonlibforengine:discaccess.obj
 0001:00029ddc       ?MakeSureDimensionSize@?$CWzArray@USt_DAFileInfo@@@@AAEXH@Z 1002addc f i programcommonlibforengine:discaccess.obj
 0001:00029eaa       ?Release@?$CWzArray@G@@AAEXXZ 1002aeaa f i programcommonlibforengine:discaccess.obj
 0001:00029eaa       ?Release@?$CWzArray@PAVCWzUnitSubType@@@@AAEXXZ 1002aeaa f i wzunit.obj
 0001:00029eaa       ?Release@?$CWzArray@PAUMeshGroupNameInfo@@@@AAEXXZ 1002aeaa f i wzunit.obj
 0001:00029eaa       ?Release@?$CWzArray@PAUWzBVExtraInfo@@@@AAEXXZ 1002aeaa f i wzunit.obj
 0001:00029eaa       ?Release@?$CWzArray@PAUWzTexAniMappingInfo@@@@AAEXXZ 1002aeaa f i wzunit.obj
 0001:00029eaa       ?Release@?$CWzArray@PAUWzBoneInfo@@@@AAEXXZ 1002aeaa f i wzunit.obj
 0001:00029eaa       ?Release@?$CWzArray@PAUWzUnitEffectInfo@@@@AAEXXZ 1002aeaa f i wzunitdraw.obj
 0001:00029eaa       ?Release@?$CWzArray@PAUWzMappingInfo@@@@AAEXXZ 1002aeaa f i wzunit.obj
 0001:00029eaa       ?Release@?$CWzArray@K@@AAEXXZ 1002aeaa f i wzunit.obj
 0001:00029eaa       ?Release@?$CWzArray@USt_DAFileInfo@@@@AAEXXZ 1002aeaa f i programcommonlibforengine:discaccess.obj
 0001:00029eaa       ?Release@?$CWzArray@PAVWzAnimationInfo@@@@AAEXXZ 1002aeaa f i wzunit.obj
 0001:00029eaa       ?Release@?$CWzArray@PAUBvAABB@@@@AAEXXZ 1002aeaa f i wzanimationInfo.obj
 0001:00029eaa       ?Release@?$CWzArray@PAUWzTexAniSetInfo@@@@AAEXXZ 1002aeaa f i wzunit.obj
 0001:00029ee3       ?Clear@?$CWzArray@G@@QAEXXZ 1002aee3 f i programcommonlibforengine:discaccess.obj
 0001:00029f0b       ?MakeSureDimensionSize@?$CWzArray@G@@AAEXH@Z 1002af0b f i programcommonlibforengine:discaccess.obj
 0001:00029fd7       ??_U@YAPAXI@Z              1002afd7 f   libcpmt:newaop.obj
 0001:00029fe2       ??0length_error@std@@QAE@ABV?$basic_string@DU?$char_traits@D@std@@V?$allocator@D@2@@1@@Z 1002afe2 f i libcpmt:string.obj
 0001:00029fff       ??0out_of_range@std@@QAE@ABV?$basic_string@DU?$char_traits@D@std@@V?$allocator@D@2@@1@@Z 1002afff f i libcpmt:string.obj
 0001:0002a01c       ?_Xlen@_String_base@std@@SAXXZ 1002b01c f   libcpmt:string.obj
 0001:0002a054       ?_Xran@_String_base@std@@SAXXZ 1002b054 f   libcpmt:string.obj
 0001:0002a08c       __initp_misc_winxfltr      1002b08c f   LIBCMT:winxfltr.obj
 0001:0002a08c       __fpclear                  1002b08c f   LIBCMT:_fpinit_.obj
 0001:0002a08d       __cfltcvt_init             1002b08d f   LIBCMT:_fpinit_.obj
 0001:0002a0ed       __fpmath                   1002b0ed f   LIBCMT:_fpinit_.obj
 0001:0002a110       ??3@YAXPAX@Z               1002b110 f   LIBCMT:delete.obj
 0001:0002a11b       ??_V@YAXPAX@Z              1002b11b f   LIBCMT:delete2.obj
 0001:0002a126       ??0bad_alloc@std@@QAE@XZ   1002b126 f i LIBCMT:new.obj
 0001:0002a141       ??2@YAPAXI@Z               1002b141 f   LIBCMT:new.obj
 0001:0002a260       ___onexitinit              1002b260 f   LIBCMT:onexit.obj
 0001:0002a291       __onexit                   1002b291 f   LIBCMT:onexit.obj
 0001:0002a2cd       _atexit                    1002b2cd f   LIBCMT:onexit.obj
 0001:0002a2e4       ?_JumpToContinuation@@YGXPAXPAUEHRegistrationNode@@@Z 1002b2e4 f   LIBCMT:_trnsctrl_.obj
 0001:0002a316       ?_CallMemberFunction0@@YGXPAX0@Z 1002b316 f   LIBCMT:_trnsctrl_.obj
 0001:0002a316       ?_CallMemberFunction2@@YGXPAX00H@Z 1002b316 f   LIBCMT:_trnsctrl_.obj
 0001:0002a316       ?_CallMemberFunction1@@YGXPAX00@Z 1002b316 f   LIBCMT:_trnsctrl_.obj
 0001:0002a31d       ?_UnwindNestedFrames@@YGXPAUEHRegistrationNode@@PAUEHExceptionRecord@@@Z 1002b31d f   LIBCMT:_trnsctrl_.obj
 0001:0002a371       ___CxxFrameHandler3        1002b371 f   LIBCMT:_trnsctrl_.obj
 0001:0002a3da       ?_CallSETranslator@@YAHPAUEHExceptionRecord@@PAUEHRegistrationNode@@PAX2PBU_s_FuncInfo@@H1@Z 1002b3da f   LIBCMT:_trnsctrl_.obj
 0001:0002a550       ?_GetRangeOfTrysToCheck@@YAPBU_s_TryBlockMapEntry@@PBU_s_FuncInfo@@HHPAI1@Z 1002b550 f   LIBCMT:_trnsctrl_.obj
 0001:0002a5c5       __CreateFrameInfo          1002b5c5 f   LIBCMT:_trnsctrl_.obj
 0001:0002a5f1       __IsExceptionObjectToBeDestroyed 1002b5f1 f   LIBCMT:_trnsctrl_.obj
 0001:0002a618       __FindAndUnlinkFrame       1002b618 f   LIBCMT:_trnsctrl_.obj
 0001:0002a66a       ?_CallCatchBlock2@@YAPAXPAUEHRegistrationNode@@PBU_s_FuncInfo@@PAXHK@Z 1002b66a f   LIBCMT:_trnsctrl_.obj
 0001:0002a6ca       @__security_check_cookie@4 1002b6ca f   LIBCMT:secchk.obj
 0001:0002a6d9       ??1type_info@@UAE@XZ       1002b6d9 f   LIBCMT:typinfo.obj
 0001:0002a6e9       ??_Etype_info@@UAEPAXI@Z   1002b6e9 f i LIBCMT:typinfo.obj
 0001:0002a6e9       ??_Gtype_info@@UAEPAXI@Z   1002b6e9 f i LIBCMT:typinfo.obj
 0001:0002a70a       ??8type_info@@QBE_NABV0@@Z 1002b70a f   LIBCMT:typinfo.obj
 0001:0002a72a       ?__ArrayUnwind@@YGXPAXIHP6EX0@Z@Z 1002b72a f   LIBCMT:ehvecdtr.obj
 0001:0002a788       ??_M@YGXPAXIHP6EX0@Z@Z     1002b788 f   LIBCMT:ehvecdtr.obj
 0001:0002a7f0       _memset                    1002b7f0 f   LIBCMT:memset.obj
 0001:0002a86a       ??_L@YGXPAXIHP6EX0@Z1@Z    1002b86a f   LIBCMT:ehvecctr.obj
 0001:0002a8cf       __initp_misc_invarg        1002b8cf f   LIBCMT:invarg.obj
 0001:0002a8de       __invoke_watson            1002b8de f   LIBCMT:invarg.obj
 0001:0002aa06       __invalid_parameter        1002ba06 f   LIBCMT:invarg.obj
 0001:0002aa2c       __invalid_parameter_noinfo 1002ba2c f   LIBCMT:invarg.obj
 0001:0002aa3c       __purecall                 1002ba3c f   LIBCMT:purevirt.obj
 0001:0002aa70       _strncpy                   1002ba70 f   LIBCMT:strncpy.obj
 0001:0002aba0       _memcpy                    1002bba0 f   LIBCMT:memcpy.obj
 0001:0002af05       ??0_LocaleUpdate@@QAE@PAUlocaleinfo_struct@@@Z 1002bf05 f i LIBCMT:stricmp.obj
 0001:0002af8c       ___ascii_stricmp           1002bf8c f   LIBCMT:stricmp.obj
 0001:0002afc5       __stricmp_l                1002bfc5 f   LIBCMT:stricmp.obj
 0001:0002b09a       __stricmp                  1002c09a f   LIBCMT:stricmp.obj
 0001:0002b09a       _stricmp                   1002c09a f   LIBCMT:stricmp.obj
 0001:0002b0f0       __CIsqrt                   1002c0f0 f   LIBCMT:_sqrt_.obj
 0001:0002b104       _sqrt                      1002c104     LIBCMT:_sqrt_.obj
 0001:0002b1aa       __strnicmp_l               1002c1aa f   LIBCMT:strnicmp.obj
 0001:0002b29c       __strnicmp                 1002c29c f   LIBCMT:strnicmp.obj
 0001:0002b2fa       __CxxThrowException@8      1002c2fa f   LIBCMT:throw.obj
 0001:0002b346       ??0exception@std@@QAE@XZ   1002c346 f   LIBCMT:stdexcpt.obj
 0001:0002b357       ??0exception@std@@QAE@ABQBD@Z 1002c357 f   LIBCMT:stdexcpt.obj
 0001:0002b3aa       ??0exception@std@@QAE@ABQBDH@Z 1002c3aa f   LIBCMT:stdexcpt.obj
 0001:0002b3c7       ??0exception@std@@QAE@ABV01@@Z 1002c3c7 f   LIBCMT:stdexcpt.obj
 0001:0002b424       ??1exception@std@@UAE@XZ   1002c424 f   LIBCMT:stdexcpt.obj
 0001:0002b43a       ?what@exception@std@@UBEPBDXZ 1002c43a f   LIBCMT:stdexcpt.obj
 0001:0002b447       ??_Eexception@std@@UAEPAXI@Z 1002c447 f i LIBCMT:stdexcpt.obj
 0001:0002b447       ??_Gexception@std@@UAEPAXI@Z 1002c447 f i LIBCMT:stdexcpt.obj
 0001:0002b468       _memcpy_s                  1002c468 f   LIBCMT:memcpy_s.obj
 0001:0002b4e5       _memmove_s                 1002c4e5 f   LIBCMT:memmove_s.obj
 0001:0002b550       __ftol2_sse                1002c550 f   LIBCMT:ftol2.obj
 0001:0002b559       __ftol2_pentium4           1002c559 f   LIBCMT:ftol2.obj
 0001:0002b56c       __ftol2_sse_excpt          1002c56c f   LIBCMT:ftol2.obj
 0001:0002b586       __ftol2                    1002c586 f   LIBCMT:ftol2.obj
 0001:0002b5fb       _rand                      1002c5fb f   LIBCMT:rand.obj
 0001:0002b620       _memmove                   1002c620 f   LIBCMT:memmove.obj
 0001:0002b985       __CRT_INIT@12              1002c985 f   LIBCMT:dllcrt0.obj
 0001:0002bbb0       __DllMainCRTStartup@12     1002cbb0 f   LIBCMT:dllcrt0.obj
 0001:0002bbe0       __except_handler4          1002cbe0 f   LIBCMT:chandler4.obj
 0001:0002bd70       _sin                       1002cd70 f   LIBCMT:_sin_.obj
 0001:0002bdb0       __CIsin                    1002cdb0 f   LIBCMT:_sin_.obj
 0001:0002bdeb       __CIsin_default            1002cdeb f   LIBCMT:_sin_.obj
 0001:0002bdff       __sin_default              1002cdff     LIBCMT:_sin_.obj
 0001:0002bea0       _cos                       1002cea0 f   LIBCMT:_cos_.obj
 0001:0002bee0       __CIcos                    1002cee0 f   LIBCMT:_cos_.obj
 0001:0002bf1b       __CIcos_default            1002cf1b f   LIBCMT:_cos_.obj
 0001:0002bf2f       __cos_default              1002cf2f     LIBCMT:_cos_.obj
 0001:0002bfd0       _acos                      1002cfd0 f   LIBCMT:_acos_.obj
 0001:0002c010       __CIacos                   1002d010 f   LIBCMT:_acos_.obj
 0001:0002c04b       __CIacos_default           1002d04b f   LIBCMT:_acos_.obj
 0001:0002c05f       __acos_default             1002d05f     LIBCMT:_acos_.obj
 0001:0002c120       _strrchr                   1002d120 f   LIBCMT:strrchr.obj
 0001:0002c14d       __vsnprintf_l              1002d14d f   LIBCMT:vsnprint.obj
 0001:0002c200       __vsnprintf                1002d200 f   LIBCMT:vsnprint.obj
 0001:0002c21d       _sprintf                   1002d21d f   LIBCMT:sprintf.obj
 0001:0002c48c       __splitpath                1002d48c f   LIBCMT:splitpat.obj
 0001:0002c4e0       _strlen                    1002d4e0 f   LIBCMT:strlen.obj
 0001:0002c56b       __EH_prolog3               1002d56b f   LIBCMT:ehprolg3.obj
 0001:0002c59e       __EH_prolog3_catch         1002d59e f   LIBCMT:ehprolg3.obj
 0001:0002c5d4       __forcdecpt_l              1002d5d4 f   LIBCMT:cvt.obj
 0001:0002c647       __cropzeros_l              1002d647 f   LIBCMT:cvt.obj
 0001:0002c6c9       __positive                 1002d6c9 f   LIBCMT:cvt.obj
 0001:0002c6e5       __fassign_l                1002d6e5 f   LIBCMT:cvt.obj
 0001:0002c727       __fassign                  1002d727 f   LIBCMT:cvt.obj
 0001:0002c760       __forcdecpt                1002d760 f   LIBCMT:cvt.obj
 0001:0002c773       __cropzeros                1002d773 f   LIBCMT:cvt.obj
 0001:0002c8f5       __cftoe_l                  1002d8f5 f   LIBCMT:cvt.obj
 0001:0002c9c5       __cftoe                    1002d9c5 f   LIBCMT:cvt.obj
 0001:0002c9e5       __cftoa_l                  1002d9e5 f   LIBCMT:cvt.obj
 0001:0002ce4f       __cftof_l                  1002de4f f   LIBCMT:cvt.obj
 0001:0002cf0a       __cftog_l                  1002df0a f   LIBCMT:cvt.obj
 0001:0002d004       __cfltcvt_l                1002e004 f   LIBCMT:cvt.obj
 0001:0002d08c       __cfltcvt                  1002e08c f   LIBCMT:cvt.obj
 0001:0002d0af       __initp_misc_cfltcvt_tab   1002e0af f   LIBCMT:cmiscdat.obj
 0001:0002d0d0       __setdefaultprecision      1002e0d0 f   LIBCMT:fp8.obj
 0001:0002d0fb       __ms_p5_test_fdiv          1002e0fb f   LIBCMT:_testfdiv_.obj
 0001:0002d139       __ms_p5_mp_test_fdiv       1002e139 f   LIBCMT:_testfdiv_.obj
 0001:0002d162       _free                      1002e162 f   LIBCMT:free.obj
 0001:0002d1f0       _V6_HeapAlloc              1002e1f0 f   LIBCMT:malloc.obj
 0001:0002d23f       _malloc                    1002e23f f   LIBCMT:malloc.obj
 0001:0002d309       __initp_heap_handler       1002e309 f   LIBCMT:handler.obj
 0001:0002d318       __callnewh                 1002e318 f   LIBCMT:handler.obj
 0001:0002d340       __encode_pointer           1002e340 f   LIBCMT:tidtable.obj
 0001:0002d3b2       __encoded_null             1002e3b2 f   LIBCMT:tidtable.obj
 0001:0002d3bb       __decode_pointer           1002e3bb f   LIBCMT:tidtable.obj
 0001:0002d42d       ___crtTlsAlloc@4           1002e42d f   LIBCMT:tidtable.obj
 0001:0002d436       ___set_flsgetvalue         1002e436 f   LIBCMT:tidtable.obj
 0001:0002d46a       __mtterm                   1002e46a f   LIBCMT:tidtable.obj
 0001:0002d4a7       __initptd                  1002e4a7 f   LIBCMT:tidtable.obj
 0001:0002d58e       __getptd_noexit            1002e58e f   LIBCMT:tidtable.obj
 0001:0002d607       __getptd                   1002e607 f   LIBCMT:tidtable.obj
 0001:0002d621       __freefls@4                1002e621 f   LIBCMT:tidtable.obj
 0001:0002d750       __freeptd                  1002e750 f   LIBCMT:tidtable.obj
 0001:0002d7be       __mtinit                   1002e7be f   LIBCMT:tidtable.obj
 0001:0002d94b       __malloc_crt               1002e94b f   LIBCMT:crtheap.obj
 0001:0002d990       __calloc_crt               1002e990 f   LIBCMT:crtheap.obj
 0001:0002d9dc       __realloc_crt              1002e9dc f   LIBCMT:crtheap.obj
 0001:0002da2a       __msize                    1002ea2a f   LIBCMT:msize.obj
 0001:0002dacd       __crt_waiting_on_module_handle 1002eacd f   LIBCMT:crt0dat.obj
 0001:0002dafd       __amsg_exit                1002eafd f   LIBCMT:crt0dat.obj
 0001:0002db26       ___crtCorExitProcess       1002eb26 f   LIBCMT:crt0dat.obj
 0001:0002db51       ___crtExitProcess          1002eb51 f   LIBCMT:crt0dat.obj
 0001:0002db69       __lockexit                 1002eb69 f   LIBCMT:crt0dat.obj
 0001:0002db72       __unlockexit               1002eb72 f   LIBCMT:crt0dat.obj
 0001:0002db98       __initterm_e               1002eb98 f   LIBCMT:crt0dat.obj
 0001:0002dbbc       __cinit                    1002ebbc f   LIBCMT:crt0dat.obj
 0001:0002dd6d       __exit                     1002ed6d f   LIBCMT:crt0dat.obj
 0001:0002dd83       __cexit                    1002ed83 f   LIBCMT:crt0dat.obj
 0001:0002dd92       __init_pointers            1002ed92 f   LIBCMT:crt0dat.obj
 0001:0002dde0       __SEH_prolog4              1002ede0 f   LIBCMT:sehprolg4.obj
 0001:0002de25       __SEH_epilog4              1002ee25 f   LIBCMT:sehprolg4.obj
 0001:0002de39       ??0bad_exception@std@@QAE@PBD@Z 1002ee39 f i LIBCMT:frame.obj
 0001:0002de57       ??1bad_exception@std@@UAE@XZ 1002ee57 f i LIBCMT:frame.obj
 0001:0002de62       ??_Ebad_exception@std@@UAEPAXI@Z 1002ee62 f i LIBCMT:frame.obj
 0001:0002de62       ??_Gbad_exception@std@@UAEPAXI@Z 1002ee62 f i LIBCMT:frame.obj
 0001:0002de89       ___TypeMatch               1002ee89 f   LIBCMT:frame.obj
 0001:0002dee8       ___FrameUnwindFilter       1002eee8 f   LIBCMT:frame.obj
 0001:0002df31       ___FrameUnwindToState      1002ef31 f   LIBCMT:frame.obj
 0001:0002e057       ___DestructExceptionObject 1002f057 f   LIBCMT:frame.obj
 0001:0002e0ac       ___AdjustPointer           1002f0ac f   LIBCMT:frame.obj
 0001:0002e335       ___BuildCatchObjectHelper  1002f335 f   LIBCMT:frame.obj
 0001:0002e4b4       ___BuildCatchObject        1002f4b4 f   LIBCMT:frame.obj
 0001:0002e9ef       ??0bad_exception@std@@QAE@ABV01@@Z 1002f9ef f i LIBCMT:frame.obj
 0001:0002ea0c       ___InternalCxxFrameHandler 1002fa0c f   LIBCMT:frame.obj
 0001:0002eaf2       ?terminate@@YAXXZ          1002faf2 f   LIBCMT:hooks.obj
 0001:0002eb2b       ?unexpected@@YAXXZ         1002fb2b f   LIBCMT:hooks.obj
 0001:0002eb3e       ?_inconsistency@@YAXXZ     1002fb3e f   LIBCMT:hooks.obj
 0001:0002eb76       __initp_eh_hooks           1002fb76 f   LIBCMT:hooks.obj
 0001:0002eb90       __CallSettingFrame@12      1002fb90 f   LIBCMT:lowhelpr.obj
 0001:0002ebb7       __NLG_Return               1002fbb7     LIBCMT:lowhelpr.obj
 0001:0002ebdc       ___report_gsfailure        1002fbdc f   LIBCMT:gs_report.obj
 0001:0002ece2       ?_Type_info_dtor@type_info@@CAXPAV1@@Z 1002fce2 f   LIBCMT:typname.obj
 0001:0002ed60       _strcmp                    1002fd60 f   LIBCMT:strcmp.obj
 0001:0002ee3f       __VEC_memzero              1002fe3f f   LIBCMT:p4_memset.obj
 0001:0002ef1e       __get_sse2_info            1002ff1e f   LIBCMT:cpu_disp.obj
 0001:0002ef80       ___sse2_available_init     1002ff80 f   LIBCMT:cpu_disp.obj
 0001:0002ef8d       __crt_debugger_hook        1002ff8d f   LIBCMT:dbghook.obj
 0001:0002ef95       _abort                     1002ff95 f   LIBCMT:abort.obj
 0001:0002f0ac       __set_abort_behavior       100300ac f   LIBCMT:abort.obj
 0001:0002f0cd       __NMSG_WRITE               100300cd f   LIBCMT:crt0msg.obj
 0001:0002f278       __FF_MSGBANNER             10030278 f   LIBCMT:crt0msg.obj
 0001:0002f2b1       __initp_misc_purevirt      100302b1 f   LIBCMT:inithelp.obj
 0001:0002f347       __VEC_memcpy               10030347 f   LIBCMT:p4_memcpy.obj
 0001:0002f650       ___updatetmbcinfo          10030650 f   LIBCMT:mbctype.obj
 0001:0002f770       __setmbcp_nolock           10030770 f   LIBCMT:mbctype.obj
 0001:0002f955       __setmbcp                  10030955 f   LIBCMT:mbctype.obj
 0001:0002faef       ___initmbctable            10030aef f   LIBCMT:mbctype.obj
 0001:0002fb0d       ___freetlocinfo            10030b0d f   LIBCMT:setlocal.obj
 0001:0002fc56       ___addlocaleref            10030c56 f   LIBCMT:setlocal.obj
 0001:0002fce5       ___removelocaleref         10030ce5 f   LIBCMT:setlocal.obj
 0001:0002fdbc       ___updatetlocinfo          10030dbc f   LIBCMT:setlocal.obj
 0001:0002fe32       __tolower_l                10030e32 f   LIBCMT:tolower.obj
 0001:0002ff47       _tolower                   10030f47 f   LIBCMT:tolower.obj
 0001:0002ff73       __get_errno_from_oserr     10030f73 f   LIBCMT:dosmap.obj
 0001:0002ffb5       __errno                    10030fb5 f   LIBCMT:dosmap.obj
 0001:0002ffc8       ___doserrno                10030fc8 f   LIBCMT:dosmap.obj
 0001:0002ffdb       __dosmaperr                10030fdb f   LIBCMT:dosmap.obj
 0001:00030000       __trandisp1                10031000 f   LIBCMT:_87disp_.obj
 0001:00030067       __trandisp2                10031067 f   LIBCMT:_87disp_.obj
 0001:000300f3       __rttospopde               100310f3     LIBCMT:_87disp_.obj
 0001:000300f8       __rttospop                 100310f8     LIBCMT:_87disp_.obj
 0001:000300fa       __rtnospop                 100310fa     LIBCMT:_87disp_.obj
 0001:000300fc       __rttosnpop                100310fc     LIBCMT:_87disp_.obj
 0001:000300fd       __rtnospopde               100310fd     LIBCMT:_87disp_.obj
 0001:00030104       __rtzeropop                10031104     LIBCMT:_87disp_.obj
 0001:00030106       __rtzeronpop               10031106     LIBCMT:_87disp_.obj
 0001:0003010b       __rtonepop                 1003110b     LIBCMT:_87disp_.obj
 0001:0003010d       __rtonenpop                1003110d     LIBCMT:_87disp_.obj
 0001:00030112       __tosnan1                  10031112     LIBCMT:_87disp_.obj
 0001:0003013d       __nosnan2                  1003113d     LIBCMT:_87disp_.obj
 0001:0003013f       __tosnan2                  1003113f     LIBCMT:_87disp_.obj
 0001:00030167       __nan2                     10031167     LIBCMT:_87disp_.obj
 0001:000301a6       __rtindfpop                100311a6     LIBCMT:_87disp_.obj
 0001:000301a8       __rtindfnpop               100311a8     LIBCMT:_87disp_.obj
 0001:000301b9       __rttosnpopde              100311b9     LIBCMT:_87disp_.obj
 0001:000301c3       __rtchsifneg               100311c3     LIBCMT:_87disp_.obj
 0001:000301d0       __startTwoArgErrorHandling 100311d0 f   LIBCMT:_genexcep_.obj
 0001:000301e7       __startOneArgErrorHandling 100311e7 f   LIBCMT:_genexcep_.obj
 0001:00030230       __twoToTOS                 10031230 f   LIBCMT:_common_.obj
 0001:00030245       __load_CW                  10031245 f   LIBCMT:_common_.obj
 0001:0003025c       __convertTOStoQNaN         1003125c f   LIBCMT:_common_.obj
 0001:00030275       __fload_withFB             10031275 f   LIBCMT:_common_.obj
 0001:000302b8       __checkTOS_withFB          100312b8 f   LIBCMT:_common_.obj
 0001:000302ce       __fast_exit                100312ce f   LIBCMT:_common_.obj
 0001:000302db       __math_exit                100312db f   LIBCMT:_common_.obj
 0001:00030305       __check_overflow_exit      10031305 f   LIBCMT:_common_.obj
 0001:00030319       __check_range_exit         10031319 f   LIBCMT:_common_.obj
 0001:000303c0       ___ascii_strnicmp          100313c0 f   LIBCMT:_strnicm.obj
 0001:00030421       _strcpy_s                  10031421 f   LIBCMT:strcpy_s.obj
 0001:00030489       __ioinit                   10031489 f   LIBCMT:ioinit.obj
 0001:000306dd       __ioterm                   100316dd f   LIBCMT:ioinit.obj
 0001:0003072b       __setenvp                  1003172b f   LIBCMT:stdenvp.obj
 0001:000309a3       __setargv                  100319a3 f   LIBCMT:stdargv.obj
 0001:00030a5e       ___crtGetEnvironmentStringsA 10031a5e f   LIBCMT:a_env.obj
 0001:00030b95       __RTC_Initialize           10031b95 f   LIBCMT:_initsect_.obj
 0001:00030bbb       __RTC_Terminate            10031bbb f   LIBCMT:_initsect_.obj
 0001:00030be1       __heap_init                10031be1 f   LIBCMT:heapinit.obj
 0001:00030c11       __heap_term                10031c11 f   LIBCMT:heapinit.obj
 0001:00030c85       __XcptFilter               10031c85 f   LIBCMT:winxfltr.obj
 0001:00030de5       ___CppXcptFilter           10031de5 f   LIBCMT:winxfltr.obj
 0001:00030e05       ___security_init_cookie    10031e05 f   LIBCMT:gs_support.obj
 0001:00030e9c       __local_unwind4            10031e9c f   LIBCMT:exsup4.obj
 0001:00030f72       __seh_longjmp_unwind4@4    10031f72 f   LIBCMT:exsup4.obj
 0001:00030f8e       @_EH4_CallFilterFunc@8     10031f8e f   LIBCMT:exsup4.obj
 0001:00030fa5       @_EH4_TransferToHandler@8  10031fa5 f   LIBCMT:exsup4.obj
 0001:00030fbe       @_EH4_GlobalUnwind@4       10031fbe f   LIBCMT:exsup4.obj
 0001:00030fd8       @_EH4_LocalUnwind@16       10031fd8 f   LIBCMT:exsup4.obj
 0001:00030ff0       __ValidateImageBase        10031ff0 f   LIBCMT:pesect.obj
 0001:00031030       __FindPESection            10032030 f   LIBCMT:pesect.obj
 0001:00031080       __IsNonwritableInCurrentImage 10032080 f   LIBCMT:pesect.obj
 0001:0003113d       __sse2_mathfcns_init       1003213d f   LIBCMT:_mathfcns_.obj
 0001:00031160       __CIsin_pentium4           10032160 f   LIBCMT:_sin_pentium4_.obj
 0001:00031178       __sin_pentium4             10032178     LIBCMT:_sin_pentium4_.obj
 0001:00031330       __CIcos_pentium4           10032330 f   LIBCMT:_cos_pentium4_.obj
 0001:00031348       __cos_pentium4             10032348     LIBCMT:_cos_pentium4_.obj
 0001:000314e0       __CIacos_pentium4          100324e0 f   LIBCMT:_acos_pentium4_.obj
 0001:000314f8       __acos_pentium4            100324f8     LIBCMT:_acos_pentium4_.obj
 0001:00031a34       __flsbuf                   10032a34 f   LIBCMT:_flsbuf.obj
 0001:00031c3e       __output_l                 10032c3e f   LIBCMT:output.obj
 0001:00032829       __ismbblead_l              10033829 f   LIBCMT:ismbbyte.obj
 0001:00032842       __ismbblead                10033842 f   LIBCMT:ismbbyte.obj
 0001:0003285a       __mbsnbcpy_s               1003385a f   LIBCMT:mbsnbcpy_s.obj
 0001:00032877       __isdigit_l                10033877 f i LIBCMT:_ctype.obj
 0001:000328c8       _isdigit                   100338c8 f i LIBCMT:_ctype.obj
 0001:000328f6       __atodbl_l                 100338f6 f   LIBCMT:atodbl.obj
 0001:0003299e       __atoflt_l                 1003399e f   LIBCMT:atodbl.obj
 0001:00032a46       __fptostr                  10033a46 f   LIBCMT:_fptostr.obj
 0001:00032b05       ___dtold                   10033b05 f   LIBCMT:_cfout_.obj
 0001:00032bc2       __fltout2                  10033bc2 f   LIBCMT:_cfout_.obj
 0001:00032c60       __alldvrm                  10033c60 f   LIBCMT:lldvrm.obj
 0001:00032d40       __aullshr                  10033d40 f   LIBCMT:ullshr.obj
 0001:00032d5f       __fptrap                   10033d5f f   LIBCMT:crt0fp.obj
 0001:00032d68       __controlfp_s              10033d68 f   LIBCMT:_contrlfp_.obj
 0001:00032dd4       __mtinitlocks              10033dd4 f   LIBCMT:mlock.obj
 0001:00032e1f       __mtdeletelocks            10033e1f f   LIBCMT:mlock.obj
 0001:00032e76       __unlock                   10033e76 f   LIBCMT:mlock.obj
 0001:00032e8d       __mtinitlocknum            10033e8d f   LIBCMT:mlock.obj
 0001:00032f50       __lock                     10033f50 f   LIBCMT:mlock.obj
 0001:00032f83       ___sbh_find_block          10033f83 f   LIBCMT:sbheap.obj
 0001:00032fb3       ___sbh_free_block          10033fb3 f   LIBCMT:sbheap.obj
 0001:000332c9       ___sbh_alloc_new_region    100342c9 f   LIBCMT:sbheap.obj
 0001:00033379       ___sbh_alloc_new_group     10034379 f   LIBCMT:sbheap.obj
 0001:00033481       ___sbh_resize_block        10034481 f   LIBCMT:sbheap.obj
 0001:00033762       ___sbh_alloc_block         10034762 f   LIBCMT:sbheap.obj
 0001:00033a47       __calloc_impl              10034a47 f   LIBCMT:calloc_impl.obj
 0001:00033b65       _realloc                   10034b65 f   LIBCMT:realloc.obj
 0001:00033d80       __initp_misc_winsig        10034d80 f   LIBCMT:winsig.obj
 0001:00033dd5       ___get_sigabrt             10034dd5 f   LIBCMT:winsig.obj
 0001:00033de2       _raise                     10034de2 f   LIBCMT:winsig.obj
 0001:00033f92       __initp_misc_rand_s        10034f92 f   LIBCMT:rand_s.obj
 0001:00033fa1       __initp_misc_initcrit      10034fa1 f   LIBCMT:initcrit.obj
 0001:00033fb0       ___crtInitCritSecAndSpinCount 10034fb0 f   LIBCMT:initcrit.obj
 0001:00034010       ?_ValidateRead@@YAHPBXI@Z  10035010 f   LIBCMT:validate.obj
 0001:00034010       ?_ValidateExecute@@YAHP6GHXZ@Z 10035010 f   LIBCMT:validate.obj
 0001:00034010       ?_ValidateWrite@@YAHPAXI@Z 10035010 f   LIBCMT:validate.obj
 0001:00034024       __global_unwind2           10035024 f   LIBCMT:exsup.obj
 0001:00034089       __local_unwind2            10035089 f   LIBCMT:exsup.obj
 0001:0003410d       __abnormal_termination     1003510d f   LIBCMT:exsup.obj
 0001:00034130       __NLG_Notify1              10035130 f   LIBCMT:exsup.obj
 0001:00034139       __NLG_Notify               10035139 f   LIBCMT:exsup.obj
 0001:00034150       __NLG_Dispatch2            10035150     LIBCMT:exsup.obj
 0001:00034150       __NLG_Dispatch             10035150     LIBCMT:exsup.obj
 0001:00034158       __NLG_Call                 10035158 f   LIBCMT:exsup.obj
 0001:0003415a       __NLG_Return2              1003515a     LIBCMT:exsup.obj
 0001:0003415b       ___crtMessageBoxA          1003515b f   LIBCMT:crtmbox.obj
 0001:000342c4       _strcat_s                  100352c4 f   LIBCMT:strcat_s.obj
 0001:00034338       _strncpy_s                 10035338 f   LIBCMT:strncpy_s.obj
 0001:000343ed       __set_error_mode           100353ed f   LIBCMT:errmode.obj
 0001:00034438       __freea                    10035438 f i LIBCMT:a_loc.obj
 0001:000347fd       ___crtLCMapStringA         100357fd f   LIBCMT:a_map.obj
 0001:000349fc       ___crtGetStringTypeA       100359fc f   LIBCMT:a_str.obj
 0001:00034a3e       ___free_lc_time            10035a3e f   LIBCMT:inittime.obj
 0001:00034bd3       ___free_lconv_num          10035bd3 f   LIBCMT:initnum.obj
 0001:00034c18       ___free_lconv_mon          10035c18 f   LIBCMT:initmon.obj
 0001:00034cb0       _strcspn                   10035cb0 f   LIBCMT:strcspn.obj
 0001:00034d00       _strpbrk                   10035d00 f   LIBCMT:strpbrk.obj
 0001:00034d40       __isleadbyte_l             10035d40 f i LIBCMT:_wctype.obj
 0001:00034d78       _isleadbyte                10035d78 f i LIBCMT:_wctype.obj
 0001:00034d8b       __isctype_l                10035d8b f   LIBCMT:isctype.obj
 0001:00034e43       __87except                 10035e43 f   LIBCMT:_87except_.obj
 0001:00034f82       ___libm_error_support      10035f82 f   LIBCMT:_libm_error_.obj
 0001:00035232       __lseeki64_nolock          10036232 f   LIBCMT:lseeki64.obj
 0001:000352b7       __lseeki64                 100362b7 f   LIBCMT:lseeki64.obj
 0001:000353d0       __write_nolock             100363d0 f   LIBCMT:write.obj
 0001:00035b03       __write                    10036b03 f   LIBCMT:write.obj
 0001:00035bdf       __getbuf                   10036bdf f   LIBCMT:_getbuf.obj
 0001:00035c28       __isatty                   10036c28 f   LIBCMT:isatty.obj
 0001:00035c8c       ___iob_func                10036c8c f   LIBCMT:_file.obj
 0001:00035c92       ___initstdio               10036c92 f   LIBCMT:_file.obj
 0001:00035d43       ___endstdio                10036d43 f   LIBCMT:_file.obj
 0001:00035d63       __lock_file                10036d63 f   LIBCMT:_file.obj
 0001:00035da4       __lock_file2               10036da4 f   LIBCMT:_file.obj
 0001:00035dd6       __unlock_file              10036dd6 f   LIBCMT:_file.obj
 0001:00035e12       __unlock_file2             10036e12 f   LIBCMT:_file.obj
 0001:00035e41       __fileno                   10036e41 f   LIBCMT:fileno.obj
 0001:00035e73       __get_printf_count_output  10036e73 f   LIBCMT:printf.obj
 0001:00035e89       __wctomb_s_l               10036e89 f   LIBCMT:wctomb.obj
 0001:00035ff5       _wctomb_s                  10036ff5 f   LIBCMT:wctomb.obj
 0001:00036020       __aulldvrm                 10037020 f   LIBCMT:ulldvrm.obj
 0001:000360b5       __mbsnbcpy_s_l             100370b5 f   LIBCMT:mbsnbcpy_s_l.obj
 0001:000362c4       __ld12tod                  100372c4 f   LIBCMT:_intrncvt_.obj
 0001:00036808       __ld12tof                  10037808 f   LIBCMT:_intrncvt_.obj
 0001:00036d4c       ___strgtold12_l            10037d4c f   LIBCMT:_strgtold_.obj
 0001:00037444       _$I10_OUTPUT               10038444 f   LIBCMT:_x10fout_.obj
 0001:00037e96       __control87                10038e96 f i LIBCMT:_ieee87_.obj
 0001:000381b0       __allmul                   100391b0 f   LIBCMT:llmul.obj
 0001:000381e4       _atol                      100391e4 f   LIBCMT:atox.obj
 0001:00038200       __alloca_probe_16          10039200 f   LIBCMT:alloca16.obj
 0001:00038216       __alloca_probe_8           10039216     LIBCMT:alloca16.obj
 0001:0003822c       ___ansicp                  1003922c f   LIBCMT:convrtcp.obj
 0001:00038275       ___convertcp               10039275 f   LIBCMT:convrtcp.obj
 0001:00038429       __raise_exc_ex             10039429 f   LIBCMT:_fpexcept_.obj
 0001:00038705       __raise_exc                10039705 f   LIBCMT:_fpexcept_.obj
 0001:00038728       __handle_exc               10039728 f   LIBCMT:_fpexcept_.obj
 0001:0003890a       __set_errno_from_matherr   1003990a f   LIBCMT:_fpexcept_.obj
 0001:00038937       __matherr                  10039937 f   LIBCMT:_matherr_.obj
 0001:0003893a       __statfp                   1003993a f   LIBCMT:_fpctrl_.obj
 0001:0003894a       __clrfp                    1003994a f   LIBCMT:_fpctrl_.obj
 0001:0003895b       __ctrlfp                   1003995b f   LIBCMT:_fpctrl_.obj
 0001:00038984       __set_statfp               10039984 f   LIBCMT:_fpctrl_.obj
 0001:000389dc       ___set_fpsr_sse2           100399dc f   LIBCMT:_fpctrl_.obj
 0001:00038a4e       __free_osfhnd              10039a4e f   LIBCMT:osfinfo.obj
 0001:00038ad4       __get_osfhandle            10039ad4 f   LIBCMT:osfinfo.obj
 0001:00038b4b       ___lock_fhandle            10039b4b f   LIBCMT:osfinfo.obj
 0001:00038beb       __unlock_fhandle           10039beb f   LIBCMT:osfinfo.obj
 0001:00038c12       __putwch_nolock            10039c12 f   LIBCMT:putwch.obj
 0001:00038cd7       __mbtowc_l                 10039cd7 f   LIBCMT:mbtowc.obj
 0001:00038dee       _mbtowc                    10039dee f   LIBCMT:mbtowc.obj
 0001:00038e10       __chkstk                   10039e10 f   LIBCMT:chkstk.obj
 0001:00038e10       __alloca_probe             10039e10     LIBCMT:chkstk.obj
 0001:00038e3b       __fcloseall                10039e3b f   LIBCMT:closeall.obj
 0001:00038eda       __flush                    10039eda f   LIBCMT:fflush.obj
 0001:00038f42       __fflush_nolock            10039f42 f   LIBCMT:fflush.obj
 0001:00039064       __flushall                 1003a064 f   LIBCMT:fflush.obj
 0001:0003929c       _strtol                    1003a29c f   LIBCMT:strtol.obj
 0001:000392c7       ___mtold12                 1003a2c7 f   LIBCMT:_mantold_.obj
 0001:00039495       __set_exp                  1003a495 f   LIBCMT:_util_.obj
 0001:000394c1       __decomp                   1003a4c1 f   LIBCMT:_util_.obj
 0001:0003957a       ___initconout              1003a57a f   LIBCMT:initcon.obj
 0001:00039599       ___termcon                 1003a599 f   LIBCMT:initcon.obj
 0001:000395c6       __fclose_nolock            1003a5c6 f   LIBCMT:fclose.obj
 0001:0003963d       _fclose                    1003a63d f   LIBCMT:fclose.obj
 0001:000396b9       __commit                   1003a6b9 f   LIBCMT:commit.obj
 0001:0003979a       __close_nolock             1003a79a f   LIBCMT:close.obj
 0001:00039836       __close                    1003a836 f   LIBCMT:close.obj
 0001:00039903       __freebuf                  1003a903 f   LIBCMT:_freebuf.obj
 0001:00039950       _strchr                    1003a950 f   LIBCMT:strchr.obj
 0001:00039956       ___from_strstr_to_strchr   1003a956     LIBCMT:strchr.obj
 0001:00039a10       ??1CAutoFree@@QAE@XZ       1003aa10 f   wzFilePacker_static:wzFilePacker.obj
 0001:00039a20       ?CONVERT_PATHCHAR@CPackFile@@CAXPAD@Z 1003aa20 f i wzFilePacker_static:wzFilePacker.obj
 0001:00039a80       ??0CPackFile@@QAE@XZ       1003aa80 f   wzFilePacker_static:wzFilePacker.obj
 0001:00039ab0       ?Close@CPackFile@@QAEXXZ   1003aab0 f   wzFilePacker_static:wzFilePacker.obj
 0001:00039ad0       ?OpenFile@CPackFile@@QAEPAXPBDK@Z 1003aad0 f   wzFilePacker_static:wzFilePacker.obj
 0001:00039b00       ?FileExists@CPackFile@@QAEHPBD@Z 1003ab00 f   wzFilePacker_static:wzFilePacker.obj
 0001:00039b20       ?DeleteFileA@CPackFile@@QAEHPBD@Z 1003ab20 f   wzFilePacker_static:wzFilePacker.obj
 0001:00039b20       ?RemoveDirectoryA@CPackFile@@QAEHPBD@Z 1003ab20 f   wzFilePacker_static:wzFilePacker.obj
 0001:00039b40       ?CreateDirectoryA@CPackFile@@QAEHPBD@Z 1003ab40 f   wzFilePacker_static:wzFilePacker.obj
 0001:00039b70       ?CloseFile@CPackFile@@QAEXPAX@Z 1003ab70 f   wzFilePacker_static:wzFilePacker.obj
 0001:00039b80       ?GetFileProperties@CPackFile@@QAEHPAXPAUFileProperties@@@Z 1003ab80 f   wzFilePacker_static:wzFilePacker.obj
 0001:00039c30       ?ReadFile@CPackFile@@QAEHPAX0K@Z 1003ac30 f   wzFilePacker_static:wzFilePacker.obj
 0001:00039c50       ?WriteFile@CPackFile@@QAEHPAXPBXK@Z 1003ac50 f   wzFilePacker_static:wzFilePacker.obj
 0001:00039c70       ?GetFileSize@CPackFile@@QAEHPAXPA_K@Z 1003ac70 f   wzFilePacker_static:wzFilePacker.obj
 0001:00039c80       ?GetFilePointer@CPackFile@@QAEHPAXPA_K@Z 1003ac80 f   wzFilePacker_static:wzFilePacker.obj
 0001:00039c90       ?SetFilePointer@CPackFile@@QAEHPAX_KK@Z 1003ac90 f   wzFilePacker_static:wzFilePacker.obj
 0001:00039cb0       ?AddFile@CPackFile@@QAEHPBD0@Z 1003acb0 f   wzFilePacker_static:wzFilePacker.obj
 0001:00039dc0       ??1CPackFile@@QAE@XZ       1003adc0 f   wzFilePacker_static:wzFilePacker.obj
 0001:00039dd0       ?Open@CPackFile@@QAEPAXPBD0K@Z 1003add0 f   wzFilePacker_static:wzFilePacker.obj
 0001:00039ef0       @geVFile_CloseAPI@0        1003aef0 f   wzFilePacker_static:vfile.obj
 0001:00039fb0       @geVFile_Open_Detail@20    1003afb0 f   wzFilePacker_static:vfile.obj
 0001:0003a0a0       @geVFile_Open@12           1003b0a0 f   wzFilePacker_static:vfile.obj
 0001:0003a190       @geVFile_DeleteFile@8      1003b190 f   wzFilePacker_static:vfile.obj
 0001:0003a1a0       @geVFile_FileExists@8      1003b1a0 f   wzFilePacker_static:vfile.obj
 0001:0003a1b0       @geVFile_Close@4           1003b1b0 f   wzFilePacker_static:vfile.obj
 0001:0003a200       @geVFile_GetS@12           1003b200 f   wzFilePacker_static:vfile.obj
 0001:0003a220       @geVFile_Read@12           1003b220 f   wzFilePacker_static:vfile.obj
 0001:0003a250       @geVFile_Write@12          1003b250 f   wzFilePacker_static:vfile.obj
 0001:0003a280       @geVFile_Seek@16           1003b280 f   wzFilePacker_static:vfile.obj
 0001:0003a2a0       @geVFile_Tell@8            1003b2a0 f   wzFilePacker_static:vfile.obj
 0001:0003a2b0       @geVFile_Size@8            1003b2b0 f   wzFilePacker_static:vfile.obj
 0001:0003a2c0       @geVFile_GetProperties@8   1003b2c0 f   wzFilePacker_static:vfile.obj
 0001:0003a2d0       @geVFile_EnlargeDirectorySize@8 1003b2d0 f   wzFilePacker_static:vfile.obj
 0001:0003a2e0       @geVFile_SetVersion@8      1003b2e0 f   wzFilePacker_static:vfile.obj
 0001:0003a2f0       @geVFile_IsPrevVersion@4   1003b2f0 f   wzFilePacker_static:vfile.obj
 0001:0003a300       @geVFile_OpenNewSystem@20  1003b300 f   wzFilePacker_static:vfile.obj
 0001:0003a440       _CopyVFile                 1003b440 f   wzFilePacker_static:vFile_util.obj
 0001:0003a5b0       _CopyOneFile               1003b5b0 f   wzFilePacker_static:vFile_util.obj
 0001:0003a630       _MakeDirectory             1003b630 f   wzFilePacker_static:vFile_util.obj
 0001:0003a720       _geRam_Allocate            1003b720 f   wzFilePacker_static:Ram.obj
 0001:0003a740       _geRam_Free_               1003b740 f   wzFilePacker_static:Ram.obj
 0001:0003a750       _geRam_Realloc             1003b750 f   wzFilePacker_static:Ram.obj
 0001:0003a7b0       _Encrypt                   1003b7b0 f   wzFilePacker_static:fsvfs.obj
 0001:0003a7f0       _Decrypt                   1003b7f0 f   wzFilePacker_static:fsvfs.obj
 0001:0003c1d0       @FSVFS_GetAPIs@0           1003d1d0 f   wzFilePacker_static:fsvfs.obj
 0001:0003c990       @FSMemory_GetAPIs@0        1003d990 f   wzFilePacker_static:FSMEMORY.obj
 0001:0003d610       @FSDos_GetAPIs@0           1003e610 f   wzFilePacker_static:fsdos.obj
 0001:0003d620       _DirTree_Create            1003e620 f   wzFilePacker_static:dirtree.obj
 0001:0003d670       _DirTree_Destroy           1003e670 f   wzFilePacker_static:dirtree.obj
 0001:0003d910       _DirTree_SetFileSize       1003e910 f   wzFilePacker_static:dirtree.obj
 0001:0003d930       _DirTree_GetFileSize       1003e930 f   wzFilePacker_static:dirtree.obj
 0001:0003d950       _DirTree_WriteToFile       1003e950 f   wzFilePacker_static:dirtree.obj
 0001:0003d980       _DirTree_GetSize           1003e980 f   wzFilePacker_static:dirtree.obj
 0001:0003dda0       _DirTree_CreateFromFile    1003eda0 f   wzFilePacker_static:dirtree.obj
 0001:0003e120       _DirTree_FindExact         1003f120 f   wzFilePacker_static:dirtree.obj
 0001:0003e180       _DirTree_FindPartial       1003f180 f   wzFilePacker_static:dirtree.obj
 0001:0003e200       _DirTree_AddFile           1003f200 f   wzFilePacker_static:dirtree.obj
 0001:0003e2d0       _DirTree_Remove            1003f2d0 f   wzFilePacker_static:dirtree.obj
 0001:0003e360       _DirTree_SetFileAttributes 1003f360 f   wzFilePacker_static:dirtree.obj
 0001:0003e380       _DirTree_GetFileAttributes 1003f380 f   wzFilePacker_static:dirtree.obj
 0001:0003e390       _DirTree_SetFileOffset     1003f390 f   wzFilePacker_static:dirtree.obj
 0001:0003e3b0       _DirTree_GetFileOffset     1003f3b0 f   wzFilePacker_static:dirtree.obj
 0001:0003e3d0       _DirTree_SetFileTime       1003f3d0 f   wzFilePacker_static:dirtree.obj
 0001:0003e3f0       _DirTree_GetFileTime       1003f3f0 f   wzFilePacker_static:dirtree.obj
 0001:0003e410       _DirTree_SetFileHints      1003f410 f   wzFilePacker_static:dirtree.obj
 0001:0003e480       _DirTree_GetFileHints      1003f480 f   wzFilePacker_static:dirtree.obj
 0001:0003e4a0       _DirTree_GetName           1003f4a0 f   wzFilePacker_static:dirtree.obj
 0001:0003e4e0       _DirTree_FileExists        1003f4e0 f   wzFilePacker_static:dirtree.obj
 0001:0003e500       _DirTree_CreateFinder      1003f500 f   wzFilePacker_static:dirtree.obj
 0001:0003e630       _DirTree_DestroyFinder     1003f630 f   wzFilePacker_static:dirtree.obj
 0001:0003e670       _DirTree_FinderGetNextFile 1003f670 f   wzFilePacker_static:dirtree.obj
 0001:0003e730       _DirTree_SetAllFileOffset  1003f730 f   wzFilePacker_static:dirtree.obj
 0001:0003e7e0       _DuplicateString           1003f7e0 f   wzFilePacker_static:dirtree-common.obj
 0001:0003e820       _GetNextDir                1003f820 f   wzFilePacker_static:dirtree-common.obj
 0001:0003e850       _MatchPattern              1003f850 f   wzFilePacker_static:dirtree-common.obj
 0001:0003e8b0       _PathHasDir                1003f8b0 f   wzFilePacker_static:dirtree-common.obj
 0001:0003e8c6       _RtlUnwind@16              1003f8c6 f   kernel32:KERNEL32.dll
 0001:0003e8cc       __mbsstr_l                 1003f8cc f   LIBCMT:mbsstr.obj
 0001:0003ea0d       __mbsstr                   1003fa0d f   LIBCMT:mbsstr.obj
 0001:0003ea30       _memchr                    1003fa30 f   LIBCMT:memchr.obj
 0001:0003eae0       _strstr                    1003fae0 f   LIBCMT:strstr.obj
 0001:0003fe60       ??__Finstance@?1??Instance@CWzdShareInfo@@SAPAV1@XZ@YAXXZ 10040e60 f i dllaccess.obj
 0001:0003fe6f       ??__Fs_discAccess@?4??CheckDiscAccessExistence@CWzdBase@@SAPAVCDiscAccess@@XZ@YAXXZ 10040e6f f i wzdbase.obj
 0002:00000000       __imp__LeaveCriticalSection@4 10041000     kernel32:KERNEL32.dll
 0002:00000004       __imp__EnterCriticalSection@4 10041004     kernel32:KERNEL32.dll
 0002:00000008       __imp__GetModuleFileNameA@12 10041008     kernel32:KERNEL32.dll
 0002:0000000c       __imp__WriteFile@20        1004100c     kernel32:KERNEL32.dll
 0002:00000010       __imp__InitializeCriticalSection@4 10041010     kernel32:KERNEL32.dll
 0002:00000014       __imp__DeleteCriticalSection@4 10041014     kernel32:KERNEL32.dll
 0002:00000018       __imp__CreateFileA@28      10041018     kernel32:KERNEL32.dll
 0002:0000001c       __imp__CloseHandle@4       1004101c     kernel32:KERNEL32.dll
 0002:00000020       __imp__SetFilePointer@16   10041020     kernel32:KERNEL32.dll
 0002:00000024       __imp__ReadFile@20         10041024     kernel32:KERNEL32.dll
 0002:00000028       __imp__FindClose@4         10041028     kernel32:KERNEL32.dll
 0002:0000002c       __imp__FindFirstFileA@8    1004102c     kernel32:KERNEL32.dll
 0002:00000030       __imp__GetFileSize@8       10041030     kernel32:KERNEL32.dll
 0002:00000034       __imp__GetFileInformationByHandle@8 10041034     kernel32:KERNEL32.dll
 0002:00000038       __imp__CopyFileA@12        10041038     kernel32:KERNEL32.dll
 0002:0000003c       __imp__DeleteFileA@4       1004103c     kernel32:KERNEL32.dll
 0002:00000040       __imp__CreateDirectoryA@8  10041040     kernel32:KERNEL32.dll
 0002:00000044       __imp__RemoveDirectoryA@4  10041044     kernel32:KERNEL32.dll
 0002:00000048       __imp__RtlUnwind@16        10041048     kernel32:KERNEL32.dll
 0002:0000004c       __imp__TerminateProcess@8  1004104c     kernel32:KERNEL32.dll
 0002:00000050       __imp__GetCurrentProcess@0 10041050     kernel32:KERNEL32.dll
 0002:00000054       __imp__UnhandledExceptionFilter@4 10041054     kernel32:KERNEL32.dll
 0002:00000058       __imp__SetUnhandledExceptionFilter@4 10041058     kernel32:KERNEL32.dll
 0002:0000005c       __imp__IsDebuggerPresent@0 1004105c     kernel32:KERNEL32.dll
 0002:00000060       __imp__RaiseException@16   10041060     kernel32:KERNEL32.dll
 0002:00000064       __imp__GetCurrentThreadId@0 10041064     kernel32:KERNEL32.dll
 0002:00000068       __imp__GetCommandLineA@0   10041068     kernel32:KERNEL32.dll
 0002:0000006c       __imp__GetProcAddress@8    1004106c     kernel32:KERNEL32.dll
 0002:00000070       __imp__GetModuleHandleA@4  10041070     kernel32:KERNEL32.dll
 0002:00000074       __imp__GetLastError@0      10041074     kernel32:KERNEL32.dll
 0002:00000078       __imp__HeapFree@12         10041078     kernel32:KERNEL32.dll
 0002:0000007c       __imp__HeapAlloc@12        1004107c     kernel32:KERNEL32.dll
 0002:00000080       __imp__GetModuleHandleW@4  10041080     kernel32:KERNEL32.dll
 0002:00000084       __imp__TlsGetValue@4       10041084     kernel32:KERNEL32.dll
 0002:00000088       __imp__TlsAlloc@0          10041088     kernel32:KERNEL32.dll
 0002:0000008c       __imp__TlsSetValue@8       1004108c     kernel32:KERNEL32.dll
 0002:00000090       __imp__TlsFree@4           10041090     kernel32:KERNEL32.dll
 0002:00000094       __imp__InterlockedIncrement@4 10041094     kernel32:KERNEL32.dll
 0002:00000098       __imp__SetLastError@4      10041098     kernel32:KERNEL32.dll
 0002:0000009c       __imp__InterlockedDecrement@4 1004109c     kernel32:KERNEL32.dll
 0002:000000a0       __imp__Sleep@4             100410a0     kernel32:KERNEL32.dll
 0002:000000a4       __imp__HeapSize@12         100410a4     kernel32:KERNEL32.dll
 0002:000000a8       __imp__ExitProcess@4       100410a8     kernel32:KERNEL32.dll
 0002:000000ac       __imp__GetStdHandle@4      100410ac     kernel32:KERNEL32.dll
 0002:000000b0       __imp__GetCPInfo@8         100410b0     kernel32:KERNEL32.dll
 0002:000000b4       __imp__GetACP@0            100410b4     kernel32:KERNEL32.dll
 0002:000000b8       __imp__GetOEMCP@0          100410b8     kernel32:KERNEL32.dll
 0002:000000bc       __imp__IsValidCodePage@4   100410bc     kernel32:KERNEL32.dll
 0002:000000c0       __imp__SetHandleCount@4    100410c0     kernel32:KERNEL32.dll
 0002:000000c4       __imp__GetFileType@4       100410c4     kernel32:KERNEL32.dll
 0002:000000c8       __imp__GetStartupInfoA@4   100410c8     kernel32:KERNEL32.dll
 0002:000000cc       __imp__FreeEnvironmentStringsA@4 100410cc     kernel32:KERNEL32.dll
 0002:000000d0       __imp__GetEnvironmentStrings@0 100410d0     kernel32:KERNEL32.dll
 0002:000000d4       __imp__FreeEnvironmentStringsW@4 100410d4     kernel32:KERNEL32.dll
 0002:000000d8       __imp__WideCharToMultiByte@32 100410d8     kernel32:KERNEL32.dll
 0002:000000dc       __imp__GetEnvironmentStringsW@0 100410dc     kernel32:KERNEL32.dll
 0002:000000e0       __imp__HeapCreate@12       100410e0     kernel32:KERNEL32.dll
 0002:000000e4       __imp__HeapDestroy@4       100410e4     kernel32:KERNEL32.dll
 0002:000000e8       __imp__VirtualFree@12      100410e8     kernel32:KERNEL32.dll
 0002:000000ec       __imp__QueryPerformanceCounter@4 100410ec     kernel32:KERNEL32.dll
 0002:000000f0       __imp__GetTickCount@0      100410f0     kernel32:KERNEL32.dll
 0002:000000f4       __imp__GetCurrentProcessId@0 100410f4     kernel32:KERNEL32.dll
 0002:000000f8       __imp__GetSystemTimeAsFileTime@4 100410f8     kernel32:KERNEL32.dll
 0002:000000fc       __imp__VirtualAlloc@16     100410fc     kernel32:KERNEL32.dll
 0002:00000100       __imp__HeapReAlloc@16      10041100     kernel32:KERNEL32.dll
 0002:00000104       __imp__LoadLibraryA@4      10041104     kernel32:KERNEL32.dll
 0002:00000108       __imp__InitializeCriticalSectionAndSpinCount@8 10041108     kernel32:KERNEL32.dll
 0002:0000010c       __imp__GetLocaleInfoA@16   1004110c     kernel32:KERNEL32.dll
 0002:00000110       __imp__LCMapStringA@24     10041110     kernel32:KERNEL32.dll
 0002:00000114       __imp__MultiByteToWideChar@24 10041114     kernel32:KERNEL32.dll
 0002:00000118       __imp__LCMapStringW@24     10041118     kernel32:KERNEL32.dll
 0002:0000011c       __imp__GetStringTypeA@20   1004111c     kernel32:KERNEL32.dll
 0002:00000120       __imp__GetStringTypeW@16   10041120     kernel32:KERNEL32.dll
 0002:00000124       __imp__GetConsoleCP@0      10041124     kernel32:KERNEL32.dll
 0002:00000128       __imp__GetConsoleMode@8    10041128     kernel32:KERNEL32.dll
 0002:0000012c       __imp__SetStdHandle@8      1004112c     kernel32:KERNEL32.dll
 0002:00000130       __imp__WriteConsoleA@20    10041130     kernel32:KERNEL32.dll
 0002:00000134       __imp__GetConsoleOutputCP@0 10041134     kernel32:KERNEL32.dll
 0002:00000138       __imp__WriteConsoleW@20    10041138     kernel32:KERNEL32.dll
 0002:0000013c       __imp__FlushFileBuffers@4  1004113c     kernel32:KERNEL32.dll
 0002:00000140       __imp__lstrlenA@4          10041140     kernel32:KERNEL32.dll
 0002:00000144       __imp__lstrcpyA@8          10041144     kernel32:KERNEL32.dll
 0002:00000148       __imp__FindNextFileA@8     10041148     kernel32:KERNEL32.dll
 0002:0000014c       __imp__OutputDebugStringA@4 1004114c     kernel32:KERNEL32.dll
 0002:00000150       __imp__SetFilePointerEx@20 10041150     kernel32:KERNEL32.dll
 0002:00000154       __imp__GetFileSizeEx@8     10041154     kernel32:KERNEL32.dll
 0002:00000158       __imp__SetEndOfFile@4      10041158     kernel32:KERNEL32.dll
 0002:0000015c       __imp__SetFileAttributesA@8 1004115c     kernel32:KERNEL32.dll
 0002:00000160       __imp__SetFileTime@16      10041160     kernel32:KERNEL32.dll
 0002:00000164       __imp__GetFileAttributesA@4 10041164     kernel32:KERNEL32.dll
 0002:00000168       __imp__MoveFileA@8         10041168     kernel32:KERNEL32.dll
 0002:0000016c       \177KERNEL32_NULL_THUNK_DATA 1004116c     kernel32:KERNEL32.dll
 0002:00000170       __imp__wsprintfA           10041170     user32:USER32.dll
 0002:00000174       __imp__SendMessageA@16     10041174     user32:USER32.dll
 0002:00000178       __imp__wvsprintfA@12       10041178     user32:USER32.dll
 0002:0000017c       \177USER32_NULL_THUNK_DATA 1004117c     user32:USER32.dll
 0002:00000180       ___xc_a                    10041180     LIBCMT:crt0init.obj
 0002:00000188       ___xc_z                    10041188     LIBCMT:crt0init.obj
 0002:0000018c       ___xi_a                    1004118c     LIBCMT:crt0init.obj
 0002:000001a4       ___xi_z                    100411a4     LIBCMT:crt0init.obj
 0002:000001a8       ___xp_a                    100411a8     LIBCMT:crt0init.obj
 0002:000001b4       ___xp_z                    100411b4     LIBCMT:crt0init.obj
 0002:000001b8       ___xt_a                    100411b8     LIBCMT:crt0init.obj
 0002:000001bc       ___xt_z                    100411bc     LIBCMT:crt0init.obj
 0002:000001dc       ??_C@_0P@GHFPNOJB@bad?5allocation?$AA@ 100411dc     dllaccess.obj
 0002:000001f0       __real@3eb0c6f7a0000000    100411f0     dllaccess.obj
 0002:000001fc       ??_7CWzdAnimation@@6B@     100411fc     wzdanimation.obj
 0002:000002d8       ??_C@_04PCBDJJAJ@WZAD?$AA@ 100412d8     wzdanimation.obj
 0002:000002e0       __real@3f800000            100412e0     wzdanimation.obj
 0002:000002e4       ??_C@_0N@LKIIPJHE@Unknown?5bone?$AA@ 100412e4     wzdanimation.obj
 0002:000002f8       __real@3ff0000000000000    100412f8     wzdanimation.obj
 0002:00000300       __real@3f847ae140000000    10041300     wzdanimation.obj
 0002:00000308       ??_C@_02PCIJFNDE@?$AN?6?$AA@ 10041308     wzdanimation.obj
 0002:0000030c       ??_C@_0BA@GPOHJINM@?7?7?$CFs?5?$CFs?5?$CFs?5?$CFs?$AN?6?$AA@ 1004130c     wzdanimation.obj
 0002:0000031c       ??_C@_09LGNBNLNK@?7?$CFs?5?$CFs?5?$CFs?$AA@ 1004131c     wzdanimation.obj
 0002:00000328       ??_C@_06FDPNKFMM@?7?$CFd?5?$CFd?$AA@ 10041328     wzdanimation.obj
 0002:00000330       ??_C@_09JFFAJOPD@node?5?$CFd?$AN?6?$AA@ 10041330     wzdanimation.obj
 0002:0000033c       ??_C@_0BH@MMPCAMON@Use?5Key?5Frame?3?5FALSE?$AN?6?$AA@ 1004133c     wzdanimation.obj
 0002:00000354       ??_C@_0BG@ECOHNLHH@Use?5Key?5Frame?3?5TRUE?$AN?6?$AA@ 10041354     wzdanimation.obj
 0002:0000036c       ??_C@_09FBPMNOOG@?$CF3d?5?7?$CFd?$AN?6?$AA@ 1004136c     wzdanimation.obj
 0002:00000378       ??_C@_0N@OBLKBBLO@key?5frames?$AN?6?$AA@ 10041378     wzdanimation.obj
 0002:00000388       ??_C@_07CPCAKLLB@end?$AN?6?$AN?6?$AA@ 10041388     wzdanimation.obj
 0002:00000390       ??_C@_0BB@JPLLOLAC@?$CF3d?5?7?$CC?$CFs?$CC?5?7?$CF3d?$AN?6?$AA@ 10041390     wzdanimation.obj
 0002:000003a4       ??_C@_0M@MNKCMBEH@nodes?5?7?$CFd?$AN?6?$AA@ 100413a4     wzdanimation.obj
 0002:000003b4       ??_7CWzdBase@@6B@          100413b4     wzdbase.obj
 0002:00000490       ??_C@_0BE@KGMIADMF@version?5?$CFd?4?$CF02d?$AN?6?$AN?6?$AA@ 10041490     wzdbase.obj
 0002:000004a4       ??_C@_06GBACDPPA@?$FL?$CFs?$FN?$AN?6?$AA@ 100414a4     wzdbase.obj
 0002:000004b4       ??_7CWzdMesh@@6B@          100414b4     wzdmesh.obj
 0002:00000590       ??_C@_04PLAJGAGN@WZMD?$AA@ 10041590     wzdmesh.obj
 0002:00000598       ??_C@_0BE@FFEKHNGD@?$CF4d?5?$CF3d?5?7?$CFs?5?$CFs?5?$CFs?$AN?6?$AA@ 10041598     wzdmesh.obj
 0002:000005ac       ??_C@_0M@DOFPGONO@vertex?5?$CFd?$AN?6?$AA@ 100415ac     wzdmesh.obj
 0002:000005b8       ??_C@_03LJIJAGL@tga?$AA@   100415b8     wzdmesh.obj
 0002:000005bc       ??_C@_0BE@FPPMHEOJ@DrawLevelCount?5?$CFd?$AN?6?$AA@ 100415bc     wzdmesh.obj
 0002:000005d0       ??_C@_0BD@DNNPELG@?$CF4d?5?7?$CF4d?5?$CF4d?5?$CF4d?$AN?6?$AA@ 100415d0     wzdmesh.obj
 0002:000005e4       ??_C@_0O@LOGMMKHL@facelist?5?$CFd?$AN?6?$AA@ 100415e4     wzdmesh.obj
 0002:000005f4       ??_C@_0O@PCEEEHDI@uv?$CI?5?$CFs?0?$CFs?5?$CJ?$AN?6?$AA@ 100415f4     wzdmesh.obj
 0002:00000604       ??_C@_0O@POFFAEJA@binormal?$CI?$CFs?$CJ?5?$AA@ 10041604     wzdmesh.obj
 0002:00000614       ??_C@_01GBGANLPD@0?$AA@    10041614     wzdmesh.obj
 0002:00000618       ??_C@_01HIHLOKLC@1?$AA@    10041618     wzdmesh.obj
 0002:0000061c       ??_C@_0BD@FIIFFNPB@tangent?$CI?$CFs?0?$CFs?0?$CFs?$CJ?5?$AA@ 1004161c     wzdmesh.obj
 0002:00000630       ??_C@_0BB@PEFGNHPE@color2?$CI?50x?$CFX?5?$CJ?5?7?$AA@ 10041630     wzdmesh.obj
 0002:00000644       ??_C@_0BA@PIALIMKI@color?$CI?50x?$CFX?5?$CJ?5?7?$AA@ 10041644     wzdmesh.obj
 0002:00000654       ??_C@_0BF@PPFDJLEM@normal?$CI?5?$CFs?0?$CFs?0?$CFs?5?$CJ?5?7?$AA@ 10041654     wzdmesh.obj
 0002:0000066c       ??_C@_0P@JDJMDLLO@?$CF4d?5?7?$CF4d?5?$CF4d?5?7?$AA@ 1004166c     wzdmesh.obj
 0002:0000067c       ??_C@_0M@PIGCEAPC@vplist?5?$CFd?$AN?6?$AA@ 1004167c     wzdmesh.obj
 0002:00000688       ??_C@_0BC@OFOOILOF@MaterialType?5?$CFd?$AN?6?$AA@ 10041688     wzdmesh.obj
 0002:0000069c       ??_C@_0DH@CLCOOEEF@meshgroup?5?$CFd?5?7Diffuse?$CI?$CFs?$CJ?7Specul@ 1004169c     wzdmesh.obj
 0002:000006d4       ??_C@_0BE@KBGONEAB@MeshGroupLayer?5?$CFd?$AN?6?$AA@ 100416d4     wzdmesh.obj
 0002:000006e8       ??_C@_0BG@GIMFKGLM@total?5vertpack?5?$CFd?$AN?6?$AN?6?$AA@ 100416e8     wzdmesh.obj
 0002:00000700       ??_C@_0O@PGGBDLPL@meshlist?5?$CFd?$AN?6?$AA@ 10041700     wzdmesh.obj
 0002:00000710       __real@0000000000000000    10041710     wzdmesh.obj
 0002:00000718       ??_C@_0O@CIGJBMFA@No?5Group?5Name?$AA@ 10041718     wzdmesh.obj
 0002:00000728       ??_C@_07FHEGEDBL@?5?7?$CFd?5?$CFs?$AA@ 10041728     wzdmesh.obj
 0002:00000730       ??_C@_02DPKJAMEF@?$CFd?$AA@ 10041730     wzdmesh.obj
 0002:00000734       ??_C@_0O@NHCNJLDF@Skinning?5?$CFd?$AN?6?$AA@ 10041734     wzdmesh.obj
 0002:00000742       ??_C@_00CNPNBAHC@?$AA@     10041742     wzdmesh.obj
 0002:0000074c       ??_7CWzdMeshConstructor@@6B@ 1004174c     wzdmeshconstructor.obj
 0002:00000828       ??_C@_02HNJCDPAF@m_?$AA@   10041828     wzdmeshconstructor.obj
 0002:00000830       ??_7length_error@std@@6B@  10041830     wzdmeshsorter.obj
 0002:00000838       ??_C@_0BD@OLBABOEK@vector?$DMT?$DO?5too?5long?$AA@ 10041838     wzdmeshsorter.obj
 0002:0000084c       ?npos@?$basic_string@DU?$char_traits@D@std@@V?$allocator@D@2@@std@@2IB 1004184c     wzdmeshsorter.obj
 0002:00000854       ??_7logic_error@std@@6B@   10041854     wzdmeshsorter.obj
 0002:0000085c       ??_C@_0BB@MOGOBHAF@list?$DMT?$DO?5too?5long?$AA@ 1004185c     wzdmeshsorter.obj
 0002:00000874       ??_7bad_alloc@std@@6B@     10041874     wzdmeshsorter.obj
 0002:0000087c       __real@3f4ccccd            1004187c     wzdshareinfo.obj
 0002:00000880       __real@3f19999a            10041880     wzdshareinfo.obj
 0002:00000884       __real@3e4ccccd            10041884     wzdshareinfo.obj
 0002:00000890       __mask@@NegFloat@          10041890     wzdshareinfo.obj
 0002:000008a4       ??_7CWzAniState@@6B@       100418a4     wzanistate.obj
 0002:000008a8       __real@3f9eb851e0000000    100418a8     wzanistate.obj
 0002:000008b0       __real@4024000000000000    100418b0     wzanistate.obj
 0002:000008b8       __real@408f400000000000    100418b8     wzanistate.obj
 0002:000008c0       __real@3f50624de0000000    100418c0     wzanistate.obj
 0002:000008c8       __real@bff0000000000000    100418c8     wzanistate.obj
 0002:000008d0       __real@4059000000000000    100418d0     wzshadowvolume.obj
 0002:000008d8       __real@4000000000000000    100418d8     wzshadowvolume.obj
 0002:000008e0       __real@42c80000            100418e0     wzshadowvolume.obj
 0002:000008e8       __real@beb0c6f7a0000000    100418e8     wzsilhouette.obj
 0002:000008f0       __real@3ba3d70a            100418f0     wzsilhouette.obj
 0002:000008f4       __real@3c75c28f            100418f4     wzsilhouette.obj
 0002:000008fc       ??_7CWzUnit@@6B@           100418fc     wzunit.obj
 0002:00000918       ??_C@_04KDPOIAPE@WZUT?$AA@ 10041918     wzunit_loadsave.obj
 0002:00000920       __real@bf800000            10041920     wzunit_loadsave.obj
 0002:00000928       ??_7CWzUnitDraw@@6B@       10041928     wzunitdraw.obj
 0002:00000930       __real@3f000000            10041930     wzunitdraw.obj
 0002:00000938       ??_7CWzUnitEditable@@6B@   10041938     wzuniteditable.obj
 0002:00000958       ??_7CWzUnitSkeleton@@6B@   10041958     wzunitskeleton.obj
 0002:00000964       ??_7CWzAniStateCB@@6B@     10041964     wzunitskeleton.obj
 0002:00000970       __real@3fe0000000000000    10041970     wzunitskeleton.obj
 0002:000009d8       ??_C@_0BE@JONHPENG@map?1set?$DMT?$DO?5too?5long?$AA@ 100419d8     wzunitskeleton.obj
 0002:000009f0       ??_7out_of_range@std@@6B@  100419f0     wzunitskeleton.obj
 0002:000009f8       ??_C@_0BM@PAPJHAGI@invalid?5map?1set?$DMT?$DO?5iterator?$AA@ 100419f8     wzunitskeleton.obj
 0002:00000a18       ??_7CWzUnitSubType@@6B@    10041a18     wzunitsubtype.obj
 0002:00000a28       __real@43fa0000            10041a28     wzunitsubtype.obj
 0002:00000a30       ??_7CWzUnitSubTypeEditable@@6B@ 10041a30     wzunitsubtypeeditable.obj
 0002:00000a40       __real@3fd0000000000000    10041a40     common:wzmath.obj
 0002:00000a48       __real@3a83126f            10041a48     common:wzmath.obj
 0002:00000a50       __real@3ee4f8b580000000    10041a50     common:wzmath.obj
 0002:00000a58       __real@5368d4a5            10041a58     common:boundingvolume.obj
 0002:00000a5c       __real@d368d4a5            10041a5c     common:boundingvolume.obj
 0002:00000a60       __real@3f1a36e2e0000000    10041a60     common:mathassistant.obj
 0002:00000a68       __real@40490fdb            10041a68     common:mathassistant.obj
 0002:00000a70       ??_7WzLogSystem@WzLog@@6B@ 10041a70     programcommonlibforengine:wzlogsystem.obj
 0002:00000a78       ??_7?$CWzSingleton@VWzLogSystem@WzLog@@@@6B@ 10041a78     programcommonlibforengine:wzlogsystem.obj
 0002:00000a7c       ??_C@_07JLNOKKCE@0x?$CF02X?5?$AA@ 10041a7c     programcommonlibforengine:wzarchive.obj
 0002:00000a88       ??_7?$CWzList@USt_ChunkStack@@@@6B@ 10041a88     programcommonlibforengine:wzarchive.obj
 0002:00000a8c       ??_C@_06DNBDMDIL@?$CF?$CF?4?$CFdf?$AA@ 10041a8c     programcommonlibforengine:filenbuffer.obj
 0002:00000a94       ??_C@_04HDOCAJNK@?$CFs?$CFs?$AA@ 10041a94     programcommonlibforengine:filenbuffer.obj
 0002:00000a9c       ??_C@_0N@PKIBJLNA@WzFilePacker?$AA@ 10041a9c     programcommonlibforengine:discaccess.obj
 0002:00000aac       ??_C@_09LGACLDHG@Hard?5disk?$AA@ 10041aac     programcommonlibforengine:discaccess.obj
 0002:00000ab8       ??_C@_04OHJIHAFH@None?$AA@ 10041ab8     programcommonlibforengine:discaccess.obj
 0002:00000ae4       ??_7?$CWzHandleManager@USt_DAFileInfo@@@@6B@ 10041ae4     programcommonlibforengine:discaccess.obj
 0002:00000ae8       ??_C@_0BA@JFNIOLAK@string?5too?5long?$AA@ 10041ae8     libcpmt:string.obj
 0002:00000af8       ??_C@_0BI@CFPLBAOH@invalid?5string?5position?$AA@ 10041af8     libcpmt:string.obj
 0002:00000b10       __FPinit                   10041b10     LIBCMT:_fpinit_.obj
 0002:00000b14       __FPmtinit                 10041b14     LIBCMT:_fpinit_.obj
 0002:00000b18       __FPmtterm                 10041b18     LIBCMT:_fpinit_.obj
 0002:00000b20       ??_7type_info@@6B@         10041b20     LIBCMT:typinfo.obj
 0002:00000b48       ??_7exception@std@@6B@     10041b48     LIBCMT:stdexcpt.obj
 0002:00000b50       ??_C@_0BC@EOODALEL@Unknown?5exception?$AA@ 10041b50     LIBCMT:stdexcpt.obj
 0002:00000b64       __pRawDllMain              10041b64     LIBCMT:dllcrt0.obj
 0002:00000b64       __pDefaultRawDllMain       10041b64     LIBCMT:dllcrt0.obj
 0002:00000b68       ??_C@_05KLBDPFGC@e?$CL000?$AA@ 10041b68     LIBCMT:cvt.obj
 0002:00000b70       __real@4150017ec0000000    10041b70     LIBCMT:_testfdiv_.obj
 0002:00000b78       __real@4147ffff80000000    10041b78     LIBCMT:_testfdiv_.obj
 0002:00000b80       ??_C@_0BK@NHEOCAHP@IsProcessorFeaturePresent?$AA@ 10041b80     LIBCMT:_testfdiv_.obj
 0002:00000b9c       ??_C@_08CPNIBGIE@KERNEL32?$AA@ 10041b9c     LIBCMT:_testfdiv_.obj
 0002:00000ba8       ??_C@_0O@NLDKAIKN@EncodePointer?$AA@ 10041ba8     LIBCMT:tidtable.obj
 0002:00000bb8       ??_C@_1BK@DBDEIDLH@?$AAK?$AAE?$AAR?$AAN?$AAE?$AAL?$AA3?$AA2?$AA?4?$AAD?$AAL?$AAL?$AA?$AA@ 10041bb8     LIBCMT:tidtable.obj
 0002:00000bd4       ??_C@_0O@KBPMFGHI@DecodePointer?$AA@ 10041bd4     LIBCMT:tidtable.obj
 0002:00000be4       ??_C@_07PEJMOBNF@FlsFree?$AA@ 10041be4     LIBCMT:tidtable.obj
 0002:00000bec       ??_C@_0M@JCPCPOEF@FlsSetValue?$AA@ 10041bec     LIBCMT:tidtable.obj
 0002:00000bf8       ??_C@_0M@GDNOONDI@FlsGetValue?$AA@ 10041bf8     LIBCMT:tidtable.obj
 0002:00000c04       ??_C@_08KNHFBNJ@FlsAlloc?$AA@ 10041c04     LIBCMT:tidtable.obj
 0002:00000c10       ??_C@_0P@MIGLKIOC@CorExitProcess?$AA@ 10041c10     LIBCMT:crt0dat.obj
 0002:00000c20       ??_C@_1BI@BGOHAHKC@?$AAm?$AAs?$AAc?$AAo?$AAr?$AAe?$AAe?$AA?4?$AAd?$AAl?$AAl?$AA?$AA@ 10041c20     LIBCMT:crt0dat.obj
 0002:00000c38       __pDestructExceptionObject 10041c38     LIBCMT:frame.obj
 0002:00000c40       ??_7bad_exception@std@@6B@ 10041c40     LIBCMT:frame.obj
 0002:00000c48       ??_C@_0O@DPKOEFFH@bad?5exception?$AA@ 10041c48     LIBCMT:frame.obj
 0002:00000c60       ??_C@_0P@GGKDKEEG@runtime?5error?5?$AA@ 10041c60     LIBCMT:crt0msg.obj
 0002:00000c70       ??_C@_0O@MJNIPGOH@TLOSS?5error?$AN?6?$AA@ 10041c70     LIBCMT:crt0msg.obj
 0002:00000c80       ??_C@_0N@BONNPDHF@SING?5error?$AN?6?$AA@ 10041c80     LIBCMT:crt0msg.obj
 0002:00000c90       ??_C@_0P@MBDAJNE@DOMAIN?5error?$AN?6?$AA@ 10041c90     LIBCMT:crt0msg.obj
 0002:00000ca0       ??_C@_0JL@DFDOOABL@R6034?$AN?6An?5application?5has?5made?5a@ 10041ca0     LIBCMT:crt0msg.obj
 0002:00000d40       ??_C@_0PH@EPAFIJ@R6033?$AN?6?9?5Attempt?5to?5use?5MSIL?5cod@ 10041d40     LIBCMT:crt0msg.obj
 0002:00000e38       ??_C@_0DD@BKEEABMM@R6032?$AN?6?9?5not?5enough?5space?5for?5lo@ 10041e38     LIBCMT:crt0msg.obj
 0002:00000e70       ??_C@_0GD@OFKILIED@R6031?$AN?6?9?5Attempt?5to?5initialize?5t@ 10041e70     LIBCMT:crt0msg.obj
 0002:00000ed4       ??_C@_0BP@LPMHJOKI@R6030?$AN?6?9?5CRT?5not?5initialized?$AN?6?$AA@ 10041ed4     LIBCMT:crt0msg.obj
 0002:00000ef4       ??_C@_0CF@KJDAIALP@R6028?$AN?6?9?5unable?5to?5initialize?5he@ 10041ef4     LIBCMT:crt0msg.obj
 0002:00000f1c       ??_C@_0DF@GAKBPDFP@R6027?$AN?6?9?5not?5enough?5space?5for?5lo@ 10041f1c     LIBCMT:crt0msg.obj
 0002:00000f54       ??_C@_0DF@IBLNNAIG@R6026?$AN?6?9?5not?5enough?5space?5for?5st@ 10041f54     LIBCMT:crt0msg.obj
 0002:00000f8c       ??_C@_0CG@IOHKGFNJ@R6025?$AN?6?9?5pure?5virtual?5function?5c@ 10041f8c     LIBCMT:crt0msg.obj
 0002:00000fb4       ??_C@_0DF@JIJJFJDC@R6024?$AN?6?9?5not?5enough?5space?5for?5_o@ 10041fb4     LIBCMT:crt0msg.obj
 0002:00000fec       ??_C@_0CJ@EGEJHFME@R6019?$AN?6?9?5unable?5to?5open?5console?5@ 10041fec     LIBCMT:crt0msg.obj
 0002:00001018       ??_C@_0CB@GNHNIELH@R6018?$AN?6?9?5unexpected?5heap?5error?$AN?6@ 10042018     LIBCMT:crt0msg.obj
 0002:0000103c       ??_C@_0CN@FOLDKNG@R6017?$AN?6?9?5unexpected?5multithread?5@ 1004203c     LIBCMT:crt0msg.obj
 0002:0000106c       ??_C@_0CM@FAHFJNHO@R6016?$AN?6?9?5not?5enough?5space?5for?5th@ 1004206c     LIBCMT:crt0msg.obj
 0002:00001098       ??_C@_0JG@LBKMGKLD@?$AN?6This?5application?5has?5requested@ 10042098     LIBCMT:crt0msg.obj
 0002:00001130       ??_C@_0CM@FLCNIPKK@R6009?$AN?6?9?5not?5enough?5space?5for?5en@ 10042130     LIBCMT:crt0msg.obj
 0002:0000115c       ??_C@_0CK@KMMJOAPP@R6008?$AN?6?9?5not?5enough?5space?5for?5ar@ 1004215c     LIBCMT:crt0msg.obj
 0002:00001188       ??_C@_0CN@LEKKICBM@R6002?$AN?6?9?5floating?5point?5support?5@ 10042188     LIBCMT:crt0msg.obj
 0002:000011b8       ??_C@_0CF@GOGNBNAK@Microsoft?5Visual?5C?$CL?$CL?5Runtime?5Lib@ 100421b8     LIBCMT:crt0msg.obj
 0002:000011e0       ??_C@_02PHMGELLB@?6?6?$AA@ 100421e0     LIBCMT:crt0msg.obj
 0002:000011e4       ??_C@_03KHICJKCI@?4?4?4?$AA@ 100421e4     LIBCMT:crt0msg.obj
 0002:000011e8       ??_C@_0BH@DNAGHKFM@?$DMprogram?5name?5unknown?$DO?$AA@ 100421e8     LIBCMT:crt0msg.obj
 0002:00001200       ??_C@_0BK@OFGJDLJJ@Runtime?5Error?$CB?6?6Program?3?5?$AA@ 10042200     LIBCMT:crt0msg.obj
 0002:000012a0       ??_C@_01NEMOKFLO@?$DN?$AA@ 100422a0     LIBCMT:setlocal.obj
 0002:000012b8       __DEFAULT_CW_in_mem        100422b8     LIBCMT:_common_.obj
 0002:000012ba       __pi_by_2_to_61            100422ba     LIBCMT:_common_.obj
 0002:000012f8       __XcptActTab               100422f8     LIBCMT:winxfltr.obj
 0002:00003ce0       ??_C@_1O@CEDCILHN@?$AA?$CI?$AAn?$AAu?$AAl?$AAl?$AA?$CJ?$AA?$AA@ 10044ce0     LIBCMT:output.obj
 0002:00003cf0       ??_C@_06OJHGLDPL@?$CInull?$CJ?$AA@ 10044cf0     LIBCMT:output.obj
 0002:00003cf8       ___lookuptable             10044cf8     LIBCMT:output.obj
 0002:00003d54       ??_C@_0BK@CFCOFLF@?5Complete?5Object?5Locator?8?$AA@ 10044d54     LIBCMT:undname.obj
 0002:00003d70       ??_C@_0BN@MECKDCOJ@?5Class?5Hierarchy?5Descriptor?8?$AA@ 10044d70     LIBCMT:undname.obj
 0002:00003d90       ??_C@_0BD@LGICGFMM@?5Base?5Class?5Array?8?$AA@ 10044d90     LIBCMT:undname.obj
 0002:00003da4       ??_C@_0BM@LDKODKLH@?5Base?5Class?5Descriptor?5at?5?$CI?$AA@ 10044da4     LIBCMT:undname.obj
 0002:00003dc0       ??_C@_0BC@DAFEJGAK@?5Type?5Descriptor?8?$AA@ 10044dc0     LIBCMT:undname.obj
 0002:00003dd4       ??_C@_0BM@PMGGMLDN@?$GAlocal?5static?5thread?5guard?8?$AA@ 10044dd4     LIBCMT:undname.obj
 0002:00003df0       ??_C@_0CL@FGIJHLCE@?$GAmanaged?5vector?5copy?5constructor@ 10044df0     LIBCMT:undname.obj
 0002:00003e1c       ??_C@_0CJ@GJELGAMM@?$GAvector?5vbase?5copy?5constructor?5i@ 10044e1c     LIBCMT:undname.obj
 0002:00003e48       ??_C@_0CD@CGAJBKEJ@?$GAvector?5copy?5constructor?5iterato@ 10044e48     LIBCMT:undname.obj
 0002:00003e6c       ??_C@_0CB@PDBIFEP@?$GAdynamic?5atexit?5destructor?5for?5?8@ 10044e6c     LIBCMT:undname.obj
 0002:00003e90       ??_C@_0BL@CLIPGLGB@?$GAdynamic?5initializer?5for?5?8?$AA@ 10044e90     LIBCMT:undname.obj
 0002:00003eac       ??_C@_0CM@FCBBDIGB@?$GAeh?5vector?5vbase?5copy?5constructo@ 10044eac     LIBCMT:undname.obj
 0002:00003ed8       ??_C@_0CG@HLDDJMAG@?$GAeh?5vector?5copy?5constructor?5iter@ 10044ed8     LIBCMT:undname.obj
 0002:00003f00       ??_C@_0CF@IMGKMJNO@?$GAmanaged?5vector?5destructor?5itera@ 10044f00     LIBCMT:undname.obj
 0002:00003f28       ??_C@_0CG@CFDHKGGD@?$GAmanaged?5vector?5constructor?5iter@ 10044f28     LIBCMT:undname.obj
 0002:00003f50       ??_C@_0BN@CKNJLHMB@?$GAplacement?5delete?$FL?$FN?5closure?8?$AA@ 10044f50     LIBCMT:undname.obj
 0002:00003f70       ??_C@_0BL@CNOONJFP@?$GAplacement?5delete?5closure?8?$AA@ 10044f70     LIBCMT:undname.obj
 0002:00003f8c       ??_C@_0P@HJKNJFNN@?$GAomni?5callsig?8?$AA@ 10044f8c     LIBCMT:undname.obj
 0002:00003f9c       ??_C@_09LBNFPBCA@?5delete?$FL?$FN?$AA@ 10044f9c     LIBCMT:undname.obj
 0002:00003fa8       ??_C@_06FHBGPFGH@?5new?$FL?$FN?$AA@ 10044fa8     LIBCMT:undname.obj
 0002:00003fb0       ??_C@_0CE@IIHCMGGL@?$GAlocal?5vftable?5constructor?5closu@ 10044fb0     LIBCMT:undname.obj
 0002:00003fd4       ??_C@_0BA@KKLDJDLB@?$GAlocal?5vftable?8?$AA@ 10044fd4     LIBCMT:undname.obj
 0002:00003fe4       ??_C@_05KHLCHHI@?$GARTTI?$AA@ 10044fe4     LIBCMT:undname.obj
 0002:00003fec       ??_C@_03KLGMFNMG@?$GAEH?$AA@ 10044fec     LIBCMT:undname.obj
 0002:00003ff0       ??_C@_0BA@KBCDOMBN@?$GAudt?5returning?8?$AA@ 10044ff0     LIBCMT:undname.obj
 0002:00004000       ??_C@_0BL@LLKPOHJI@?$GAcopy?5constructor?5closure?8?$AA@ 10045000     LIBCMT:undname.obj
 0002:0000401c       ??_C@_0CH@OOJPLCPH@?$GAeh?5vector?5vbase?5constructor?5ite@ 1004501c     LIBCMT:undname.obj
 0002:00004044       ??_C@_0CA@GCEOPDGL@?$GAeh?5vector?5destructor?5iterator?8?$AA@ 10045044     LIBCMT:undname.obj
 0002:00004064       ??_C@_0CB@JONCMFFK@?$GAeh?5vector?5constructor?5iterator?8@ 10045064     LIBCMT:undname.obj
 0002:00004088       ??_C@_0BL@NILFHHPC@?$GAvirtual?5displacement?5map?8?$AA@ 10045088     LIBCMT:undname.obj
 0002:000040a4       ??_C@_0CE@IKBNEHA@?$GAvector?5vbase?5constructor?5iterat@ 100450a4     LIBCMT:undname.obj
 0002:000040c8       ??_C@_0BN@LFPFMEDL@?$GAvector?5destructor?5iterator?8?$AA@ 100450c8     LIBCMT:undname.obj
 0002:000040e8       ??_C@_0BO@PFGOCPJJ@?$GAvector?5constructor?5iterator?8?$AA@ 100450e8     LIBCMT:undname.obj
 0002:00004108       ??_C@_0BN@IMDCHIKM@?$GAscalar?5deleting?5destructor?8?$AA@ 10045108     LIBCMT:undname.obj
 0002:00004128       ??_C@_0BO@OBMKPJIG@?$GAdefault?5constructor?5closure?8?$AA@ 10045128     LIBCMT:undname.obj
 0002:00004148       ??_C@_0BN@DEGPLNFK@?$GAvector?5deleting?5destructor?8?$AA@ 10045148     LIBCMT:undname.obj
 0002:00004168       ??_C@_0BD@JDLKDPAB@?$GAvbase?5destructor?8?$AA@ 10045168     LIBCMT:undname.obj
 0002:0000417c       ??_C@_08OBABFOLI@?$GAstring?8?$AA@ 1004517c     LIBCMT:undname.obj
 0002:00004188       ??_C@_0BF@KDPPACIK@?$GAlocal?5static?5guard?8?$AA@ 10045188     LIBCMT:undname.obj
 0002:000041a0       ??_C@_08LLFFHHDJ@?$GAtypeof?8?$AA@ 100451a0     LIBCMT:undname.obj
 0002:000041ac       ??_C@_07FEEIOKP@?$GAvcall?8?$AA@ 100451ac     LIBCMT:undname.obj
 0002:000041b4       ??_C@_09BLBHBJP@?$GAvbtable?8?$AA@ 100451b4     LIBCMT:undname.obj
 0002:000041c0       ??_C@_09IFPLHPGF@?$GAvftable?8?$AA@ 100451c0     LIBCMT:undname.obj
 0002:000041cc       ??_C@_02MHEGNOJ@?$FO?$DN?$AA@ 100451cc     LIBCMT:undname.obj
 0002:000041d0       ??_C@_02DHLNPPGH@?$HM?$DN?$AA@ 100451d0     LIBCMT:undname.obj
 0002:000041d4       ??_C@_02FGJGFEAB@?$CG?$DN?$AA@ 100451d4     LIBCMT:undname.obj
 0002:000041d8       ??_C@_03CDNPDDLA@?$DM?$DM?$DN?$AA@ 100451d8     LIBCMT:undname.obj
 0002:000041dc       ??_C@_03IKFCCPFF@?$DO?$DO?$DN?$AA@ 100451dc     LIBCMT:undname.obj
 0002:000041e0       ??_C@_02FENAOKFI@?$CF?$DN?$AA@ 100451e0     LIBCMT:undname.obj
 0002:000041e4       ??_C@_02FJEHGPIO@?1?$DN?$AA@ 100451e4     LIBCMT:undname.obj
 0002:000041e8       ??_C@_02FKMDLLOA@?9?$DN?$AA@ 100451e8     LIBCMT:undname.obj
 0002:000041ec       ??_C@_02FOEOMHFC@?$CL?$DN?$AA@ 100451ec     LIBCMT:undname.obj
 0002:000041f0       ??_C@_02FPIMKNGF@?$CK?$DN?$AA@ 100451f0     LIBCMT:undname.obj
 0002:000041f4       ??_C@_02NONPIBCD@?$HM?$HM?$AA@ 100451f4     LIBCMT:undname.obj
 0002:000041f8       ??_C@_02PPKAJPJL@?$CG?$CG?$AA@ 100451f8     LIBCMT:undname.obj
 0002:000041fc       ??_C@_01DNKMNLPK@?$HM?$AA@ 100451fc     LIBCMT:undname.obj
 0002:00004200       ??_C@_01JKBOJNNK@?$FO?$AA@ 10045200     LIBCMT:undname.obj
 0002:00004204       ??_C@_01PJKLJHI@?$HO?$AA@  10045204     LIBCMT:undname.obj
 0002:00004208       ??_C@_02HCKGKOFO@?$CI?$CJ?$AA@ 10045208     LIBCMT:undname.obj
 0002:0000420c       ??_C@_01IHBHIGKO@?0?$AA@   1004520c     LIBCMT:undname.obj
 0002:00004210       ??_C@_02EEKDKGMJ@?$DO?$DN?$AA@ 10045210     LIBCMT:undname.obj
 0002:00004214       ??_C@_01PPODPGHN@?$DO?$AA@ 10045214     LIBCMT:undname.obj
 0002:00004218       ??_C@_02EHCHHCKH@?$DM?$DN?$AA@ 10045218     LIBCMT:undname.obj
 0002:0000421c       ??_C@_01MNNFJEPP@?$DM?$AA@ 1004521c     LIBCMT:undname.obj
 0002:00004220       ??_C@_01FGNFDNOH@?$CF?$AA@ 10045220     LIBCMT:undname.obj
 0002:00004224       ??_C@_01KMDKNFGN@?1?$AA@   10045224     LIBCMT:undname.obj
 0002:00004228       ??_C@_03MNHNFDLC@?9?$DO?$CK?$AA@ 10045228     LIBCMT:undname.obj
 0002:0000422c       ??_C@_01HNPIGOCE@?$CG?$AA@ 1004522c     LIBCMT:undname.obj
 0002:00004230       ??_C@_01MIFGBAGJ@?$CL?$AA@ 10045230     LIBCMT:undname.obj
 0002:00004234       ??_C@_01JOAMLHOP@?9?$AA@   10045234     LIBCMT:undname.obj
 0002:00004238       ??_C@_02BAABKJLB@?9?9?$AA@ 10045238     LIBCMT:undname.obj
 0002:0000423c       ??_C@_02ECNGHCIF@?$CL?$CL?$AA@ 1004523c     LIBCMT:undname.obj
 0002:00004240       ??_C@_01NBENCBCI@?$CK?$AA@ 10045240     LIBCMT:undname.obj
 0002:00004244       ??_C@_02HBOOOICD@?9?$DO?$AA@ 10045244     LIBCMT:undname.obj
 0002:00004248       ??_C@_08LHJFAFGD@operator?$AA@ 10045248     LIBCMT:undname.obj
 0002:00004254       ??_C@_02GPECMEKF@?$FL?$FN?$AA@ 10045254     LIBCMT:undname.obj
 0002:00004258       ??_C@_02FDNJECIE@?$CB?$DN?$AA@ 10045258     LIBCMT:undname.obj
 0002:0000425c       ??_C@_02EGOFBIJA@?$DN?$DN?$AA@ 1004525c     LIBCMT:undname.obj
 0002:00004260       ??_C@_01DCLJPIOD@?$CB?$AA@ 10045260     LIBCMT:undname.obj
 0002:00004264       ??_C@_02FODMEDOG@?$DM?$DM?$AA@ 10045264     LIBCMT:undname.obj
 0002:00004268       ??_C@_02GPIOPFAK@?$DO?$DO?$AA@ 10045268     LIBCMT:undname.obj
 0002:0000426c       ??_C@_07FPCDHGMM@?5delete?$AA@ 1004526c     LIBCMT:undname.obj
 0002:00004274       ??_C@_04NIHEBCM@?5new?$AA@ 10045274     LIBCMT:undname.obj
 0002:0000427c       ??_C@_0M@GFIIJFMG@__unaligned?$AA@ 1004527c     LIBCMT:undname.obj
 0002:00004288       ??_C@_0L@PILCLIHE@__restrict?$AA@ 10045288     LIBCMT:undname.obj
 0002:00004294       ??_C@_07JOMMBBKO@__ptr64?$AA@ 10045294     LIBCMT:undname.obj
 0002:0000429c       ??_C@_09HIJEGCPM@__clrcall?$AA@ 1004529c     LIBCMT:undname.obj
 0002:000042a8       ??_C@_0L@JMKHOMEK@__fastcall?$AA@ 100452a8     LIBCMT:undname.obj
 0002:000042b4       ??_C@_0L@NPHFGOKO@__thiscall?$AA@ 100452b4     LIBCMT:undname.obj
 0002:000042c0       ??_C@_09IFJBGAPI@__stdcall?$AA@ 100452c0     LIBCMT:undname.obj
 0002:000042cc       ??_C@_08GHMPAG@__pascal?$AA@ 100452cc     LIBCMT:undname.obj
 0002:000042d8       ??_C@_07KOLFKCDI@__cdecl?$AA@ 100452d8     LIBCMT:undname.obj
 0002:000042e0       ??_C@_08EHJDFFNH@__based?$CI?$AA@ 100452e0     LIBCMT:undname.obj
 0002:00004470       ??_C@_0BI@DFKBFLJE@GetProcessWindowStation?$AA@ 10045470     LIBCMT:crtmbox.obj
 0002:00004488       ??_C@_0BK@CIDNPOGP@GetUserObjectInformationA?$AA@ 10045488     LIBCMT:crtmbox.obj
 0002:000044a4       ??_C@_0BD@HHGDFDBJ@GetLastActivePopup?$AA@ 100454a4     LIBCMT:crtmbox.obj
 0002:000044b8       ??_C@_0BA@HNOPNCHB@GetActiveWindow?$AA@ 100454b8     LIBCMT:crtmbox.obj
 0002:000044c8       ??_C@_0M@CHKKJDAI@MessageBoxA?$AA@ 100454c8     LIBCMT:crtmbox.obj
 0002:000044d4       ??_C@_0L@NDEGIDAG@USER32?4DLL?$AA@ 100454d4     LIBCMT:crtmbox.obj
 0002:000044e0       __real@00000000            100454e0     wzdanimation.obj
 0002:000044e0       ??_C@_13NOLLCAOD@?$AA?$AA?$AA?$AA@ 100454e0     LIBCMT:a_map.obj
 0002:000044e8       ___newctype                100454e8     LIBCMT:ctype.obj
 0002:000047e8       __wctype                   100457e8     LIBCMT:ctype.obj
 0002:000049f0       ___newclmap                100459f0     LIBCMT:ctype.obj
 0002:00004b70       ___newcumap                10045b70     LIBCMT:ctype.obj
 0002:00004cf0       ??_C@_08JCCMCCIL@HH?3mm?3ss?$AA@ 10045cf0     LIBCMT:strftime.obj
 0002:00004cfc       ??_C@_0BE@CKGJFCPC@dddd?0?5MMMM?5dd?0?5yyyy?$AA@ 10045cfc     LIBCMT:strftime.obj
 0002:00004d10       ??_C@_08BPBNCDIB@MM?1dd?1yy?$AA@ 10045d10     LIBCMT:strftime.obj
 0002:00004d1c       ??_C@_02CJNFDJBF@PM?$AA@   10045d1c     LIBCMT:strftime.obj
 0002:00004d20       ??_C@_02DEDBPAFC@AM?$AA@   10045d20     LIBCMT:strftime.obj
 0002:00004d24       ??_C@_08EDHMEBNP@December?$AA@ 10045d24     LIBCMT:strftime.obj
 0002:00004d30       ??_C@_08HCHEGEOA@November?$AA@ 10045d30     LIBCMT:strftime.obj
 0002:00004d3c       ??_C@_07JJNFCEND@October?$AA@ 10045d3c     LIBCMT:strftime.obj
 0002:00004d44       ??_C@_09BHHEALKD@September?$AA@ 10045d44     LIBCMT:strftime.obj
 0002:00004d50       ??_C@_06LBBHFDDG@August?$AA@ 10045d50     LIBCMT:strftime.obj
 0002:00004d58       ??_C@_04MIEPOIFP@July?$AA@ 10045d58     LIBCMT:strftime.obj
 0002:00004d60       ??_C@_04CNLMGBGM@June?$AA@ 10045d60     LIBCMT:strftime.obj
 0002:00004d68       ??_C@_05DMJDNLEJ@April?$AA@ 10045d68     LIBCMT:strftime.obj
 0002:00004d70       ??_C@_05HPCKOFNC@March?$AA@ 10045d70     LIBCMT:strftime.obj
 0002:00004d78       ??_C@_08GNJGEPFN@February?$AA@ 10045d78     LIBCMT:strftime.obj
 0002:00004d84       ??_C@_07CGJPFGJA@January?$AA@ 10045d84     LIBCMT:strftime.obj
 0002:00004d8c       ??_C@_03MKABNOCG@Dec?$AA@  10045d8c     LIBCMT:strftime.obj
 0002:00004d90       ??_C@_03JPJOFNIA@Nov?$AA@  10045d90     LIBCMT:strftime.obj
 0002:00004d94       ??_C@_03BMAOKBAD@Oct?$AA@  10045d94     LIBCMT:strftime.obj
 0002:00004d98       ??_C@_03GGCAPAJC@Sep?$AA@  10045d98     LIBCMT:strftime.obj
 0002:00004d9c       ??_C@_03IFJFEIGA@Aug?$AA@  10045d9c     LIBCMT:strftime.obj
 0002:00004da0       ??_C@_03LBGABGKK@Jul?$AA@  10045da0     LIBCMT:strftime.obj
 0002:00004da4       ??_C@_03IDFGHECI@Jun?$AA@  10045da4     LIBCMT:strftime.obj
 0002:00004da8       ??_C@_03CNMDKL@May?$AA@    10045da8     LIBCMT:strftime.obj
 0002:00004dac       ??_C@_03LEOLGMJP@Apr?$AA@  10045dac     LIBCMT:strftime.obj
 0002:00004db0       ??_C@_03ODNJBKGA@Mar?$AA@  10045db0     LIBCMT:strftime.obj
 0002:00004db4       ??_C@_03HJBDCHOM@Feb?$AA@  10045db4     LIBCMT:strftime.obj
 0002:00004db8       ??_C@_03JIHJHPIE@Jan?$AA@  10045db8     LIBCMT:strftime.obj
 0002:00004dbc       ??_C@_08INBOOONO@Saturday?$AA@ 10045dbc     LIBCMT:strftime.obj
 0002:00004dc8       ??_C@_06JECMNKMI@Friday?$AA@ 10045dc8     LIBCMT:strftime.obj
 0002:00004dd0       ??_C@_08HACCIKIA@Thursday?$AA@ 10045dd0     LIBCMT:strftime.obj
 0002:00004ddc       ??_C@_09DLIGFAKA@Wednesday?$AA@ 10045ddc     LIBCMT:strftime.obj
 0002:00004de8       ??_C@_07BAAGCFCM@Tuesday?$AA@ 10045de8     LIBCMT:strftime.obj
 0002:00004df0       ??_C@_06JLEDEDGH@Monday?$AA@ 10045df0     LIBCMT:strftime.obj
 0002:00004df8       ??_C@_06OOPIFAJ@Sunday?$AA@ 10045df8     LIBCMT:strftime.obj
 0002:00004e00       ??_C@_03FEFJNEK@Sat?$AA@   10045e00     LIBCMT:strftime.obj
 0002:00004e04       ??_C@_03IDIOELNC@Fri?$AA@  10045e04     LIBCMT:strftime.obj
 0002:00004e08       ??_C@_03IOFIKPDN@Thu?$AA@  10045e08     LIBCMT:strftime.obj
 0002:00004e0c       ??_C@_03MHOMLAJA@Wed?$AA@  10045e0c     LIBCMT:strftime.obj
 0002:00004e10       ??_C@_03NAGEINEP@Tue?$AA@  10045e10     LIBCMT:strftime.obj
 0002:00004e14       ??_C@_03PDAGKDH@Mon?$AA@   10045e14     LIBCMT:strftime.obj
 0002:00004e18       ??_C@_03KOEHGMDN@Sun?$AA@  10045e18     LIBCMT:strftime.obj
 0002:00004e88       ??_C@_03IIINPABG@tan?$AA@  10045e88     LIBCMT:_libm_error_.obj
 0002:00004e8c       ??_C@_03LALBNOCG@cos?$AA@  10045e8c     LIBCMT:_libm_error_.obj
 0002:00004e90       ??_C@_03BLEJJJBH@sin?$AA@  10045e90     LIBCMT:_libm_error_.obj
 0002:00004e94       ??_C@_04EHEDPDJG@modf?$AA@ 10045e94     LIBCMT:_libm_error_.obj
 0002:00004e9c       ??_C@_05PBJFFIGL@floor?$AA@ 10045e9c     LIBCMT:_libm_error_.obj
 0002:00004ea4       ??_C@_04GFPJNGEK@ceil?$AA@ 10045ea4     LIBCMT:_libm_error_.obj
 0002:00004eac       ??_C@_04MLLJIGOK@atan?$AA@ 10045eac     LIBCMT:_libm_error_.obj
 0002:00004eb4       ??_C@_05EOHGHCHD@exp10?$AA@ 10045eb4     LIBCMT:_libm_error_.obj
 0002:00004ebc       ??_C@_04PDIFKINK@acos?$AA@ 10045ebc     LIBCMT:_libm_error_.obj
 0002:00004ec4       ??_C@_04FIHNOPOL@asin?$AA@ 10045ec4     LIBCMT:_libm_error_.obj
 0002:00004ecc       ??_C@_03MGHMBJCF@log?$AA@  10045ecc     LIBCMT:_libm_error_.obj
 0002:00004ed0       ??_C@_05HGHHAHAP@log10?$AA@ 10045ed0     LIBCMT:_libm_error_.obj
 0002:00004ed8       ??_C@_03KHJOGHMM@exp?$AA@  10045ed8     LIBCMT:_libm_error_.obj
 0002:00004edc       ??_C@_03JGHBODFD@pow?$AA@  10045edc     LIBCMT:_libm_error_.obj
 0002:00004ee0       ___lookuptable_s           10045ee0     LIBCMT:outputs.obj
 0002:00004f3c       ??_C@_06IMKFLFPG@1?$CDQNAN?$AA@ 10045f3c     LIBCMT:_x10fout_.obj
 0002:00004f44       ??_C@_05DNEBIAHO@1?$CDINF?$AA@ 10045f44     LIBCMT:_x10fout_.obj
 0002:00004f4c       ??_C@_05PHHOCPM@1?$CDIND?$AA@ 10045f4c     LIBCMT:_x10fout_.obj
 0002:00004f54       ??_C@_06PGGFOGJG@1?$CDSNAN?$AA@ 10045f54     LIBCMT:_x10fout_.obj
 0002:00004f5c       ___dnames                  10045f5c     LIBCMT:timeset.obj
 0002:00004f74       ___mnames                  10045f74     LIBCMT:timeset.obj
 0002:00004f9c       ??_C@_0L@KDOEJCKC@_nextafter?$AA@ 10045f9c     LIBCMT:_fpexcept_.obj
 0002:00004fa8       ??_C@_05JGDBENOH@_logb?$AA@ 10045fa8     LIBCMT:_fpexcept_.obj
 0002:00004fb0       ??_C@_03ONILCKOB@_yn?$AA@  10045fb0     LIBCMT:_fpexcept_.obj
 0002:00004fb4       ??_C@_03NAKIGLHK@_y1?$AA@  10045fb4     LIBCMT:_fpexcept_.obj
 0002:00004fb8       ??_C@_03MJLDFKDL@_y0?$AA@  10045fb8     LIBCMT:_fpexcept_.obj
 0002:00004fbc       ??_C@_05GKKHEGJL@frexp?$AA@ 10045fbc     LIBCMT:_fpexcept_.obj
 0002:00004fc4       ??_C@_04KEPJIHGP@fmod?$AA@ 10045fc4     LIBCMT:_fpexcept_.obj
 0002:00004fcc       ??_C@_06MEIMCGCF@_hypot?$AA@ 10045fcc     LIBCMT:_fpexcept_.obj
 0002:00004fd4       ??_C@_05KBKMEMPO@_cabs?$AA@ 10045fd4     LIBCMT:_fpexcept_.obj
 0002:00004fdc       ??_C@_05CEJMAHNP@ldexp?$AA@ 10045fdc     LIBCMT:_fpexcept_.obj
 0002:00004fe4       ??_C@_04ODHECPBC@fabs?$AA@ 10045fe4     LIBCMT:_fpexcept_.obj
 0002:00004fec       ??_C@_04EIAKFFMI@sqrt?$AA@ 10045fec     LIBCMT:_fpexcept_.obj
 0002:00004ff4       ??_C@_05KNGEOGJB@atan2?$AA@ 10045ff4     LIBCMT:_fpexcept_.obj
 0002:00004ffc       ??_C@_04FJHINJAO@tanh?$AA@ 10045ffc     LIBCMT:_fpexcept_.obj
 0002:00005004       ??_C@_04HPJJNFIM@cosh?$AA@ 10046004     LIBCMT:_fpexcept_.obj
 0002:0000500c       ??_C@_04COOMCNPB@sinh?$AA@ 1004600c     LIBCMT:_fpexcept_.obj
 0002:00005014       ??_C@_07GPDNMNG@CONOUT$?$AA@ 10046014     LIBCMT:initcon.obj
 0002:00005238       __real@4f800000            10046238     wzFilePacker_static:wzFilePacker.obj
 0002:00005aa0       ??_C@_0BI@LCBABOGN@header?5is?5Final?5Version?$AA@ 10046aa0     wzFilePacker_static:fsvfs.obj
 0002:00005ab8       ??_C@_0P@FOHJAHFG@header?5invalid?$AA@ 10046ab8     wzFilePacker_static:fsvfs.obj
 0002:00005ac8       ??_C@_0DM@MLIJDPNB@Now?5Packing?5File?5Version?5?3?5?$CFd?0?5P@ 10046ac8     wzFilePacker_static:fsvfs.obj
 0002:00005b04       ??_C@_0DA@JPDHOIDD@?$CK?$CK?$CK?$CK?$CK?$CK?$CK?$CK?$CK?$CK?$CK?$CK?$CK?$CK?$CK?$CK?5N2_UpdateFilePo@ 10046b04     wzFilePacker_static:fsvfs.obj
 0002:00005b34       ??_C@_0CO@LGMGIONK@?$CK?$CK?$CK?$CK?$CK?$CK?$CK?$CK?$CK?$CK?$CK?$CK?$CK?$CK?$CK?$CK?5N2_SetFilePoint@ 10046b34     wzFilePacker_static:fsvfs.obj
 0002:00005b64       ??_C@_0DF@IHAPMOPK@?$CL?$CL?$CL?$CL?$CL?$CL?$CL?$CL?$CL?$CL?5ReadFail_4_Error?5?3?5?G?O@ 10046b64     wzFilePacker_static:fsvfs.obj
 0002:00005b9c       ??_C@_0DH@HABJGGNC@?$CL?$CL?$CL?$CL?$CL?$CL?$CL?$CL?$CL?$CL?5ReadFail_3_Error?5?3?5?$MA?P@ 10046b9c     wzFilePacker_static:fsvfs.obj
 0002:00005bd4       ??_C@_0DG@LCJJILDN@?$CL?$CL?$CL?$CL?$CL?$CL?$CL?$CL?$CL?$CL?5ReadFail_2_Error?5?3?5?$LP?$MA@ 10046bd4     wzFilePacker_static:fsvfs.obj
 0002:00005c0c       ??_C@_0CG@GENKINJN@?$CL?$CL?$CL?$CL?$CL?$CL?$CL?$CL?$CL?$CL?5ReadFail_1_ErrorCode?5@ 10046c0c     wzFilePacker_static:fsvfs.obj
 0002:00005c34       ??_C@_0BH@MMBDGEON@Remove?5Fsvfs?5Tree?5Fail?$AA@ 10046c34     wzFilePacker_static:fsvfs.obj
 0002:00005c4c       ??_C@_0BK@PKGCLKLI@Remove?5Fsvfs?5Tree?5SUCCESS?$AA@ 10046c4c     wzFilePacker_static:fsvfs.obj
 0002:00005c68       ??_C@_0BM@OPDJPMGP@Not?5File?5SameName?5Tree?9Node?$AA@ 10046c68     wzFilePacker_static:fsvfs.obj
 0002:000060b8       ??_C@_02CEGDFPFP@?4?2?$AA@ 100470b8     wzFilePacker_static:fsdos.obj
 0002:000060bc       ??_C@_0BP@PFJFMKGH@Win32_SetFilePointer_Error?3?$CFd?6?$AA@ 100470bc     wzFilePacker_static:fsdos.obj
 0002:00006530       __load_config_used         10047530     LIBCMT:loadcfg.obj
 0002:000065ec       ??_R4CWzdAnimation@@6B@    100475ec     wzdanimation.obj
 0002:00006600       ??_R3CWzdAnimation@@8      10047600     wzdanimation.obj
 0002:00006610       ??_R2CWzdAnimation@@8      10047610     wzdanimation.obj
 0002:0000661c       ??_R1A@?0A@EA@CWzdAnimation@@8 1004761c     wzdanimation.obj
 0002:00006638       ??_R1A@?0A@EA@CWzdBase@@8  10047638     wzdanimation.obj
 0002:00006654       ??_R3CWzdBase@@8           10047654     wzdanimation.obj
 0002:00006664       ??_R2CWzdBase@@8           10047664     wzdanimation.obj
 0002:0000666c       ??_R4CWzdBase@@6B@         1004766c     wzdbase.obj
 0002:00006680       ??_R4CWzdMesh@@6B@         10047680     wzdmesh.obj
 0002:00006694       ??_R3CWzdMesh@@8           10047694     wzdmesh.obj
 0002:000066a4       ??_R2CWzdMesh@@8           100476a4     wzdmesh.obj
 0002:000066b8       ??_R1A@?0A@EA@CWzdMesh@@8  100476b8     wzdmesh.obj
 0002:000066d4       ??_R1A@?0A@EA@CWzdMeshConstructor@@8 100476d4     wzdmesh.obj
 0002:000066f0       ??_R3CWzdMeshConstructor@@8 100476f0     wzdmesh.obj
 0002:00006700       ??_R2CWzdMeshConstructor@@8 10047700     wzdmesh.obj
 0002:00006710       ??_R4CWzdMeshConstructor@@6B@ 10047710     wzdmeshconstructor.obj
 0002:00006724       ??_R4length_error@std@@6B@ 10047724     wzdmeshsorter.obj
 0002:00006738       ??_R3length_error@std@@8   10047738     wzdmeshsorter.obj
 0002:00006748       ??_R2length_error@std@@8   10047748     wzdmeshsorter.obj
 0002:00006758       ??_R1A@?0A@EA@length_error@std@@8 10047758     wzdmeshsorter.obj
 0002:00006774       ??_R1A@?0A@EA@logic_error@std@@8 10047774     wzdmeshsorter.obj
 0002:00006790       ??_R3logic_error@std@@8    10047790     wzdmeshsorter.obj
 0002:000067a0       ??_R2logic_error@std@@8    100477a0     wzdmeshsorter.obj
 0002:000067ac       ??_R1A@?0A@EA@exception@std@@8 100477ac     wzdmeshsorter.obj
 0002:000067c8       ??_R3exception@std@@8      100477c8     wzdmeshsorter.obj
 0002:000067d8       ??_R2exception@std@@8      100477d8     wzdmeshsorter.obj
 0002:000067e0       ??_R4logic_error@std@@6B@  100477e0     wzdmeshsorter.obj
 0002:000067f4       ??_R4bad_alloc@std@@6B@    100477f4     wzdmeshsorter.obj
 0002:00006808       ??_R3bad_alloc@std@@8      10047808     wzdmeshsorter.obj
 0002:00006818       ??_R2bad_alloc@std@@8      10047818     wzdmeshsorter.obj
 0002:00006824       ??_R1A@?0A@EA@bad_alloc@std@@8 10047824     wzdmeshsorter.obj
 0002:00006840       ??_R4CWzAniState@@6B@      10047840     wzanistate.obj
 0002:00006854       ??_R3CWzAniState@@8        10047854     wzanistate.obj
 0002:00006864       ??_R2CWzAniState@@8        10047864     wzanistate.obj
 0002:0000686c       ??_R1A@?0A@EA@CWzAniState@@8 1004786c     wzanistate.obj
 0002:00006888       ??_R4CWzUnit@@6B@          10047888     wzunit.obj
 0002:0000689c       ??_R3CWzUnit@@8            1004789c     wzunit.obj
 0002:000068ac       ??_R2CWzUnit@@8            100478ac     wzunit.obj
 0002:000068b4       ??_R1A@?0A@EA@CWzUnit@@8   100478b4     wzunit.obj
 0002:000068d0       ??_R4CWzUnitDraw@@6B@      100478d0     wzunitdraw.obj
 0002:000068e4       ??_R3CWzUnitDraw@@8        100478e4     wzunitdraw.obj
 0002:000068f4       ??_R2CWzUnitDraw@@8        100478f4     wzunitdraw.obj
 0002:000068fc       ??_R1A@?0A@EA@CWzUnitDraw@@8 100478fc     wzunitdraw.obj
 0002:00006918       ??_R4CWzUnitEditable@@6B@  10047918     wzuniteditable.obj
 0002:0000692c       ??_R3CWzUnitEditable@@8    1004792c     wzuniteditable.obj
 0002:0000693c       ??_R2CWzUnitEditable@@8    1004793c     wzuniteditable.obj
 0002:00006948       ??_R1A@?0A@EA@CWzUnitEditable@@8 10047948     wzuniteditable.obj
 0002:00006964       ??_R4CWzAniStateCB@@6B@    10047964     wzunitskeleton.obj
 0002:00006978       ??_R3CWzAniStateCB@@8      10047978     wzunitskeleton.obj
 0002:00006988       ??_R2CWzAniStateCB@@8      10047988     wzunitskeleton.obj
 0002:00006990       ??_R1A@?0A@EA@CWzAniStateCB@@8 10047990     wzunitskeleton.obj
 0002:000069ac       ??_R4CWzUnitSkeleton@@6B@  100479ac     wzunitskeleton.obj
 0002:000069c0       ??_R3CWzUnitSkeleton@@8    100479c0     wzunitskeleton.obj
 0002:000069d0       ??_R2CWzUnitSkeleton@@8    100479d0     wzunitskeleton.obj
 0002:000069dc       ??_R1A@?0A@EA@CWzUnitSkeleton@@8 100479dc     wzunitskeleton.obj
 0002:000069f8       ??_R4out_of_range@std@@6B@ 100479f8     wzunitskeleton.obj
 0002:00006a0c       ??_R3out_of_range@std@@8   10047a0c     wzunitskeleton.obj
 0002:00006a1c       ??_R2out_of_range@std@@8   10047a1c     wzunitskeleton.obj
 0002:00006a2c       ??_R1A@?0A@EA@out_of_range@std@@8 10047a2c     wzunitskeleton.obj
 0002:00006a48       ??_R4CWzUnitSubType@@6B@   10047a48     wzunitsubtype.obj
 0002:00006a5c       ??_R3CWzUnitSubType@@8     10047a5c     wzunitsubtype.obj
 0002:00006a6c       ??_R2CWzUnitSubType@@8     10047a6c     wzunitsubtype.obj
 0002:00006a74       ??_R1A@?0A@EA@CWzUnitSubType@@8 10047a74     wzunitsubtype.obj
 0002:00006a90       ??_R4CWzUnitSubTypeEditable@@6B@ 10047a90     wzunitsubtypeeditable.obj
 0002:00006aa4       ??_R3CWzUnitSubTypeEditable@@8 10047aa4     wzunitsubtypeeditable.obj
 0002:00006ab4       ??_R2CWzUnitSubTypeEditable@@8 10047ab4     wzunitsubtypeeditable.obj
 0002:00006ac0       ??_R1A@?0A@EA@CWzUnitSubTypeEditable@@8 10047ac0     wzunitsubtypeeditable.obj
 0002:00006adc       ??_R4?$CWzSingleton@VWzLogSystem@WzLog@@@@6B@ 10047adc     programcommonlibforengine:wzlogsystem.obj
 0002:00006af0       ??_R3?$CWzSingleton@VWzLogSystem@WzLog@@@@8 10047af0     programcommonlibforengine:wzlogsystem.obj
 0002:00006b00       ??_R2?$CWzSingleton@VWzLogSystem@WzLog@@@@8 10047b00     programcommonlibforengine:wzlogsystem.obj
 0002:00006b08       ??_R1A@?0A@EA@?$CWzSingleton@VWzLogSystem@WzLog@@@@8 10047b08     programcommonlibforengine:wzlogsystem.obj
 0002:00006b24       ??_R4WzLogSystem@WzLog@@6B@ 10047b24     programcommonlibforengine:wzlogsystem.obj
 0002:00006b38       ??_R3WzLogSystem@WzLog@@8  10047b38     programcommonlibforengine:wzlogsystem.obj
 0002:00006b48       ??_R2WzLogSystem@WzLog@@8  10047b48     programcommonlibforengine:wzlogsystem.obj
 0002:00006b54       ??_R1A@?0A@EA@WzLogSystem@WzLog@@8 10047b54     programcommonlibforengine:wzlogsystem.obj
 0002:00006b70       ??_R4?$CWzList@USt_ChunkStack@@@@6B@ 10047b70     programcommonlibforengine:wzarchive.obj
 0002:00006b84       ??_R3?$CWzList@USt_ChunkStack@@@@8 10047b84     programcommonlibforengine:wzarchive.obj
 0002:00006b94       ??_R2?$CWzList@USt_ChunkStack@@@@8 10047b94     programcommonlibforengine:wzarchive.obj
 0002:00006b9c       ??_R1A@?0A@EA@?$CWzList@USt_ChunkStack@@@@8 10047b9c     programcommonlibforengine:wzarchive.obj
 0002:00006bb8       ??_R4?$CWzHandleManager@USt_DAFileInfo@@@@6B@ 10047bb8     programcommonlibforengine:discaccess.obj
 0002:00006bcc       ??_R3?$CWzHandleManager@USt_DAFileInfo@@@@8 10047bcc     programcommonlibforengine:discaccess.obj
 0002:00006bdc       ??_R2?$CWzHandleManager@USt_DAFileInfo@@@@8 10047bdc     programcommonlibforengine:discaccess.obj
 0002:00006be4       ??_R1A@?0A@EA@?$CWzHandleManager@USt_DAFileInfo@@@@8 10047be4     programcommonlibforengine:discaccess.obj
 0002:00006c00       ??_R4type_info@@6B@        10047c00     LIBCMT:typinfo.obj
 0002:00006c14       ??_R3type_info@@8          10047c14     LIBCMT:typinfo.obj
 0002:00006c24       ??_R2type_info@@8          10047c24     LIBCMT:typinfo.obj
 0002:00006c2c       ??_R1A@?0A@EA@type_info@@8 10047c2c     LIBCMT:typinfo.obj
 0002:00006c48       ??_R4exception@std@@6B@    10047c48     LIBCMT:stdexcpt.obj
 0002:00006c5c       ??_R4bad_exception@std@@6B@ 10047c5c     LIBCMT:frame.obj
 0002:00006c70       ??_R3bad_exception@std@@8  10047c70     LIBCMT:frame.obj
 0002:00006c80       ??_R2bad_exception@std@@8  10047c80     LIBCMT:frame.obj
 0002:00006c8c       ??_R1A@?0A@EA@bad_exception@std@@8 10047c8c     LIBCMT:frame.obj
 0002:00006cb0       ___safe_se_handler_table   10047cb0     <linker-defined>
 0002:00006e68       ___rtc_iaa                 10047e68     LIBCMT:_initsect_.obj
 0002:00006e6c       ___rtc_izz                 10047e6c     LIBCMT:_initsect_.obj
 0002:00006e70       ___rtc_taa                 10047e70     LIBCMT:_initsect_.obj
 0002:00006e74       ___rtc_tzz                 10047e74     LIBCMT:_initsect_.obj
 0002:000072f8       __TI3?AVlength_error@std@@ 100482f8     wzdmeshsorter.obj
 0002:00007308       __CTA3?AVlength_error@std@@ 10048308     wzdmeshsorter.obj
 0002:00007318       __CT??_R0?AVlength_error@std@@@8??0length_error@std@@QAE@ABV01@@Z40 10048318     wzdmeshsorter.obj
 0002:00007334       __CT??_R0?AVlogic_error@std@@@8??0logic_error@std@@QAE@ABV01@@Z40 10048334     wzdmeshsorter.obj
 0002:00007350       __CT??_R0?AVexception@std@@@8??0exception@std@@QAE@ABV01@@Z12 10048350     wzdmeshsorter.obj
 0002:000074d4       __TI2?AVbad_alloc@std@@    100484d4     wzdmeshsorter.obj
 0002:000074e4       __CTA2?AVbad_alloc@std@@   100484e4     wzdmeshsorter.obj
 0002:000074f0       __CT??_R0?AVbad_alloc@std@@@8??0bad_alloc@std@@QAE@ABV01@@Z12 100484f0     wzdmeshsorter.obj
 0002:000081c4       __TI3?AVout_of_range@std@@ 100491c4     wzunitskeleton.obj
 0002:00008200       __CTA3?AVout_of_range@std@@ 10049200     wzunitskeleton.obj
 0002:00008210       __CT??_R0?AVout_of_range@std@@@8??0out_of_range@std@@QAE@ABV01@@Z40 10049210     wzunitskeleton.obj
 0002:000089fc       __TI2?AVbad_exception@std@@ 100499fc     LIBCMT:frame.obj
 0002:00008a0c       __CTA2?AVbad_exception@std@@ 10049a0c     LIBCMT:frame.obj
 0002:00008a18       __CT??_R0?AVbad_exception@std@@@8??0bad_exception@std@@QAE@ABV01@@Z12 10049a18     LIBCMT:frame.obj
 0002:00008d1c       __IMPORT_DESCRIPTOR_KERNEL32 10049d1c     kernel32:KERNEL32.dll
 0002:00008d30       __IMPORT_DESCRIPTOR_USER32 10049d30     user32:USER32.dll
 0002:00008d44       __NULL_IMPORT_DESCRIPTOR   10049d44     kernel32:KERNEL32.dll
 0003:00000008       ??_R0?AVCWzdAnimation@@@8  1004d008     wzdanimation.obj
 0003:00000024       ??_R0?AVCWzdBase@@@8       1004d024     wzdanimation.obj
 0003:00000044       ??_R0?AVCWzdMesh@@@8       1004d044     wzdmesh.obj
 0003:0000005c       ??_R0?AVCWzdMeshConstructor@@@8 1004d05c     wzdmesh.obj
 0003:00000088       ??_R0?AVlength_error@std@@@8 1004d088     wzdmeshsorter.obj
 0003:000000a8       ??_R0?AVlogic_error@std@@@8 1004d0a8     wzdmeshsorter.obj
 0003:000000c8       ??_R0?AVexception@std@@@8  1004d0c8     wzdmeshsorter.obj
 0003:000000e4       ??_R0?AVbad_alloc@std@@@8  1004d0e4     wzdmeshsorter.obj
 0003:0000010c       ??_R0?AVCWzAniState@@@8    1004d10c     wzanistate.obj
 0003:00000134       ??_R0?AVCWzUnit@@@8        1004d134     wzunit.obj
 0003:00000154       ??_R0?AVCWzUnitDraw@@@8    1004d154     wzunitdraw.obj
 0003:00000174       ??_R0?AVCWzUnitEditable@@@8 1004d174     wzuniteditable.obj
 0003:00000198       ??_R0?AVCWzAniStateCB@@@8  1004d198     wzunitskeleton.obj
 0003:000001b4       ??_R0?AVCWzUnitSkeleton@@@8 1004d1b4     wzunitskeleton.obj
 0003:000001d4       ??_R0?AVout_of_range@std@@@8 1004d1d4     wzunitskeleton.obj
 0003:000001f4       ??_R0?AVCWzUnitSubType@@@8 1004d1f4     wzunitsubtype.obj
 0003:00000214       ??_R0?AVCWzUnitSubTypeEditable@@@8 1004d214     wzunitsubtypeeditable.obj
 0003:00000240       ?g_MatMulFunc@@3P6APAUWzMatrix@@PAU1@PBU1@1@ZA 1004d240     common:wzmath.obj
 0003:00000244       ?g_MatMul4x3Func@@3P6APAUWzMatrix@@PAU1@PBU1@1@ZA 1004d244     common:wzmath.obj
 0003:00000248       ?g_MatRotXFunc@@3P6APAUWzMatrix@@PAU1@M@ZA 1004d248     common:wzmath.obj
 0003:0000024c       ?g_MatRotYFunc@@3P6APAUWzMatrix@@PAU1@M@ZA 1004d24c     common:wzmath.obj
 0003:00000250       ?g_MatRotZFunc@@3P6APAUWzMatrix@@PAU1@M@ZA 1004d250     common:wzmath.obj
 0003:00000254       ?g_QuatMulFunc@@3P6APAUWzQuaternion@@PAU1@PBU1@1@ZA 1004d254     common:wzmath.obj
 0003:00000260       ?_PMPM@@3PAIA              1004d260     common:wzmath.obj
 0003:00000270       ?_PPMM@@3PAIA              1004d270     common:wzmath.obj
 0003:00000280       ?_MPPM@@3PAIA              1004d280     common:wzmath.obj
 0003:00000290       ?_PM@@3PAIA                1004d290     common:wzmath.obj
 0003:000002a0       ?_MP@@3PAIA                1004d2a0     common:wzmath.obj
 0003:000002a8       ??_R0?AV?$CWzSingleton@VWzLogSystem@WzLog@@@@@8 1004d2a8     programcommonlibforengine:wzlogsystem.obj
 0003:000002dc       ??_R0?AVWzLogSystem@WzLog@@@8 1004d2dc     programcommonlibforengine:wzlogsystem.obj
 0003:000002fc       ??_R0?AV?$CWzList@USt_ChunkStack@@@@@8 1004d2fc     programcommonlibforengine:wzarchive.obj
 0003:0000032c       ?g_lpszDiscType@@3PAPBDA   1004d32c     programcommonlibforengine:discaccess.obj
 0003:00000338       ??_R0?AV?$CWzHandleManager@USt_DAFileInfo@@@@@8 1004d338     programcommonlibforengine:discaccess.obj
 0003:00000374       __fltused                  1004d374     LIBCMT:_fpinit_.obj
 0003:00000378       __ldused                   1004d378     LIBCMT:_fpinit_.obj
 0003:00000380       ___security_cookie         1004d380     LIBCMT:gs_cookie.obj
 0003:00000384       ___security_cookie_complement 1004d384     LIBCMT:gs_cookie.obj
 0003:0000038c       ??_R0?AVtype_info@@@8      1004d38c     LIBCMT:typinfo.obj
 0003:000003f0       __cfltcvt_tab              1004d3f0     LIBCMT:cmiscdat.obj
 0003:00000418       ___flsindex                1004d418     LIBCMT:tidtable.obj
 0003:0000041c       ___getvalueindex           1004d41c     LIBCMT:tidtable.obj
 0003:00000420       __aexit_rtn                1004d420     LIBCMT:crt0dat.obj
 0003:00000428       ??_R0?AVbad_exception@std@@@8 1004d428     LIBCMT:frame.obj
 0003:00000460       ___abort_behavior          1004d460     LIBCMT:abort.obj
 0003:00000520       ___initialmbcinfo          1004d520     LIBCMT:mbctype.obj
 0003:00000740       __mbctype                  1004d740     LIBCMT:mbctype.obj
 0003:00000848       __mbcasemap                1004d848     LIBCMT:mbctype.obj
 0003:00000948       ___ptmbcinfo               1004d948     LIBCMT:mbctype.obj
 0003:00000a44       ___globallocalestatus      1004da44     LIBCMT:glstatus.obj
 0003:00000a48       ___clocalestr              1004da48     LIBCMT:nlsdata2.obj
 0003:00000a50       ___initiallocinfo          1004da50     LIBCMT:nlsdata2.obj
 0003:00000b28       ___ptlocinfo               1004db28     LIBCMT:nlsdata2.obj
 0003:00000b2c       ___lc_clike                1004db2c     LIBCMT:nlsdata2.obj
 0003:00000b30       ___initiallocalestructinfo 1004db30     LIBCMT:nlsdata2.obj
 0003:00000cb0       __indefinite               1004dcb0     LIBCMT:_87disp_.obj
 0003:00000cba       __piby2                    1004dcba     LIBCMT:_87disp_.obj
 0003:00000ce0       ___badioinfo               1004dce0     LIBCMT:ioinit.obj
 0003:00000d20       __amblksiz                 1004dd20     LIBCMT:heapinit.obj
 0003:00000d24       __First_FPE_Indx           1004dd24     LIBCMT:winxfltr.obj
 0003:00000d28       __Num_FPE                  1004dd28     LIBCMT:winxfltr.obj
 0003:00000d2c       __XcptActTabSize           1004dd2c     LIBCMT:winxfltr.obj
 0003:00000d30       __XcptActTabCount          1004dd30     LIBCMT:winxfltr.obj
 0003:00000d40       ___nullstring              1004dd40     LIBCMT:output.obj
 0003:00000d44       ___wnullstring             1004dd44     LIBCMT:output.obj
 0003:00000e70       __NLG_Destination          1004de70     LIBCMT:exsup.obj
 0003:00000e80       __pctype                   1004de80     LIBCMT:ctype.obj
 0003:00000e84       __pwctype                  1004de84     LIBCMT:ctype.obj
 0003:00000e88       ___lc_time_c               1004de88     LIBCMT:strftime.obj
 0003:00000f40       ___lc_time_curr            1004df40     LIBCMT:strftime.obj
 0003:00000f44       ___lconv_static_decimal    1004df44     LIBCMT:lconv.obj
 0003:00000f48       ___lconv_c                 1004df48     LIBCMT:lconv.obj
 0003:00000f78       ___lconv                   1004df78     LIBCMT:lconv.obj
 0003:00000f7c       ___mb_cur_max              1004df7c     LIBCMT:nlsdata1.obj
 0003:00000f80       ___decimal_point           1004df80     LIBCMT:nlsdata1.obj
 0003:00000f84       ___decimal_point_length    1004df84     LIBCMT:nlsdata1.obj
 0003:00000f90       __iob                      1004df90     LIBCMT:_file.obj
 0003:00001240       __timezone                 1004e240     LIBCMT:timeset.obj
 0003:00001244       __daylight                 1004e244     LIBCMT:timeset.obj
 0003:00001248       __dstbias                  1004e248     LIBCMT:timeset.obj
 0003:000012d0       __tzname                   1004e2d0     LIBCMT:timeset.obj
 0003:000013d8       __matherr_flag             1004e3d8     LIBCMT:_matherr_.obj
 0003:00001400       __pow10pos                 1004e400     LIBCMT:_constpow_.obj
 0003:00001560       __pow10neg                 1004e560     LIBCMT:_constpow_.obj
 0003:000016bc       __lpdays                   1004e6bc     LIBCMT:days.obj
 0003:000016f0       __days                     1004e6f0     LIBCMT:days.obj
 0003:00001728       __d_inf                    1004e728     LIBCMT:_util_.obj
 0003:00001730       __d_ind                    1004e730     LIBCMT:_util_.obj
 0003:00001738       __d_max                    1004e738     LIBCMT:_util_.obj
 0003:00001740       __d_min                    1004e740     LIBCMT:_util_.obj
 0003:00001748       __d_mzero                  1004e748     LIBCMT:_util_.obj
 0003:00001750       __coninpfh                 1004e750     LIBCMT:initcon.obj
 0003:00001754       __confh                    1004e754     LIBCMT:initcon.obj
 0003:00001774       _cchCurDir                 1004e774     wzFilePacker_static:vFile_util.obj
 0003:000018c0       __lookuptrailbytes         1004e8c0     LIBCMT:read.obj
 0003:000019c0       ?s_instance@?$CWzSingleton@VWzLogSystem@WzLog@@@@0PAVWzLogSystem@WzLog@@A 1004e9c0     dllaccess.obj
 0003:000019c8       ?instance@?1??Instance@CWzdShareInfo@@SAPAV2@XZ@4V2@A 1004e9c8     dllaccess.obj
 0003:00001a14       ??_B?1??Instance@CWzdShareInfo@@SAPAV1@XZ@51 1004ea14     dllaccess.obj
 0003:00001a18       ?dummy@?1??GetBvAABB@CWzdBase@@UBEABUBvAABB@@XZ@4U3@A 1004ea18     wzdanimation.obj
 0003:00001a30       ?dummy@?1??GetBvSphere@CWzdBase@@UBEABUBvSphere@@XZ@4U3@A 1004ea30     wzdanimation.obj
 0003:00001a40       ?fInWX@?1??QuaternionToMatrix@@YAPAUWzMatrix@@PAU2@PBUWzQuaternion@@@Z@4MA 1004ea40     wzdanimation.obj
 0003:00001a44       ?fInWY@?1??QuaternionToMatrix@@YAPAUWzMatrix@@PAU2@PBUWzQuaternion@@@Z@4MA 1004ea44     wzdanimation.obj
 0003:00001a48       ?fInWZ@?1??QuaternionToMatrix@@YAPAUWzMatrix@@PAU2@PBUWzQuaternion@@@Z@4MA 1004ea48     wzdanimation.obj
 0003:00001a4c       ?fInYZ@?1??QuaternionToMatrix@@YAPAUWzMatrix@@PAU2@PBUWzQuaternion@@@Z@4MA 1004ea4c     wzdanimation.obj
 0003:00001a50       ?fInXZ@?1??QuaternionToMatrix@@YAPAUWzMatrix@@PAU2@PBUWzQuaternion@@@Z@4MA 1004ea50     wzdanimation.obj
 0003:00001a54       ?fInXY@?1??QuaternionToMatrix@@YAPAUWzMatrix@@PAU2@PBUWzQuaternion@@@Z@4MA 1004ea54     wzdanimation.obj
 0003:00001a58       ?fInZZ@?1??QuaternionToMatrix@@YAPAUWzMatrix@@PAU2@PBUWzQuaternion@@@Z@4MA 1004ea58     wzdanimation.obj
 0003:00001a5c       ?fInYY@?1??QuaternionToMatrix@@YAPAUWzMatrix@@PAU2@PBUWzQuaternion@@@Z@4MA 1004ea5c     wzdanimation.obj
 0003:00001a60       ?fInXX@?1??QuaternionToMatrix@@YAPAUWzMatrix@@PAU2@PBUWzQuaternion@@@Z@4MA 1004ea60     wzdanimation.obj
 0003:00001a64       ?s_pDiscAccess@CWzdBase@@1PAVCDiscAccess@@A 1004ea64     wzdbase.obj
 0003:00001a68       ?s_discAccess@?4??CheckDiscAccessExistence@CWzdBase@@SAPAVCDiscAccess@@XZ@4V3@A 1004ea68     wzdbase.obj
 0003:00003cb4       ??_B?4??CheckDiscAccessExistence@CWzdBase@@SAPAVCDiscAccess@@XZ@54 10050cb4     wzdbase.obj
 0003:00003cb8       ?m_dummyData@?$CWzArray@PAUBvAABB@@@@0PAUBvAABB@@A 10050cb8     wzanimationInfo.obj
 0003:00003cbc       ?m_dummyData@?$CWzHandleManager@PAUSt_WzdContainer@@@@1PAUSt_WzdContainer@@A 10050cbc     wzanistate.obj
 0003:00003cc0       ?m_dummyData@?$CWzHashTable@PAXVCKey_HashTableStr@@@@1PAXA 10050cc0     wzanistate.obj
 0003:00003cc4       ?m_dummyData@?$CWzArray@G@@0GA 10050cc4     wzanistate.obj
 0003:00003cc8       ?m_dummyData@?$CWzArray@PAUSt_WzdContainer@@@@0PAUSt_WzdContainer@@A 10050cc8     wzanistate.obj
 0003:00003ccc       ?m_dummyData@?$CWzArray@K@@0KA 10050ccc     wzunit.obj
 0003:00003cd0       ?m_dummyData@?$CWzArray@PAVWzAnimationInfo@@@@0PAVWzAnimationInfo@@A 10050cd0     wzunit.obj
 0003:00003cd4       ?m_dummyData@?$CWzArray@PAUWzBoneInfo@@@@0PAUWzBoneInfo@@A 10050cd4     wzunit.obj
 0003:00003cd8       ?m_dummyData@?$CWzArray@PAVCWzUnitSubType@@@@0PAVCWzUnitSubType@@A 10050cd8     wzunit.obj
 0003:00003cdc       ?m_dummyData@?$CWzArray@PAUMeshGroupNameInfo@@@@0PAUMeshGroupNameInfo@@A 10050cdc     wzunit.obj
 0003:00003ce0       ?m_dummyData@?$CWzArray@PAUWzMappingInfo@@@@0PAUWzMappingInfo@@A 10050ce0     wzunit.obj
 0003:00003ce4       ?m_dummyData@?$CWzArray@PAUWzTexAniMappingInfo@@@@0PAUWzTexAniMappingInfo@@A 10050ce4     wzunit.obj
 0003:00003ce8       ?m_dummyData@?$CWzArray@PAUWzTexAniSetInfo@@@@0PAUWzTexAniSetInfo@@A 10050ce8     wzunit.obj
 0003:00003cec       ?m_dummyData@?$CWzArray@PAUWzBVExtraInfo@@@@0PAUWzBVExtraInfo@@A 10050cec     wzunit.obj
 0003:00003cf0       ?m_dummyData@?$CWzArray@PAUWzRenderInfo@@@@0PAUWzRenderInfo@@A 10050cf0     wzunitdraw.obj
 0003:00003cf4       ?m_dummyData@?$CWzArray@PAUWzUnitEffectInfo@@@@0PAUWzUnitEffectInfo@@A 10050cf4     wzunitdraw.obj
 0003:00003d04       ?m_dummyData@?$CWzArray@PAUWzBoneScaling@@@@0PAUWzBoneScaling@@A 10050d04     wzunitskeleton.obj
 0003:00003d08       ?m_dummyData@?$CWzArray@PAUWzDecoration@@@@0PAUWzDecoration@@A 10050d08     wzunitsubtype.obj
 0003:00004238       ?m_dummyData@?$CWzList@USt_ChunkStack@@@@1USt_ChunkStack@@A 10051238     programcommonlibforengine:wzarchive.obj
 0003:00004344       ?m_dummyData@?$CWzHandleManager@USt_DAFileInfo@@@@1USt_DAFileInfo@@A 10051344     programcommonlibforengine:discaccess.obj
 0003:0000434c       ?m_nullData@?$CWzHandleManager@USt_DAFileInfo@@@@1USt_DAFileInfo@@A 1005134c     programcommonlibforengine:discaccess.obj
 0003:00004354       ?m_dummyData@?$CWzArray@USt_DAFileInfo@@@@0USt_DAFileInfo@@A 10051354     programcommonlibforengine:discaccess.obj
 0003:0000435c       ___fastflag                1005135c     LIBCMT:_fpinit_.obj
 0003:00004360       __adjust_fdiv              10051360     LIBCMT:_fpinit_.obj
 0003:00004374       ___pInvalidArgHandler      10051374     LIBCMT:invarg.obj
 0003:0000437c       __aenvptr                  1005137c     LIBCMT:dllcrt0.obj
 0003:00004380       __wenvptr                  10051380     LIBCMT:dllcrt0.obj
 0003:00004384       ___error_mode              10051384     LIBCMT:dllcrt0.obj
 0003:00004388       ___app_type                10051388     LIBCMT:dllcrt0.obj
 0003:0000438c       ?_pnhHeap@@3P6AHI@ZA       1005138c     LIBCMT:handler.obj
 0003:00004390       _gpFlsAlloc                10051390     LIBCMT:tidtable.obj
 0003:00004394       _gpFlsGetValue             10051394     LIBCMT:tidtable.obj
 0003:00004398       _gpFlsSetValue             10051398     LIBCMT:tidtable.obj
 0003:0000439c       _gpFlsFree                 1005139c     LIBCMT:tidtable.obj
 0003:000043a0       __maxwait                  100513a0     LIBCMT:crtheap.obj
 0003:000043a4       __umaskval                 100513a4     LIBCMT:crt0dat.obj
 0003:000043a8       ___argc                    100513a8     LIBCMT:crt0dat.obj
 0003:000043ac       ___argv                    100513ac     LIBCMT:crt0dat.obj
 0003:000043b0       ___wargv                   100513b0     LIBCMT:crt0dat.obj
 0003:000043b4       __environ                  100513b4     LIBCMT:crt0dat.obj
 0003:000043b8       ___initenv                 100513b8     LIBCMT:crt0dat.obj
 0003:000043bc       __wenviron                 100513bc     LIBCMT:crt0dat.obj
 0003:000043c0       ___winitenv                100513c0     LIBCMT:crt0dat.obj
 0003:000043c4       __pgmptr                   100513c4     LIBCMT:crt0dat.obj
 0003:000043c8       __wpgmptr                  100513c8     LIBCMT:crt0dat.obj
 0003:000043cc       __exitflag                 100513cc     LIBCMT:crt0dat.obj
 0003:000043d0       __C_Termination_Done       100513d0     LIBCMT:crt0dat.obj
 0003:000043d4       __C_Exit_Done              100513d4     LIBCMT:crt0dat.obj
 0003:000043d8       ?__pInconsistency@@3P6AXXZA 100513d8     LIBCMT:hooks.obj
 0003:00004a2c       ___pPurecall               10051a2c     LIBCMT:inithelp.obj
 0003:00004a34       ___mbulinfo                10051a34     LIBCMT:mbctype.obj
 0003:00004a40       ___mbcodepage              10051a40     LIBCMT:mbctype.obj
 0003:00004a44       ___ismbcodepage            10051a44     LIBCMT:mbctype.obj
 0003:00004a48       ___mblcid                  10051a48     LIBCMT:mbctype.obj
 0003:00004a4c       ___locale_changed          10051a4c     LIBCMT:setlocal.obj
 0003:00004a50       ___lc_handle               10051a50     LIBCMT:nlsdata2.obj
 0003:00004a68       ___lc_codepage             10051a68     LIBCMT:nlsdata2.obj
 0003:00004a6c       ___lc_collate_cp           10051a6c     LIBCMT:nlsdata2.obj
 0003:00004b7c       __crtheap                  10051b7c     LIBCMT:heapinit.obj
 0003:00004b80       __outputformat             10051b80     LIBCMT:outputformat.obj
 0003:00004cd8       ___sbh_pHeaderDefer        10051cd8     LIBCMT:sbheap.obj
 0003:00004cdc       __newmode                  10051cdc     LIBCMT:_newmode.obj
 0003:00004d10       ?pArgList@UnDecorator@@0PAVReplicator@@A 10051d10     LIBCMT:undname.obj
 0003:00004d14       ?pZNameList@UnDecorator@@0PAVReplicator@@A 10051d14     LIBCMT:undname.obj
 0003:00004d18       ?pTemplateArgList@UnDecorator@@0PAVReplicator@@A 10051d18     LIBCMT:undname.obj
 0003:00004d1c       ?gName@UnDecorator@@0PBDB  10051d1c     LIBCMT:undname.obj
 0003:00004d20       ?name@UnDecorator@@0PBDB   10051d20     LIBCMT:undname.obj
 0003:00004d24       ?outputString@UnDecorator@@0PADA 10051d24     LIBCMT:undname.obj
 0003:00004d28       ?maxStringLength@UnDecorator@@0HA 10051d28     LIBCMT:undname.obj
 0003:00004d2c       ?disableFlags@UnDecorator@@0KA 10051d2c     LIBCMT:undname.obj
 0003:00004d30       ?m_pGetParameter@UnDecorator@@0P6APADJ@ZA 10051d30     LIBCMT:undname.obj
 0003:00004d34       ?fExplicitTemplateParams@UnDecorator@@0_NA 10051d34     LIBCMT:undname.obj
 0003:00004d35       ?fGetTemplateArgumentList@UnDecorator@@0_NA 10051d35     LIBCMT:undname.obj
 0003:00004d54       ___lconv_static_null       10051d54     LIBCMT:lconv.obj
 0003:00004d5c       __cflush                   10051d5c     LIBCMT:_file.obj
 0003:00004e20       __stdbuf                   10051e20     LIBCMT:_sftbuf.obj
 0003:00004e28       ?autofree@@3VCAutoFree@@A  10051e28     wzFilePacker_static:wzFilePacker.obj
 0003:00004e38       _dwTreeCount               10051e38     wzFilePacker_static:vfile.obj
 0003:00004e3c       _g_nTreeArrayCount         10051e3c     wzFilePacker_static:vfile.obj
 0003:00004e40       _g_ulStartBinaryOffset     10051e40     wzFilePacker_static:vfile.obj
 0003:00004e48       _g_ulTatalBinarySize       10051e48     wzFilePacker_static:vfile.obj
 0003:00004e54       _bCurDirCreated            10051e54     wzFilePacker_static:vFile_util.obj
 0003:00005764       __commode                  10052764     LIBCMT:ncommode.obj
 0003:00005768       __fmode                    10052768     LIBCMT:txtmode.obj
 0003:0000576c       ___piob                    1005276c     <common>
 0003:00005780       __bufin                    10052780     <common>
 0003:00006780       __nstream                  10053780     <common>
 0003:00006784       __pmatherr                 10053784     <common>
 0003:00006788       ___sbh_cntHeaderList       10053788     <common>
 0003:0000678c       ___sbh_pHeaderList         1005378c     <common>
 0003:00006790       ___sbh_threshold           10053790     <common>
 0003:00006794       ___sbh_pHeaderScan         10053794     <common>
 0003:00006798       ___sbh_sizeHeaderList      10053798     <common>
 0003:0000679c       ___sbh_indGroupDefer       1005379c     <common>
 0003:000067a0       ___use_sse2_mathfcns       100537a0     <common>
 0003:000067a4       ___active_heap             100537a4     <common>
 0003:000067a8       __nhandle                  100537a8     <common>
 0003:000067c0       ___pioinfo                 100537c0     <common>
 0003:000068c0       __debugger_hook_dummy      100538c0     <common>
 0003:000068c4       ___sse2_available          100538c4     <common>
 0003:000068c8       ___env_initialized         100538c8     <common>
 0003:000068cc       ___onexitend               100538cc     <common>
 0003:000068d0       ___onexitbegin             100538d0     <common>
 0003:000068d4       ___mbctype_initialized     100538d4     <common>
 0003:000068d8       ___dyn_tls_init_callback   100538d8     <common>
 0003:000068dc       __acmdln                   100538dc     <common>
 0003:000068e0       _StupidUnusedPointer       100538e0     <common>
 0003:00006900       _g_TreeList                10053900     <common>

 entry point at        0001:0002bbb0

 Static symbols

 0001:0000aa13       __catch$?_Buynode@?$list@HV?$allocator@H@std@@@std@@IAEPAU_Node@?$_List_nod@HV?$allocator@H@std@@@2@XZ$0 1000ba13 f i wzdmeshsorter.obj
 0001:0000ae10       __catch$?_Insert_n@?$vector@HV?$allocator@H@std@@@std@@IAEXV?$_Vector_const_iterator@HV?$allocator@H@std@@@2@IABH@Z$0 1000be10 f i wzdmeshsorter.obj
 0001:0000b03b       __catch$?_Insert_n@?$vector@HV?$allocator@H@std@@@std@@IAEXV?$_Vector_const_iterator@HV?$allocator@H@std@@@2@IABH@Z$2 1000c03b f i wzdmeshsorter.obj
 0001:0000b8a3       __catch$?_Buynode@?$list@HV?$allocator@H@std@@@std@@IAEPAU_Node@?$_List_nod@HV?$allocator@H@std@@@2@PAU342@0ABH@Z$0 1000c8a3 f i wzdmeshsorter.obj
 0001:0000bc33       __catch$?_Copy@?$basic_string@DU?$char_traits@D@std@@V?$allocator@D@2@@std@@IAEXII@Z$0 1000cc33 f i wzdmeshsorter.obj
 0001:0000bc5f       __catch$?_Copy@?$basic_string@DU?$char_traits@D@std@@V?$allocator@D@2@@std@@IAEXII@Z$1 1000cc5f f i wzdmeshsorter.obj
 0001:0000fafd       __catch$?_Insert_n@?$vector@UWzSoundInfo@@V?$allocator@UWzSoundInfo@@@std@@@std@@IAEXV?$_Vector_const_iterator@UWzSoundInfo@@V?$allocator@UWzSoundInfo@@@std@@@2@IABUWzSoundInfo@@@Z$0 10010afd f i wzanimationInfo.obj
 0001:0000fe0e       __catch$?_Insert_n@?$vector@UWzSoundInfo@@V?$allocator@UWzSoundInfo@@@std@@@std@@IAEXV?$_Vector_const_iterator@UWzSoundInfo@@V?$allocator@UWzSoundInfo@@@std@@@2@IABUWzSoundInfo@@@Z$2 10010e0e f i wzanimationInfo.obj
 0001:000103b0       __catch$?_Insert_n@?$vector@UWzEffectInfo@@V?$allocator@UWzEffectInfo@@@std@@@std@@IAEXV?$_Vector_const_iterator@UWzEffectInfo@@V?$allocator@UWzEffectInfo@@@std@@@2@IABUWzEffectInfo@@@Z$0 100113b0 f i wzanimationInfo.obj
 0001:00010675       __catch$?_Insert_n@?$vector@UWzEffectInfo@@V?$allocator@UWzEffectInfo@@@std@@@std@@IAEXV?$_Vector_const_iterator@UWzEffectInfo@@V?$allocator@UWzEffectInfo@@@std@@@2@IABUWzEffectInfo@@@Z$2 10011675 f i wzanimationInfo.obj
 0001:00010b70       __catch$?_Insert_n@?$vector@UWzCustomInfo@@V?$allocator@UWzCustomInfo@@@std@@@std@@IAEXV?$_Vector_const_iterator@UWzCustomInfo@@V?$allocator@UWzCustomInfo@@@std@@@2@IABUWzCustomInfo@@@Z$0 10011b70 f i wzanimationInfo.obj
 0001:00010e35       __catch$?_Insert_n@?$vector@UWzCustomInfo@@V?$allocator@UWzCustomInfo@@@std@@@std@@IAEXV?$_Vector_const_iterator@UWzCustomInfo@@V?$allocator@UWzCustomInfo@@@std@@@2@IABUWzCustomInfo@@@Z$2 10011e35 f i wzanimationInfo.obj
 0001:000114ab       __catch$??0?$vector@HV?$allocator@H@std@@@std@@QAE@ABV01@@Z$0 100124ab f i wzanimationInfo.obj
 0001:00011ce6       __catch$??$_Uninit_fill_n@PAUWzSoundInfo@@IU1@V?$allocator@UWzSoundInfo@@@std@@@std@@YAXPAUWzSoundInfo@@IABU1@AAV?$allocator@UWzSoundInfo@@@0@U_Nonscalar_ptr_iterator_tag@0@U_Range_checked_iterator_tag@0@@Z$0 10012ce6 f i wzanimationInfo.obj
 0001:00011da7       __catch$??$_Uninit_fill_n@PAUWzEffectInfo@@IU1@V?$allocator@UWzEffectInfo@@@std@@@std@@YAXPAUWzEffectInfo@@IABU1@AAV?$allocator@UWzEffectInfo@@@0@U_Nonscalar_ptr_iterator_tag@0@U_Range_checked_iterator_tag@0@@Z$0 10012da7 f i wzanimationInfo.obj
 0001:00011e5e       __catch$??$_Uninit_fill_n@PAUWzCustomInfo@@IU1@V?$allocator@UWzCustomInfo@@@std@@@std@@YAXPAUWzCustomInfo@@IABU1@AAV?$allocator@UWzCustomInfo@@@0@U_Nonscalar_ptr_iterator_tag@0@U_Range_checked_iterator_tag@0@@Z$0 10012e5e f i wzanimationInfo.obj
 0001:00012495       __catch$??$_Uninit_copy@PAUWzSoundInfo@@PAU1@V?$allocator@UWzSoundInfo@@@std@@@std@@YAPAUWzSoundInfo@@PAU1@00AAV?$allocator@UWzSoundInfo@@@0@U_Nonscalar_ptr_iterator_tag@0@U_Range_checked_iterator_tag@0@@Z$0 10013495 f i wzanimationInfo.obj
 0001:0001255d       __catch$??$_Uninit_copy@PAUWzEffectInfo@@PAU1@V?$allocator@UWzEffectInfo@@@std@@@std@@YAPAUWzEffectInfo@@PAU1@00AAV?$allocator@UWzEffectInfo@@@0@U_Nonscalar_ptr_iterator_tag@0@U_Range_checked_iterator_tag@0@@Z$0 1001355d f i wzanimationInfo.obj
 0001:0001261b       __catch$??$_Uninit_copy@PAUWzCustomInfo@@PAU1@V?$allocator@UWzCustomInfo@@@std@@@std@@YAPAUWzCustomInfo@@PAU1@00AAV?$allocator@UWzCustomInfo@@@0@U_Nonscalar_ptr_iterator_tag@0@U_Range_checked_iterator_tag@0@@Z$0 1001361b f i wzanimationInfo.obj
 0001:0001e6e5       __catch$?_Buynode@?$_Tree@V?$_Tmap_traits@HUWzVector@@U?$less@H@std@@V?$allocator@U?$pair@$$CBHUWzVector@@@std@@@3@$0A@@std@@@std@@IAEPAU_Node@?$_Tree_nod@V?$_Tmap_traits@HUWzVector@@U?$less@H@std@@V?$allocator@U?$pair@$$CBHUWzVector@@@std@@@3@$0A@@std@@@2@PAU342@00ABU?$pair@$$CBHUWzVector@@@2@D@Z$0 1001f6e5 f i wzunitskeleton.obj
 0001:0001ee67       __catch$?_Buynode@?$_Tree@V?$_Tmap_traits@HUWzVector@@U?$less@H@std@@V?$allocator@U?$pair@$$CBHUWzVector@@@std@@@3@$0A@@std@@@std@@IAEPAU_Node@?$_Tree_nod@V?$_Tmap_traits@HUWzVector@@U?$less@H@std@@V?$allocator@U?$pair@$$CBHUWzVector@@@std@@@3@$0A@@std@@@2@XZ$0 1001fe67 f i wzunitskeleton.obj
 0001:0002a1a6       __onexit_nolock            1002b1a6 f   LIBCMT:onexit.obj
 0001:0002a3a7       ?CatchGuardHandler@@YA?AW4_EXCEPTION_DISPOSITION@@PAUEHExceptionRecord@@PAUCatchGuardRN@@PAX2@Z 1002b3a7 f   LIBCMT:_trnsctrl_.obj
 0001:0002a4b1       ?TranslatorGuardHandler@@YA?AW4_EXCEPTION_DISPOSITION@@PAUEHExceptionRecord@@PAUTranslatorGuardRN@@PAX2@Z 1002b4b1 f   LIBCMT:_trnsctrl_.obj
 0001:0002baba       ___DllMainCRTStartup       1002caba f   LIBCMT:dllcrt0.obj
 0001:0002c29a       __splitpath_helper         1002d29a f   LIBCMT:splitpat.obj
 0001:0002c741       __shift                    1002d741 f   LIBCMT:cvt.obj
 0001:0002c786       __cftoe2_l                 1002d786 f   LIBCMT:cvt.obj
 0001:0002cd58       __cftof2_l                 1002dd58 f   LIBCMT:cvt.obj
 0001:0002db7b       __initterm                 1002eb7b f   LIBCMT:crt0dat.obj
 0001:0002dc41       _doexit                    1002ec41 f   LIBCMT:crt0dat.obj
 0001:0002e012       ?ExFilterRethrow@@YAHPAU_EXCEPTION_POINTERS@@@Z 1002f012 f   LIBCMT:frame.obj
 0001:0002e0d5       ?IsInExceptionSpec@@YAEPAUEHExceptionRecord@@PBU_s_ESTypeList@@@Z 1002f0d5 f   LIBCMT:frame.obj
 0001:0002e150       ?CallUnexpected@@YAXPBU_s_ESTypeList@@@Z 1002f150 f   LIBCMT:frame.obj
 0001:0002e181       __catch$?CallUnexpected@@YAXPBU_s_ESTypeList@@@Z$0 1002f181 f   LIBCMT:frame.obj
 0001:0002e199       ?CallCatchBlock@@YAPAXPAUEHExceptionRecord@@PAUEHRegistrationNode@@PAU_CONTEXT@@PBU_s_FuncInfo@@PAXHK@Z 1002f199 f   LIBCMT:frame.obj
 0001:0002e546       ?CatchIt@@YAXPAUEHExceptionRecord@@PAUEHRegistrationNode@@PAU_CONTEXT@@PAXPBU_s_FuncInfo@@PBU_s_HandlerType@@PBU_s_CatchableType@@PBU_s_TryBlockMapEntry@@H1E@Z 1002f546 f   LIBCMT:frame.obj
 0001:0002e5b4       ?FindHandlerForForeignException@@YAXPAUEHExceptionRecord@@PAUEHRegistrationNode@@PAU_CONTEXT@@PAXPBU_s_FuncInfo@@HH1@Z 1002f5b4 f   LIBCMT:frame.obj
 0001:0002e6a8       ?FindHandler@@YAXPAUEHExceptionRecord@@PAUEHRegistrationNode@@PAU_CONTEXT@@PAXPBU_s_FuncInfo@@EH1@Z 1002f6a8 f   LIBCMT:frame.obj
 0001:0002ede8       _fastzero_I                1002fde8 f   LIBCMT:p4_memset.obj
 0001:0002eece       _has_osfxsr_set            1002fece f   LIBCMT:cpu_disp.obj
 0001:0002f2c0       _fastcopy_I                100302c0 f   LIBCMT:p4_memcpy.obj
 0001:0002f42a       ?CPtoLCID@@YAHH@Z          1003042a f   LIBCMT:mbctype.obj
 0001:0002f459       ?setSBCS@@YAXPAUthreadmbcinfostruct@@@Z 10030459 f   LIBCMT:mbctype.obj
 0001:0002f4bd       ?setSBUpLow@@YAXPAUthreadmbcinfostruct@@@Z 100304bd f   LIBCMT:mbctype.obj
 0001:0002f6f4       ?getSystemCP@@YAHH@Z       100306f4 f   LIBCMT:mbctype.obj
 0001:0002fd7e       __updatetlocinfoEx_nolock  10030d7e f   LIBCMT:setlocal.obj
 0001:00030809       _parse_cmdline             10031809 f   LIBCMT:stdargv.obj
 0001:00030f2c       __unwind_handler4          10031f2c f   LIBCMT:exsup4.obj
 0001:00031b98       _write_char                10032b98 f   LIBCMT:output.obj
 0001:00031bcb       _write_multi_char          10032bcb f   LIBCMT:output.obj
 0001:00031bf1       _write_string              10032bf1 f   LIBCMT:output.obj
 0001:000327d6       ?x_ismbbtype_l@@YAHPAUlocaleinfo_struct@@IHH@Z 100337d6 f   LIBCMT:ismbbyte.obj
 0001:00033d9e       _siglookup                 10034d9e f   LIBCMT:winsig.obj
 0001:00034044       __unwind_handler           10035044 f   LIBCMT:exsup.obj
 0001:00034458       ?__crtLCMapStringA_stat@@YAHPAUlocaleinfo_struct@@KKPBDHPADHHH@Z 10035458 f   LIBCMT:a_map.obj
 0001:00034842       ?__crtGetStringTypeA_stat@@YAHPAUlocaleinfo_struct@@KPBDHPAGHHH@Z 10035842 f   LIBCMT:a_str.obj
 0001:00037d68       __hw_cw                    10038d68 f   LIBCMT:_ieee87_.obj
 0001:00037df6       ___hw_cw_sse2              10038df6 f   LIBCMT:_ieee87_.obj
 0001:00038f8a       _flsall                    10039f8a f   LIBCMT:fflush.obj
 0001:0003906d       ?strtoxl@@YAKPAUlocaleinfo_struct@@PBDPAPBDHH@Z 1003a06d f   LIBCMT:strtol.obj
 0001:00039ea0       @geVFile_RegisterFileSystemInternal@8 1003aea0 f   wzFilePacker_static:vfile.obj
 0001:00039f10       _RegisterBuiltInAPIs       1003af10 f   wzFilePacker_static:vfile.obj
 0001:00039f80       @CheckOpenFlags@4          1003af80 f   wzFilePacker_static:vfile.obj
 0001:0003a700       _geRam_DoCriticalCallback  1003b700 f   wzFilePacker_static:Ram.obj
 0001:0003a830       @FSVFS_FinderCreate@12     1003b830 f   wzFilePacker_static:fsvfs.obj
 0001:0003a8a0       @FSVFS_FinderGetNextFile@4 1003b8a0 f   wzFilePacker_static:fsvfs.obj
 0001:0003a8c0       @FSVFS_FinderGetProperties@8 1003b8c0 f   wzFilePacker_static:fsvfs.obj
 0001:0003a920       @FSVFS_FinderDestroy@4     1003b920 f   wzFilePacker_static:fsvfs.obj
 0001:0003a950       @FSVFS_OpenNewSystem@16    1003b950 f   wzFilePacker_static:fsvfs.obj
 0001:0003b030       @FSVFS_Disperse@16         1003c030 f   wzFilePacker_static:fsvfs.obj
 0001:0003b030       @FSMemory_Disperse@16      1003c030 f   wzFilePacker_static:fsvfs.obj
 0001:0003b030       @FSMemory_RenameFile@16    1003c030 f   wzFilePacker_static:fsvfs.obj
 0001:0003b030       @FSVFS_RenameFile@16       1003c030 f   wzFilePacker_static:fsvfs.obj
 0001:0003b030       @FSVFS_UpdateContext@16    1003c030 f   wzFilePacker_static:fsvfs.obj
 0001:0003b030       @FSVFS_SetSize@12          1003c030 f   wzFilePacker_static:fsvfs.obj
 0001:0003b030       @FSDos_UpdateContext@16    1003c030 f   wzFilePacker_static:fsvfs.obj
 0001:0003b030       @FSDos_Disperse@16         1003c030 f   wzFilePacker_static:fsvfs.obj
 0001:0003b030       @FSMemory_SetSize@12       1003c030 f   wzFilePacker_static:fsvfs.obj
 0001:0003b040       @FSVFS_MakeSpace@24        1003c040 f   wzFilePacker_static:fsvfs.obj
 0001:0003b2e0       @FSVFS_EnlargeDirectorySize@8 1003c2e0 f   wzFilePacker_static:fsvfs.obj
 0001:0003b3c0       @FSVFS_Close@4             1003c3c0 f   wzFilePacker_static:fsvfs.obj
 0001:0003b530       @ForceFilePos@4            1003c530 f   wzFilePacker_static:fsvfs.obj
 0001:0003b550       _ClampOperationSize        1003c550 f   wzFilePacker_static:fsvfs.obj
 0001:0003b590       @UpdateFilePos@4           1003c590 f   wzFilePacker_static:fsvfs.obj
 0001:0003b670       @FSVFS_GetS@12             1003c670 f   wzFilePacker_static:fsvfs.obj
 0001:0003b6c0       @FSVFS_Read@12             1003c6c0 f   wzFilePacker_static:fsvfs.obj
 0001:0003b830       @FSVFS_Write@12            1003c830 f   wzFilePacker_static:fsvfs.obj
 0001:0003b890       @FSVFS_Seek@16             1003c890 f   wzFilePacker_static:fsvfs.obj
 0001:0003b920       @FSVFS_EOF@4               1003c920 f   wzFilePacker_static:fsvfs.obj
 0001:0003b940       @FSVFS_Tell@8              1003c940 f   wzFilePacker_static:fsvfs.obj
 0001:0003b960       @FSVFS_Size@8              1003c960 f   wzFilePacker_static:fsvfs.obj
 0001:0003b980       @FSVFS_GetProperties@8     1003c980 f   wzFilePacker_static:fsvfs.obj
 0001:0003b9d0       @FSVFS_SetAttributes@8     1003c9d0 f   wzFilePacker_static:fsvfs.obj
 0001:0003b9f0       @FSVFS_SetTime@8           1003c9f0 f   wzFilePacker_static:fsvfs.obj
 0001:0003ba00       @FSVFS_SetHints@8          1003ca00 f   wzFilePacker_static:fsvfs.obj
 0001:0003ba10       @FSVFS_FileExists@12       1003ca10 f   wzFilePacker_static:fsvfs.obj
 0001:0003ba30       _FSVFS_GetVoidSpace        1003ca30 f   wzFilePacker_static:fsvfs.obj
 0001:0003bec0       _FSVFS_SetVoidSpace        1003cec0 f   wzFilePacker_static:fsvfs.obj
 0001:0003c1e0       @FSVFS_Open@20             1003d1e0 f   wzFilePacker_static:fsvfs.obj
 0001:0003c3a0       @FSVFS_DeleteFile@12       1003d3a0 f   wzFilePacker_static:fsvfs.obj
 0001:0003c4e0       @FSMemory_FinderDestroy@4  1003d4e0 f   wzFilePacker_static:FSMEMORY.obj
 0001:0003c4f0       @FSMemory_Open@20          1003d4f0 f   wzFilePacker_static:FSMEMORY.obj
 0001:0003c500       @FSMemory_OpenNewSystem@16 1003d500 f   wzFilePacker_static:FSMEMORY.obj
 0001:0003c5c0       @FSMemory_UpdateContext@16 1003d5c0 f   wzFilePacker_static:FSMEMORY.obj
 0001:0003c5f0       @FSMemory_Close@4          1003d5f0 f   wzFilePacker_static:FSMEMORY.obj
 0001:0003c630       @ClampOperationSize@12     1003d630 f   wzFilePacker_static:FSMEMORY.obj
 0001:0003c670       @DataPtr@4                 1003d670 f   wzFilePacker_static:FSMEMORY.obj
 0001:0003c680       @FSMemory_GetS@12          1003d680 f   wzFilePacker_static:FSMEMORY.obj
 0001:0003c6e0       @FSMemory_Read@12          1003d6e0 f   wzFilePacker_static:FSMEMORY.obj
 0001:0003c740       @TestForExpansion@12       1003d740 f   wzFilePacker_static:FSMEMORY.obj
 0001:0003c7c0       @FSMemory_Write@12         1003d7c0 f   wzFilePacker_static:FSMEMORY.obj
 0001:0003c840       @FSMemory_Seek@16          1003d840 f   wzFilePacker_static:FSMEMORY.obj
 0001:0003c910       @FSMemory_EOF@4            1003d910 f   wzFilePacker_static:FSMEMORY.obj
 0001:0003c930       @FSMemory_Tell@8           1003d930 f   wzFilePacker_static:FSMEMORY.obj
 0001:0003c950       @FSMemory_Size@8           1003d950 f   wzFilePacker_static:FSMEMORY.obj
 0001:0003c970       @FSMemory_DeleteFile@12    1003d970 f   wzFilePacker_static:FSMEMORY.obj
 0001:0003c970       @FSMemory_FinderCreate@12  1003d970 f   wzFilePacker_static:FSMEMORY.obj
 0001:0003c970       @FSMemory_FileExists@12    1003d970 f   wzFilePacker_static:FSMEMORY.obj
 0001:0003c980       @FSMemory_SetTime@8        1003d980 f   wzFilePacker_static:FSMEMORY.obj
 0001:0003c980       @FSMemory_SetAttributes@8  1003d980 f   wzFilePacker_static:FSMEMORY.obj
 0001:0003c980       @FSMemory_EnlargeDirectorySize@8 1003d980 f   wzFilePacker_static:FSMEMORY.obj
 0001:0003c980       @FSMemory_FinderGetProperties@8 1003d980 f   wzFilePacker_static:FSMEMORY.obj
 0001:0003c980       @FSMemory_FinderGetNextFile@4 1003d980 f   wzFilePacker_static:FSMEMORY.obj
 0001:0003c980       @FSMemory_GetProperties@8  1003d980 f   wzFilePacker_static:FSMEMORY.obj
 0001:0003c980       @FSMemory_SetHints@8       1003d980 f   wzFilePacker_static:FSMEMORY.obj
 0001:0003c980       @FSDos_EnlargeDirectorySize@8 1003d980 f   wzFilePacker_static:FSMEMORY.obj
 0001:0003c980       @FSDos_SetHints@8          1003d980 f   wzFilePacker_static:FSMEMORY.obj
 0001:0003c9a0       _BuildFileName             1003d9a0 f   wzFilePacker_static:fsdos.obj
 0001:0003ca70       @FSDos_FinderCreate@12     1003da70 f   wzFilePacker_static:fsdos.obj
 0001:0003cb40       @FSDos_FinderGetNextFile@4 1003db40 f   wzFilePacker_static:fsdos.obj
 0001:0003cbb0       @FSDos_FinderGetProperties@8 1003dbb0 f   wzFilePacker_static:fsdos.obj
 0001:0003cc30       @FSDos_FinderDestroy@4     1003dc30 f   wzFilePacker_static:fsdos.obj
 0001:0003cc60       _IsRootDirectory           1003dc60 f   wzFilePacker_static:fsdos.obj
 0001:0003ccb0       @FSDos_Open@20             1003dcb0 f   wzFilePacker_static:fsdos.obj
 0001:0003ceb0       @FSDos_OpenNewSystem@16    1003deb0 f   wzFilePacker_static:fsdos.obj
 0001:0003ced0       @FSDos_Close@4             1003ded0 f   wzFilePacker_static:fsdos.obj
 0001:0003cf20       @FSDos_GetS@12             1003df20 f   wzFilePacker_static:fsdos.obj
 0001:0003d000       @FSDos_Read@12             1003e000 f   wzFilePacker_static:fsdos.obj
 0001:0003d060       @FSDos_Write@12            1003e060 f   wzFilePacker_static:fsdos.obj
 0001:0003d0a0       @FSDos_Seek@16             1003e0a0 f   wzFilePacker_static:fsdos.obj
 0001:0003d160       @FSDos_EOF@4               1003e160 f   wzFilePacker_static:fsdos.obj
 0001:0003d1f0       @FSDos_Tell@8              1003e1f0 f   wzFilePacker_static:fsdos.obj
 0001:0003d260       @FSDos_Size@8              1003e260 f   wzFilePacker_static:fsdos.obj
 0001:0003d2d0       @FSDos_GetProperties@8     1003e2d0 f   wzFilePacker_static:fsdos.obj
 0001:0003d390       @FSDos_SetSize@12          1003e390 f   wzFilePacker_static:fsdos.obj
 0001:0003d3e0       @FSDos_SetAttributes@8     1003e3e0 f   wzFilePacker_static:fsdos.obj
 0001:0003d410       @FSDos_SetTime@8           1003e410 f   wzFilePacker_static:fsdos.obj
 0001:0003d440       @FSDos_FileExists@12       1003e440 f   wzFilePacker_static:fsdos.obj
 0001:0003d4d0       @FSDos_DeleteFile@12       1003e4d0 f   wzFilePacker_static:fsdos.obj
 0001:0003d560       @FSDos_RenameFile@16       1003e560 f   wzFilePacker_static:fsdos.obj
 0001:0003d6d0       _WriteTree                 1003e6d0 f   wzFilePacker_static:dirtree.obj
 0001:0003d850       _DirTree_WriteToFile1      1003e850 f   wzFilePacker_static:dirtree.obj
 0001:0003d9f0       _ReadTree                  1003e9f0 f   wzFilePacker_static:dirtree.obj
 0001:0003dc40       _ReadTreeCount             1003ec40 f   wzFilePacker_static:dirtree.obj
 0001:0003eb70       __unwindfunclet$?Instance@CWzdShareInfo@@SAPAV1@XZ$0 1003fb70 f   dllaccess.obj
 0001:0003eb7e       __ehhandler$?Instance@CWzdShareInfo@@SAPAV1@XZ 1003fb7e f   dllaccess.obj
 0001:0003eb99       __unwindfunclet$??0CWzdAnimation@@QAE@XZ$0 1003fb99 f   wzdanimation.obj
 0001:0003eba1       __ehhandler$??0CWzdAnimation@@QAE@XZ 1003fba1 f   wzdanimation.obj
 0001:0003ebbc       __unwindfunclet$??1CWzdAnimation@@UAE@XZ$0 1003fbbc f   wzdanimation.obj
 0001:0003ebc4       __ehhandler$??1CWzdAnimation@@UAE@XZ 1003fbc4 f   wzdanimation.obj
 0001:0003ebdf       __unwindfunclet$?AllocKeyFrames@CWzdAnimation@@UAEXXZ$0 1003fbdf f   wzdanimation.obj
 0001:0003ebe9       __ehhandler$?AllocKeyFrames@CWzdAnimation@@UAEXXZ 1003fbe9 f   wzdanimation.obj
 0001:0003ec04       __unwindfunclet$?Create@CWzdBase@@UAEHPBDPAEH@Z$0 1003fc04 f   wzdbase.obj
 0001:0003ec0f       __ehhandler$?Create@CWzdBase@@UAEHPBDPAEH@Z 1003fc0f f   wzdbase.obj
 0001:0003ec37       __unwindfunclet$?Save@CWzdBase@@UAEHPBDH@Z$0 1003fc37 f   wzdbase.obj
 0001:0003ec42       __ehhandler$?Save@CWzdBase@@UAEHPBDH@Z 1003fc42 f   wzdbase.obj
 0001:0003ec6a       __unwindfunclet$?Save@CWzdBase@@UAEHPBDPAXH@Z$0 1003fc6a f   wzdbase.obj
 0001:0003ec75       __ehhandler$?Save@CWzdBase@@UAEHPBDPAXH@Z 1003fc75 f   wzdbase.obj
 0001:0003ec9d       __unwindfunclet$?CheckDiscAccessExistence@CWzdBase@@SAPAVCDiscAccess@@XZ$0 1003fc9d f   wzdbase.obj
 0001:0003ecab       __ehhandler$?CheckDiscAccessExistence@CWzdBase@@SAPAVCDiscAccess@@XZ 1003fcab f   wzdbase.obj
 0001:0003ecc6       __unwindfunclet$??0CWzdMesh@@QAE@XZ$0 1003fcc6 f   wzdmesh.obj
 0001:0003ecce       __ehhandler$??0CWzdMesh@@QAE@XZ 1003fcce f   wzdmesh.obj
 0001:0003ece9       __unwindfunclet$??1CWzdMesh@@UAE@XZ$0 1003fce9 f   wzdmesh.obj
 0001:0003ecf1       __ehhandler$??1CWzdMesh@@UAE@XZ 1003fcf1 f   wzdmesh.obj
 0001:0003ed0c       __unwindfunclet$?Serialize@CWzdMesh@@MAEHPAVCWzArchive@@@Z$0 1003fd0c f   wzdmesh.obj
 0001:0003ed14       __ehhandler$?Serialize@CWzdMesh@@MAEHPAVCWzArchive@@@Z 1003fd14 f   wzdmesh.obj
 0001:0003ed2f       __unwindfunclet$?SerializeMeshGroup@CWzdMesh@@IAEHPAVCWzArchive@@@Z$0 1003fd2f f   wzdmesh.obj
 0001:0003ed3c       __ehhandler$?SerializeMeshGroup@CWzdMesh@@IAEHPAVCWzArchive@@@Z 1003fd3c f   wzdmesh.obj
 0001:0003ed64       __unwindfunclet$??0CWzdMeshConstructor@@QAE@XZ$0 1003fd64 f   wzdmeshconstructor.obj
 0001:0003ed6c       __ehhandler$??0CWzdMeshConstructor@@QAE@XZ 1003fd6c f   wzdmeshconstructor.obj
 0001:0003ed87       __unwindfunclet$??1CWzdMeshConstructor@@UAE@XZ$0 1003fd87 f   wzdmeshconstructor.obj
 0001:0003ed8f       __ehhandler$??1CWzdMeshConstructor@@UAE@XZ 1003fd8f f   wzdmeshconstructor.obj
 0001:0003edaa       __unwindfunclet$?AllocForMesh@CWzdMeshConstructor@@UAEHXZ$0 1003fdaa f   wzdmeshconstructor.obj
 0001:0003edb4       __ehhandler$?AllocForMesh@CWzdMeshConstructor@@UAEHXZ 1003fdb4 f   wzdmeshconstructor.obj
 0001:0003edcf       __unwindfunclet$?MakeSureMeshGroupSize@CWzdMeshConstructor@@IAEXH@Z$0 1003fdcf f   wzdmeshconstructor.obj
 0001:0003edd9       __ehhandler$?MakeSureMeshGroupSize@CWzdMeshConstructor@@IAEXH@Z 1003fdd9 f   wzdmeshconstructor.obj
 0001:0003edf4       __unwindfunclet$?SortBones@CWzdMeshSorter@@AAEHPAHPAUSt_BoneConnection@@@Z$2 1003fdf4 f   wzdmeshsorter.obj
 0001:0003ee0d       __ehhandler$?SortBones@CWzdMeshSorter@@AAEHPAHPAUSt_BoneConnection@@@Z 1003fe0d f   wzdmeshsorter.obj
 0001:0003ee2b       __unwindfunclet$?SortFaces@CWzdMeshSorter@@AAEXHPBH@Z$1 1003fe2b f   wzdmeshsorter.obj
 0001:0003ee33       __ehhandler$?SortFaces@CWzdMeshSorter@@AAEXHPBH@Z 1003fe33 f   wzdmeshsorter.obj
 0001:0003ee51       __unwindfunclet$??1?$vector@HV?$allocator@H@std@@@std@@QAE@XZ$0 1003fe51 f   wzdmeshsorter.obj
 0001:0003ee59       __ehhandler$??1?$vector@HV?$allocator@H@std@@@std@@QAE@XZ 1003fe59 f   wzdmeshsorter.obj
 0001:0003ee74       __unwindfunclet$??0?$list@HV?$allocator@H@std@@@std@@QAE@XZ$0 1003fe74 f   wzdmeshsorter.obj
 0001:0003ee7c       __ehhandler$??0?$list@HV?$allocator@H@std@@@std@@QAE@XZ 1003fe7c f   wzdmeshsorter.obj
 0001:0003ee97       __unwindfunclet$??1?$list@HV?$allocator@H@std@@@std@@QAE@XZ$0 1003fe97 f   wzdmeshsorter.obj
 0001:0003ee9f       __ehhandler$??1?$list@HV?$allocator@H@std@@@std@@QAE@XZ 1003fe9f f   wzdmeshsorter.obj
 0001:0003eeba       __ehhandler$?_Buynode@?$list@HV?$allocator@H@std@@@std@@IAEPAU_Node@?$_List_nod@HV?$allocator@H@std@@@2@XZ 1003feba f   wzdmeshsorter.obj
 0001:0003eed5       __ehhandler$?_Insert_n@?$vector@HV?$allocator@H@std@@@std@@IAEXV?$_Vector_const_iterator@HV?$allocator@H@std@@@2@IABH@Z 1003fed5 f   wzdmeshsorter.obj
 0001:0003eef3       __unwindfunclet$??0?$_Container_base_aux_alloc_real@V?$allocator@UWzSoundInfo@@@std@@@std@@IAE@V?$allocator@UWzSoundInfo@@@1@@Z$0 1003fef3 f   wzdmeshsorter.obj
 0001:0003eef3       __unwindfunclet$??0?$_Container_base_aux_alloc_real@V?$allocator@UWzEffectInfo@@@std@@@std@@IAE@V?$allocator@UWzEffectInfo@@@1@@Z$0 1003fef3 f   wzdmeshsorter.obj
 0001:0003eef3       __unwindfunclet$??0?$_Container_base_aux_alloc_real@V?$allocator@UWzCustomInfo@@@std@@@std@@IAE@V?$allocator@UWzCustomInfo@@@1@@Z$0 1003fef3 f   wzdmeshsorter.obj
 0001:0003eef3       __unwindfunclet$??0?$_Container_base_aux_alloc_real@V?$allocator@H@std@@@std@@IAE@V?$allocator@H@1@@Z$0 1003fef3 f   wzdmeshsorter.obj
 0001:0003eef3       __unwindfunclet$??0?$_Container_base_aux_alloc_real@V?$allocator@U?$pair@$$CBHUWzVector@@@std@@@std@@@std@@IAE@V?$allocator@U?$pair@$$CBHUWzVector@@@std@@@1@@Z$0 1003fef3 f   wzdmeshsorter.obj
 0001:0003eefb       __ehhandler$??0?$_Container_base_aux_alloc_real@V?$allocator@U?$pair@$$CBHUWzVector@@@std@@@std@@@std@@IAE@V?$allocator@U?$pair@$$CBHUWzVector@@@std@@@1@@Z 1003fefb f   wzdmeshsorter.obj
 0001:0003eefb       __ehhandler$??0?$_Container_base_aux_alloc_real@V?$allocator@H@std@@@std@@IAE@V?$allocator@H@1@@Z 1003fefb f   wzdmeshsorter.obj
 0001:0003eefb       __ehhandler$??0?$_Container_base_aux_alloc_real@V?$allocator@UWzEffectInfo@@@std@@@std@@IAE@V?$allocator@UWzEffectInfo@@@1@@Z 1003fefb f   wzdmeshsorter.obj
 0001:0003eefb       __ehhandler$??0?$_Container_base_aux_alloc_real@V?$allocator@UWzSoundInfo@@@std@@@std@@IAE@V?$allocator@UWzSoundInfo@@@1@@Z 1003fefb f   wzdmeshsorter.obj
 0001:0003eefb       __ehhandler$??0?$_Container_base_aux_alloc_real@V?$allocator@UWzCustomInfo@@@std@@@std@@IAE@V?$allocator@UWzCustomInfo@@@1@@Z 1003fefb f   wzdmeshsorter.obj
 0001:0003ef16       __ehhandler$?_Buynode@?$list@HV?$allocator@H@std@@@std@@IAEPAU_Node@?$_List_nod@HV?$allocator@H@std@@@2@PAU342@0ABH@Z 1003ff16 f   wzdmeshsorter.obj
 0001:0003ef31       __unwindfunclet$?_Incsize@?$list@HV?$allocator@H@std@@@std@@IAEXI@Z$0 1003ff31 f   wzdmeshsorter.obj
 0001:0003ef39       __ehhandler$?_Incsize@?$list@HV?$allocator@H@std@@@std@@IAEXI@Z 1003ff39 f   wzdmeshsorter.obj
 0001:0003ef57       __unwindfunclet$??0logic_error@std@@QAE@ABV01@@Z$0 1003ff57 f   wzdmeshsorter.obj
 0001:0003ef57       __unwindfunclet$??0logic_error@std@@QAE@ABV?$basic_string@DU?$char_traits@D@std@@V?$allocator@D@2@@1@@Z$0 1003ff57 f   wzdmeshsorter.obj
 0001:0003ef5f       __ehhandler$??0logic_error@std@@QAE@ABV?$basic_string@DU?$char_traits@D@std@@V?$allocator@D@2@@1@@Z 1003ff5f f   wzdmeshsorter.obj
 0001:0003ef5f       __ehhandler$??0logic_error@std@@QAE@ABV01@@Z 1003ff5f f   wzdmeshsorter.obj
 0001:0003ef7a       __ehhandler$?_Copy@?$basic_string@DU?$char_traits@D@std@@V?$allocator@D@2@@std@@IAEXII@Z 1003ff7a f   wzdmeshsorter.obj
 0001:0003ef98       __unwindfunclet$??0WzAnimationInfo@@QAE@XZ$0 1003ff98 f   wzanimationInfo.obj
 0001:0003efa6       __unwindfunclet$??0WzAnimationInfo@@QAE@XZ$1 1003ffa6 f   wzanimationInfo.obj
 0001:0003efb4       __unwindfunclet$??0WzAnimationInfo@@QAE@XZ$2 1003ffb4 f   wzanimationInfo.obj
 0001:0003efc2       __unwindfunclet$??0WzAnimationInfo@@QAE@XZ$3 1003ffc2 f   wzanimationInfo.obj
 0001:0003efd3       __ehhandler$??0WzAnimationInfo@@QAE@XZ 1003ffd3 f   wzanimationInfo.obj
 0001:0003eff1       __unwindfunclet$??1WzAnimationInfo@@QAE@XZ$0 1003fff1 f   wzanimationInfo.obj
 0001:0003efff       __unwindfunclet$??1WzAnimationInfo@@QAE@XZ$1 1003ffff f   wzanimationInfo.obj
 0001:0003f00d       __unwindfunclet$??1WzAnimationInfo@@QAE@XZ$2 1004000d f   wzanimationInfo.obj
 0001:0003f01b       __unwindfunclet$??1WzAnimationInfo@@QAE@XZ$3 1004001b f   wzanimationInfo.obj
 0001:0003f02c       __unwindfunclet$??1WzAnimationInfo@@QAE@XZ$4 1004002c f   wzanimationInfo.obj
 0001:0003f034       __unwindfunclet$??1WzAnimationInfo@@QAE@XZ$7 10040034 f   wzanimationInfo.obj
 0001:0003f03c       __unwindfunclet$??1WzAnimationInfo@@QAE@XZ$10 1004003c f   wzanimationInfo.obj
 0001:0003f047       __ehhandler$??1WzAnimationInfo@@QAE@XZ 10040047 f   wzanimationInfo.obj
 0001:0003f065       __unwindfunclet$?AddSound@WzAnimationInfo@@QAEXHMH@Z$0 10040065 f   wzanimationInfo.obj
 0001:0003f06d       __unwindfunclet$?AddSound@WzAnimationInfo@@QAEXHMH@Z$5 1004006d f   wzanimationInfo.obj
 0001:0003f078       __ehhandler$?AddSound@WzAnimationInfo@@QAEXHMH@Z 10040078 f   wzanimationInfo.obj
 0001:0003f096       __unwindfunclet$??1?$vector@UWzSoundInfo@@V?$allocator@UWzSoundInfo@@@std@@@std@@QAE@XZ$0 10040096 f   wzanimationInfo.obj
 0001:0003f09e       __ehhandler$??1?$vector@UWzSoundInfo@@V?$allocator@UWzSoundInfo@@@std@@@std@@QAE@XZ 1004009e f   wzanimationInfo.obj
 0001:0003f0b9       __unwindfunclet$??0?$vector@UWzCustomInfo@@V?$allocator@UWzCustomInfo@@@std@@@std@@QAE@XZ$0 100400b9 f   wzanimationInfo.obj
 0001:0003f0b9       __unwindfunclet$??0?$vector@HV?$allocator@H@std@@@std@@QAE@XZ$0 100400b9 f   wzanimationInfo.obj
 0001:0003f0b9       __unwindfunclet$??0?$vector@UWzEffectInfo@@V?$allocator@UWzEffectInfo@@@std@@@std@@QAE@XZ$0 100400b9 f   wzanimationInfo.obj
 0001:0003f0b9       __unwindfunclet$??0?$vector@UWzSoundInfo@@V?$allocator@UWzSoundInfo@@@std@@@std@@QAE@XZ$0 100400b9 f   wzanimationInfo.obj
 0001:0003f0c4       __ehhandler$??0?$vector@HV?$allocator@H@std@@@std@@QAE@XZ 100400c4 f   wzanimationInfo.obj
 0001:0003f0c4       __ehhandler$??0?$vector@UWzCustomInfo@@V?$allocator@UWzCustomInfo@@@std@@@std@@QAE@XZ 100400c4 f   wzanimationInfo.obj
 0001:0003f0c4       __ehhandler$??0?$vector@UWzSoundInfo@@V?$allocator@UWzSoundInfo@@@std@@@std@@QAE@XZ 100400c4 f   wzanimationInfo.obj
 0001:0003f0c4       __ehhandler$??0?$vector@UWzEffectInfo@@V?$allocator@UWzEffectInfo@@@std@@@std@@QAE@XZ 100400c4 f   wzanimationInfo.obj
 0001:0003f0e2       __unwindfunclet$??1?$vector@UWzCustomInfo@@V?$allocator@UWzCustomInfo@@@std@@@std@@QAE@XZ$0 100400e2 f   wzanimationInfo.obj
 0001:0003f0e2       __unwindfunclet$??1?$vector@UWzEffectInfo@@V?$allocator@UWzEffectInfo@@@std@@@std@@QAE@XZ$0 100400e2 f   wzanimationInfo.obj
 0001:0003f0ea       __ehhandler$??1?$vector@UWzEffectInfo@@V?$allocator@UWzEffectInfo@@@std@@@std@@QAE@XZ 100400ea f   wzanimationInfo.obj
 0001:0003f0ea       __ehhandler$??1?$vector@UWzCustomInfo@@V?$allocator@UWzCustomInfo@@@std@@@std@@QAE@XZ 100400ea f   wzanimationInfo.obj
 0001:0003f105       __unwindfunclet$?_Insert_n@?$vector@UWzSoundInfo@@V?$allocator@UWzSoundInfo@@@std@@@std@@IAEXV?$_Vector_const_iterator@UWzSoundInfo@@V?$allocator@UWzSoundInfo@@@std@@@2@IABUWzSoundInfo@@@Z$4 10040105 f   wzanimationInfo.obj
 0001:0003f10d       __unwindfunclet$?_Insert_n@?$vector@UWzSoundInfo@@V?$allocator@UWzSoundInfo@@@std@@@std@@IAEXV?$_Vector_const_iterator@UWzSoundInfo@@V?$allocator@UWzSoundInfo@@@std@@@2@IABUWzSoundInfo@@@Z$24 1004010d f   wzanimationInfo.obj
 0001:0003f118       __unwindfunclet$?_Insert_n@?$vector@UWzSoundInfo@@V?$allocator@UWzSoundInfo@@@std@@@std@@IAEXV?$_Vector_const_iterator@UWzSoundInfo@@V?$allocator@UWzSoundInfo@@@std@@@2@IABUWzSoundInfo@@@Z$5 10040118 f   wzanimationInfo.obj
 0001:0003f120       __unwindfunclet$?_Insert_n@?$vector@UWzSoundInfo@@V?$allocator@UWzSoundInfo@@@std@@@std@@IAEXV?$_Vector_const_iterator@UWzSoundInfo@@V?$allocator@UWzSoundInfo@@@std@@@2@IABUWzSoundInfo@@@Z$29 10040120 f   wzanimationInfo.obj
 0001:0003f12b       __ehhandler$?_Insert_n@?$vector@UWzSoundInfo@@V?$allocator@UWzSoundInfo@@@std@@@std@@IAEXV?$_Vector_const_iterator@UWzSoundInfo@@V?$allocator@UWzSoundInfo@@@std@@@2@IABUWzSoundInfo@@@Z 1004012b f   wzanimationInfo.obj
 0001:0003f149       __unwindfunclet$?_Xlen@?$vector@UWzEffectInfo@@V?$allocator@UWzEffectInfo@@@std@@@std@@KAXXZ$0 10040149 f   wzanimationInfo.obj
 0001:0003f149       __unwindfunclet$?_Xlen@?$vector@HV?$allocator@H@std@@@std@@KAXXZ$0 10040149 f   wzanimationInfo.obj
 0001:0003f149       __unwindfunclet$?_Xlen@?$vector@UWzSoundInfo@@V?$allocator@UWzSoundInfo@@@std@@@std@@KAXXZ$0 10040149 f   wzanimationInfo.obj
 0001:0003f149       __unwindfunclet$?_Xlen@?$vector@UWzCustomInfo@@V?$allocator@UWzCustomInfo@@@std@@@std@@KAXXZ$0 10040149 f   wzanimationInfo.obj
 0001:0003f151       __ehhandler$?_Xlen@?$vector@UWzSoundInfo@@V?$allocator@UWzSoundInfo@@@std@@@std@@KAXXZ 10040151 f   wzanimationInfo.obj
 0001:0003f151       __ehhandler$?_Xlen@?$vector@HV?$allocator@H@std@@@std@@KAXXZ 10040151 f   wzanimationInfo.obj
 0001:0003f151       __ehhandler$?_Xlen@?$vector@UWzCustomInfo@@V?$allocator@UWzCustomInfo@@@std@@@std@@KAXXZ 10040151 f   wzanimationInfo.obj
 0001:0003f151       __ehhandler$?_Xlen@?$vector@UWzEffectInfo@@V?$allocator@UWzEffectInfo@@@std@@@std@@KAXXZ 10040151 f   wzanimationInfo.obj
 0001:0003f16f       __ehhandler$?_Insert_n@?$vector@UWzEffectInfo@@V?$allocator@UWzEffectInfo@@@std@@@std@@IAEXV?$_Vector_const_iterator@UWzEffectInfo@@V?$allocator@UWzEffectInfo@@@std@@@2@IABUWzEffectInfo@@@Z 1004016f f   wzanimationInfo.obj
 0001:0003f18d       __ehhandler$?_Insert_n@?$vector@UWzCustomInfo@@V?$allocator@UWzCustomInfo@@@std@@@std@@IAEXV?$_Vector_const_iterator@UWzCustomInfo@@V?$allocator@UWzCustomInfo@@@std@@@2@IABUWzCustomInfo@@@Z 1004018d f   wzanimationInfo.obj
 0001:0003f1ab       __unwindfunclet$??0?$vector@HV?$allocator@H@std@@@std@@QAE@ABV01@@Z$2 100401ab f   wzanimationInfo.obj
 0001:0003f1b6       __ehhandler$??0?$vector@HV?$allocator@H@std@@@std@@QAE@ABV01@@Z 100401b6 f   wzanimationInfo.obj
 0001:0003f1d4       __ehhandler$??$_Uninit_fill_n@PAUWzSoundInfo@@IU1@V?$allocator@UWzSoundInfo@@@std@@@std@@YAXPAUWzSoundInfo@@IABU1@AAV?$allocator@UWzSoundInfo@@@0@U_Nonscalar_ptr_iterator_tag@0@U_Range_checked_iterator_tag@0@@Z 100401d4 f   wzanimationInfo.obj
 0001:0003f1ef       __ehhandler$??$_Uninit_fill_n@PAUWzEffectInfo@@IU1@V?$allocator@UWzEffectInfo@@@std@@@std@@YAXPAUWzEffectInfo@@IABU1@AAV?$allocator@UWzEffectInfo@@@0@U_Nonscalar_ptr_iterator_tag@0@U_Range_checked_iterator_tag@0@@Z 100401ef f   wzanimationInfo.obj
 0001:0003f20a       __ehhandler$??$_Uninit_fill_n@PAUWzCustomInfo@@IU1@V?$allocator@UWzCustomInfo@@@std@@@std@@YAXPAUWzCustomInfo@@IABU1@AAV?$allocator@UWzCustomInfo@@@0@U_Nonscalar_ptr_iterator_tag@0@U_Range_checked_iterator_tag@0@@Z 1004020a f   wzanimationInfo.obj
 0001:0003f225       __ehhandler$??$_Uninit_copy@PAUWzSoundInfo@@PAU1@V?$allocator@UWzSoundInfo@@@std@@@std@@YAPAUWzSoundInfo@@PAU1@00AAV?$allocator@UWzSoundInfo@@@0@U_Nonscalar_ptr_iterator_tag@0@U_Range_checked_iterator_tag@0@@Z 10040225 f   wzanimationInfo.obj
 0001:0003f240       __ehhandler$??$_Uninit_copy@PAUWzEffectInfo@@PAU1@V?$allocator@UWzEffectInfo@@@std@@@std@@YAPAUWzEffectInfo@@PAU1@00AAV?$allocator@UWzEffectInfo@@@0@U_Nonscalar_ptr_iterator_tag@0@U_Range_checked_iterator_tag@0@@Z 10040240 f   wzanimationInfo.obj
 0001:0003f25b       __ehhandler$??$_Uninit_copy@PAUWzCustomInfo@@PAU1@V?$allocator@UWzCustomInfo@@@std@@@std@@YAPAUWzCustomInfo@@PAU1@00AAV?$allocator@UWzCustomInfo@@@0@U_Nonscalar_ptr_iterator_tag@0@U_Range_checked_iterator_tag@0@@Z 1004025b f   wzanimationInfo.obj
 0001:0003f276       __unwindfunclet$??$_Construct@UWzSoundInfo@@U1@@std@@YAXPAUWzSoundInfo@@ABU1@@Z$0 10040276 f   wzanimationInfo.obj
 0001:0003f284       __ehhandler$??$_Construct@UWzSoundInfo@@U1@@std@@YAXPAUWzSoundInfo@@ABU1@@Z 10040284 f   wzanimationInfo.obj
 0001:0003f29f       __unwindfunclet$??_GWzSoundInfo@@QAEPAXI@Z$1 1004029f f   wzanimationInfo.obj
 0001:0003f29f       __unwindfunclet$??1WzSoundInfo@@QAE@XZ$1 1004029f f   wzanimationInfo.obj
 0001:0003f2a7       __ehhandler$??_GWzSoundInfo@@QAEPAXI@Z 100402a7 f   wzanimationInfo.obj
 0001:0003f2a7       __ehhandler$??1WzSoundInfo@@QAE@XZ 100402a7 f   wzanimationInfo.obj
 0001:0003f2c2       __unwindfunclet$??0CWzAniState@@QAE@XZ$0 100402c2 f   wzanistate.obj
 0001:0003f2d0       __unwindfunclet$??0CWzAniState@@QAE@XZ$1 100402d0 f   wzanistate.obj
 0001:0003f2de       __ehhandler$??0CWzAniState@@QAE@XZ 100402de f   wzanistate.obj
 0001:0003f2fc       __unwindfunclet$??1CWzAniState@@UAE@XZ$0 100402fc f   wzanistate.obj
 0001:0003f307       __unwindfunclet$??1CWzAniState@@UAE@XZ$1 10040307 f   wzanistate.obj
 0001:0003f312       __unwindfunclet$??1CWzAniState@@UAE@XZ$2 10040312 f   wzanistate.obj
 0001:0003f31a       __ehhandler$??1CWzAniState@@UAE@XZ 1004031a f   wzanistate.obj
 0001:0003f335       __unwindfunclet$?FindWzd@CManagerWzdLoader@@QAEPAXPBD@Z$0 10040335 f   wzanistate.obj
 0001:0003f33d       __ehhandler$?FindWzd@CManagerWzdLoader@@QAEPAXPBD@Z 1004033d f   wzanistate.obj
 0001:0003f358       __unwindfunclet$?GetWzdInfo@CManagerWzdLoader@@QAEPAUSt_WzdContainer@@PAX@Z$0 10040358 f   wzanistate.obj
 0001:0003f360       __ehhandler$?GetWzdInfo@CManagerWzdLoader@@QAEPAUSt_WzdContainer@@PAX@Z 10040360 f   wzanistate.obj
 0001:0003f37b       __unwindfunclet$?GetC@?$CWzHashTableStr@PAX@@QBEABQAXPBD@Z$0 1004037b f   wzanistate.obj
 0001:0003f383       __ehhandler$?GetC@?$CWzHashTableStr@PAX@@QBEABQAXPBD@Z 10040383 f   wzanistate.obj
 0001:0003f39e       __unwindfunclet$??0CWzUnit@@QAE@XZ$0 1004039e f   wzunit.obj
 0001:0003f3a9       __unwindfunclet$??0CWzUnit@@QAE@XZ$1 100403a9 f   wzunit.obj
 0001:0003f3b4       __unwindfunclet$??0CWzUnit@@QAE@XZ$2 100403b4 f   wzunit.obj
 0001:0003f3bf       __unwindfunclet$??0CWzUnit@@QAE@XZ$3 100403bf f   wzunit.obj
 0001:0003f3ca       __unwindfunclet$??0CWzUnit@@QAE@XZ$4 100403ca f   wzunit.obj
 0001:0003f3d5       __unwindfunclet$??0CWzUnit@@QAE@XZ$5 100403d5 f   wzunit.obj
 0001:0003f3e0       __unwindfunclet$??0CWzUnit@@QAE@XZ$6 100403e0 f   wzunit.obj
 0001:0003f3eb       __unwindfunclet$??0CWzUnit@@QAE@XZ$7 100403eb f   wzunit.obj
 0001:0003f3f9       __unwindfunclet$??0CWzUnit@@QAE@XZ$8 100403f9 f   wzunit.obj
 0001:0003f407       __unwindfunclet$??0CWzUnit@@QAE@XZ$9 10040407 f   wzunit.obj
 0001:0003f415       __unwindfunclet$??0CWzUnit@@QAE@XZ$10 10040415 f   wzunit.obj
 0001:0003f423       __unwindfunclet$??0CWzUnit@@QAE@XZ$11 10040423 f   wzunit.obj
 0001:0003f431       __unwindfunclet$??0CWzUnit@@QAE@XZ$12 10040431 f   wzunit.obj
 0001:0003f43f       __ehhandler$??0CWzUnit@@QAE@XZ 1004043f f   wzunit.obj
 0001:0003f45a       __unwindfunclet$??1CWzUnit@@UAE@XZ$0 1004045a f   wzunit.obj
 0001:0003f465       __unwindfunclet$??1CWzUnit@@UAE@XZ$1 10040465 f   wzunit.obj
 0001:0003f470       __unwindfunclet$??1CWzUnit@@UAE@XZ$2 10040470 f   wzunit.obj
 0001:0003f47b       __unwindfunclet$??1CWzUnit@@UAE@XZ$3 1004047b f   wzunit.obj
 0001:0003f486       __unwindfunclet$??1CWzUnit@@UAE@XZ$4 10040486 f   wzunit.obj
 0001:0003f491       __unwindfunclet$??1CWzUnit@@UAE@XZ$5 10040491 f   wzunit.obj
 0001:0003f49c       __unwindfunclet$??1CWzUnit@@UAE@XZ$6 1004049c f   wzunit.obj
 0001:0003f4a7       __unwindfunclet$??1CWzUnit@@UAE@XZ$7 100404a7 f   wzunit.obj
 0001:0003f4b5       __unwindfunclet$??1CWzUnit@@UAE@XZ$8 100404b5 f   wzunit.obj
 0001:0003f4c3       __unwindfunclet$??1CWzUnit@@UAE@XZ$9 100404c3 f   wzunit.obj
 0001:0003f4d1       __unwindfunclet$??1CWzUnit@@UAE@XZ$10 100404d1 f   wzunit.obj
 0001:0003f4df       __unwindfunclet$??1CWzUnit@@UAE@XZ$11 100404df f   wzunit.obj
 0001:0003f4ed       __unwindfunclet$??1CWzUnit@@UAE@XZ$12 100404ed f   wzunit.obj
 0001:0003f4fb       __ehhandler$??1CWzUnit@@UAE@XZ 100404fb f   wzunit.obj
 0001:0003f516       __unwindfunclet$?AddAnimationInfo@CWzUnit@@QAEXABVWzAnimationInfo@@@Z$0 10040516 f   wzunit.obj
 0001:0003f520       __ehhandler$?AddAnimationInfo@CWzUnit@@QAEXABVWzAnimationInfo@@@Z 10040520 f   wzunit.obj
 0001:0003f53b       __unwindfunclet$?CreateSubType@CWzUnit@@QAEPAVCWzUnitSubType@@XZ$0 1004053b f   wzunit.obj
 0001:0003f545       __ehhandler$?CreateSubType@CWzUnit@@QAEPAVCWzUnitSubType@@XZ 10040545 f   wzunit.obj
 0001:0003f560       __unwindfunclet$?AddTexAniSetInfo@CWzUnit@@QAEXABUWzTexAniSetInfo@@@Z$0 10040560 f   wzunit.obj
 0001:0003f56a       __ehhandler$?AddTexAniSetInfo@CWzUnit@@QAEXABUWzTexAniSetInfo@@@Z 1004056a f   wzunit.obj
 0001:0003f585       __unwindfunclet$??0WzTexAniSetInfo@@QAE@XZ$0 10040585 f   wzunit.obj
 0001:0003f590       __ehhandler$??0WzTexAniSetInfo@@QAE@XZ 10040590 f   wzunit.obj
 0001:0003f5ab       __unwindfunclet$?Save@CWzUnit@@UAEHPBD@Z$0 100405ab f   wzunit_loadsave.obj
 0001:0003f5b6       __ehhandler$?Save@CWzUnit@@UAEHPBD@Z 100405b6 f   wzunit_loadsave.obj
 0001:0003f5de       __unwindfunclet$?Load@CWzUnit@@UAEHPBD@Z$0 100405de f   wzunit_loadsave.obj
 0001:0003f5e9       __ehhandler$?Load@CWzUnit@@UAEHPBD@Z 100405e9 f   wzunit_loadsave.obj
 0001:0003f611       __unwindfunclet$?SerializeAnimInfo@CWzUnit@@AAEHPAVCWzArchive@@@Z$0 10040611 f   wzunit_loadsave.obj
 0001:0003f61c       __ehhandler$?SerializeAnimInfo@CWzUnit@@AAEHPAVCWzArchive@@@Z 1004061c f   wzunit_loadsave.obj
 0001:0003f644       __unwindfunclet$?SerializeMappingInfo@CWzUnit@@AAEHPAVCWzArchive@@@Z$0 10040644 f   wzunit_loadsave.obj
 0001:0003f64f       __ehhandler$?SerializeMappingInfo@CWzUnit@@AAEHPAVCWzArchive@@@Z 1004064f f   wzunit_loadsave.obj
 0001:0003f677       __unwindfunclet$??0CWzUnitDraw@@QAE@K@Z$0 10040677 f   wzunitdraw.obj
 0001:0003f682       __unwindfunclet$??0CWzUnitDraw@@QAE@K@Z$1 10040682 f   wzunitdraw.obj
 0001:0003f68d       __unwindfunclet$??0CWzUnitDraw@@QAE@K@Z$2 1004068d f   wzunitdraw.obj
 0001:0003f698       __unwindfunclet$??0CWzUnitDraw@@QAE@K@Z$3 10040698 f   wzunitdraw.obj
 0001:0003f6a3       __ehhandler$??0CWzUnitDraw@@QAE@K@Z 100406a3 f   wzunitdraw.obj
 0001:0003f6be       __unwindfunclet$??1CWzUnitDraw@@UAE@XZ$0 100406be f   wzunitdraw.obj
 0001:0003f6c9       __unwindfunclet$??1CWzUnitDraw@@UAE@XZ$1 100406c9 f   wzunitdraw.obj
 0001:0003f6d4       __unwindfunclet$??1CWzUnitDraw@@UAE@XZ$2 100406d4 f   wzunitdraw.obj
 0001:0003f6df       __unwindfunclet$??1CWzUnitDraw@@UAE@XZ$3 100406df f   wzunitdraw.obj
 0001:0003f6ea       __ehhandler$??1CWzUnitDraw@@UAE@XZ 100406ea f   wzunitdraw.obj
 0001:0003f705       __unwindfunclet$?SetAniRefUnitDraw@CWzUnitDraw@@QAEXPAV1@@Z$0 10040705 f   wzunitdraw.obj
 0001:0003f70f       __ehhandler$?SetAniRefUnitDraw@CWzUnitDraw@@QAEXPAV1@@Z 1004070f f   wzunitdraw.obj
 0001:0003f72a       __unwindfunclet$?UpdateSilhouette@CWzUnitDraw@@QAEXPAVCWzdBase@@ABUWzVector@@PBU3@@Z$0 1004072a f   wzunitdraw.obj
 0001:0003f734       __ehhandler$?UpdateSilhouette@CWzUnitDraw@@QAEXPAVCWzdBase@@ABUWzVector@@PBU3@@Z 10040734 f   wzunitdraw.obj
 0001:0003f74f       __unwindfunclet$?UpdateShadowVolume@CWzUnitDraw@@QAEXPAVCWzdBase@@ABUWzVector@@PBU3@K@Z$0 1004074f f   wzunitdraw.obj
 0001:0003f759       __ehhandler$?UpdateShadowVolume@CWzUnitDraw@@QAEXPAVCWzdBase@@ABUWzVector@@PBU3@K@Z 10040759 f   wzunitdraw.obj
 0001:0003f774       __unwindfunclet$?AddTexAniID@CWzUnitEditable@@QAEXK@Z$0 10040774 f   wzuniteditable.obj
 0001:0003f77c       __ehhandler$?AddTexAniID@CWzUnitEditable@@QAEXK@Z 1004077c f   wzuniteditable.obj
 0001:0003f797       __unwindfunclet$?CreateSubType@CWzUnitEditable@@QAEPAVCWzUnitSubType@@XZ$0 10040797 f   wzuniteditable.obj
 0001:0003f7a1       __ehhandler$?CreateSubType@CWzUnitEditable@@QAEPAVCWzUnitSubType@@XZ 100407a1 f   wzuniteditable.obj
 0001:0003f7bc       __unwindfunclet$??0CWzUnitSkeleton@@AAE@XZ$0 100407bc f   wzunitskeleton.obj
 0001:0003f7c4       __unwindfunclet$??0CWzUnitSkeleton@@AAE@XZ$1 100407c4 f   wzunitskeleton.obj
 0001:0003f7cf       __unwindfunclet$??0CWzUnitSkeleton@@AAE@XZ$2 100407cf f   wzunitskeleton.obj
 0001:0003f7da       __unwindfunclet$??0CWzUnitSkeleton@@AAE@XZ$3 100407da f   wzunitskeleton.obj
 0001:0003f7e8       __unwindfunclet$??0CWzUnitSkeleton@@AAE@XZ$4 100407e8 f   wzunitskeleton.obj
 0001:0003f7f6       __ehhandler$??0CWzUnitSkeleton@@AAE@XZ 100407f6 f   wzunitskeleton.obj
 0001:0003f811       __unwindfunclet$??0CWzUnitSkeleton@@QAE@PAVCWzUnitDraw@@@Z$0 10040811 f   wzunitskeleton.obj
 0001:0003f819       __unwindfunclet$??0CWzUnitSkeleton@@QAE@PAVCWzUnitDraw@@@Z$1 10040819 f   wzunitskeleton.obj
 0001:0003f824       __unwindfunclet$??0CWzUnitSkeleton@@QAE@PAVCWzUnitDraw@@@Z$2 10040824 f   wzunitskeleton.obj
 0001:0003f82f       __unwindfunclet$??0CWzUnitSkeleton@@QAE@PAVCWzUnitDraw@@@Z$3 1004082f f   wzunitskeleton.obj
 0001:0003f83d       __unwindfunclet$??0CWzUnitSkeleton@@QAE@PAVCWzUnitDraw@@@Z$4 1004083d f   wzunitskeleton.obj
 0001:0003f84b       __unwindfunclet$??0CWzUnitSkeleton@@QAE@PAVCWzUnitDraw@@@Z$5 1004084b f   wzunitskeleton.obj
 0001:0003f859       __ehhandler$??0CWzUnitSkeleton@@QAE@PAVCWzUnitDraw@@@Z 10040859 f   wzunitskeleton.obj
 0001:0003f874       __unwindfunclet$??1CWzUnitSkeleton@@UAE@XZ$0 10040874 f   wzunitskeleton.obj
 0001:0003f87c       __unwindfunclet$??1CWzUnitSkeleton@@UAE@XZ$1 1004087c f   wzunitskeleton.obj
 0001:0003f887       __unwindfunclet$??1CWzUnitSkeleton@@UAE@XZ$2 10040887 f   wzunitskeleton.obj
 0001:0003f892       __unwindfunclet$??1CWzUnitSkeleton@@UAE@XZ$3 10040892 f   wzunitskeleton.obj
 0001:0003f8a0       __unwindfunclet$??1CWzUnitSkeleton@@UAE@XZ$4 100408a0 f   wzunitskeleton.obj
 0001:0003f8ae       __unwindfunclet$??1CWzUnitSkeleton@@UAE@XZ$5 100408ae f   wzunitskeleton.obj
 0001:0003f8bc       __unwindfunclet$??1CWzUnitSkeleton@@UAE@XZ$8 100408bc f   wzunitskeleton.obj
 0001:0003f8c4       __ehhandler$??1CWzUnitSkeleton@@UAE@XZ 100408c4 f   wzunitskeleton.obj
 0001:0003f8df       __unwindfunclet$??1WzTransformParam@@QAE@XZ$2 100408df f   wzunitskeleton.obj
 0001:0003f8e7       __ehhandler$??1WzTransformParam@@QAE@XZ 100408e7 f   wzunitskeleton.obj
 0001:0003f902       __unwindfunclet$??0?$_Tree@V?$_Tmap_traits@HUWzVector@@U?$less@H@std@@V?$allocator@U?$pair@$$CBHUWzVector@@@std@@@3@$0A@@std@@@std@@QAE@ABU?$less@H@1@ABV?$allocator@U?$pair@$$CBHUWzVector@@@std@@@1@@Z$0 10040902 f   wzunitskeleton.obj
 0001:0003f90a       __ehhandler$??0?$_Tree@V?$_Tmap_traits@HUWzVector@@U?$less@H@std@@V?$allocator@U?$pair@$$CBHUWzVector@@@std@@@3@$0A@@std@@@std@@QAE@ABU?$less@H@1@ABV?$allocator@U?$pair@$$CBHUWzVector@@@std@@@1@@Z 1004090a f   wzunitskeleton.obj
 0001:0003f925       __unwindfunclet$?_Insert@?$_Tree@V?$_Tmap_traits@HUWzVector@@U?$less@H@std@@V?$allocator@U?$pair@$$CBHUWzVector@@@std@@@3@$0A@@std@@@std@@IAE?AViterator@12@_NPAU_Node@?$_Tree_nod@V?$_Tmap_traits@HUWzVector@@U?$less@H@std@@V?$allocator@U?$pair@$$CBHUWzVector@@@std@@@3@$0A@@std@@@2@ABU?$pair@$$CBHUWzVector@@@2@@Z$0 10040925 f   wzunitskeleton.obj
 0001:0003f92d       __ehhandler$?_Insert@?$_Tree@V?$_Tmap_traits@HUWzVector@@U?$less@H@std@@V?$allocator@U?$pair@$$CBHUWzVector@@@std@@@3@$0A@@std@@@std@@IAE?AViterator@12@_NPAU_Node@?$_Tree_nod@V?$_Tmap_traits@HUWzVector@@U?$less@H@std@@V?$allocator@U?$pair@$$CBHUWzVector@@@std@@@3@$0A@@std@@@2@ABU?$pair@$$CBHUWzVector@@@2@@Z 1004092d f   wzunitskeleton.obj
 0001:0003f94b       __ehhandler$?_Buynode@?$_Tree@V?$_Tmap_traits@HUWzVector@@U?$less@H@std@@V?$allocator@U?$pair@$$CBHUWzVector@@@std@@@3@$0A@@std@@@std@@IAEPAU_Node@?$_Tree_nod@V?$_Tmap_traits@HUWzVector@@U?$less@H@std@@V?$allocator@U?$pair@$$CBHUWzVector@@@std@@@3@$0A@@std@@@2@PAU342@00ABU?$pair@$$CBHUWzVector@@@2@D@Z 1004094b f   wzunitskeleton.obj
 0001:0003f966       __unwindfunclet$?erase@?$_Tree@V?$_Tmap_traits@HUWzVector@@U?$less@H@std@@V?$allocator@U?$pair@$$CBHUWzVector@@@std@@@3@$0A@@std@@@std@@QAE?AViterator@12@Vconst_iterator@12@@Z$0 10040966 f   wzunitskeleton.obj
 0001:0003f96e       __ehhandler$?erase@?$_Tree@V?$_Tmap_traits@HUWzVector@@U?$less@H@std@@V?$allocator@U?$pair@$$CBHUWzVector@@@std@@@3@$0A@@std@@@std@@QAE?AViterator@12@Vconst_iterator@12@@Z 1004096e f   wzunitskeleton.obj
 0001:0003f98c       __ehhandler$?_Buynode@?$_Tree@V?$_Tmap_traits@HUWzVector@@U?$less@H@std@@V?$allocator@U?$pair@$$CBHUWzVector@@@std@@@3@$0A@@std@@@std@@IAEPAU_Node@?$_Tree_nod@V?$_Tmap_traits@HUWzVector@@U?$less@H@std@@V?$allocator@U?$pair@$$CBHUWzVector@@@std@@@3@$0A@@std@@@2@XZ 1004098c f   wzunitskeleton.obj
 0001:0003f9a7       __unwindfunclet$??0CWzUnitSubType@@QAE@XZ$0 100409a7 f   wzunitsubtype.obj
 0001:0003f9b2       __unwindfunclet$??0CWzUnitSubType@@QAE@XZ$1 100409b2 f   wzunitsubtype.obj
 0001:0003f9bd       __unwindfunclet$??0CWzUnitSubType@@QAE@XZ$2 100409bd f   wzunitsubtype.obj
 0001:0003f9c8       __ehhandler$??0CWzUnitSubType@@QAE@XZ 100409c8 f   wzunitsubtype.obj
 0001:0003f9e3       __unwindfunclet$??1CWzUnitSubType@@UAE@XZ$0 100409e3 f   wzunitsubtype.obj
 0001:0003f9ee       __unwindfunclet$??1CWzUnitSubType@@UAE@XZ$1 100409ee f   wzunitsubtype.obj
 0001:0003f9f9       __unwindfunclet$??1CWzUnitSubType@@UAE@XZ$2 100409f9 f   wzunitsubtype.obj
 0001:0003fa04       __ehhandler$??1CWzUnitSubType@@UAE@XZ 10040a04 f   wzunitsubtype.obj
 0001:0003fa1f       __unwindfunclet$?AddRenderInfo@CWzUnitSubType@@QAEXPBUWzRenderInfo@@@Z$0 10040a1f f   wzunitsubtype.obj
 0001:0003fa29       __ehhandler$?AddRenderInfo@CWzUnitSubType@@QAEXPBUWzRenderInfo@@@Z 10040a29 f   wzunitsubtype.obj
 0001:0003fa44       __unwindfunclet$?InitializeWzLogSystem@@YAXXZ$0 10040a44 f   programcommonlibforengine:wzlogsystem.obj
 0001:0003fa4e       __ehhandler$?InitializeWzLogSystem@@YAXXZ 10040a4e f   programcommonlibforengine:wzlogsystem.obj
 0001:0003fa69       __unwindfunclet$??0CWzArchive@@QAE@XZ$0 10040a69 f   programcommonlibforengine:wzarchive.obj
 0001:0003fa74       __ehhandler$??0CWzArchive@@QAE@XZ 10040a74 f   programcommonlibforengine:wzarchive.obj
 0001:0003fa8f       __unwindfunclet$??1CWzArchive@@QAE@XZ$0 10040a8f f   programcommonlibforengine:wzarchive.obj
 0001:0003fa9a       __ehhandler$??1CWzArchive@@QAE@XZ 10040a9a f   programcommonlibforengine:wzarchive.obj
 0001:0003fab5       __unwindfunclet$?CreateDiscAccess@CWzArchive@@AAEXXZ$0 10040ab5 f   programcommonlibforengine:wzarchive.obj
 0001:0003fabf       __ehhandler$?CreateDiscAccess@CWzArchive@@AAEXXZ 10040abf f   programcommonlibforengine:wzarchive.obj
 0001:0003fada       __unwindfunclet$??0CDiscAccess@@QAE@XZ$0 10040ada f   programcommonlibforengine:discaccess.obj
 0001:0003fae8       __unwindfunclet$??0CDiscAccess@@QAE@XZ$1 10040ae8 f   programcommonlibforengine:discaccess.obj
 0001:0003faf6       __ehhandler$??0CDiscAccess@@QAE@XZ 10040af6 f   programcommonlibforengine:discaccess.obj
 0001:0003fb11       __unwindfunclet$??1CDiscAccess@@QAE@XZ$0 10040b11 f   programcommonlibforengine:discaccess.obj
 0001:0003fb1f       __unwindfunclet$??1CDiscAccess@@QAE@XZ$1 10040b1f f   programcommonlibforengine:discaccess.obj
 0001:0003fb2d       __ehhandler$??1CDiscAccess@@QAE@XZ 10040b2d f   programcommonlibforengine:discaccess.obj
 0001:0003fb48       __unwindfunclet$?OpenDisc_Packer@CDiscAccess@@QAEHKPBD0W4ENUM_OPEN_PACKER_TYPE@@@Z$0 10040b48 f   programcommonlibforengine:discaccess.obj
 0001:0003fb50       __unwindfunclet$?OpenDisc_Packer@CDiscAccess@@QAEHKPBD0W4ENUM_OPEN_PACKER_TYPE@@@Z$1 10040b50 f   programcommonlibforengine:discaccess.obj
 0001:0003fb5a       __ehhandler$?OpenDisc_Packer@CDiscAccess@@QAEHKPBD0W4ENUM_OPEN_PACKER_TYPE@@@Z 10040b5a f   programcommonlibforengine:discaccess.obj
 0001:0003fb75       __unwindfunclet$?CloseDisc@CDiscAccess@@QAEXK@Z$0 10040b75 f   programcommonlibforengine:discaccess.obj
 0001:0003fb7d       __ehhandler$?CloseDisc@CDiscAccess@@QAEXK@Z 10040b7d f   programcommonlibforengine:discaccess.obj
 0001:0003fb98       __unwindfunclet$?OpenFile@CDiscAccess@@QAEPAXKPBDKKW4ENUM_OPEN_DISPOSITION@@@Z$0 10040b98 f   programcommonlibforengine:discaccess.obj
 0001:0003fba0       __ehhandler$?OpenFile@CDiscAccess@@QAEPAXKPBDKKW4ENUM_OPEN_DISPOSITION@@@Z 10040ba0 f   programcommonlibforengine:discaccess.obj
 0001:0003fbc8       __unwindfunclet$?CloseFile@CDiscAccess@@QAEHPAX@Z$0 10040bc8 f   programcommonlibforengine:discaccess.obj
 0001:0003fbd0       __ehhandler$?CloseFile@CDiscAccess@@QAEHPAX@Z 10040bd0 f   programcommonlibforengine:discaccess.obj
 0001:0003fbeb       __unwindfunclet$?SeekFile@CDiscAccess@@QAEKPAXJW4ENUM_SEEK_ORIGIN@@@Z$0 10040beb f   programcommonlibforengine:discaccess.obj
 0001:0003fbf3       __ehhandler$?SeekFile@CDiscAccess@@QAEKPAXJW4ENUM_SEEK_ORIGIN@@@Z 10040bf3 f   programcommonlibforengine:discaccess.obj
 0001:0003fc0e       __unwindfunclet$?ReadFile@CDiscAccess@@QAEKPAX0K@Z$0 10040c0e f   programcommonlibforengine:discaccess.obj
 0001:0003fc16       __ehhandler$?ReadFile@CDiscAccess@@QAEKPAX0K@Z 10040c16 f   programcommonlibforengine:discaccess.obj
 0001:0003fc31       __unwindfunclet$?WriteFile@CDiscAccess@@QAEKPAXPBXK@Z$0 10040c31 f   programcommonlibforengine:discaccess.obj
 0001:0003fc39       __ehhandler$?WriteFile@CDiscAccess@@QAEKPAXPBXK@Z 10040c39 f   programcommonlibforengine:discaccess.obj
 0001:0003fc54       __unwindfunclet$?FileExists@CDiscAccess@@QAEHKPBD@Z$0 10040c54 f   programcommonlibforengine:discaccess.obj
 0001:0003fc5c       __ehhandler$?FileExists@CDiscAccess@@QAEHKPBD@Z 10040c5c f   programcommonlibforengine:discaccess.obj
 0001:0003fc84       __unwindfunclet$?GetFileSize@CDiscAccess@@QAEKPAX@Z$0 10040c84 f   programcommonlibforengine:discaccess.obj
 0001:0003fc8c       __ehhandler$?GetFileSize@CDiscAccess@@QAEKPAX@Z 10040c8c f   programcommonlibforengine:discaccess.obj
 0001:0003fca7       __unwindfunclet$?GetFileInformationByHandle@CDiscAccess@@QAEHPAXPAUSt_FileInformation@@@Z$0 10040ca7 f   programcommonlibforengine:discaccess.obj
 0001:0003fcaf       __ehhandler$?GetFileInformationByHandle@CDiscAccess@@QAEHPAXPAUSt_FileInformation@@@Z 10040caf f   programcommonlibforengine:discaccess.obj
 0001:0003fcd7       __unwindfunclet$?CopyFileA@CDiscAccess@@QAEHKPBD0@Z$0 10040cd7 f   programcommonlibforengine:discaccess.obj
 0001:0003fcdf       __ehhandler$?CopyFileA@CDiscAccess@@QAEHKPBD0@Z 10040cdf f   programcommonlibforengine:discaccess.obj
 0001:0003fd07       __unwindfunclet$?DeleteFileA@CDiscAccess@@QAEHKPBD@Z$0 10040d07 f   programcommonlibforengine:discaccess.obj
 0001:0003fd0f       __ehhandler$?DeleteFileA@CDiscAccess@@QAEHKPBD@Z 10040d0f f   programcommonlibforengine:discaccess.obj
 0001:0003fd37       __unwindfunclet$?CreateDirectoryA@CDiscAccess@@QAEHKPBD@Z$0 10040d37 f   programcommonlibforengine:discaccess.obj
 0001:0003fd3f       __ehhandler$?CreateDirectoryA@CDiscAccess@@QAEHKPBD@Z 10040d3f f   programcommonlibforengine:discaccess.obj
 0001:0003fd67       __unwindfunclet$?RemoveDirectoryA@CDiscAccess@@QAEHKPBD@Z$0 10040d67 f   programcommonlibforengine:discaccess.obj
 0001:0003fd6f       __ehhandler$?RemoveDirectoryA@CDiscAccess@@QAEHKPBD@Z 10040d6f f   programcommonlibforengine:discaccess.obj
 0001:0003fd97       __unwindfunclet$??0?$CWzHandleManager@USt_DAFileInfo@@@@QAE@XZ$0 10040d97 f   programcommonlibforengine:discaccess.obj
 0001:0003fda2       __unwindfunclet$??0?$CWzHandleManager@USt_DAFileInfo@@@@QAE@XZ$1 10040da2 f   programcommonlibforengine:discaccess.obj
 0001:0003fdad       __unwindfunclet$??0?$CWzHandleManager@USt_DAFileInfo@@@@QAE@XZ$2 10040dad f   programcommonlibforengine:discaccess.obj
 0001:0003fdb8       __ehhandler$??0?$CWzHandleManager@USt_DAFileInfo@@@@QAE@XZ 10040db8 f   programcommonlibforengine:discaccess.obj
 0001:0003fdd3       __unwindfunclet$??1?$CWzHandleManager@USt_DAFileInfo@@@@UAE@XZ$0 10040dd3 f   programcommonlibforengine:discaccess.obj
 0001:0003fdde       __unwindfunclet$??1?$CWzHandleManager@USt_DAFileInfo@@@@UAE@XZ$1 10040dde f   programcommonlibforengine:discaccess.obj
 0001:0003fde9       __ehhandler$??1?$CWzHandleManager@USt_DAFileInfo@@@@UAE@XZ 10040de9 f   programcommonlibforengine:discaccess.obj
 0001:0003fe04       __unwindfunclet$?_Xlen@_String_base@std@@SAXXZ$0 10040e04 f   libcpmt:string.obj
 0001:0003fe04       __unwindfunclet$?_Xran@_String_base@std@@SAXXZ$0 10040e04 f   libcpmt:string.obj
 0001:0003fe0c       __ehhandler$?_Xran@_String_base@std@@SAXXZ 10040e0c f   libcpmt:string.obj
 0001:0003fe0c       __ehhandler$?_Xlen@_String_base@std@@SAXXZ 10040e0c f   libcpmt:string.obj
 0001:0003fe27       __ehhandler$?CallUnexpected@@YAXPBU_s_ESTypeList@@@Z 10040e27 f   LIBCMT:frame.obj
 0001:0003fe50       ??__Eautofree@@YAXXZ       10040e50 f   wzFilePacker_static:wzFilePacker.obj
 0001:0003fe7e       ??__Fnomem@?5???2@YAPAXI@Z@YAXXZ 10040e7e f   LIBCMT:new.obj
 0001:0003fea0       ??__Fautofree@@YAXXZ       10040ea0 f   wzFilePacker_static:wzFilePacker.obj

 Exports

  ordinal    name

        1    ??4WzAnimationInfo@@QAEAAV0@ABV0@@Z (public: class WzAnimationInfo & __thiscall WzAnimationInfo::operator=(class WzAnimationInfo const &))
        2    ?AddAnimationInfo@CWzUnit@@QAEXABVWzAnimationInfo@@@Z (public: void __thiscall CWzUnit::AddAnimationInfo(class WzAnimationInfo const &))
        3    ?AddBV@WzAnimationInfo@@QAEXPBUBvAABB@@@Z (public: void __thiscall WzAnimationInfo::AddBV(struct BvAABB const *))
        4    ?AddBVExtraInfo@CWzUnit@@QAEXABUWzBVExtraInfo@@@Z (public: void __thiscall CWzUnit::AddBVExtraInfo(struct WzBVExtraInfo const &))
        5    ?AddBoneInfo@CWzUnit@@QAEXABUWzBoneInfo@@@Z (public: void __thiscall CWzUnit::AddBoneInfo(struct WzBoneInfo const &))
        6    ?AddBoneScaling@CWzUnitSubType@@QAEXPBUWzBoneScaling@@@Z (public: void __thiscall CWzUnitSubType::AddBoneScaling(struct WzBoneScaling const *))
        7    ?AddCustomInfo@WzAnimationInfo@@QAEXPBUWzCustomInfo@@@Z (public: void __thiscall WzAnimationInfo::AddCustomInfo(struct WzCustomInfo const *))
        8    ?AddDecoration@CWzUnitSubType@@QAEXPBUWzDecoration@@@Z (public: void __thiscall CWzUnitSubType::AddDecoration(struct WzDecoration const *))
        9    ?AddDiffuseMapInfo@CWzUnit@@QAEXHABUWzMappingInfo@@@Z (public: void __thiscall CWzUnit::AddDiffuseMapInfo(int,struct WzMappingInfo const &))
       10    ?AddEffectInfo@WzAnimationInfo@@QAEXPBUWzEffectInfo@@@Z (public: void __thiscall WzAnimationInfo::AddEffectInfo(struct WzEffectInfo const *))
       11    ?AddFilterInfo@CWzUnit@@QAEXHABUWzMappingInfo@@@Z (public: void __thiscall CWzUnit::AddFilterInfo(int,struct WzMappingInfo const &))
       12    ?AddGlowMapInfo@CWzUnit@@QAEXHABUWzMappingInfo@@@Z (public: void __thiscall CWzUnit::AddGlowMapInfo(int,struct WzMappingInfo const &))
       13    ?AddInternalMapInfo@CWzUnit@@QAEXHABUWzMappingInfo@@@Z (public: void __thiscall CWzUnit::AddInternalMapInfo(int,struct WzMappingInfo const &))
       14    ?AddMeshGroupNameInfo@CWzUnit@@QAEXABUMeshGroupNameInfo@@@Z (public: void __thiscall CWzUnit::AddMeshGroupNameInfo(struct MeshGroupNameInfo const &))
       15    ?AddNormalMapInfo@CWzUnit@@QAEXHABUWzMappingInfo@@@Z (public: void __thiscall CWzUnit::AddNormalMapInfo(int,struct WzMappingInfo const &))
       16    ?AddRenderInfo@CWzUnitSubType@@QAEXPBUWzRenderInfo@@@Z (public: void __thiscall CWzUnitSubType::AddRenderInfo(struct WzRenderInfo const *))
       17    ?AddSound@WzAnimationInfo@@QAEXHMH@Z (public: void __thiscall WzAnimationInfo::AddSound(int,float,int))
       18    ?AddSoundInfo@WzAnimationInfo@@QAEXPBUWzSoundInfo@@@Z (public: void __thiscall WzAnimationInfo::AddSoundInfo(struct WzSoundInfo const *))
       19    ?AddSpecularMapInfo@CWzUnit@@QAEXHABUWzMappingInfo@@@Z (public: void __thiscall CWzUnit::AddSpecularMapInfo(int,struct WzMappingInfo const &))
       20    ?AddTexAniID@CWzUnitEditable@@QAEXK@Z (public: void __thiscall CWzUnitEditable::AddTexAniID(unsigned long))
       21    ?AddTexAniMapInfo@CWzUnit@@QAEXHABUWzTexAniMappingInfo@@@Z (public: void __thiscall CWzUnit::AddTexAniMapInfo(int,struct WzTexAniMappingInfo const &))
       22    ?AddTexAniSetInfo@CWzUnit@@QAEXABUWzTexAniSetInfo@@@Z (public: void __thiscall CWzUnit::AddTexAniSetInfo(struct WzTexAniSetInfo const &))
       23    ?AddTexIDInTexAniSetInfo@CWzUnitEditable@@QAEXKH@Z (public: void __thiscall CWzUnitEditable::AddTexIDInTexAniSetInfo(unsigned long,int))
       24    ?AddUnitEffectInfo@CWzUnitDraw@@QAEXPBUWzUnitEffectInfo@@@Z (public: void __thiscall CWzUnitDraw::AddUnitEffectInfo(struct WzUnitEffectInfo const *))
       25    ?AddWzdFileName@CWzUnit@@QAEXPBD@Z (public: void __thiscall CWzUnit::AddWzdFileName(char const *))
       26    ?CheckLoadState@CWzUnit@@AAEXXZ (private: void __thiscall CWzUnit::CheckLoadState(void))
       27    ?ClearAllSound@WzAnimationInfo@@QAEXXZ (public: void __thiscall WzAnimationInfo::ClearAllSound(void))
       28    ?ClearAllUnitEffectInfo@CWzUnitDraw@@QAEXXZ (public: void __thiscall CWzUnitDraw::ClearAllUnitEffectInfo(void))
       29    ?ClearSoundIndex@WzAnimationInfo@@QAEXH@Z (public: void __thiscall WzAnimationInfo::ClearSoundIndex(int))
       30    ?CopySubType@CWzUnitEditable@@QAEXHH@Z (public: void __thiscall CWzUnitEditable::CopySubType(int,int))
       31    ?CreateSubType@CWzUnit@@QAEPAVCWzUnitSubType@@XZ (public: class CWzUnitSubType * __thiscall CWzUnit::CreateSubType(void))
       32    ?CreateSubType@CWzUnitEditable@@QAEPAVCWzUnitSubType@@XZ (public: class CWzUnitSubType * __thiscall CWzUnitEditable::CreateSubType(void))
       33    ?DelAnimationInfoByIndex@CWzUnitEditable@@QAEXH@Z (public: void __thiscall CWzUnitEditable::DelAnimationInfoByIndex(int))
       34    ?DelBVExtraInfoByIndex@CWzUnitEditable@@QAEXH@Z (public: void __thiscall CWzUnitEditable::DelBVExtraInfoByIndex(int))
       35    ?DelBoneInfoByIndex@CWzUnitEditable@@QAEXH@Z (public: void __thiscall CWzUnitEditable::DelBoneInfoByIndex(int))
       36    ?DelBoneScaling@CWzUnitSubTypeEditable@@QAEXH@Z (public: void __thiscall CWzUnitSubTypeEditable::DelBoneScaling(int))
       37    ?DelCustomIndex@WzAnimationInfo@@QAEXH@Z (public: void __thiscall WzAnimationInfo::DelCustomIndex(int))
       38    ?DelDecoration@CWzUnitSubTypeEditable@@QAEXH@Z (public: void __thiscall CWzUnitSubTypeEditable::DelDecoration(int))
       39    ?DelEffectIndex@WzAnimationInfo@@QAEXH@Z (public: void __thiscall WzAnimationInfo::DelEffectIndex(int))
       40    ?DelInternalMapInfoByIndex@CWzUnitEditable@@QAEXH@Z (public: void __thiscall CWzUnitEditable::DelInternalMapInfoByIndex(int))
       41    ?DelRenderInfo@CWzUnitSubTypeEditable@@QAEXH@Z (public: void __thiscall CWzUnitSubTypeEditable::DelRenderInfo(int))
       42    ?DelSoundIndex@WzAnimationInfo@@QAEXHH@Z (public: void __thiscall WzAnimationInfo::DelSoundIndex(int,int))
       43    ?DelSoundSetIndex@WzAnimationInfo@@QAEXH@Z (public: void __thiscall WzAnimationInfo::DelSoundSetIndex(int))
       44    ?DelSubType@CWzUnitEditable@@QAEXH@Z (public: void __thiscall CWzUnitEditable::DelSubType(int))
       45    ?DelTexAniMapInfoByIndex@CWzUnitEditable@@QAEXH@Z (public: void __thiscall CWzUnitEditable::DelTexAniMapInfoByIndex(int))
       46    ?DelTexAniSetInfoByIndex@CWzUnitEditable@@QAEXH@Z (public: void __thiscall CWzUnitEditable::DelTexAniSetInfoByIndex(int))
       47    ?DelTexIDInTexAniSetInfo@CWzUnitEditable@@QAEXHH@Z (public: void __thiscall CWzUnitEditable::DelTexIDInTexAniSetInfo(int,int))
       48    ?DelWzdFileName@CWzUnitEditable@@QAEXH@Z (public: void __thiscall CWzUnitEditable::DelWzdFileName(int))
       49    ?DeleteAllBV@WzAnimationInfo@@QAEXXZ (public: void __thiscall WzAnimationInfo::DeleteAllBV(void))
       50    ?EnableLodByForce@CWzUnitEditable@@QAEX_N@Z (public: void __thiscall CWzUnitEditable::EnableLodByForce(bool))
       51    ?EnableShadowCast@CWzUnitDraw@@QAEXHH@Z (public: void __thiscall CWzUnitDraw::EnableShadowCast(int,int))
       52    ?EnableShadowReceive@CWzUnitDraw@@QAEXHH@Z (public: void __thiscall CWzUnitDraw::EnableShadowReceive(int,int))
       53    ?FindWzdPtr@CWzUnit@@AAEXH@Z (private: void __thiscall CWzUnit::FindWzdPtr(int))
       54    ?GetAnimationInfo@CWzUnit@@QAEPAVWzAnimationInfo@@K@Z (public: class WzAnimationInfo * __thiscall CWzUnit::GetAnimationInfo(unsigned long))
       55    ?GetBoneInfo@CWzUnit@@QAEPAUWzBoneInfo@@K@Z (public: struct WzBoneInfo * __thiscall CWzUnit::GetBoneInfo(unsigned long))
       56    ?GetCustomInfo@WzAnimationInfo@@QAEPAUWzCustomInfo@@H@Z (public: struct WzCustomInfo * __thiscall WzAnimationInfo::GetCustomInfo(int))
       57    ?GetEffectInfo@WzAnimationInfo@@QAEPAUWzEffectInfo@@H@Z (public: struct WzEffectInfo * __thiscall WzAnimationInfo::GetEffectInfo(int))
       58    ?GetInverseAndTransformBuffer@CWzUnitDraw@@QAEPAUWzMatrix@@H@Z (public: struct WzMatrix * __thiscall CWzUnitDraw::GetInverseAndTransformBuffer(int))
       59    ?GetMeshGroupIndexByName@CWzUnit@@QAEHPBD@Z (public: int __thiscall CWzUnit::GetMeshGroupIndexByName(char const *))
       60    ?GetNumCustomInfo@WzAnimationInfo@@QBEHXZ (public: int __thiscall WzAnimationInfo::GetNumCustomInfo(void)const )
       61    ?GetNumEffectInfo@WzAnimationInfo@@QBEHXZ (public: int __thiscall WzAnimationInfo::GetNumEffectInfo(void)const )
       62    ?GetNumSound@WzAnimationInfo@@QBEHH@Z (public: int __thiscall WzAnimationInfo::GetNumSound(int)const )
       63    ?GetNumSoundInfo@WzAnimationInfo@@QBEHXZ (public: int __thiscall WzAnimationInfo::GetNumSoundInfo(void)const )
       64    ?GetNumSoundSet@WzAnimationInfo@@QBEHXZ (public: int __thiscall WzAnimationInfo::GetNumSoundSet(void)const )
       65    ?GetSound@WzAnimationInfo@@QBEHHH@Z (public: int __thiscall WzAnimationInfo::GetSound(int,int)const )
       66    ?GetSoundFrame@WzAnimationInfo@@QBEMH@Z (public: float __thiscall WzAnimationInfo::GetSoundFrame(int)const )
       67    ?GetSoundInfo@WzAnimationInfo@@QAEPAUWzSoundInfo@@H@Z (public: struct WzSoundInfo * __thiscall WzAnimationInfo::GetSoundInfo(int))
       68    ?GetTexAniSetInfo@CWzUnit@@QAEPAUWzTexAniSetInfo@@K@Z (public: struct WzTexAniSetInfo * __thiscall CWzUnit::GetTexAniSetInfo(unsigned long))
       69    ?GetTransformBuffer@CWzUnitDraw@@QAEPAUWzMatrix@@H@Z (public: struct WzMatrix * __thiscall CWzUnitDraw::GetTransformBuffer(int))
       70    ?GetWzdFileName@CWzUnit@@QAEXPADH@Z (public: void __thiscall CWzUnit::GetWzdFileName(char *,int))
       71    ?InitShadowCastRecvInfo@CWzUnitDraw@@QAEXXZ (public: void __thiscall CWzUnitDraw::InitShadowCastRecvInfo(void))
       72    ?IsEnableShadowCast@CWzUnitDraw@@QAEHH@Z (public: int __thiscall CWzUnitDraw::IsEnableShadowCast(int))
       73    ?IsEnableShadowReceive@CWzUnitDraw@@QAEHH@Z (public: int __thiscall CWzUnitDraw::IsEnableShadowReceive(int))
       74    ?IsVoiceChannel@WzAnimationInfo@@QBEHH@Z (public: int __thiscall WzAnimationInfo::IsVoiceChannel(int)const )
       75    ?Process@CWzUnitDraw@@QAEXPBUWzMatrix@@@Z (public: void __thiscall CWzUnitDraw::Process(struct WzMatrix const *))
       76    ?ProgressFrame@CWzUnitDraw@@QAE?AW4ENUM_ANI_FRAME_STATUS@@MPAUWzEvent@@PAM@Z (public: enum ENUM_ANI_FRAME_STATUS __thiscall CWzUnitDraw::ProgressFrame(float,struct WzEvent *,float *))
       77    ?RemoveUnitEffectInfo@CWzUnitDraw@@QAEXH@Z (public: void __thiscall CWzUnitDraw::RemoveUnitEffectInfo(int))
       78    ?ResetBVExtra@CWzUnitDraw@@QAEXXZ (public: void __thiscall CWzUnitDraw::ResetBVExtra(void))
       79    ?SetAniRefUnitDraw@CWzUnitDraw@@QAEXPAV1@@Z (public: void __thiscall CWzUnitDraw::SetAniRefUnitDraw(class CWzUnitDraw *))
       80    ?SetAnimationInfoByIndex@CWzUnitEditable@@QAEXPBVWzAnimationInfo@@H@Z (public: void __thiscall CWzUnitEditable::SetAnimationInfoByIndex(class WzAnimationInfo const *,int))
       81    ?SetBVExtraInfoByIndex@CWzUnitEditable@@QAEXPBUWzBVExtraInfo@@H@Z (public: void __thiscall CWzUnitEditable::SetBVExtraInfoByIndex(struct WzBVExtraInfo const *,int))
       82    ?SetBlendInterpolationFrame@CWzUnitDraw@@QAEXHH@Z (public: void __thiscall CWzUnitDraw::SetBlendInterpolationFrame(int,int))
       83    ?SetBoneInfoByIndex@CWzUnitEditable@@QAEXPBUWzBoneInfo@@H@Z (public: void __thiscall CWzUnitEditable::SetBoneInfoByIndex(struct WzBoneInfo const *,int))
       84    ?SetBoneScaling@CWzUnitSubTypeEditable@@QAEXPBUWzBoneScaling@@H@Z (public: void __thiscall CWzUnitSubTypeEditable::SetBoneScaling(struct WzBoneScaling const *,int))
       85    ?SetBoundingVolume@CWzUnitDraw@@QAEXABUWzBoundingVolume@@@Z (public: void __thiscall CWzUnitDraw::SetBoundingVolume(struct WzBoundingVolume const &))
       86    ?SetCurrentAnimation@CWzUnitDraw@@QAEXKHHH@Z (public: void __thiscall CWzUnitDraw::SetCurrentAnimation(unsigned long,int,int,int))
       87    ?SetCurrentBlendAnimation@CWzUnitDraw@@QAEXKHHMHM@Z (public: void __thiscall CWzUnitDraw::SetCurrentBlendAnimation(unsigned long,int,int,float,int,float))
       88    ?SetCustomInfo@WzAnimationInfo@@QAEXPBUWzCustomInfo@@H@Z (public: void __thiscall WzAnimationInfo::SetCustomInfo(struct WzCustomInfo const *,int))
       89    ?SetDecoration@CWzUnitSubTypeEditable@@QAEXPBUWzDecoration@@H@Z (public: void __thiscall CWzUnitSubTypeEditable::SetDecoration(struct WzDecoration const *,int))
       90    ?SetDiffuseMapInfoByIndex@CWzUnitEditable@@QAEXPBUWzMappingInfo@@H@Z (public: void __thiscall CWzUnitEditable::SetDiffuseMapInfoByIndex(struct WzMappingInfo const *,int))
       91    ?SetEffectApplyRotation@CWzUnitDraw@@QAEXPAXH@Z (public: void __thiscall CWzUnitDraw::SetEffectApplyRotation(void *,int))
       92    ?SetEffectInfo@WzAnimationInfo@@QAEXPBUWzEffectInfo@@H@Z (public: void __thiscall WzAnimationInfo::SetEffectInfo(struct WzEffectInfo const *,int))
       93    ?SetEffectPosition@CWzUnitDraw@@QAEXPAXABUWzVector@@@Z (public: void __thiscall CWzUnitDraw::SetEffectPosition(void *,struct WzVector const &))
       94    ?SetEffectRotation@CWzUnitDraw@@QAEXPAXABUWzQuaternion@@@Z (public: void __thiscall CWzUnitDraw::SetEffectRotation(void *,struct WzQuaternion const &))
       95    ?SetEffectScale@CWzUnitDraw@@QAEXPAXABUWzVector@@@Z (public: void __thiscall CWzUnitDraw::SetEffectScale(void *,struct WzVector const &))
       96    ?SetGlowMapInfoByIndex@CWzUnitEditable@@QAEXPBUWzMappingInfo@@H@Z (public: void __thiscall CWzUnitEditable::SetGlowMapInfoByIndex(struct WzMappingInfo const *,int))
       97    ?SetHasBVInfo@CWzUnitEditable@@QAEXH@Z (public: void __thiscall CWzUnitEditable::SetHasBVInfo(int))
       98    ?SetInternalMapInfoByIndex@CWzUnitEditable@@QAEXPBUWzMappingInfo@@H@Z (public: void __thiscall CWzUnitEditable::SetInternalMapInfoByIndex(struct WzMappingInfo const *,int))
       99    ?SetInterpolationFrame@CWzUnitDraw@@QAEXH@Z (public: void __thiscall CWzUnitDraw::SetInterpolationFrame(int))
      100    ?SetNormalMapInfoByIndex@CWzUnitEditable@@QAEXPBUWzMappingInfo@@H@Z (public: void __thiscall CWzUnitEditable::SetNormalMapInfoByIndex(struct WzMappingInfo const *,int))
      101    ?SetPosition@CWzUnitDraw@@QAEXABUWzVector@@H@Z (public: void __thiscall CWzUnitDraw::SetPosition(struct WzVector const &,int))
      102    ?SetPosition@CWzUnitDraw@@QAEXMMMH@Z (public: void __thiscall CWzUnitDraw::SetPosition(float,float,float,int))
      103    ?SetRenderInfo@CWzUnitSubTypeEditable@@QAEXPBUWzRenderInfo@@H@Z (public: void __thiscall CWzUnitSubTypeEditable::SetRenderInfo(struct WzRenderInfo const *,int))
      104    ?SetRotation@CWzUnitDraw@@QAEXABUWzVector@@H@Z (public: void __thiscall CWzUnitDraw::SetRotation(struct WzVector const &,int))
      105    ?SetRotation@CWzUnitDraw@@QAEXMMMH@Z (public: void __thiscall CWzUnitDraw::SetRotation(float,float,float,int))
      106    ?SetScale@CWzUnitDraw@@QAEXABUWzVector@@H@Z (public: void __thiscall CWzUnitDraw::SetScale(struct WzVector const &,int))
      107    ?SetScale@CWzUnitDraw@@QAEXMH@Z (public: void __thiscall CWzUnitDraw::SetScale(float,int))
      108    ?SetScale@CWzUnitDraw@@QAEXMMMH@Z (public: void __thiscall CWzUnitDraw::SetScale(float,float,float,int))
      109    ?SetSoundFrame@WzAnimationInfo@@QAEXMH@Z (public: void __thiscall WzAnimationInfo::SetSoundFrame(float,int))
      110    ?SetSpecularMapInfoByIndex@CWzUnitEditable@@QAEXPBUWzMappingInfo@@H@Z (public: void __thiscall CWzUnitEditable::SetSpecularMapInfoByIndex(struct WzMappingInfo const *,int))
      111    ?SetSubType@CWzUnitDraw@@QAEXH@Z (public: void __thiscall CWzUnitDraw::SetSubType(int))
      112    ?SetTexAniMapInfoByIndex@CWzUnitEditable@@QAEXPBUWzTexAniMappingInfo@@H@Z (public: void __thiscall CWzUnitEditable::SetTexAniMapInfoByIndex(struct WzTexAniMappingInfo const *,int))
      113    ?SetTexAniSetInfoByIndex@CWzUnitEditable@@QAEXPBUWzTexAniSetInfo@@H@Z (public: void __thiscall CWzUnitEditable::SetTexAniSetInfoByIndex(struct WzTexAniSetInfo const *,int))
      114    ?SetVoiceChannel@WzAnimationInfo@@QAEXHH@Z (public: void __thiscall WzAnimationInfo::SetVoiceChannel(int,int))
      115    ?SetWzUnit@CWzUnitDraw@@QAEXPAVCWzUnit@@H@Z (public: void __thiscall CWzUnitDraw::SetWzUnit(class CWzUnit *,int))
      116    ?SetWzdFileName@CWzUnitEditable@@QAEXPBDH@Z (public: void __thiscall CWzUnitEditable::SetWzdFileName(char const *,int))
      117    ?UnSetBlendAnimation@CWzUnitDraw@@QAEXXZ (public: void __thiscall CWzUnitDraw::UnSetBlendAnimation(void))
      118    ?UpdateBoundingVolumeWithMatrix@CWzUnitDraw@@QAEXPAUWzMatrix@@@Z (public: void __thiscall CWzUnitDraw::UpdateBoundingVolumeWithMatrix(struct WzMatrix *))
      119    ?UpdateShadowVolume@CWzUnitDraw@@QAEXPAVCWzdBase@@ABUWzVector@@PBU3@K@Z (public: void __thiscall CWzUnitDraw::UpdateShadowVolume(class CWzdBase *,struct WzVector const &,struct WzVector const *,unsigned long))
      120    ?UpdateSilhouette@CWzUnitDraw@@QAEXPAVCWzdBase@@ABUWzVector@@PBU3@@Z (public: void __thiscall CWzUnitDraw::UpdateSilhouette(class CWzdBase *,struct WzVector const &,struct WzVector const *))
      121    _Func_ContactWzd
               exported name: Func_ContactWzd
